 config_device_type_edit

 Timestamp is 614c8039 (Thu Sep 23 13:25:13 2021)

 Preferred load address is 10000000

 Start         Length     Name                   Class
 0001:00000000 000000c6H .text$di                CODE
 0001:000000d0 0000edbcH .text$mn                CODE
 0001:0000ee8c 0000280aH .text$x                 CODE
 0001:00011696 00000042H .text$yd                CODE
 0002:00000000 00000fb4H .idata$5                DATA
 0002:00000fb4 00000004H .CRT$XCA                DATA
 0002:00000fb8 00000018H .CRT$XCU                DATA
 0002:00000fd0 00000004H .CRT$XCZ                DATA
 0002:00000fd4 00000004H .CRT$XIA                DATA
 0002:00000fd8 00000004H .CRT$XIAA               DATA
 0002:00000fdc 00000004H .CRT$XIC                DATA
 0002:00000fe0 00000004H .CRT$XIZ                DATA
 0002:00000ff0 00005098H .rdata                  DATA
 0002:00006088 000013b4H .rdata$r                DATA
 0002:0000743c 00000004H .rtc$IAA                DATA
 0002:00007440 00000004H .rtc$IZZ                DATA
 0002:00007444 00000004H .rtc$TAA                DATA
 0002:00007448 00000004H .rtc$TZZ                DATA
 0002:00007450 000026b4H .xdata$x                DATA
 0002:00009b10 00000699H .edata                  DATA
 0002:0000a1ac 00000050H .idata$2                DATA
 0002:0000a1fc 00000014H .idata$3                DATA
 0002:0000a210 00000fb4H .idata$4                DATA
 0002:0000b1c4 0000a354H .idata$6                DATA
 0003:00000000 000000c4H .data                   DATA
 0003:000000c4 00000638H .data$r                 DATA
 0003:00000700 00000464H .bss                    DATA
 0004:00000000 000000a0H .rsrc$01                DATA
 0004:000000a0 00000620H .rsrc$02                DATA

  Address         Publics by Value              Rva+Base       Lib:Object

 0000:00000000       ___safe_se_handler_count   00000000     <absolute>
 0000:00000000       __except_list              00000000     <absolute>
 0000:00000000       ___guard_flags             00000000     <absolute>
 0000:00000000       ___guard_fids_table        00000000     <absolute>
 0000:00000000       ___safe_se_handler_table   00000000     <absolute>
 0000:00000000       ___guard_fids_count        00000000     <absolute>
 0000:00009876       __ldused                   00009876     <absolute>
 0000:00009876       __fltused                  00009876     <absolute>
 0000:00000000       ___ImageBase               10000000     <linker-defined>
 0001:000000d0       ??0?$QGuardedPtr@VQDockWindow@@@@QAE@XZ 100010d0 f i device_type_edit.obj
 0001:000000d0       ??0?$QGuardedPtr@VtoolWindow@@@@QAE@XZ 100010d0 f i device_type_edit.obj
 0001:000000d0       ??0?$QGuardedPtr@VQPopupMenu@@@@QAE@XZ 100010d0 f i device_type_edit.obj
 0001:00000111       ??0config_plugin_base@@QAE@ABVQString@@00@Z 10001111 f i device_type_edit.obj
 0001:0000019e       ??0device_type_edit@@QAE@ABVQString@@00@Z 1000119e f   device_type_edit.obj
 0001:00000739       ??1?$QDict@VQAction@@@@UAE@XZ 10001739 f i device_type_edit.obj
 0001:0000076c       ??1?$QGuardedPtr@VtoolWindow@@@@QAE@XZ 1000176c f i device_type_edit.obj
 0001:0000076c       ??1?$QGuardedPtr@VQDockWindow@@@@QAE@XZ 1000176c f i device_type_edit.obj
 0001:0000076c       ??1?$QGuardedPtr@VQPopupMenu@@@@QAE@XZ 1000176c f i device_type_edit.obj
 0001:00000771       ??1?$QPtrList@VQPopupMenu@@@@UAE@XZ 10001771 f i device_type_edit.obj
 0001:000007a4       ??1QDockWindowList@@UAE@XZ 100017a4 f i device_type_edit.obj
 0001:000007ed       ??1QPopupMenuList@@UAE@XZ  100017ed f i device_type_edit.obj
 0001:0000081f       ??1config_plugin_base@@UAE@XZ 1000181f f i device_type_edit.obj
 0001:00000879       ??1device_type_edit@@UAE@XZ 10001879 f   device_type_edit.obj
 0001:00000958       ??4?$QGuardedPtr@VQDockWindow@@@@QAEAAV0@PAVQDockWindow@@@Z 10001958 f i device_type_edit.obj
 0001:00000958       ??4?$QGuardedPtr@VQPopupMenu@@@@QAEAAV0@PAVQPopupMenu@@@Z 10001958 f i device_type_edit.obj
 0001:00000958       ??4?$QGuardedPtr@VtoolWindow@@@@QAEAAV0@PAVtoolWindow@@@Z 10001958 f i device_type_edit.obj
 0001:000009b6       ??_EQDockWindow@@WCI@AEPAXI@Z 100019b6 f i device_type_edit.obj
 0001:000009be       ??_EQPopupMenu@@WCI@AEPAXI@Z 100019be f i device_type_edit.obj
 0001:000009c6       ??_EQPopupMenu@@WIM@AEPAXI@Z 100019c6 f i device_type_edit.obj
 0001:000009d1       ??_EQToolBar@@WCI@AEPAXI@Z 100019d1 f i device_type_edit.obj
 0001:000009d9       ??_Econfig_plugin_base@@WCI@AEPAXI@Z 100019d9 f i device_type_edit.obj
 0001:000009e1       ??_Edevice_type_edit@@WCI@AEPAXI@Z 100019e1 f i device_type_edit.obj
 0001:000009e9       ??_E?$QDict@VQAction@@@@UAEPAXI@Z 100019e9 f i device_type_edit.obj
 0001:000009e9       ??_G?$QDict@VQAction@@@@UAEPAXI@Z 100019e9 f i device_type_edit.obj
 0001:00000a08       ??_E?$QPtrList@VQPopupMenu@@@@UAEPAXI@Z 10001a08 f i device_type_edit.obj
 0001:00000a08       ??_G?$QPtrList@VQPopupMenu@@@@UAEPAXI@Z 10001a08 f i device_type_edit.obj
 0001:00000a27       ??_EQAction@@UAEPAXI@Z     10001a27 f i device_type_edit.obj
 0001:00000a27       ??_GQAction@@UAEPAXI@Z     10001a27 f i device_type_edit.obj
 0001:00000a47       ??_EQDockWindow@@UAEPAXI@Z 10001a47 f i device_type_edit.obj
 0001:00000a47       ??_GQDockWindow@@UAEPAXI@Z 10001a47 f i device_type_edit.obj
 0001:00000a67       ??_GQDockWindowList@@UAEPAXI@Z 10001a67 f i device_type_edit.obj
 0001:00000a67       ??_EQDockWindowList@@UAEPAXI@Z 10001a67 f i device_type_edit.obj
 0001:00000a86       ??_GQGuardedPtrPrivate@@UAEPAXI@Z 10001a86 f i device_type_edit.obj
 0001:00000a86       ??_EQGuardedPtrPrivate@@UAEPAXI@Z 10001a86 f i device_type_edit.obj
 0001:00000aa6       ??_GQPopupMenu@@UAEPAXI@Z  10001aa6 f i device_type_edit.obj
 0001:00000aa6       ??_EQPopupMenu@@UAEPAXI@Z  10001aa6 f i device_type_edit.obj
 0001:00000ac6       ??_EQPopupMenuList@@UAEPAXI@Z 10001ac6 f i device_type_edit.obj
 0001:00000ac6       ??_GQPopupMenuList@@UAEPAXI@Z 10001ac6 f i device_type_edit.obj
 0001:00000ae5       ??_EQToolBar@@UAEPAXI@Z    10001ae5 f i device_type_edit.obj
 0001:00000ae5       ??_GQToolBar@@UAEPAXI@Z    10001ae5 f i device_type_edit.obj
 0001:00000b05       ??_Econfig_plugin_base@@UAEPAXI@Z 10001b05 f i device_type_edit.obj
 0001:00000b05       ??_Gconfig_plugin_base@@UAEPAXI@Z 10001b05 f i device_type_edit.obj
 0001:00000b24       ??_Edevice_type_edit@@UAEPAXI@Z 10001b24 f i device_type_edit.obj
 0001:00000b24       ??_Gdevice_type_edit@@UAEPAXI@Z 10001b24 f i device_type_edit.obj
 0001:00000b43       ?about@config_plugin_base@@UAE?AVQString@@XZ 10001b43 f i device_type_edit.obj
 0001:00000b99       ?about@device_type_edit@@UAE?AVQString@@XZ 10001b99 f   device_type_edit.obj
 0001:00000c41       ?activate@device_type_edit@@UAEX_N@Z 10001c41 f   device_type_edit.obj
 0001:00000e49       ?apply@config_plugin_base@@UAEXXZ 10001e49 f i device_type_edit.obj
 0001:00000e4a       ?apply@device_type_edit@@UAEXXZ 10001e4a f   device_type_edit.obj
 0001:0000127b       ?clear@?$QDict@VQAction@@@@UAEXXZ 1000227b f i device_type_edit.obj
 0001:00001281       ?clear@?$QPtrList@VQListViewItem@@@@UAEXXZ 10002281 f i device_type_editdlgimpl.obj
 0001:00001281       ?clear@?$QPtrList@VQPopupMenu@@@@UAEXXZ 10002281 f i device_type_edit.obj
 0001:00001287       ?closeEvent@config_plugin_base@@UAEXPAVQCloseEvent@@@Z 10002287 f i device_type_edit.obj
 0001:00001295       ?closeEvent@device_type_edit@@UAEXPAVQCloseEvent@@@Z 10002295 f   device_type_edit.obj
 0001:000013a2       ?count@?$QDict@VQAction@@@@UBEIXZ 100023a2 f i device_type_edit.obj
 0001:000013a6       ?db@@YAXABVQString@@@Z     100023a6 f   device_type_edit.obj
 0001:000013ee       ?deleteItem@?$QPtrList@VQPopupMenu@@@@EAEXPAX@Z 100023ee f i device_type_edit.obj
 0001:000013ee       ?deleteItem@?$QDict@VQAction@@@@EAEXPAX@Z 100023ee f i device_type_edit.obj
 0001:00001409       ?deleteType@device_type_edit@@AAEXABVQString@@@Z 10002409 f   device_type_edit.obj
 0001:0000157c       ?deref@?$QGuardedPtr@VQPopupMenu@@@@AAEXXZ 1000257c f i device_type_edit.obj
 0001:0000157c       ?deref@?$QGuardedPtr@VtoolWindow@@@@AAEXXZ 1000257c f i device_type_edit.obj
 0001:0000157c       ?deref@?$QGuardedPtr@VQDockWindow@@@@AAEXXZ 1000257c f i device_type_edit.obj
 0001:00001591       ?isDirty@config_plugin_base@@UAE_NXZ 10002591 f i device_type_edit.obj
 0001:00001591       ?validate@config_plugin_base@@UAE_NXZ 10002591 f i device_type_edit.obj
 0001:00001591       ?qt_static_property@cfg_ListView@@SA_NPAVQObject@@HHPAVQVariant@@@Z 10002591 f i cfg_widgets001:moc_cfg_ListView.obj
 0001:00001594       ?isDirty@device_type_edit@@UAE_NXZ 10002594 f   device_type_edit.obj
 0001:0000159b       ?markDirty@device_type_edit@@AAEXXZ 1000259b f   device_type_edit.obj
 0001:0000169d       ?menus@config_plugin_base@@UAE?AVQPopupMenuList@@XZ 1000269d f i device_type_edit.obj
 0001:000016c0       ?menus@device_type_edit@@UAE?AVQPopupMenuList@@XZ 100026c0 f   device_type_edit.obj
 0001:0000170a       ?metaObject@device_type_edit@@UBEPAVQMetaObject@@XZ 1000270a f i device_type_edit.obj
 0001:0000170f       ?navigate@config_plugin_base@@UAEXABVQString@@0@Z 1000270f f i device_type_edit.obj
 0001:00001712       ?navigate@device_type_edit@@UAEXABVQString@@0@Z 10002712 f   device_type_edit.obj
 0001:0000178e       ?reply@config_plugin_base@@UAEXPAVresponse@@@Z 1000278e f i device_type_edit.obj
 0001:0000178e       ?activate@config_plugin_base@@UAEX_N@Z 1000278e f i device_type_edit.obj
 0001:00001791       ?reply@device_type_edit@@UAEXPAVresponse@@@Z 10002791 f   device_type_edit.obj
 0001:00001f01       ?resizeEvent@device_type_edit@@UAEXPAVQResizeEvent@@@Z 10002f01 f   device_type_edit.obj
 0001:00001f36       ?selectType@device_type_edit@@AAEXABVQString@@@Z 10002f36 f   device_type_edit.obj
 0001:00002186       ?toolbars@config_plugin_base@@UAE?AVQDockWindowList@@XZ 10003186 f i device_type_edit.obj
 0001:000021a9       ?toolbars@device_type_edit@@UAE?AVQDockWindowList@@XZ 100031a9 f   device_type_edit.obj
 0001:00002201       ??0device_type_editDlg@@QAE@ABVQString@@PAVQWidget@@PBDI@Z 10003201 f   device_type_editdlgimpl.obj
 0001:00002661       ??1?$QPtrList@VQListViewItem@@@@UAE@XZ 10003661 f i device_type_editdlgimpl.obj
 0001:00002694       ??1?$QPtrListIterator@VQFileInfo@@@@QAE@XZ 10003694 f i device_type_editdlgimpl.obj
 0001:0000269a       ??1device_type_editDlg@@UAE@XZ 1000369a f   device_type_editdlgimpl.obj
 0001:0000270b       ??_Edevice_type_editDlg@@WCI@AEPAXI@Z 1000370b f i device_type_editdlgimpl.obj
 0001:00002713       ??_E?$QPtrList@VQListViewItem@@@@UAEPAXI@Z 10003713 f i device_type_editdlgimpl.obj
 0001:00002713       ??_G?$QPtrList@VQListViewItem@@@@UAEPAXI@Z 10003713 f i device_type_editdlgimpl.obj
 0001:00002732       ??_EQDomDocument@@UAEPAXI@Z 10003732 f i device_type_editdlgimpl.obj
 0001:00002732       ??_GQDomDocument@@UAEPAXI@Z 10003732 f i device_type_editdlgimpl.obj
 0001:00002752       ??_GQDomElement@@UAEPAXI@Z 10003752 f i device_type_editdlgimpl.obj
 0001:00002752       ??_EQDomElement@@UAEPAXI@Z 10003752 f i device_type_editdlgimpl.obj
 0001:00002772       ??_GQListViewItem@@UAEPAXI@Z 10003772 f i device_type_editdlgimpl.obj
 0001:00002772       ??_EQListViewItem@@UAEPAXI@Z 10003772 f i device_type_editdlgimpl.obj
 0001:00002792       ??_Edevice_type_editDlg@@UAEPAXI@Z 10003792 f i device_type_editdlgimpl.obj
 0001:00002792       ??_Gdevice_type_editDlg@@UAEPAXI@Z 10003792 f i device_type_editdlgimpl.obj
 0001:000027b1       ?apply@device_type_editDlg@@QAEXXZ 100037b1 f   device_type_editdlgimpl.obj
 0001:000027c2       ?checkParamClipboard@device_type_editDlg@@AAEXXZ 100037c2 f   device_type_editdlgimpl.obj
 0001:000028a0       ?clear@device_type_editDlg@@AAEXXZ 100038a0 f   device_type_editdlgimpl.obj
 0001:000028c3       ?clearParamView@device_type_editDlg@@AAEXXZ 100038c3 f   device_type_editdlgimpl.obj
 0001:00002983       ?count@?$QPtrList@VQPopupMenu@@@@UBEIXZ 10003983 f i device_type_edit.obj
 0001:00002983       ?count@?$QPtrList@VQListViewItem@@@@UBEIXZ 10003983 f i device_type_editdlgimpl.obj
 0001:00002987       ?deleteItem@?$QPtrList@VQListViewItem@@@@EAEXPAX@Z 10003987 f i device_type_editdlgimpl.obj
 0001:000029a1       ?devTypeChange@device_type_editDlg@@AAEXH@Z 100039a1 f   device_type_editdlgimpl.obj
 0001:00002aa1       ?displayEnum@device_type_editDlg@@AAEXPAVQDomElement@@@Z 10003aa1 f   device_type_editdlgimpl.obj
 0001:00002d7f       ?displayRange@device_type_editDlg@@AAEXPAVQDomElement@@@Z 10003d7f f   device_type_editdlgimpl.obj
 0001:000032cd       ?displayString@device_type_editDlg@@AAEXPAVQDomElement@@@Z 100042cd f   device_type_editdlgimpl.obj
 0001:000034a4       ?enumDblClick@device_type_editDlg@@AAEXPAVQListViewItem@@ABVQPoint@@H@Z 100044a4 f   device_type_editdlgimpl.obj
 0001:000034e7       ?enumDeleteState@device_type_editDlg@@AAEXXZ 100044e7 f   device_type_editdlgimpl.obj
 0001:00003530       ?enumDeleteState@device_type_editDlg@@AAE_NVQString@@@Z 10004530 f   device_type_editdlgimpl.obj
 0001:0000373c       ?enumNewState@device_type_editDlg@@AAEXXZ 1000473c f   device_type_editdlgimpl.obj
 0001:00003b27       ?enumPaste@device_type_editDlg@@AAEXXZ 10004b27 f   device_type_editdlgimpl.obj
 0001:00004033       ?loadElement@device_type_editDlg@@AAE_NPAVQDomElement@@@Z 10005033 f   device_type_editdlgimpl.obj
 0001:0000436c       ?loadFile@device_type_editDlg@@AAE_NABVQString@@0@Z 1000536c f   device_type_editdlgimpl.obj
 0001:00004812       ?loadParamLvi@device_type_editDlg@@AAEXVQString@@PAVQDomElement@@@Z 10005812 f   device_type_editdlgimpl.obj
 0001:00004a47       ?loadTemplates@device_type_editDlg@@AAEXVQString@@@Z 10005a47 f   device_type_editdlgimpl.obj
 0001:00004b96       ?markDirty@device_type_editDlg@@AAEXH@Z 10005b96 f   device_type_editdlgimpl.obj
 0001:00004b96       ?markDirty@device_type_editDlg@@AAEXABVQString@@@Z 10005b96 f   device_type_editdlgimpl.obj
 0001:00004b9e       ?markDirty@device_type_editDlg@@AAEXPAVQListViewItem@@H@Z 10005b9e f   device_type_editdlgimpl.obj
 0001:00004ba6       ?markDirty@device_type_editDlg@@AAEXXZ 10005ba6 f   device_type_editdlgimpl.obj
 0001:00004bcb       ?metaObject@device_type_editDlg@@UBEPAVQMetaObject@@XZ 10005bcb f i device_type_editdlgimpl.obj
 0001:00004bd0       ?newGetNewParamName@device_type_editDlg@@AAE?AVQString@@V2@@Z 10005bd0 f   device_type_editdlgimpl.obj
 0001:00004eef       ?paramCopy@device_type_editDlg@@AAEXXZ 10005eef f   device_type_editdlgimpl.obj
 0001:0000517f       ?paramDelete@device_type_editDlg@@AAEXXZ 1000617f f   device_type_editdlgimpl.obj
 0001:000053c6       ?paramNew@device_type_editDlg@@AAEXXZ 100063c6 f   device_type_editdlgimpl.obj
 0001:00005589       ?paramPaste@device_type_editDlg@@AAEXXZ 10006589 f   device_type_editdlgimpl.obj
 0001:000059c4       ?paramRename@device_type_editDlg@@AAEXXZ 100069c4 f   device_type_editdlgimpl.obj
 0001:00005ae7       ?removeSettings@device_type_editDlg@@AAE_NPAVQDomElement@@VQString@@@Z 10006ae7 f   device_type_editdlgimpl.obj
 0001:00005f67       ?saveElement@device_type_editDlg@@AAE_NPAVQDomElement@@@Z 10006f67 f   device_type_editdlgimpl.obj
 0001:00006289       ?saveEnum@device_type_editDlg@@AAE_NPAVQDomElement@@@Z 10007289 f   device_type_editdlgimpl.obj
 0001:0000655a       ?saveFile@device_type_editDlg@@AAE_NABVQString@@0@Z 1000755a f   device_type_editdlgimpl.obj
 0001:00006648       ?saveRange@device_type_editDlg@@AAE_NPAVQDomElement@@@Z 10007648 f   device_type_editdlgimpl.obj
 0001:00006d40       ?saveString@device_type_editDlg@@AAE_NPAVQDomElement@@@Z 10007d40 f   device_type_editdlgimpl.obj
 0001:00006fa9       ?selectParam@device_type_editDlg@@AAEXPAVQListViewItem@@@Z 10007fa9 f   device_type_editdlgimpl.obj
 0001:0000726e       ?selectParam@device_type_editDlg@@AAEXXZ 1000826e f   device_type_editdlgimpl.obj
 0001:0000735d       ??0paramLVI@@QAE@PAVQListView@@@Z 1000835d f   paramLVI.obj
 0001:00007379       ??1paramLVI@@UAE@XZ        10008379 f   paramLVI.obj
 0001:00007385       ??_EparamLVI@@UAEPAXI@Z    10008385 f i paramLVI.obj
 0001:00007385       ??_GparamLVI@@UAEPAXI@Z    10008385 f i paramLVI.obj
 0001:000073a4       ?compare@paramLVI@@UBEHPAVQListViewItem@@H_N@Z 100083a4 f   paramLVI.obj
 0001:0000754c       ??_Gplugindesc@@UAEPAXI@Z  1000854c f i plugindesc.obj
 0001:0000754c       ??_Gconfig_plugin_desc_base@@UAEPAXI@Z 1000854c f i plugindesc.obj
 0001:0000754c       ??_Econfig_plugin_desc_base@@UAEPAXI@Z 1000854c f i plugindesc.obj
 0001:0000754c       ??_Eplugindesc@@UAEPAXI@Z  1000854c f i plugindesc.obj
 0001:0000756c       ?create@plugindesc@@UAEPAVconfig_plugin_base@@ABVQString@@00@Z 1000856c f   plugindesc.obj
 0001:000075a7       ?keys@plugindesc@@UAE?AVQStringList@@ABVQString@@0@Z 100085a7 f   plugindesc.obj
 0001:00007602       ?pixmap@plugindesc@@UAE?AVQPixmap@@ABVQString@@@Z 10008602 f   plugindesc.obj
 0001:00007621       _load_bncs_config_plugin_desc 10008621 f   plugindesc.obj
 0001:00007637       ??0toolWindow@@QAE@PAVQWidget@@PBDI@Z 10008637 f   toolwindowimpl.obj
 0001:00007719       ??1toolWindow@@UAE@XZ      10008719 f   toolwindowimpl.obj
 0001:00007758       ??_EtoolWindow@@WCI@AEPAXI@Z 10008758 f i toolwindowimpl.obj
 0001:00007760       ??_GtoolWindow@@UAEPAXI@Z  10008760 f i toolwindowimpl.obj
 0001:00007760       ??_EtoolWindow@@UAEPAXI@Z  10008760 f i toolwindowimpl.obj
 0001:0000777f       ?deleteFile@toolWindow@@AAEXXZ 1000877f f   toolwindowimpl.obj
 0001:0000794c       ?loadFile@toolWindow@@QAE_NVQString@@@Z 1000894c f   toolwindowimpl.obj
 0001:00007ca6       ?metaObject@toolWindow@@UBEPAVQMetaObject@@XZ 10008ca6 f i toolwindowimpl.obj
 0001:00007cab       ?newFile@toolWindow@@AAEXXZ 10008cab f   toolwindowimpl.obj
 0001:000081e4       ?saveFile@toolWindow@@QAE_NVQString@@@Z 100091e4 f   toolwindowimpl.obj
 0001:000082ac       ?selectFamily@toolWindow@@AAE?AVQString@@V2@0@Z 100092ac f   toolwindowimpl.obj
 0001:00008395       ?selectType@toolWindow@@AAEXPAVQListViewItem@@@Z 10009395 f   toolwindowimpl.obj
 0001:000083d6       ??0device_type_editDlgBase@@QAE@PAVQWidget@@PBDI@Z 100093d6 f   device_type_editdlg.obj
 0001:0000a4a5       ??1device_type_editDlgBase@@UAE@XZ 1000b4a5 f   device_type_editdlg.obj
 0001:0000a4e5       ??_EQCheckBox@@WCI@AEPAXI@Z 1000b4e5 f i device_type_editdlg.obj
 0001:0000a4ed       ??_EQComboBox@@WCI@AEPAXI@Z 1000b4ed f i device_type_editdlg.obj
 0001:0000a4f5       ??_EQGridLayout@@WCI@AEPAXI@Z 1000b4f5 f i device_type_editdlg.obj
 0001:0000a4fd       ??_EQGroupBox@@WCI@AEPAXI@Z 1000b4fd f i device_type_editdlg.obj
 0001:0000a505       ??_EQHBoxLayout@@WCI@AEPAXI@Z 1000b505 f i device_type_editdlg.obj
 0001:0000a50d       ??_EQLabel@@WCI@AEPAXI@Z   1000b50d f i device_type_editdlg.obj
 0001:0000a515       ??_EQLineEdit@@WCI@AEPAXI@Z 1000b515 f i device_type_editdlg.obj
 0001:0000a51d       ??_EQListView@@WCI@AEPAXI@Z 1000b51d f i device_type_editdlg.obj
 0001:0000a525       ??_EQPushButton@@WCI@AEPAXI@Z 1000b525 f i device_type_editdlg.obj
 0001:0000a52d       ??_EQSpinBox@@WCI@AEPAXI@Z 1000b52d f i device_type_editdlg.obj
 0001:0000a535       ??_EQSpinBox@@WGM@AEPAXI@Z 1000b535 f i device_type_editdlg.obj
 0001:0000a53d       ??_EQVBoxLayout@@WCI@AEPAXI@Z 1000b53d f i device_type_editdlg.obj
 0001:0000a545       ??_EQWidget@@WCI@AEPAXI@Z  1000b545 f i device_type_editdlg.obj
 0001:0000a54d       ??_EQWidgetStack@@WCI@AEPAXI@Z 1000b54d f i device_type_editdlg.obj
 0001:0000a555       ??_Edevice_type_editDlgBase@@WCI@AEPAXI@Z 1000b555 f i device_type_editdlg.obj
 0001:0000a55d       ??_EQCheckBox@@UAEPAXI@Z   1000b55d f i device_type_editdlg.obj
 0001:0000a55d       ??_GQCheckBox@@UAEPAXI@Z   1000b55d f i device_type_editdlg.obj
 0001:0000a57d       ??_GQComboBox@@UAEPAXI@Z   1000b57d f i device_type_editdlg.obj
 0001:0000a57d       ??_EQComboBox@@UAEPAXI@Z   1000b57d f i device_type_editdlg.obj
 0001:0000a59d       ??_EQGridLayout@@UAEPAXI@Z 1000b59d f i device_type_editdlg.obj
 0001:0000a59d       ??_GQGridLayout@@UAEPAXI@Z 1000b59d f i device_type_editdlg.obj
 0001:0000a5bd       ??_GQGroupBox@@UAEPAXI@Z   1000b5bd f i device_type_editdlg.obj
 0001:0000a5bd       ??_EQGroupBox@@UAEPAXI@Z   1000b5bd f i device_type_editdlg.obj
 0001:0000a5dd       ??_GQHBoxLayout@@UAEPAXI@Z 1000b5dd f i device_type_editdlg.obj
 0001:0000a5dd       ??_EQHBoxLayout@@UAEPAXI@Z 1000b5dd f i device_type_editdlg.obj
 0001:0000a5fd       ??_GQLabel@@UAEPAXI@Z      1000b5fd f i device_type_editdlg.obj
 0001:0000a5fd       ??_EQLabel@@UAEPAXI@Z      1000b5fd f i device_type_editdlg.obj
 0001:0000a61d       ??_EQLineEdit@@UAEPAXI@Z   1000b61d f i device_type_editdlg.obj
 0001:0000a61d       ??_GQLineEdit@@UAEPAXI@Z   1000b61d f i device_type_editdlg.obj
 0001:0000a63d       ??_EQListView@@UAEPAXI@Z   1000b63d f i device_type_editdlg.obj
 0001:0000a63d       ??_GQListView@@UAEPAXI@Z   1000b63d f i device_type_editdlg.obj
 0001:0000a65d       ??_EQPushButton@@UAEPAXI@Z 1000b65d f i device_type_editdlg.obj
 0001:0000a65d       ??_GQPushButton@@UAEPAXI@Z 1000b65d f i device_type_editdlg.obj
 0001:0000a67d       ??_EQSpacerItem@@UAEPAXI@Z 1000b67d f i device_type_editdlg.obj
 0001:0000a67d       ??_GQSpacerItem@@UAEPAXI@Z 1000b67d f i device_type_editdlg.obj
 0001:0000a69d       ??_GQSpinBox@@UAEPAXI@Z    1000b69d f i device_type_editdlg.obj
 0001:0000a69d       ??_EQSpinBox@@UAEPAXI@Z    1000b69d f i device_type_editdlg.obj
 0001:0000a6bd       ??_GQVBoxLayout@@UAEPAXI@Z 1000b6bd f i device_type_editdlg.obj
 0001:0000a6bd       ??_EQVBoxLayout@@UAEPAXI@Z 1000b6bd f i device_type_editdlg.obj
 0001:0000a6dd       ??_EQWidget@@UAEPAXI@Z     1000b6dd f i device_type_editdlg.obj
 0001:0000a6dd       ??_GQWidget@@UAEPAXI@Z     1000b6dd f i device_type_editdlg.obj
 0001:0000a6fd       ??_EQWidgetStack@@UAEPAXI@Z 1000b6fd f i device_type_editdlg.obj
 0001:0000a6fd       ??_GQWidgetStack@@UAEPAXI@Z 1000b6fd f i device_type_editdlg.obj
 0001:0000a71d       ??_Gdevice_type_editDlgBase@@UAEPAXI@Z 1000b71d f i device_type_editdlg.obj
 0001:0000a71d       ??_Edevice_type_editDlgBase@@UAEPAXI@Z 1000b71d f i device_type_editdlg.obj
 0001:0000a73c       ?languageChange@device_type_editDlgBase@@MAEXXZ 1000b73c f   device_type_editdlg.obj
 0001:0000b36d       ?metaObject@device_type_editDlgBase@@UBEPAVQMetaObject@@XZ 1000c36d f i device_type_editdlg.obj
 0001:0000b372       ?className@device_type_edit@@UBEPBDXZ 1000c372 f   moc_device_type_edit.obj
 0001:0000b378       ?command@device_type_edit@@IAEXVQString@@0@Z 1000c378 f   moc_device_type_edit.obj
 0001:0000b438       ?qt_cast@device_type_edit@@UAEPAXPBD@Z 1000c438 f   moc_device_type_edit.obj
 0001:0000b466       ?qt_emit@device_type_edit@@UAE_NHPAUQUObject@@@Z 1000c466 f   moc_device_type_edit.obj
 0001:0000b4ca       ?qt_invoke@device_type_edit@@UAE_NHPAUQUObject@@@Z 1000c4ca f   moc_device_type_edit.obj
 0001:0000b51c       ?staticMetaObject@device_type_edit@@SAPAVQMetaObject@@XZ 1000c51c f   moc_device_type_edit.obj
 0001:0000b5f8       ?className@device_type_editDlgBase@@UBEPBDXZ 1000c5f8 f   moc_device_type_editdlg.obj
 0001:0000b5fe       ?qt_cast@device_type_editDlgBase@@UAEPAXPBD@Z 1000c5fe f   moc_device_type_editdlg.obj
 0001:0000b62c       ?qt_invoke@device_type_editDlgBase@@UAE_NHPAUQUObject@@@Z 1000c62c f   moc_device_type_editdlg.obj
 0001:0000b65e       ?qt_property@device_type_edit@@UAE_NHHPAVQVariant@@@Z 1000c65e f   moc_device_type_edit.obj
 0001:0000b65e       ?qt_property@device_type_editDlgBase@@UAE_NHHPAVQVariant@@@Z 1000c65e f   moc_device_type_editdlg.obj
 0001:0000b65e       ?qt_property@toolWindowBase@@UAE_NHHPAVQVariant@@@Z 1000c65e f   moc_toolwindow.obj
 0001:0000b668       ?staticMetaObject@device_type_editDlgBase@@SAPAVQMetaObject@@XZ 1000c668 f   moc_device_type_editdlg.obj
 0001:0000b6b2       ?tr@device_type_editDlgBase@@SA?AVQString@@PBD0@Z 1000c6b2 f   moc_device_type_editdlg.obj
 0001:0000b6f5       ?className@device_type_editDlg@@UBEPBDXZ 1000c6f5 f   moc_device_type_editdlgimpl.obj
 0001:0000b6fb       ?command@device_type_editDlg@@IAEXVQString@@0@Z 1000c6fb f   moc_device_type_editdlgimpl.obj
 0001:0000b7bb       ?dirty@device_type_editDlg@@IAEXXZ 1000c7bb f   moc_device_type_editdlgimpl.obj
 0001:0000b7d2       ?qt_cast@device_type_editDlg@@UAEPAXPBD@Z 1000c7d2 f   moc_device_type_editdlgimpl.obj
 0001:0000b7ff       ?qt_emit@device_type_editDlg@@UAE_NHPAUQUObject@@@Z 1000c7ff f   moc_device_type_editdlgimpl.obj
 0001:0000b86d       ?qt_invoke@device_type_editDlg@@UAE_NHPAUQUObject@@@Z 1000c86d f   moc_device_type_editdlgimpl.obj
 0001:0000b9c9       ?qt_property@toolWindow@@UAE_NHHPAVQVariant@@@Z 1000c9c9 f   moc_toolwindowimpl.obj
 0001:0000b9c9       ?qt_property@device_type_editDlg@@UAE_NHHPAVQVariant@@@Z 1000c9c9 f   moc_device_type_editdlgimpl.obj
 0001:0000b9d2       ?staticMetaObject@device_type_editDlg@@SAPAVQMetaObject@@XZ 1000c9d2 f   moc_device_type_editdlgimpl.obj
 0001:0000bbb3       ?className@toolWindowBase@@UBEPBDXZ 1000cbb3 f   moc_toolwindow.obj
 0001:0000bbb9       ?qt_cast@toolWindowBase@@UAEPAXPBD@Z 1000cbb9 f   moc_toolwindow.obj
 0001:0000bbe7       ?qt_emit@device_type_editDlgBase@@UAE_NHPAUQUObject@@@Z 1000cbe7 f   moc_device_type_editdlg.obj
 0001:0000bbe7       ?qt_emit@toolWindowBase@@UAE_NHPAUQUObject@@@Z 1000cbe7 f   moc_toolwindow.obj
 0001:0000bbf1       ?qt_invoke@toolWindowBase@@UAE_NHPAUQUObject@@@Z 1000cbf1 f   moc_toolwindow.obj
 0001:0000bc23       ?staticMetaObject@toolWindowBase@@SAPAVQMetaObject@@XZ 1000cc23 f   moc_toolwindow.obj
 0001:0000bc6d       ?tr@toolWindowBase@@SA?AVQString@@PBD0@Z 1000cc6d f   moc_toolwindow.obj
 0001:0000bcb0       ?className@toolWindow@@UBEPBDXZ 1000ccb0 f   moc_toolwindowimpl.obj
 0001:0000bcb6       ?dirty@toolWindow@@IAEXXZ  1000ccb6 f   moc_toolwindowimpl.obj
 0001:0000bccf       ?qt_cast@toolWindow@@UAEPAXPBD@Z 1000cccf f   moc_toolwindowimpl.obj
 0001:0000bcfc       ?qt_emit@toolWindow@@UAE_NHPAUQUObject@@@Z 1000ccfc f   moc_toolwindowimpl.obj
 0001:0000bd4d       ?qt_invoke@toolWindow@@UAE_NHPAUQUObject@@@Z 1000cd4d f   moc_toolwindowimpl.obj
 0001:0000bd98       ?staticMetaObject@toolWindow@@SAPAVQMetaObject@@XZ 1000cd98 f   moc_toolwindowimpl.obj
 0001:0000be65       ?typeDeleted@toolWindow@@IAEXABVQString@@@Z 1000ce65 f   moc_toolwindowimpl.obj
 0001:0000bea4       ?typeSelected@toolWindow@@IAEXABVQString@@@Z 1000cea4 f   moc_toolwindowimpl.obj
 0001:0000bee1       ??0toolWindowBase@@QAE@PAVQWidget@@PBDI@Z 1000cee1 f   toolwindow.obj
 0001:0000c28c       ??1toolWindowBase@@UAE@XZ  1000d28c f   toolwindow.obj
 0001:0000c29f       ??_EQTabWidget@@WCI@AEPAXI@Z 1000d29f f i toolwindow.obj
 0001:0000c2a7       ??_EtoolWindowBase@@WCI@AEPAXI@Z 1000d2a7 f i toolwindow.obj
 0001:0000c2af       ??_GQTabWidget@@UAEPAXI@Z  1000d2af f i toolwindow.obj
 0001:0000c2af       ??_EQTabWidget@@UAEPAXI@Z  1000d2af f i toolwindow.obj
 0001:0000c2cf       ??_GtoolWindowBase@@UAEPAXI@Z 1000d2cf f i toolwindow.obj
 0001:0000c2cf       ??_EtoolWindowBase@@UAEPAXI@Z 1000d2cf f i toolwindow.obj
 0001:0000c2ee       ?languageChange@toolWindowBase@@MAEXXZ 1000d2ee f   toolwindow.obj
 0001:0000c44b       ?metaObject@toolWindowBase@@UBEPAVQMetaObject@@XZ 1000d44b f i toolwindow.obj
 0001:0000c450       ?setName@QWidget@@UAEXPBD@Z 1000d450 f   qt-mt323:qt-mt323.dll
 0001:0000c456       ?closeEvent@QWidget@@MAEXPAVQCloseEvent@@@Z 1000d456 f   qt-mt323:qt-mt323.dll
 0001:0000c45c       ?activateItemAt@QPopupMenu@@UAEXH@Z 1000d45c f   qt-mt323:qt-mt323.dll
 0001:0000c462       ?addTo@QAction@@UAE_NPAVQWidget@@@Z 1000d462 f   qt-mt323:qt-mt323.dll
 0001:0000c468       ?addedTo@QAction@@MAEXHPAVQPopupMenu@@@Z 1000d468 f   qt-mt323:qt-mt323.dll
 0001:0000c46e       ?addedTo@QAction@@MAEXPAVQWidget@@0@Z 1000d46e f   qt-mt323:qt-mt323.dll
 0001:0000c474       ?adjustSize@QWidget@@UAEXXZ 1000d474 f   qt-mt323:qt-mt323.dll
 0001:0000c47a       ?checkConnectArgs@QObject@@MAE_NPBDPBV1@0@Z 1000d47a f   qt-mt323:qt-mt323.dll
 0001:0000c480       ?childEvent@QObject@@MAEXPAVQChildEvent@@@Z 1000d480 f   qt-mt323:qt-mt323.dll
 0001:0000c486       ?className@QAction@@UBEPBDXZ 1000d486 f   qt-mt323:qt-mt323.dll
 0001:0000c48c       ?className@QDockWindow@@UBEPBDXZ 1000d48c f   qt-mt323:qt-mt323.dll
 0001:0000c492       ?className@QGuardedPtrPrivate@@UBEPBDXZ 1000d492 f   qt-mt323:qt-mt323.dll
 0001:0000c498       ?className@QPopupMenu@@UBEPBDXZ 1000d498 f   qt-mt323:qt-mt323.dll
 0001:0000c49e       ?className@QToolBar@@UBEPBDXZ 1000d49e f   qt-mt323:qt-mt323.dll
 0001:0000c4a4       ?className@QWidget@@UBEPBDXZ 1000d4a4 f   qt-mt323:qt-mt323.dll
 0001:0000c4aa       ?clear@?$QPtrList@VQDockWindow@@@@UAEXXZ 1000d4aa f   qt-mt323:qt-mt323.dll
 0001:0000c4b0       ?clear@QToolBar@@UAEXXZ    1000d4b0 f   qt-mt323:qt-mt323.dll
 0001:0000c4b6       ?close@QWidget@@UAE_N_N@Z  1000d4b6 f   qt-mt323:qt-mt323.dll
 0001:0000c4bc       ?closeEvent@QPopupMenu@@MAEXPAVQCloseEvent@@@Z 1000d4bc f   qt-mt323:qt-mt323.dll
 0001:0000c4c2       ?cmd@QPaintDevice@@MAE_NHPAVQPainter@@PATQPDevCmdParam@@@Z 1000d4c2 f   qt-mt323:qt-mt323.dll
 0001:0000c4c8       ?compareItems@QGList@@MAEHPAX0@Z 1000d4c8 f   qt-mt323:qt-mt323.dll
 0001:0000c4ce       ?connectNotify@QObject@@MAEXPBD@Z 1000d4ce f   qt-mt323:qt-mt323.dll
 0001:0000c4d4       ?contextMenuEvent@QDockWindow@@MAEXPAVQContextMenuEvent@@@Z 1000d4d4 f   qt-mt323:qt-mt323.dll
 0001:0000c4da       ?contextMenuEvent@QWidget@@MAEXPAVQContextMenuEvent@@@Z 1000d4da f   qt-mt323:qt-mt323.dll
 0001:0000c4e0       ?count@?$QPtrList@VQDockWindow@@@@UBEIXZ 1000d4e0 f   qt-mt323:qt-mt323.dll
 0001:0000c4e6       ?create@QWidget@@MAEXPAUHWND__@@_N1@Z 1000d4e6 f   qt-mt323:qt-mt323.dll
 0001:0000c4ec       ?customEvent@QObject@@MAEXPAVQCustomEvent@@@Z 1000d4ec f   qt-mt323:qt-mt323.dll
 0001:0000c4f2       ?customWhatsThis@QPopupMenu@@UBE_NXZ 1000d4f2 f   qt-mt323:qt-mt323.dll
 0001:0000c4f8       ?customWhatsThis@QWidget@@UBE_NXZ 1000d4f8 f   qt-mt323:qt-mt323.dll
 0001:0000c4fe       ?deleteItem@?$QPtrList@VQDockWindow@@@@EAEXPAX@Z 1000d4fe f   qt-mt323:qt-mt323.dll
 0001:0000c504       ?destroy@QWidget@@MAEX_N0@Z 1000d504 f   qt-mt323:qt-mt323.dll
 0001:0000c50a       ?disconnectNotify@QObject@@MAEXPBD@Z 1000d50a f   qt-mt323:qt-mt323.dll
 0001:0000c510       ?dock@QDockWindow@@UAEXXZ  1000d510 f   qt-mt323:qt-mt323.dll
 0001:0000c516       ?dragEnterEvent@QWidget@@MAEXPAVQDragEnterEvent@@@Z 1000d516 f   qt-mt323:qt-mt323.dll
 0001:0000c51c       ?dragLeaveEvent@QWidget@@MAEXPAVQDragLeaveEvent@@@Z 1000d51c f   qt-mt323:qt-mt323.dll
 0001:0000c522       ?dragMoveEvent@QWidget@@MAEXPAVQDragMoveEvent@@@Z 1000d522 f   qt-mt323:qt-mt323.dll
 0001:0000c528       ?drawContents@QDockWindow@@MAEXPAVQPainter@@@Z 1000d528 f   qt-mt323:qt-mt323.dll
 0001:0000c52e       ?drawContents@QPopupMenu@@MAEXPAVQPainter@@@Z 1000d52e f   qt-mt323:qt-mt323.dll
 0001:0000c534       ?drawFrame@QDockWindow@@MAEXPAVQPainter@@@Z 1000d534 f   qt-mt323:qt-mt323.dll
 0001:0000c53a       ?drawFrame@QFrame@@MAEXPAVQPainter@@@Z 1000d53a f   qt-mt323:qt-mt323.dll
 0001:0000c540       ?dropEvent@QWidget@@MAEXPAVQDropEvent@@@Z 1000d540 f   qt-mt323:qt-mt323.dll
 0001:0000c546       ?enabledChange@QPopupMenu@@MAEX_N@Z 1000d546 f   qt-mt323:qt-mt323.dll
 0001:0000c54c       ?enabledChange@QWidget@@MAEX_N@Z 1000d54c f   qt-mt323:qt-mt323.dll
 0001:0000c552       ?enterEvent@QWidget@@MAEXPAVQEvent@@@Z 1000d552 f   qt-mt323:qt-mt323.dll
 0001:0000c558       ?event@QDockWindow@@MAE_NPAVQEvent@@@Z 1000d558 f   qt-mt323:qt-mt323.dll
 0001:0000c55e       ?event@QObject@@UAE_NPAVQEvent@@@Z 1000d55e f   qt-mt323:qt-mt323.dll
 0001:0000c564       ?event@QToolBar@@UAE_NPAVQEvent@@@Z 1000d564 f   qt-mt323:qt-mt323.dll
 0001:0000c56a       ?event@QWidget@@MAE_NPAVQEvent@@@Z 1000d56a f   qt-mt323:qt-mt323.dll
 0001:0000c570       ?eventFilter@QDockWindow@@UAE_NPAVQObject@@PAVQEvent@@@Z 1000d570 f   qt-mt323:qt-mt323.dll
 0001:0000c576       ?eventFilter@QObject@@UAE_NPAV1@PAVQEvent@@@Z 1000d576 f   qt-mt323:qt-mt323.dll
 0001:0000c57c       ?focusInEvent@QPopupMenu@@MAEXPAVQFocusEvent@@@Z 1000d57c f   qt-mt323:qt-mt323.dll
 0001:0000c582       ?focusInEvent@QWidget@@MAEXPAVQFocusEvent@@@Z 1000d582 f   qt-mt323:qt-mt323.dll
 0001:0000c588       ?focusNextPrevChild@QPopupMenu@@MAE_N_N@Z 1000d588 f   qt-mt323:qt-mt323.dll
 0001:0000c58e       ?focusNextPrevChild@QWidget@@MAE_N_N@Z 1000d58e f   qt-mt323:qt-mt323.dll
 0001:0000c594       ?focusOutEvent@QPopupMenu@@MAEXPAVQFocusEvent@@@Z 1000d594 f   qt-mt323:qt-mt323.dll
 0001:0000c59a       ?focusOutEvent@QWidget@@MAEXPAVQFocusEvent@@@Z 1000d59a f   qt-mt323:qt-mt323.dll
 0001:0000c5a0       ?fontChange@QWidget@@MAEXABVQFont@@@Z 1000d5a0 f   qt-mt323:qt-mt323.dll
 0001:0000c5a6       ?fontInf@QPaintDevice@@MBEHPAVQFont@@H@Z 1000d5a6 f   qt-mt323:qt-mt323.dll
 0001:0000c5ac       ?fontMet@QPaintDevice@@MBEHPAVQFont@@HPBDH@Z 1000d5ac f   qt-mt323:qt-mt323.dll
 0001:0000c5b2       ?frameChanged@QFrame@@MAEXXZ 1000d5b2 f   qt-mt323:qt-mt323.dll
 0001:0000c5b8       ?frameChanged@QPopupMenu@@EAEXXZ 1000d5b8 f   qt-mt323:qt-mt323.dll
 0001:0000c5be       ?handle@QPaintDevice@@UBEPAUHDC__@@XZ 1000d5be f   qt-mt323:qt-mt323.dll
 0001:0000c5c4       ?heightForWidth@QWidget@@UBEHH@Z 1000d5c4 f   qt-mt323:qt-mt323.dll
 0001:0000c5ca       ?hide@QPopupMenu@@UAEXXZ   1000d5ca f   qt-mt323:qt-mt323.dll
 0001:0000c5d0       ?hide@QToolBar@@UAEXXZ     1000d5d0 f   qt-mt323:qt-mt323.dll
 0001:0000c5d6       ?hide@QWidget@@UAEXXZ      1000d5d6 f   qt-mt323:qt-mt323.dll
 0001:0000c5dc       ?hideEvent@QDockWindow@@MAEXPAVQHideEvent@@@Z 1000d5dc f   qt-mt323:qt-mt323.dll
 0001:0000c5e2       ?hideEvent@QWidget@@MAEXPAVQHideEvent@@@Z 1000d5e2 f   qt-mt323:qt-mt323.dll
 0001:0000c5e8       ?imComposeEvent@QWidget@@MAEXPAVQIMEvent@@@Z 1000d5e8 f   qt-mt323:qt-mt323.dll
 0001:0000c5ee       ?imEndEvent@QWidget@@MAEXPAVQIMEvent@@@Z 1000d5ee f   qt-mt323:qt-mt323.dll
 0001:0000c5f4       ?imStartEvent@QWidget@@MAEXPAVQIMEvent@@@Z 1000d5f4 f   qt-mt323:qt-mt323.dll
 0001:0000c5fa       ?insertChild@QObject@@UAEXPAV1@@Z 1000d5fa f   qt-mt323:qt-mt323.dll
 0001:0000c600       ?keyPressEvent@QPopupMenu@@MAEXPAVQKeyEvent@@@Z 1000d600 f   qt-mt323:qt-mt323.dll
 0001:0000c606       ?keyPressEvent@QWidget@@MAEXPAVQKeyEvent@@@Z 1000d606 f   qt-mt323:qt-mt323.dll
 0001:0000c60c       ?keyReleaseEvent@QWidget@@MAEXPAVQKeyEvent@@@Z 1000d60c f   qt-mt323:qt-mt323.dll
 0001:0000c612       ?leaveEvent@QPopupMenu@@MAEXPAVQEvent@@@Z 1000d612 f   qt-mt323:qt-mt323.dll
 0001:0000c618       ?leaveEvent@QWidget@@MAEXPAVQEvent@@@Z 1000d618 f   qt-mt323:qt-mt323.dll
 0001:0000c61e       ?menuContentsChanged@QPopupMenu@@EAEXXZ 1000d61e f   qt-mt323:qt-mt323.dll
 0001:0000c624       ?menuDelPopup@QPopupMenu@@EAEXPAV1@@Z 1000d624 f   qt-mt323:qt-mt323.dll
 0001:0000c62a       ?menuInsPopup@QPopupMenu@@EAEXPAV1@@Z 1000d62a f   qt-mt323:qt-mt323.dll
 0001:0000c630       ?menuStateChanged@QPopupMenu@@EAEXXZ 1000d630 f   qt-mt323:qt-mt323.dll
 0001:0000c636       ?metaObject@QAction@@UBEPAVQMetaObject@@XZ 1000d636 f   qt-mt323:qt-mt323.dll
 0001:0000c63c       ?metaObject@QDockWindow@@UBEPAVQMetaObject@@XZ 1000d63c f   qt-mt323:qt-mt323.dll
 0001:0000c642       ?metaObject@QGuardedPtrPrivate@@UBEPAVQMetaObject@@XZ 1000d642 f   qt-mt323:qt-mt323.dll
 0001:0000c648       ?metaObject@QPopupMenu@@UBEPAVQMetaObject@@XZ 1000d648 f   qt-mt323:qt-mt323.dll
 0001:0000c64e       ?metaObject@QToolBar@@UBEPAVQMetaObject@@XZ 1000d64e f   qt-mt323:qt-mt323.dll
 0001:0000c654       ?metaObject@QWidget@@UBEPAVQMetaObject@@XZ 1000d654 f   qt-mt323:qt-mt323.dll
 0001:0000c65a       ?metric@QWidget@@MBEHH@Z   1000d65a f   qt-mt323:qt-mt323.dll
 0001:0000c660       ?minimumSizeHint@QDockWindow@@UBE?AVQSize@@XZ 1000d660 f   qt-mt323:qt-mt323.dll
 0001:0000c666       ?minimumSizeHint@QToolBar@@UBE?AVQSize@@XZ 1000d666 f   qt-mt323:qt-mt323.dll
 0001:0000c66c       ?minimumSizeHint@QWidget@@UBE?AVQSize@@XZ 1000d66c f   qt-mt323:qt-mt323.dll
 0001:0000c672       ?mouseDoubleClickEvent@QWidget@@MAEXPAVQMouseEvent@@@Z 1000d672 f   qt-mt323:qt-mt323.dll
 0001:0000c678       ?mouseMoveEvent@QPopupMenu@@MAEXPAVQMouseEvent@@@Z 1000d678 f   qt-mt323:qt-mt323.dll
 0001:0000c67e       ?mouseMoveEvent@QWidget@@MAEXPAVQMouseEvent@@@Z 1000d67e f   qt-mt323:qt-mt323.dll
 0001:0000c684       ?mousePressEvent@QPopupMenu@@MAEXPAVQMouseEvent@@@Z 1000d684 f   qt-mt323:qt-mt323.dll
 0001:0000c68a       ?mousePressEvent@QWidget@@MAEXPAVQMouseEvent@@@Z 1000d68a f   qt-mt323:qt-mt323.dll
 0001:0000c690       ?mouseReleaseEvent@QPopupMenu@@MAEXPAVQMouseEvent@@@Z 1000d690 f   qt-mt323:qt-mt323.dll
 0001:0000c696       ?mouseReleaseEvent@QWidget@@MAEXPAVQMouseEvent@@@Z 1000d696 f   qt-mt323:qt-mt323.dll
 0001:0000c69c       ?move@QWidget@@UAEXHH@Z    1000d69c f   qt-mt323:qt-mt323.dll
 0001:0000c6a2       ?moveEvent@QWidget@@MAEXPAVQMoveEvent@@@Z 1000d6a2 f   qt-mt323:qt-mt323.dll
 0001:0000c6a8       ?newItem@QPtrCollection@@MAEPAXPAX@Z 1000d6a8 f   qt-mt323:qt-mt323.dll
 0001:0000c6ae       ?paintEvent@QFrame@@MAEXPAVQPaintEvent@@@Z 1000d6ae f   qt-mt323:qt-mt323.dll
 0001:0000c6b4       ?paintEvent@QPopupMenu@@MAEXPAVQPaintEvent@@@Z 1000d6b4 f   qt-mt323:qt-mt323.dll
 0001:0000c6ba       ?paintEvent@QWidget@@MAEXPAVQPaintEvent@@@Z 1000d6ba f   qt-mt323:qt-mt323.dll
 0001:0000c6c0       ?paletteChange@QWidget@@MAEXABVQPalette@@@Z 1000d6c0 f   qt-mt323:qt-mt323.dll
 0001:0000c6c6       ?polish@QWidget@@UAEXXZ    1000d6c6 f   qt-mt323:qt-mt323.dll
 0001:0000c6cc       ?property@QObject@@UBE?AVQVariant@@PBD@Z 1000d6cc f   qt-mt323:qt-mt323.dll
 0001:0000c6d2       ?qt_cast@QAction@@UAEPAXPBD@Z 1000d6d2 f   qt-mt323:qt-mt323.dll
 0001:0000c6d8       ?qt_cast@QDockWindow@@UAEPAXPBD@Z 1000d6d8 f   qt-mt323:qt-mt323.dll
 0001:0000c6de       ?qt_cast@QGuardedPtrPrivate@@UAEPAXPBD@Z 1000d6de f   qt-mt323:qt-mt323.dll
 0001:0000c6e4       ?qt_cast@QPopupMenu@@UAEPAXPBD@Z 1000d6e4 f   qt-mt323:qt-mt323.dll
 0001:0000c6ea       ?qt_cast@QToolBar@@UAEPAXPBD@Z 1000d6ea f   qt-mt323:qt-mt323.dll
 0001:0000c6f0       ?qt_cast@QWidget@@UAEPAXPBD@Z 1000d6f0 f   qt-mt323:qt-mt323.dll
 0001:0000c6f6       ?qt_emit@QAction@@UAE_NHPAUQUObject@@@Z 1000d6f6 f   qt-mt323:qt-mt323.dll
 0001:0000c6fc       ?qt_emit@QDockWindow@@UAE_NHPAUQUObject@@@Z 1000d6fc f   qt-mt323:qt-mt323.dll
 0001:0000c702       ?qt_emit@QGuardedPtrPrivate@@UAE_NHPAUQUObject@@@Z 1000d702 f   qt-mt323:qt-mt323.dll
 0001:0000c708       ?qt_emit@QPopupMenu@@UAE_NHPAUQUObject@@@Z 1000d708 f   qt-mt323:qt-mt323.dll
 0001:0000c70e       ?qt_emit@QToolBar@@UAE_NHPAUQUObject@@@Z 1000d70e f   qt-mt323:qt-mt323.dll
 0001:0000c714       ?qt_emit@QWidget@@UAE_NHPAUQUObject@@@Z 1000d714 f   qt-mt323:qt-mt323.dll
 0001:0000c71a       ?qt_invoke@QAction@@UAE_NHPAUQUObject@@@Z 1000d71a f   qt-mt323:qt-mt323.dll
 0001:0000c720       ?qt_invoke@QDockWindow@@UAE_NHPAUQUObject@@@Z 1000d720 f   qt-mt323:qt-mt323.dll
 0001:0000c726       ?qt_invoke@QGuardedPtrPrivate@@UAE_NHPAUQUObject@@@Z 1000d726 f   qt-mt323:qt-mt323.dll
 0001:0000c72c       ?qt_invoke@QPopupMenu@@UAE_NHPAUQUObject@@@Z 1000d72c f   qt-mt323:qt-mt323.dll
 0001:0000c732       ?qt_invoke@QToolBar@@UAE_NHPAUQUObject@@@Z 1000d732 f   qt-mt323:qt-mt323.dll
 0001:0000c738       ?qt_invoke@QWidget@@UAE_NHPAUQUObject@@@Z 1000d738 f   qt-mt323:qt-mt323.dll
 0001:0000c73e       ?qt_property@QAction@@UAE_NHHPAVQVariant@@@Z 1000d73e f   qt-mt323:qt-mt323.dll
 0001:0000c744       ?qt_property@QDockWindow@@UAE_NHHPAVQVariant@@@Z 1000d744 f   qt-mt323:qt-mt323.dll
 0001:0000c74a       ?qt_property@QGuardedPtrPrivate@@UAE_NHHPAVQVariant@@@Z 1000d74a f   qt-mt323:qt-mt323.dll
 0001:0000c750       ?qt_property@QPopupMenu@@UAE_NHHPAVQVariant@@@Z 1000d750 f   qt-mt323:qt-mt323.dll
 0001:0000c756       ?qt_property@QToolBar@@UAE_NHHPAVQVariant@@@Z 1000d756 f   qt-mt323:qt-mt323.dll
 0001:0000c75c       ?qt_property@QWidget@@UAE_NHHPAVQVariant@@@Z 1000d75c f   qt-mt323:qt-mt323.dll
 0001:0000c762       ?read@QGDict@@MAEAAVQDataStream@@AAV2@AAPAX@Z 1000d762 f   qt-mt323:qt-mt323.dll
 0001:0000c768       ?read@QGList@@MAEAAVQDataStream@@AAV2@AAPAX@Z 1000d768 f   qt-mt323:qt-mt323.dll
 0001:0000c76e       ?removeChild@QObject@@UAEXPAV1@@Z 1000d76e f   qt-mt323:qt-mt323.dll
 0001:0000c774       ?removeFrom@QAction@@UAE_NPAVQWidget@@@Z 1000d774 f   qt-mt323:qt-mt323.dll
 0001:0000c77a       ?reparent@QWidget@@UAEXPAV1@IABVQPoint@@_N@Z 1000d77a f   qt-mt323:qt-mt323.dll
 0001:0000c780       ?resize@QWidget@@UAEXHH@Z  1000d780 f   qt-mt323:qt-mt323.dll
 0001:0000c786       ?resizeEvent@QDockWindow@@MAEXPAVQResizeEvent@@@Z 1000d786 f   qt-mt323:qt-mt323.dll
 0001:0000c78c       ?resizeEvent@QFrame@@MAEXPAVQResizeEvent@@@Z 1000d78c f   qt-mt323:qt-mt323.dll
 0001:0000c792       ?resizeEvent@QToolBar@@MAEXPAVQResizeEvent@@@Z 1000d792 f   qt-mt323:qt-mt323.dll
 0001:0000c798       ?resizeEvent@QWidget@@MAEXPAVQResizeEvent@@@Z 1000d798 f   qt-mt323:qt-mt323.dll
 0001:0000c79e       ?resolution@QPaintDevice@@UBEHXZ 1000d79e f   qt-mt323:qt-mt323.dll
 0001:0000c7a4       ?setAccel@QAction@@UAEXABVQKeySequence@@@Z 1000d7a4 f   qt-mt323:qt-mt323.dll
 0001:0000c7aa       ?setAcceptDrops@QWidget@@UAEX_N@Z 1000d7aa f   qt-mt323:qt-mt323.dll
 0001:0000c7b0       ?setActiveItem@QPopupMenu@@UAEXH@Z 1000d7b0 f   qt-mt323:qt-mt323.dll
 0001:0000c7b6       ?setActiveWindow@QWidget@@UAEXXZ 1000d7b6 f   qt-mt323:qt-mt323.dll
 0001:0000c7bc       ?setAutoMask@QWidget@@UAEX_N@Z 1000d7bc f   qt-mt323:qt-mt323.dll
 0001:0000c7c2       ?setBackgroundColor@QWidget@@UAEXABVQColor@@@Z 1000d7c2 f   qt-mt323:qt-mt323.dll
 0001:0000c7c8       ?setBackgroundMode@QWidget@@UAEXW4BackgroundMode@Qt@@@Z 1000d7c8 f   qt-mt323:qt-mt323.dll
 0001:0000c7ce       ?setBackgroundOrigin@QWidget@@UAEXW4BackgroundOrigin@1@@Z 1000d7ce f   qt-mt323:qt-mt323.dll
 0001:0000c7d4       ?setBackgroundPixmap@QWidget@@UAEXABVQPixmap@@@Z 1000d7d4 f   qt-mt323:qt-mt323.dll
 0001:0000c7da       ?setCaption@QDockWindow@@UAEXABVQString@@@Z 1000d7da f   qt-mt323:qt-mt323.dll
 0001:0000c7e0       ?setCaption@QWidget@@UAEXABVQString@@@Z 1000d7e0 f   qt-mt323:qt-mt323.dll
 0001:0000c7e6       ?setCheckable@QPopupMenu@@UAEX_N@Z 1000d7e6 f   qt-mt323:qt-mt323.dll
 0001:0000c7ec       ?setCloseMode@QDockWindow@@UAEXH@Z 1000d7ec f   qt-mt323:qt-mt323.dll
 0001:0000c7f2       ?setCursor@QWidget@@UAEXABVQCursor@@@Z 1000d7f2 f   qt-mt323:qt-mt323.dll
 0001:0000c7f8       ?setEnabled@QAction@@UAEX_N@Z 1000d7f8 f   qt-mt323:qt-mt323.dll
 0001:0000c7fe       ?setEnabled@QWidget@@UAEX_N@Z 1000d7fe f   qt-mt323:qt-mt323.dll
 0001:0000c804       ?setEraseColor@QWidget@@UAEXABVQColor@@@Z 1000d804 f   qt-mt323:qt-mt323.dll
 0001:0000c80a       ?setErasePixmap@QWidget@@UAEXABVQPixmap@@@Z 1000d80a f   qt-mt323:qt-mt323.dll
 0001:0000c810       ?setFirstItemActive@QPopupMenu@@EAEXXZ 1000d810 f   qt-mt323:qt-mt323.dll
 0001:0000c816       ?setFixedExtentHeight@QDockWindow@@UAEXH@Z 1000d816 f   qt-mt323:qt-mt323.dll
 0001:0000c81c       ?setFixedExtentWidth@QDockWindow@@UAEXH@Z 1000d81c f   qt-mt323:qt-mt323.dll
 0001:0000c822       ?setFocus@QWidget@@UAEXXZ  1000d822 f   qt-mt323:qt-mt323.dll
 0001:0000c828       ?setFocusPolicy@QWidget@@UAEXW4FocusPolicy@1@@Z 1000d828 f   qt-mt323:qt-mt323.dll
 0001:0000c82e       ?setFocusProxy@QWidget@@UAEXPAV1@@Z 1000d82e f   qt-mt323:qt-mt323.dll
 0001:0000c834       ?setFont@QPopupMenu@@UAEXABVQFont@@@Z 1000d834 f   qt-mt323:qt-mt323.dll
 0001:0000c83a       ?setFont@QWidget@@UAEXABVQFont@@@Z 1000d83a f   qt-mt323:qt-mt323.dll
 0001:0000c840       ?setFrameRect@QFrame@@UAEXABVQRect@@@Z 1000d840 f   qt-mt323:qt-mt323.dll
 0001:0000c846       ?setFrameStyle@QFrame@@UAEXH@Z 1000d846 f   qt-mt323:qt-mt323.dll
 0001:0000c84c       ?setGeometry@QWidget@@UAEXABVQRect@@@Z 1000d84c f   qt-mt323:qt-mt323.dll
 0001:0000c852       ?setGeometry@QWidget@@UAEXHHHH@Z 1000d852 f   qt-mt323:qt-mt323.dll
 0001:0000c858       ?setHorizontallyStretchable@QDockWindow@@UAEX_N@Z 1000d858 f   qt-mt323:qt-mt323.dll
 0001:0000c85e       ?setIcon@QWidget@@UAEXABVQPixmap@@@Z 1000d85e f   qt-mt323:qt-mt323.dll
 0001:0000c864       ?setIconSet@QAction@@UAEXABVQIconSet@@@Z 1000d864 f   qt-mt323:qt-mt323.dll
 0001:0000c86a       ?setIconText@QWidget@@UAEXABVQString@@@Z 1000d86a f   qt-mt323:qt-mt323.dll
 0001:0000c870       ?setId@QMenuData@@UAEXHH@Z 1000d870 f   qt-mt323:qt-mt323.dll
 0001:0000c876       ?setKeyCompression@QWidget@@MAEX_N@Z 1000d876 f   qt-mt323:qt-mt323.dll
 0001:0000c87c       ?setLabel@QToolBar@@UAEXABVQString@@@Z 1000d87c f   qt-mt323:qt-mt323.dll
 0001:0000c882       ?setLineWidth@QFrame@@UAEXH@Z 1000d882 f   qt-mt323:qt-mt323.dll
 0001:0000c888       ?setMargin@QFrame@@UAEXH@Z 1000d888 f   qt-mt323:qt-mt323.dll
 0001:0000c88e       ?setMask@QWidget@@UAEXABVQBitmap@@@Z 1000d88e f   qt-mt323:qt-mt323.dll
 0001:0000c894       ?setMask@QWidget@@UAEXABVQRegion@@@Z 1000d894 f   qt-mt323:qt-mt323.dll
 0001:0000c89a       ?setMaximumSize@QWidget@@UAEXHH@Z 1000d89a f   qt-mt323:qt-mt323.dll
 0001:0000c8a0       ?setMenuText@QAction@@UAEXABVQString@@@Z 1000d8a0 f   qt-mt323:qt-mt323.dll
 0001:0000c8a6       ?setMicroFocusHint@QWidget@@MAEXHHHH_NPAVQFont@@@Z 1000d8a6 f   qt-mt323:qt-mt323.dll
 0001:0000c8ac       ?setMidLineWidth@QFrame@@UAEXH@Z 1000d8ac f   qt-mt323:qt-mt323.dll
 0001:0000c8b2       ?setMinimumSize@QToolBar@@UAEXHH@Z 1000d8b2 f   qt-mt323:qt-mt323.dll
 0001:0000c8b8       ?setMinimumSize@QWidget@@UAEXHH@Z 1000d8b8 f   qt-mt323:qt-mt323.dll
 0001:0000c8be       ?setMouseTracking@QWidget@@UAEX_N@Z 1000d8be f   qt-mt323:qt-mt323.dll
 0001:0000c8c4       ?setMovingEnabled@QDockWindow@@UAEX_N@Z 1000d8c4 f   qt-mt323:qt-mt323.dll
 0001:0000c8ca       ?setName@QObject@@UAEXPBD@Z 1000d8ca f   qt-mt323:qt-mt323.dll
 0001:0000c8d0       ?setNewLine@QDockWindow@@UAEX_N@Z 1000d8d0 f   qt-mt323:qt-mt323.dll
 0001:0000c8d6       ?setOffset@QDockWindow@@UAEXH@Z 1000d8d6 f   qt-mt323:qt-mt323.dll
 0001:0000c8dc       ?setOn@QAction@@UAEX_N@Z   1000d8dc f   qt-mt323:qt-mt323.dll
 0001:0000c8e2       ?setOpaqueMoving@QDockWindow@@UAEX_N@Z 1000d8e2 f   qt-mt323:qt-mt323.dll
 0001:0000c8e8       ?setOrientation@QDockWindow@@UAEXW4Orientation@Qt@@@Z 1000d8e8 f   qt-mt323:qt-mt323.dll
 0001:0000c8ee       ?setOrientation@QToolBar@@UAEXW4Orientation@Qt@@@Z 1000d8ee f   qt-mt323:qt-mt323.dll
 0001:0000c8f4       ?setPalette@QWidget@@UAEXABVQPalette@@@Z 1000d8f4 f   qt-mt323:qt-mt323.dll
 0001:0000c8fa       ?setPaletteBackgroundColor@QWidget@@UAEXABVQColor@@@Z 1000d8fa f   qt-mt323:qt-mt323.dll
 0001:0000c900       ?setPaletteBackgroundPixmap@QWidget@@UAEXABVQPixmap@@@Z 1000d900 f   qt-mt323:qt-mt323.dll
 0001:0000c906       ?setProperty@QObject@@UAE_NPBDABVQVariant@@@Z 1000d906 f   qt-mt323:qt-mt323.dll
 0001:0000c90c       ?setResizeEnabled@QDockWindow@@UAEX_N@Z 1000d90c f   qt-mt323:qt-mt323.dll
 0001:0000c912       ?setResolution@QPaintDevice@@UAEXH@Z 1000d912 f   qt-mt323:qt-mt323.dll
 0001:0000c918       ?setSizeIncrement@QWidget@@UAEXHH@Z 1000d918 f   qt-mt323:qt-mt323.dll
 0001:0000c91e       ?setSizePolicy@QWidget@@UAEXVQSizePolicy@@@Z 1000d91e f   qt-mt323:qt-mt323.dll
 0001:0000c924       ?setStatusTip@QAction@@UAEXABVQString@@@Z 1000d924 f   qt-mt323:qt-mt323.dll
 0001:0000c92a       ?setStretchableWidget@QToolBar@@UAEXPAVQWidget@@@Z 1000d92a f   qt-mt323:qt-mt323.dll
 0001:0000c930       ?setText@QAction@@UAEXABVQString@@@Z 1000d930 f   qt-mt323:qt-mt323.dll
 0001:0000c936       ?setToggleAction@QAction@@UAEX_N@Z 1000d936 f   qt-mt323:qt-mt323.dll
 0001:0000c93c       ?setToolTip@QAction@@UAEXABVQString@@@Z 1000d93c f   qt-mt323:qt-mt323.dll
 0001:0000c942       ?setUpdatesEnabled@QWidget@@UAEX_N@Z 1000d942 f   qt-mt323:qt-mt323.dll
 0001:0000c948       ?setVerticallyStretchable@QDockWindow@@UAEX_N@Z 1000d948 f   qt-mt323:qt-mt323.dll
 0001:0000c94e       ?setWFlags@QWidget@@MAEXI@Z 1000d94e f   qt-mt323:qt-mt323.dll
 0001:0000c954       ?setWState@QWidget@@MAEXI@Z 1000d954 f   qt-mt323:qt-mt323.dll
 0001:0000c95a       ?setWhatsThis@QAction@@UAEXABVQString@@@Z 1000d95a f   qt-mt323:qt-mt323.dll
 0001:0000c960       ?setWidget@QDockWindow@@UAEXPAVQWidget@@@Z 1000d960 f   qt-mt323:qt-mt323.dll
 0001:0000c966       ?show@QPopupMenu@@UAEXXZ   1000d966 f   qt-mt323:qt-mt323.dll
 0001:0000c96c       ?show@QToolBar@@UAEXXZ     1000d96c f   qt-mt323:qt-mt323.dll
 0001:0000c972       ?show@QWidget@@UAEXXZ      1000d972 f   qt-mt323:qt-mt323.dll
 0001:0000c978       ?showEvent@QDockWindow@@MAEXPAVQShowEvent@@@Z 1000d978 f   qt-mt323:qt-mt323.dll
 0001:0000c97e       ?showEvent@QWidget@@MAEXPAVQShowEvent@@@Z 1000d97e f   qt-mt323:qt-mt323.dll
 0001:0000c984       ?showMaximized@QWidget@@UAEXXZ 1000d984 f   qt-mt323:qt-mt323.dll
 0001:0000c98a       ?showMinimized@QWidget@@UAEXXZ 1000d98a f   qt-mt323:qt-mt323.dll
 0001:0000c990       ?showNormal@QWidget@@UAEXXZ 1000d990 f   qt-mt323:qt-mt323.dll
 0001:0000c996       ?sizeHint@QDockWindow@@UBE?AVQSize@@XZ 1000d996 f   qt-mt323:qt-mt323.dll
 0001:0000c99c       ?sizeHint@QPopupMenu@@UBE?AVQSize@@XZ 1000d99c f   qt-mt323:qt-mt323.dll
 0001:0000c9a2       ?sizeHint@QWidget@@UBE?AVQSize@@XZ 1000d9a2 f   qt-mt323:qt-mt323.dll
 0001:0000c9a8       ?sizePolicy@QWidget@@UBE?AVQSizePolicy@@XZ 1000d9a8 f   qt-mt323:qt-mt323.dll
 0001:0000c9ae       ?styleChange@QFrame@@MAEXAAVQStyle@@@Z 1000d9ae f   qt-mt323:qt-mt323.dll
 0001:0000c9b4       ?styleChange@QPopupMenu@@MAEXAAVQStyle@@@Z 1000d9b4 f   qt-mt323:qt-mt323.dll
 0001:0000c9ba       ?styleChange@QToolBar@@MAEXAAVQStyle@@@Z 1000d9ba f   qt-mt323:qt-mt323.dll
 0001:0000c9c0       ?styleChange@QWidget@@MAEXAAVQStyle@@@Z 1000d9c0 f   qt-mt323:qt-mt323.dll
 0001:0000c9c6       ?tabletEvent@QWidget@@MAEXPAVQTabletEvent@@@Z 1000d9c6 f   qt-mt323:qt-mt323.dll
 0001:0000c9cc       ?timerEvent@QObject@@MAEXPAVQTimerEvent@@@Z 1000d9cc f   qt-mt323:qt-mt323.dll
 0001:0000c9d2       ?timerEvent@QPopupMenu@@MAEXPAVQTimerEvent@@@Z 1000d9d2 f   qt-mt323:qt-mt323.dll
 0001:0000c9d8       ?undock@QDockWindow@@UAEXPAVQWidget@@@Z 1000d9d8 f   qt-mt323:qt-mt323.dll
 0001:0000c9de       ?undock@QDockWindow@@UAEXXZ 1000d9de f   qt-mt323:qt-mt323.dll
 0001:0000c9e4       ?unsetCursor@QWidget@@UAEXXZ 1000d9e4 f   qt-mt323:qt-mt323.dll
 0001:0000c9ea       ?updateItem@QPopupMenu@@UAEXH@Z 1000d9ea f   qt-mt323:qt-mt323.dll
 0001:0000c9f0       ?updateMask@QWidget@@MAEXXZ 1000d9f0 f   qt-mt323:qt-mt323.dll
 0001:0000c9f6       ?wheelEvent@QWidget@@MAEXPAVQWheelEvent@@@Z 1000d9f6 f   qt-mt323:qt-mt323.dll
 0001:0000c9fc       ?winEvent@QWidget@@MAE_NPAUtagMSG@@@Z 1000d9fc f   qt-mt323:qt-mt323.dll
 0001:0000ca02       ?windowActivationChange@QWidget@@MAEX_N@Z 1000da02 f   qt-mt323:qt-mt323.dll
 0001:0000ca08       ?write@QGDict@@MBEAAVQDataStream@@AAV2@PAX@Z 1000da08 f   qt-mt323:qt-mt323.dll
 0001:0000ca0e       ?write@QGList@@MBEAAVQDataStream@@AAV2@PAX@Z 1000da0e f   qt-mt323:qt-mt323.dll
 0001:0000ca14       ?replaceChild@QDomNode@@UAE?AV1@ABV1@0@Z 1000da14 f   qt-mt323:qt-mt323.dll
 0001:0000ca1a       ?removeChild@QDomNode@@UAE?AV1@ABV1@@Z 1000da1a f   qt-mt323:qt-mt323.dll
 0001:0000ca20       ?appendChild@QDomNode@@UAE?AV1@ABV1@@Z 1000da20 f   qt-mt323:qt-mt323.dll
 0001:0000ca26       ?cloneNode@QDomNode@@UBE?AV1@_N@Z 1000da26 f   qt-mt323:qt-mt323.dll
 0001:0000ca2c       ?firstChild@QDomNode@@UBE?AV1@XZ 1000da2c f   qt-mt323:qt-mt323.dll
 0001:0000ca32       ?nextSibling@QDomNode@@UBE?AV1@XZ 1000da32 f   qt-mt323:qt-mt323.dll
 0001:0000ca38       ?acceptDrop@QListViewItem@@UBE_NPBVQMimeSource@@@Z 1000da38 f   qt-mt323:qt-mt323.dll
 0001:0000ca3e       ?activate@QListViewItem@@MAEXXZ 1000da3e f   qt-mt323:qt-mt323.dll
 0001:0000ca44       ?attributes@QDomElement@@UBE?AVQDomNamedNodeMap@@XZ 1000da44 f   qt-mt323:qt-mt323.dll
 0001:0000ca4a       ?attributes@QDomNode@@UBE?AVQDomNamedNodeMap@@XZ 1000da4a f   qt-mt323:qt-mt323.dll
 0001:0000ca50       ?cancelRename@QListViewItem@@MAEXH@Z 1000da50 f   qt-mt323:qt-mt323.dll
 0001:0000ca56       ?childNodes@QDomNode@@UBE?AVQDomNodeList@@XZ 1000da56 f   qt-mt323:qt-mt323.dll
 0001:0000ca5c       ?compare@QListViewItem@@UBEHPAV1@H_N@Z 1000da5c f   qt-mt323:qt-mt323.dll
 0001:0000ca62       ?dragEntered@QListViewItem@@MAEXXZ 1000da62 f   qt-mt323:qt-mt323.dll
 0001:0000ca68       ?dragLeft@QListViewItem@@MAEXXZ 1000da68 f   qt-mt323:qt-mt323.dll
 0001:0000ca6e       ?dropped@QListViewItem@@MAEXPAVQDropEvent@@@Z 1000da6e f   qt-mt323:qt-mt323.dll
 0001:0000ca74       ?elementsByTagName@QDomElement@@UBE?AVQDomNodeList@@ABVQString@@@Z 1000da74 f   qt-mt323:qt-mt323.dll
 0001:0000ca7a       ?elementsByTagNameNS@QDomElement@@UBE?AVQDomNodeList@@ABVQString@@0@Z 1000da7a f   qt-mt323:qt-mt323.dll
 0001:0000ca80       ?enforceSortOrder@QListViewItem@@MBEXXZ 1000da80 f   qt-mt323:qt-mt323.dll
 0001:0000ca86       ?hasAttributes@QDomNode@@UBE_NXZ 1000da86 f   qt-mt323:qt-mt323.dll
 0001:0000ca8c       ?hasChildNodes@QDomNode@@UBE_NXZ 1000da8c f   qt-mt323:qt-mt323.dll
 0001:0000ca92       ?insertAfter@QDomNode@@UAE?AV1@ABV1@0@Z 1000da92 f   qt-mt323:qt-mt323.dll
 0001:0000ca98       ?insertBefore@QDomNode@@UAE?AV1@ABV1@0@Z 1000da98 f   qt-mt323:qt-mt323.dll
 0001:0000ca9e       ?insertItem@QListViewItem@@UAEXPAV1@@Z 1000da9e f   qt-mt323:qt-mt323.dll
 0001:0000caa4       ?invalidateHeight@QListViewItem@@UAEXXZ 1000daa4 f   qt-mt323:qt-mt323.dll
 0001:0000caaa       ?isAttr@QDomNode@@UBE_NXZ  1000daaa f   qt-mt323:qt-mt323.dll
 0001:0000cab0       ?isCDATASection@QDomNode@@UBE_NXZ 1000dab0 f   qt-mt323:qt-mt323.dll
 0001:0000cab6       ?isCharacterData@QDomNode@@UBE_NXZ 1000dab6 f   qt-mt323:qt-mt323.dll
 0001:0000cabc       ?isComment@QDomNode@@UBE_NXZ 1000dabc f   qt-mt323:qt-mt323.dll
 0001:0000cac2       ?isDocument@QDomDocument@@UBE_NXZ 1000dac2 f   qt-mt323:qt-mt323.dll
 0001:0000cac8       ?isDocument@QDomNode@@UBE_NXZ 1000dac8 f   qt-mt323:qt-mt323.dll
 0001:0000cace       ?isDocumentFragment@QDomNode@@UBE_NXZ 1000dace f   qt-mt323:qt-mt323.dll
 0001:0000cad4       ?isDocumentType@QDomNode@@UBE_NXZ 1000dad4 f   qt-mt323:qt-mt323.dll
 0001:0000cada       ?isElement@QDomElement@@UBE_NXZ 1000dada f   qt-mt323:qt-mt323.dll
 0001:0000cae0       ?isElement@QDomNode@@UBE_NXZ 1000dae0 f   qt-mt323:qt-mt323.dll
 0001:0000cae6       ?isEntity@QDomNode@@UBE_NXZ 1000dae6 f   qt-mt323:qt-mt323.dll
 0001:0000caec       ?isEntityReference@QDomNode@@UBE_NXZ 1000daec f   qt-mt323:qt-mt323.dll
 0001:0000caf2       ?isNotation@QDomNode@@UBE_NXZ 1000daf2 f   qt-mt323:qt-mt323.dll
 0001:0000caf8       ?isProcessingInstruction@QDomNode@@UBE_NXZ 1000daf8 f   qt-mt323:qt-mt323.dll
 0001:0000cafe       ?isSupported@QDomNode@@UBE_NABVQString@@0@Z 1000dafe f   qt-mt323:qt-mt323.dll
 0001:0000cb04       ?isText@QDomNode@@UBE_NXZ  1000db04 f   qt-mt323:qt-mt323.dll
 0001:0000cb0a       ?key@QListViewItem@@UBE?AVQString@@H_N@Z 1000db0a f   qt-mt323:qt-mt323.dll
 0001:0000cb10       ?lastChild@QDomNode@@UBE?AV1@XZ 1000db10 f   qt-mt323:qt-mt323.dll
 0001:0000cb16       ?localName@QDomNode@@UBE?AVQString@@XZ 1000db16 f   qt-mt323:qt-mt323.dll
 0001:0000cb1c       ?namespaceURI@QDomNode@@UBE?AVQString@@XZ 1000db1c f   qt-mt323:qt-mt323.dll
 0001:0000cb22       ?nodeName@QDomNode@@UBE?AVQString@@XZ 1000db22 f   qt-mt323:qt-mt323.dll
 0001:0000cb28       ?nodeType@QDomDocument@@UBE?AW4NodeType@QDomNode@@XZ 1000db28 f   qt-mt323:qt-mt323.dll
 0001:0000cb2e       ?nodeType@QDomElement@@UBE?AW4NodeType@QDomNode@@XZ 1000db2e f   qt-mt323:qt-mt323.dll
 0001:0000cb34       ?nodeValue@QDomNode@@UBE?AVQString@@XZ 1000db34 f   qt-mt323:qt-mt323.dll
 0001:0000cb3a       ?normalize@QDomNode@@UAEXXZ 1000db3a f   qt-mt323:qt-mt323.dll
 0001:0000cb40       ?okRename@QListViewItem@@MAEXH@Z 1000db40 f   qt-mt323:qt-mt323.dll
 0001:0000cb46       ?ownerDocument@QDomNode@@UBE?AVQDomDocument@@XZ 1000db46 f   qt-mt323:qt-mt323.dll
 0001:0000cb4c       ?paintBranches@QListViewItem@@UAEXPAVQPainter@@ABVQColorGroup@@HHH@Z 1000db4c f   qt-mt323:qt-mt323.dll
 0001:0000cb52       ?paintCell@QListViewItem@@UAEXPAVQPainter@@ABVQColorGroup@@HHH@Z 1000db52 f   qt-mt323:qt-mt323.dll
 0001:0000cb58       ?paintFocus@QListViewItem@@UAEXPAVQPainter@@ABVQColorGroup@@ABVQRect@@@Z 1000db58 f   qt-mt323:qt-mt323.dll
 0001:0000cb5e       ?parentNode@QDomNode@@UBE?AV1@XZ 1000db5e f   qt-mt323:qt-mt323.dll
 0001:0000cb64       ?pixmap@QListViewItem@@UBEPBVQPixmap@@H@Z 1000db64 f   qt-mt323:qt-mt323.dll
 0001:0000cb6a       ?prefix@QDomNode@@UBE?AVQString@@XZ 1000db6a f   qt-mt323:qt-mt323.dll
 0001:0000cb70       ?previousSibling@QDomNode@@UBE?AV1@XZ 1000db70 f   qt-mt323:qt-mt323.dll
 0001:0000cb76       ?removeItem@QListViewItem@@UAEXPAV1@@Z 1000db76 f   qt-mt323:qt-mt323.dll
 0001:0000cb7c       ?rtti@QListViewItem@@UBEHXZ 1000db7c f   qt-mt323:qt-mt323.dll
 0001:0000cb82       ?setDragEnabled@QListViewItem@@UAEX_N@Z 1000db82 f   qt-mt323:qt-mt323.dll
 0001:0000cb88       ?setDropEnabled@QListViewItem@@UAEX_N@Z 1000db88 f   qt-mt323:qt-mt323.dll
 0001:0000cb8e       ?setEnabled@QListViewItem@@UAEX_N@Z 1000db8e f   qt-mt323:qt-mt323.dll
 0001:0000cb94       ?setExpandable@QListViewItem@@UAEX_N@Z 1000db94 f   qt-mt323:qt-mt323.dll
 0001:0000cb9a       ?setHeight@QListViewItem@@MAEXH@Z 1000db9a f   qt-mt323:qt-mt323.dll
 0001:0000cba0       ?setMultiLinesEnabled@QListViewItem@@UAEX_N@Z 1000dba0 f   qt-mt323:qt-mt323.dll
 0001:0000cba6       ?setNodeValue@QDomNode@@UAEXABVQString@@@Z 1000dba6 f   qt-mt323:qt-mt323.dll
 0001:0000cbac       ?setOpen@QListViewItem@@UAEX_N@Z 1000dbac f   qt-mt323:qt-mt323.dll
 0001:0000cbb2       ?setPixmap@QListViewItem@@UAEXHABVQPixmap@@@Z 1000dbb2 f   qt-mt323:qt-mt323.dll
 0001:0000cbb8       ?setPrefix@QDomNode@@UAEXABVQString@@@Z 1000dbb8 f   qt-mt323:qt-mt323.dll
 0001:0000cbbe       ?setRenameEnabled@QListViewItem@@UAEXH_N@Z 1000dbbe f   qt-mt323:qt-mt323.dll
 0001:0000cbc4       ?setSelectable@QListViewItem@@UAEX_N@Z 1000dbc4 f   qt-mt323:qt-mt323.dll
 0001:0000cbca       ?setSelected@QListViewItem@@UAEX_N@Z 1000dbca f   qt-mt323:qt-mt323.dll
 0001:0000cbd0       ?setText@QListViewItem@@UAEXHABVQString@@@Z 1000dbd0 f   qt-mt323:qt-mt323.dll
 0001:0000cbd6       ?setup@QListViewItem@@UAEXXZ 1000dbd6 f   qt-mt323:qt-mt323.dll
 0001:0000cbdc       ?sort@QListViewItem@@UAEXXZ 1000dbdc f   qt-mt323:qt-mt323.dll
 0001:0000cbe2       ?sortChildItems@QListViewItem@@UAEXH_N@Z 1000dbe2 f   qt-mt323:qt-mt323.dll
 0001:0000cbe8       ?startRename@QListViewItem@@UAEXH@Z 1000dbe8 f   qt-mt323:qt-mt323.dll
 0001:0000cbee       ?takeItem@QListViewItem@@UAEXPAV1@@Z 1000dbee f   qt-mt323:qt-mt323.dll
 0001:0000cbf4       ?text@QListViewItem@@UBE?AVQString@@H@Z 1000dbf4 f   qt-mt323:qt-mt323.dll
 0001:0000cbfa       ?width@QListViewItem@@UBEHABVQFontMetrics@@PBVQListView@@H@Z 1000dbfa f   qt-mt323:qt-mt323.dll
 0001:0000cc00       ?addChild@QScrollView@@UAEXPAVQWidget@@HH@Z 1000dc00 f   qt-mt323:qt-mt323.dll
 0001:0000cc06       ?addColumn@QListView@@UAEHABVQIconSet@@ABVQString@@H@Z 1000dc06 f   qt-mt323:qt-mt323.dll
 0001:0000cc0c       ?addColumn@QListView@@UAEHABVQString@@H@Z 1000dc0c f   qt-mt323:qt-mt323.dll
 0001:0000cc12       ?addItem@QBoxLayout@@UAEXPAVQLayoutItem@@@Z 1000dc12 f   qt-mt323:qt-mt323.dll
 0001:0000cc18       ?addItem@QGridLayout@@UAEXPAVQLayoutItem@@@Z 1000dc18 f   qt-mt323:qt-mt323.dll
 0001:0000cc1e       ?childEvent@QGroupBox@@MAEXPAVQChildEvent@@@Z 1000dc1e f   qt-mt323:qt-mt323.dll
 0001:0000cc24       ?childEvent@QLayout@@MAEXPAVQChildEvent@@@Z 1000dc24 f   qt-mt323:qt-mt323.dll
 0001:0000cc2a       ?childEvent@QWidgetStack@@MAEXPAVQChildEvent@@@Z 1000dc2a f   qt-mt323:qt-mt323.dll
 0001:0000cc30       ?className@QCheckBox@@UBEPBDXZ 1000dc30 f   qt-mt323:qt-mt323.dll
 0001:0000cc36       ?className@QComboBox@@UBEPBDXZ 1000dc36 f   qt-mt323:qt-mt323.dll
 0001:0000cc3c       ?className@QGridLayout@@UBEPBDXZ 1000dc3c f   qt-mt323:qt-mt323.dll
 0001:0000cc42       ?className@QGroupBox@@UBEPBDXZ 1000dc42 f   qt-mt323:qt-mt323.dll
 0001:0000cc48       ?className@QHBoxLayout@@UBEPBDXZ 1000dc48 f   qt-mt323:qt-mt323.dll
 0001:0000cc4e       ?className@QLabel@@UBEPBDXZ 1000dc4e f   qt-mt323:qt-mt323.dll
 0001:0000cc54       ?className@QLineEdit@@UBEPBDXZ 1000dc54 f   qt-mt323:qt-mt323.dll
 0001:0000cc5a       ?className@QListView@@UBEPBDXZ 1000dc5a f   qt-mt323:qt-mt323.dll
 0001:0000cc60       ?className@QPushButton@@UBEPBDXZ 1000dc60 f   qt-mt323:qt-mt323.dll
 0001:0000cc66       ?className@QSpinBox@@UBEPBDXZ 1000dc66 f   qt-mt323:qt-mt323.dll
 0001:0000cc6c       ?className@QVBoxLayout@@UBEPBDXZ 1000dc6c f   qt-mt323:qt-mt323.dll
 0001:0000cc72       ?className@QWidgetStack@@UBEPBDXZ 1000dc72 f   qt-mt323:qt-mt323.dll
 0001:0000cc78       ?cleanText@QSpinBox@@UBE?AVQString@@XZ 1000dc78 f   qt-mt323:qt-mt323.dll
 0001:0000cc7e       ?clear@QLineEdit@@UAEXXZ   1000dc7e f   qt-mt323:qt-mt323.dll
 0001:0000cc84       ?clear@QListView@@UAEXXZ   1000dc84 f   qt-mt323:qt-mt323.dll
 0001:0000cc8a       ?clearSelection@QListView@@UAEXXZ 1000dc8a f   qt-mt323:qt-mt323.dll
 0001:0000cc90       ?clearValidator@QLineEdit@@UAEXXZ 1000dc90 f   qt-mt323:qt-mt323.dll
 0001:0000cc96       ?contentsContextMenuEvent@QListView@@MAEXPAVQContextMenuEvent@@@Z 1000dc96 f   qt-mt323:qt-mt323.dll
 0001:0000cc9c       ?contentsDragEnterEvent@QListView@@MAEXPAVQDragEnterEvent@@@Z 1000dc9c f   qt-mt323:qt-mt323.dll
 0001:0000cca2       ?contentsDragLeaveEvent@QListView@@MAEXPAVQDragLeaveEvent@@@Z 1000dca2 f   qt-mt323:qt-mt323.dll
 0001:0000cca8       ?contentsDragMoveEvent@QListView@@MAEXPAVQDragMoveEvent@@@Z 1000dca8 f   qt-mt323:qt-mt323.dll
 0001:0000ccae       ?contentsDropEvent@QListView@@MAEXPAVQDropEvent@@@Z 1000dcae f   qt-mt323:qt-mt323.dll
 0001:0000ccb4       ?contentsMouseDoubleClickEvent@QListView@@MAEXPAVQMouseEvent@@@Z 1000dcb4 f   qt-mt323:qt-mt323.dll
 0001:0000ccba       ?contentsMouseMoveEvent@QListView@@MAEXPAVQMouseEvent@@@Z 1000dcba f   qt-mt323:qt-mt323.dll
 0001:0000ccc0       ?contentsMousePressEvent@QListView@@MAEXPAVQMouseEvent@@@Z 1000dcc0 f   qt-mt323:qt-mt323.dll
 0001:0000ccc6       ?contentsMouseReleaseEvent@QListView@@MAEXPAVQMouseEvent@@@Z 1000dcc6 f   qt-mt323:qt-mt323.dll
 0001:0000cccc       ?contentsWheelEvent@QScrollView@@MAEXPAVQWheelEvent@@@Z 1000dccc f   qt-mt323:qt-mt323.dll
 0001:0000ccd2       ?contextMenuEvent@QLineEdit@@MAEXPAVQContextMenuEvent@@@Z 1000dcd2 f   qt-mt323:qt-mt323.dll
 0001:0000ccd8       ?contextMenuEvent@QScrollView@@MAEXPAVQContextMenuEvent@@@Z 1000dcd8 f   qt-mt323:qt-mt323.dll
 0001:0000ccde       ?copy@QLineEdit@@UBEXXZ    1000dcde f   qt-mt323:qt-mt323.dll
 0001:0000cce4       ?createPopupMenu@QLineEdit@@MAEPAVQPopupMenu@@XZ 1000dce4 f   qt-mt323:qt-mt323.dll
 0001:0000ccea       ?cut@QLineEdit@@UAEXXZ     1000dcea f   qt-mt323:qt-mt323.dll
 0001:0000ccf0       ?deselect@QLineEdit@@UAEXXZ 1000dcf0 f   qt-mt323:qt-mt323.dll
 0001:0000ccf6       ?dragEnterEvent@QLineEdit@@MAEXPAVQDragEnterEvent@@@Z 1000dcf6 f   qt-mt323:qt-mt323.dll
 0001:0000ccfc       ?dragLeaveEvent@QLineEdit@@MAEXPAVQDragLeaveEvent@@@Z 1000dcfc f   qt-mt323:qt-mt323.dll
 0001:0000cd02       ?dragMoveEvent@QLineEdit@@MAEXPAVQDragMoveEvent@@@Z 1000dd02 f   qt-mt323:qt-mt323.dll
 0001:0000cd08       ?dragObject@QListView@@MAEPAVQDragObject@@XZ 1000dd08 f   qt-mt323:qt-mt323.dll
 0001:0000cd0e       ?drawButton@QCheckBox@@MAEXPAVQPainter@@@Z 1000dd0e f   qt-mt323:qt-mt323.dll
 0001:0000cd14       ?drawButton@QPushButton@@MAEXPAVQPainter@@@Z 1000dd14 f   qt-mt323:qt-mt323.dll
 0001:0000cd1a       ?drawButtonLabel@QCheckBox@@MAEXPAVQPainter@@@Z 1000dd1a f   qt-mt323:qt-mt323.dll
 0001:0000cd20       ?drawButtonLabel@QPushButton@@MAEXPAVQPainter@@@Z 1000dd20 f   qt-mt323:qt-mt323.dll
 0001:0000cd26       ?drawContents@QFrame@@MAEXPAVQPainter@@@Z 1000dd26 f   qt-mt323:qt-mt323.dll
 0001:0000cd2c       ?drawContents@QLabel@@MAEXPAVQPainter@@@Z 1000dd2c f   qt-mt323:qt-mt323.dll
 0001:0000cd32       ?drawContents@QLineEdit@@MAEXPAVQPainter@@@Z 1000dd32 f   qt-mt323:qt-mt323.dll
 0001:0000cd38       ?drawContents@QScrollView@@EAEXPAVQPainter@@@Z 1000dd38 f   qt-mt323:qt-mt323.dll
 0001:0000cd3e       ?drawContents@QScrollView@@MAEXPAVQPainter@@HHHH@Z 1000dd3e f   qt-mt323:qt-mt323.dll
 0001:0000cd44       ?drawContentsOffset@QListView@@MAEXPAVQPainter@@HHHHHH@Z 1000dd44 f   qt-mt323:qt-mt323.dll
 0001:0000cd4a       ?dropEvent@QLineEdit@@MAEXPAVQDropEvent@@@Z 1000dd4a f   qt-mt323:qt-mt323.dll
 0001:0000cd50       ?enabledChange@QButton@@MAEX_N@Z 1000dd50 f   qt-mt323:qt-mt323.dll
 0001:0000cd56       ?event@QGroupBox@@MAE_NPAVQEvent@@@Z 1000dd56 f   qt-mt323:qt-mt323.dll
 0001:0000cd5c       ?event@QLineEdit@@MAE_NPAVQEvent@@@Z 1000dd5c f   qt-mt323:qt-mt323.dll
 0001:0000cd62       ?eventFilter@QComboBox@@UAE_NPAVQObject@@PAVQEvent@@@Z 1000dd62 f   qt-mt323:qt-mt323.dll
 0001:0000cd68       ?eventFilter@QLayout@@MAE_NPAVQObject@@PAVQEvent@@@Z 1000dd68 f   qt-mt323:qt-mt323.dll
 0001:0000cd6e       ?eventFilter@QListView@@UAE_NPAVQObject@@PAVQEvent@@@Z 1000dd6e f   qt-mt323:qt-mt323.dll
 0001:0000cd74       ?eventFilter@QSpinBox@@MAE_NPAVQObject@@PAVQEvent@@@Z 1000dd74 f   qt-mt323:qt-mt323.dll
 0001:0000cd7a       ?expanding@QBoxLayout@@UBE?AW4ExpandData@QSizePolicy@@XZ 1000dd7a f   qt-mt323:qt-mt323.dll
 0001:0000cd80       ?expanding@QGridLayout@@UBE?AW4ExpandData@QSizePolicy@@XZ 1000dd80 f   qt-mt323:qt-mt323.dll
 0001:0000cd86       ?expanding@QSpacerItem@@UBE?AW4ExpandData@QSizePolicy@@XZ 1000dd86 f   qt-mt323:qt-mt323.dll
 0001:0000cd8c       ?focusInEvent@QButton@@MAEXPAVQFocusEvent@@@Z 1000dd8c f   qt-mt323:qt-mt323.dll
 0001:0000cd92       ?focusInEvent@QComboBox@@MAEXPAVQFocusEvent@@@Z 1000dd92 f   qt-mt323:qt-mt323.dll
 0001:0000cd98       ?focusInEvent@QGroupBox@@MAEXPAVQFocusEvent@@@Z 1000dd98 f   qt-mt323:qt-mt323.dll
 0001:0000cd9e       ?focusInEvent@QLineEdit@@MAEXPAVQFocusEvent@@@Z 1000dd9e f   qt-mt323:qt-mt323.dll
 0001:0000cda4       ?focusInEvent@QListView@@MAEXPAVQFocusEvent@@@Z 1000dda4 f   qt-mt323:qt-mt323.dll
 0001:0000cdaa       ?focusInEvent@QPushButton@@MAEXPAVQFocusEvent@@@Z 1000ddaa f   qt-mt323:qt-mt323.dll
 0001:0000cdb0       ?focusNextPrevChild@QScrollView@@MAE_N_N@Z 1000ddb0 f   qt-mt323:qt-mt323.dll
 0001:0000cdb6       ?focusOutEvent@QButton@@MAEXPAVQFocusEvent@@@Z 1000ddb6 f   qt-mt323:qt-mt323.dll
 0001:0000cdbc       ?focusOutEvent@QComboBox@@MAEXPAVQFocusEvent@@@Z 1000ddbc f   qt-mt323:qt-mt323.dll
 0001:0000cdc2       ?focusOutEvent@QLineEdit@@MAEXPAVQFocusEvent@@@Z 1000ddc2 f   qt-mt323:qt-mt323.dll
 0001:0000cdc8       ?focusOutEvent@QListView@@MAEXPAVQFocusEvent@@@Z 1000ddc8 f   qt-mt323:qt-mt323.dll
 0001:0000cdce       ?focusOutEvent@QPushButton@@MAEXPAVQFocusEvent@@@Z 1000ddce f   qt-mt323:qt-mt323.dll
 0001:0000cdd4       ?fontChange@QGroupBox@@MAEXABVQFont@@@Z 1000ddd4 f   qt-mt323:qt-mt323.dll
 0001:0000cdda       ?fontChange@QLabel@@MAEXABVQFont@@@Z 1000ddda f   qt-mt323:qt-mt323.dll
 0001:0000cde0       ?fontChange@QScrollView@@MAEXABVQFont@@@Z 1000dde0 f   qt-mt323:qt-mt323.dll
 0001:0000cde6       ?frameChanged@QScrollView@@MAEXXZ 1000dde6 f   qt-mt323:qt-mt323.dll
 0001:0000cdec       ?frameChanged@QWidgetStack@@MAEXXZ 1000ddec f   qt-mt323:qt-mt323.dll
 0001:0000cdf2       ?geometry@QLayout@@UBE?AVQRect@@XZ 1000ddf2 f   qt-mt323:qt-mt323.dll
 0001:0000cdf8       ?geometry@QSpacerItem@@UBE?AVQRect@@XZ 1000ddf8 f   qt-mt323:qt-mt323.dll
 0001:0000cdfe       ?hasHeightForWidth@QBoxLayout@@UBE_NXZ 1000ddfe f   qt-mt323:qt-mt323.dll
 0001:0000ce04       ?hasHeightForWidth@QGridLayout@@UBE_NXZ 1000de04 f   qt-mt323:qt-mt323.dll
 0001:0000ce0a       ?hasHeightForWidth@QLayoutItem@@UBE_NXZ 1000de0a f   qt-mt323:qt-mt323.dll
 0001:0000ce10       ?heightForWidth@QBoxLayout@@UBEHH@Z 1000de10 f   qt-mt323:qt-mt323.dll
 0001:0000ce16       ?heightForWidth@QGridLayout@@UBEHH@Z 1000de16 f   qt-mt323:qt-mt323.dll
 0001:0000ce1c       ?heightForWidth@QLabel@@UBEHH@Z 1000de1c f   qt-mt323:qt-mt323.dll
 0001:0000ce22       ?heightForWidth@QLayoutItem@@UBEHH@Z 1000de22 f   qt-mt323:qt-mt323.dll
 0001:0000ce28       ?hitButton@QButton@@MBE_NABVQPoint@@@Z 1000de28 f   qt-mt323:qt-mt323.dll
 0001:0000ce2e       ?hitButton@QCheckBox@@MBE_NABVQPoint@@@Z 1000de2e f   qt-mt323:qt-mt323.dll
 0001:0000ce34       ?imComposeEvent@QLineEdit@@MAEXPAVQIMEvent@@@Z 1000de34 f   qt-mt323:qt-mt323.dll
 0001:0000ce3a       ?imEndEvent@QLineEdit@@MAEXPAVQIMEvent@@@Z 1000de3a f   qt-mt323:qt-mt323.dll
 0001:0000ce40       ?imStartEvent@QLineEdit@@MAEXPAVQIMEvent@@@Z 1000de40 f   qt-mt323:qt-mt323.dll
 0001:0000ce46       ?insert@QLineEdit@@UAEXABVQString@@@Z 1000de46 f   qt-mt323:qt-mt323.dll
 0001:0000ce4c       ?insertItem@QListView@@UAEXPAVQListViewItem@@@Z 1000de4c f   qt-mt323:qt-mt323.dll
 0001:0000ce52       ?interpretText@QSpinBox@@MAEXXZ 1000de52 f   qt-mt323:qt-mt323.dll
 0001:0000ce58       ?invalidate@QBoxLayout@@UAEXXZ 1000de58 f   qt-mt323:qt-mt323.dll
 0001:0000ce5e       ?invalidate@QGridLayout@@UAEXXZ 1000de5e f   qt-mt323:qt-mt323.dll
 0001:0000ce64       ?invalidate@QLayoutItem@@UAEXXZ 1000de64 f   qt-mt323:qt-mt323.dll
 0001:0000ce6a       ?invertSelection@QListView@@UAEXXZ 1000de6a f   qt-mt323:qt-mt323.dll
 0001:0000ce70       ?isEmpty@QLayout@@UBE_NXZ  1000de70 f   qt-mt323:qt-mt323.dll
 0001:0000ce76       ?isEmpty@QSpacerItem@@UBE_NXZ 1000de76 f   qt-mt323:qt-mt323.dll
 0001:0000ce7c       ?iterator@QBoxLayout@@UAE?AVQLayoutIterator@@XZ 1000de7c f   qt-mt323:qt-mt323.dll
 0001:0000ce82       ?iterator@QGridLayout@@UAE?AVQLayoutIterator@@XZ 1000de82 f   qt-mt323:qt-mt323.dll
 0001:0000ce88       ?iterator@QLayoutItem@@UAE?AVQLayoutIterator@@XZ 1000de88 f   qt-mt323:qt-mt323.dll
 0001:0000ce8e       ?keyPressEvent@QButton@@MAEXPAVQKeyEvent@@@Z 1000de8e f   qt-mt323:qt-mt323.dll
 0001:0000ce94       ?keyPressEvent@QComboBox@@MAEXPAVQKeyEvent@@@Z 1000de94 f   qt-mt323:qt-mt323.dll
 0001:0000ce9a       ?keyPressEvent@QLineEdit@@MAEXPAVQKeyEvent@@@Z 1000de9a f   qt-mt323:qt-mt323.dll
 0001:0000cea0       ?keyPressEvent@QListView@@MAEXPAVQKeyEvent@@@Z 1000dea0 f   qt-mt323:qt-mt323.dll
 0001:0000cea6       ?keyReleaseEvent@QButton@@MAEXPAVQKeyEvent@@@Z 1000dea6 f   qt-mt323:qt-mt323.dll
 0001:0000ceac       ?layout@QLayout@@UAEPAV1@XZ 1000deac f   qt-mt323:qt-mt323.dll
 0001:0000ceb2       ?layout@QLayoutItem@@UAEPAVQLayout@@XZ 1000deb2 f   qt-mt323:qt-mt323.dll
 0001:0000ceb8       ?leaveEvent@QSpinBox@@MAEXPAVQEvent@@@Z 1000deb8 f   qt-mt323:qt-mt323.dll
 0001:0000cebe       ?mapTextToValue@QSpinBox@@MAEHPA_N@Z 1000debe f   qt-mt323:qt-mt323.dll
 0001:0000cec4       ?mapValueToText@QSpinBox@@MAE?AVQString@@H@Z 1000dec4 f   qt-mt323:qt-mt323.dll
 0001:0000ceca       ?maximumSize@QBoxLayout@@UBE?AVQSize@@XZ 1000deca f   qt-mt323:qt-mt323.dll
 0001:0000ced0       ?maximumSize@QGridLayout@@UBE?AVQSize@@XZ 1000ded0 f   qt-mt323:qt-mt323.dll
 0001:0000ced6       ?maximumSize@QSpacerItem@@UBE?AVQSize@@XZ 1000ded6 f   qt-mt323:qt-mt323.dll
 0001:0000cedc       ?metaObject@QCheckBox@@UBEPAVQMetaObject@@XZ 1000dedc f   qt-mt323:qt-mt323.dll
 0001:0000cee2       ?metaObject@QComboBox@@UBEPAVQMetaObject@@XZ 1000dee2 f   qt-mt323:qt-mt323.dll
 0001:0000cee8       ?metaObject@QGridLayout@@UBEPAVQMetaObject@@XZ 1000dee8 f   qt-mt323:qt-mt323.dll
 0001:0000ceee       ?metaObject@QGroupBox@@UBEPAVQMetaObject@@XZ 1000deee f   qt-mt323:qt-mt323.dll
 0001:0000cef4       ?metaObject@QHBoxLayout@@UBEPAVQMetaObject@@XZ 1000def4 f   qt-mt323:qt-mt323.dll
 0001:0000cefa       ?metaObject@QLabel@@UBEPAVQMetaObject@@XZ 1000defa f   qt-mt323:qt-mt323.dll
 0001:0000cf00       ?metaObject@QLineEdit@@UBEPAVQMetaObject@@XZ 1000df00 f   qt-mt323:qt-mt323.dll
 0001:0000cf06       ?metaObject@QListView@@UBEPAVQMetaObject@@XZ 1000df06 f   qt-mt323:qt-mt323.dll
 0001:0000cf0c       ?metaObject@QPushButton@@UBEPAVQMetaObject@@XZ 1000df0c f   qt-mt323:qt-mt323.dll
 0001:0000cf12       ?metaObject@QSpinBox@@UBEPAVQMetaObject@@XZ 1000df12 f   qt-mt323:qt-mt323.dll
 0001:0000cf18       ?metaObject@QVBoxLayout@@UBEPAVQMetaObject@@XZ 1000df18 f   qt-mt323:qt-mt323.dll
 0001:0000cf1e       ?metaObject@QWidgetStack@@UBEPAVQMetaObject@@XZ 1000df1e f   qt-mt323:qt-mt323.dll
 0001:0000cf24       ?minimumSize@QBoxLayout@@UBE?AVQSize@@XZ 1000df24 f   qt-mt323:qt-mt323.dll
 0001:0000cf2a       ?minimumSize@QGridLayout@@UBE?AVQSize@@XZ 1000df2a f   qt-mt323:qt-mt323.dll
 0001:0000cf30       ?minimumSize@QSpacerItem@@UBE?AVQSize@@XZ 1000df30 f   qt-mt323:qt-mt323.dll
 0001:0000cf36       ?minimumSizeHint@QLabel@@UBE?AVQSize@@XZ 1000df36 f   qt-mt323:qt-mt323.dll
 0001:0000cf3c       ?minimumSizeHint@QLineEdit@@UBE?AVQSize@@XZ 1000df3c f   qt-mt323:qt-mt323.dll
 0001:0000cf42       ?minimumSizeHint@QListView@@UBE?AVQSize@@XZ 1000df42 f   qt-mt323:qt-mt323.dll
 0001:0000cf48       ?minimumSizeHint@QSpinBox@@UBE?AVQSize@@XZ 1000df48 f   qt-mt323:qt-mt323.dll
 0001:0000cf4e       ?minimumSizeHint@QWidgetStack@@UBE?AVQSize@@XZ 1000df4e f   qt-mt323:qt-mt323.dll
 0001:0000cf54       ?mouseDoubleClickEvent@QComboBox@@MAEXPAVQMouseEvent@@@Z 1000df54 f   qt-mt323:qt-mt323.dll
 0001:0000cf5a       ?mouseDoubleClickEvent@QLineEdit@@MAEXPAVQMouseEvent@@@Z 1000df5a f   qt-mt323:qt-mt323.dll
 0001:0000cf60       ?mouseDoubleClickEvent@QScrollView@@MAEXPAVQMouseEvent@@@Z 1000df60 f   qt-mt323:qt-mt323.dll
 0001:0000cf66       ?mouseMoveEvent@QButton@@MAEXPAVQMouseEvent@@@Z 1000df66 f   qt-mt323:qt-mt323.dll
 0001:0000cf6c       ?mouseMoveEvent@QComboBox@@MAEXPAVQMouseEvent@@@Z 1000df6c f   qt-mt323:qt-mt323.dll
 0001:0000cf72       ?mouseMoveEvent@QLineEdit@@MAEXPAVQMouseEvent@@@Z 1000df72 f   qt-mt323:qt-mt323.dll
 0001:0000cf78       ?mouseMoveEvent@QScrollView@@MAEXPAVQMouseEvent@@@Z 1000df78 f   qt-mt323:qt-mt323.dll
 0001:0000cf7e       ?mousePressEvent@QButton@@MAEXPAVQMouseEvent@@@Z 1000df7e f   qt-mt323:qt-mt323.dll
 0001:0000cf84       ?mousePressEvent@QComboBox@@MAEXPAVQMouseEvent@@@Z 1000df84 f   qt-mt323:qt-mt323.dll
 0001:0000cf8a       ?mousePressEvent@QLineEdit@@MAEXPAVQMouseEvent@@@Z 1000df8a f   qt-mt323:qt-mt323.dll
 0001:0000cf90       ?mousePressEvent@QScrollView@@MAEXPAVQMouseEvent@@@Z 1000df90 f   qt-mt323:qt-mt323.dll
 0001:0000cf96       ?mouseReleaseEvent@QButton@@MAEXPAVQMouseEvent@@@Z 1000df96 f   qt-mt323:qt-mt323.dll
 0001:0000cf9c       ?mouseReleaseEvent@QComboBox@@MAEXPAVQMouseEvent@@@Z 1000df9c f   qt-mt323:qt-mt323.dll
 0001:0000cfa2       ?mouseReleaseEvent@QLineEdit@@MAEXPAVQMouseEvent@@@Z 1000dfa2 f   qt-mt323:qt-mt323.dll
 0001:0000cfa8       ?mouseReleaseEvent@QScrollView@@MAEXPAVQMouseEvent@@@Z 1000dfa8 f   qt-mt323:qt-mt323.dll
 0001:0000cfae       ?move@QPushButton@@UAEXHH@Z 1000dfae f   qt-mt323:qt-mt323.dll
 0001:0000cfb4       ?moveChild@QScrollView@@UAEXPAVQWidget@@HH@Z 1000dfb4 f   qt-mt323:qt-mt323.dll
 0001:0000cfba       ?paintEmptyArea@QListView@@MAEXPAVQPainter@@ABVQRect@@@Z 1000dfba f   qt-mt323:qt-mt323.dll
 0001:0000cfc0       ?paintEvent@QButton@@MAEXPAVQPaintEvent@@@Z 1000dfc0 f   qt-mt323:qt-mt323.dll
 0001:0000cfc6       ?paintEvent@QComboBox@@MAEXPAVQPaintEvent@@@Z 1000dfc6 f   qt-mt323:qt-mt323.dll
 0001:0000cfcc       ?paintEvent@QGroupBox@@MAEXPAVQPaintEvent@@@Z 1000dfcc f   qt-mt323:qt-mt323.dll
 0001:0000cfd2       ?paste@QLineEdit@@UAEXXZ   1000dfd2 f   qt-mt323:qt-mt323.dll
 0001:0000cfd8       ?popup@QComboBox@@UAEXXZ   1000dfd8 f   qt-mt323:qt-mt323.dll
 0001:0000cfde       ?prefix@QSpinBox@@UBE?AVQString@@XZ 1000dfde f   qt-mt323:qt-mt323.dll
 0001:0000cfe4       ?qt_cast@QCheckBox@@UAEPAXPBD@Z 1000dfe4 f   qt-mt323:qt-mt323.dll
 0001:0000cfea       ?qt_cast@QComboBox@@UAEPAXPBD@Z 1000dfea f   qt-mt323:qt-mt323.dll
 0001:0000cff0       ?qt_cast@QGridLayout@@UAEPAXPBD@Z 1000dff0 f   qt-mt323:qt-mt323.dll
 0001:0000cff6       ?qt_cast@QGroupBox@@UAEPAXPBD@Z 1000dff6 f   qt-mt323:qt-mt323.dll
 0001:0000cffe       ?qt_cast@QHBoxLayout@@UAEPAXPBD@Z 1000dffe f   qt-mt323:qt-mt323.dll
 0001:0000d004       ?qt_cast@QLabel@@UAEPAXPBD@Z 1000e004 f   qt-mt323:qt-mt323.dll
 0001:0000d00a       ?qt_cast@QLineEdit@@UAEPAXPBD@Z 1000e00a f   qt-mt323:qt-mt323.dll
 0001:0000d010       ?qt_cast@QListView@@UAEPAXPBD@Z 1000e010 f   qt-mt323:qt-mt323.dll
 0001:0000d016       ?qt_cast@QPushButton@@UAEPAXPBD@Z 1000e016 f   qt-mt323:qt-mt323.dll
 0001:0000d01c       ?qt_cast@QSpinBox@@UAEPAXPBD@Z 1000e01c f   qt-mt323:qt-mt323.dll
 0001:0000d022       ?qt_cast@QVBoxLayout@@UAEPAXPBD@Z 1000e022 f   qt-mt323:qt-mt323.dll
 0001:0000d028       ?qt_cast@QWidgetStack@@UAEPAXPBD@Z 1000e028 f   qt-mt323:qt-mt323.dll
 0001:0000d02e       ?qt_emit@QCheckBox@@UAE_NHPAUQUObject@@@Z 1000e02e f   qt-mt323:qt-mt323.dll
 0001:0000d034       ?qt_emit@QComboBox@@UAE_NHPAUQUObject@@@Z 1000e034 f   qt-mt323:qt-mt323.dll
 0001:0000d03a       ?qt_emit@QGridLayout@@UAE_NHPAUQUObject@@@Z 1000e03a f   qt-mt323:qt-mt323.dll
 0001:0000d040       ?qt_emit@QGroupBox@@UAE_NHPAUQUObject@@@Z 1000e040 f   qt-mt323:qt-mt323.dll
 0001:0000d046       ?qt_emit@QHBoxLayout@@UAE_NHPAUQUObject@@@Z 1000e046 f   qt-mt323:qt-mt323.dll
 0001:0000d04c       ?qt_emit@QLabel@@UAE_NHPAUQUObject@@@Z 1000e04c f   qt-mt323:qt-mt323.dll
 0001:0000d052       ?qt_emit@QLineEdit@@UAE_NHPAUQUObject@@@Z 1000e052 f   qt-mt323:qt-mt323.dll
 0001:0000d058       ?qt_emit@QListView@@UAE_NHPAUQUObject@@@Z 1000e058 f   qt-mt323:qt-mt323.dll
 0001:0000d05e       ?qt_emit@QPushButton@@UAE_NHPAUQUObject@@@Z 1000e05e f   qt-mt323:qt-mt323.dll
 0001:0000d064       ?qt_emit@QSpinBox@@UAE_NHPAUQUObject@@@Z 1000e064 f   qt-mt323:qt-mt323.dll
 0001:0000d06a       ?qt_emit@QVBoxLayout@@UAE_NHPAUQUObject@@@Z 1000e06a f   qt-mt323:qt-mt323.dll
 0001:0000d070       ?qt_emit@QWidgetStack@@UAE_NHPAUQUObject@@@Z 1000e070 f   qt-mt323:qt-mt323.dll
 0001:0000d076       ?qt_invoke@QCheckBox@@UAE_NHPAUQUObject@@@Z 1000e076 f   qt-mt323:qt-mt323.dll
 0001:0000d07c       ?qt_invoke@QComboBox@@UAE_NHPAUQUObject@@@Z 1000e07c f   qt-mt323:qt-mt323.dll
 0001:0000d082       ?qt_invoke@QGridLayout@@UAE_NHPAUQUObject@@@Z 1000e082 f   qt-mt323:qt-mt323.dll
 0001:0000d088       ?qt_invoke@QGroupBox@@UAE_NHPAUQUObject@@@Z 1000e088 f   qt-mt323:qt-mt323.dll
 0001:0000d08e       ?qt_invoke@QHBoxLayout@@UAE_NHPAUQUObject@@@Z 1000e08e f   qt-mt323:qt-mt323.dll
 0001:0000d094       ?qt_invoke@QLabel@@UAE_NHPAUQUObject@@@Z 1000e094 f   qt-mt323:qt-mt323.dll
 0001:0000d09a       ?qt_invoke@QLineEdit@@UAE_NHPAUQUObject@@@Z 1000e09a f   qt-mt323:qt-mt323.dll
 0001:0000d0a0       ?qt_invoke@QListView@@UAE_NHPAUQUObject@@@Z 1000e0a0 f   qt-mt323:qt-mt323.dll
 0001:0000d0a6       ?qt_invoke@QPushButton@@UAE_NHPAUQUObject@@@Z 1000e0a6 f   qt-mt323:qt-mt323.dll
 0001:0000d0ac       ?qt_invoke@QSpinBox@@UAE_NHPAUQUObject@@@Z 1000e0ac f   qt-mt323:qt-mt323.dll
 0001:0000d0b2       ?qt_invoke@QVBoxLayout@@UAE_NHPAUQUObject@@@Z 1000e0b2 f   qt-mt323:qt-mt323.dll
 0001:0000d0b8       ?qt_invoke@QWidgetStack@@UAE_NHPAUQUObject@@@Z 1000e0b8 f   qt-mt323:qt-mt323.dll
 0001:0000d0be       ?qt_property@QCheckBox@@UAE_NHHPAVQVariant@@@Z 1000e0be f   qt-mt323:qt-mt323.dll
 0001:0000d0c4       ?qt_property@QComboBox@@UAE_NHHPAVQVariant@@@Z 1000e0c4 f   qt-mt323:qt-mt323.dll
 0001:0000d0ca       ?qt_property@QGridLayout@@UAE_NHHPAVQVariant@@@Z 1000e0ca f   qt-mt323:qt-mt323.dll
 0001:0000d0d0       ?qt_property@QGroupBox@@UAE_NHHPAVQVariant@@@Z 1000e0d0 f   qt-mt323:qt-mt323.dll
 0001:0000d0d6       ?qt_property@QHBoxLayout@@UAE_NHHPAVQVariant@@@Z 1000e0d6 f   qt-mt323:qt-mt323.dll
 0001:0000d0dc       ?qt_property@QLabel@@UAE_NHHPAVQVariant@@@Z 1000e0dc f   qt-mt323:qt-mt323.dll
 0001:0000d0e2       ?qt_property@QLineEdit@@UAE_NHHPAVQVariant@@@Z 1000e0e2 f   qt-mt323:qt-mt323.dll
 0001:0000d0e8       ?qt_property@QListView@@UAE_NHHPAVQVariant@@@Z 1000e0e8 f   qt-mt323:qt-mt323.dll
 0001:0000d0ee       ?qt_property@QPushButton@@UAE_NHHPAVQVariant@@@Z 1000e0ee f   qt-mt323:qt-mt323.dll
 0001:0000d0f4       ?qt_property@QSpinBox@@UAE_NHHPAVQVariant@@@Z 1000e0f4 f   qt-mt323:qt-mt323.dll
 0001:0000d0fa       ?qt_property@QVBoxLayout@@UAE_NHHPAVQVariant@@@Z 1000e0fa f   qt-mt323:qt-mt323.dll
 0001:0000d100       ?qt_property@QWidgetStack@@UAE_NHHPAVQVariant@@@Z 1000e100 f   qt-mt323:qt-mt323.dll
 0001:0000d106       ?rangeChange@QSpinBox@@MAEXXZ 1000e106 f   qt-mt323:qt-mt323.dll
 0001:0000d10c       ?redo@QLineEdit@@UAEXXZ    1000e10c f   qt-mt323:qt-mt323.dll
 0001:0000d112       ?removeChild@QScrollView@@UAEXPAVQObject@@@Z 1000e112 f   qt-mt323:qt-mt323.dll
 0001:0000d118       ?removeColumn@QListView@@UAEXH@Z 1000e118 f   qt-mt323:qt-mt323.dll
 0001:0000d11e       ?removeItem@QListView@@UAEXPAVQListViewItem@@@Z 1000e11e f   qt-mt323:qt-mt323.dll
 0001:0000d124       ?resize@QPushButton@@UAEXHH@Z 1000e124 f   qt-mt323:qt-mt323.dll
 0001:0000d12a       ?resize@QScrollView@@UAEXHH@Z 1000e12a f   qt-mt323:qt-mt323.dll
 0001:0000d130       ?resizeContents@QScrollView@@UAEXHH@Z 1000e130 f   qt-mt323:qt-mt323.dll
 0001:0000d136       ?resizeEvent@QCheckBox@@MAEXPAVQResizeEvent@@@Z 1000e136 f   qt-mt323:qt-mt323.dll
 0001:0000d13c       ?resizeEvent@QComboBox@@MAEXPAVQResizeEvent@@@Z 1000e13c f   qt-mt323:qt-mt323.dll
 0001:0000d142       ?resizeEvent@QGroupBox@@MAEXPAVQResizeEvent@@@Z 1000e142 f   qt-mt323:qt-mt323.dll
 0001:0000d148       ?resizeEvent@QLabel@@MAEXPAVQResizeEvent@@@Z 1000e148 f   qt-mt323:qt-mt323.dll
 0001:0000d14e       ?resizeEvent@QLineEdit@@MAEXPAVQResizeEvent@@@Z 1000e14e f   qt-mt323:qt-mt323.dll
 0001:0000d154       ?resizeEvent@QListView@@MAEXPAVQResizeEvent@@@Z 1000e154 f   qt-mt323:qt-mt323.dll
 0001:0000d15a       ?resizeEvent@QPushButton@@MAEXPAVQResizeEvent@@@Z 1000e15a f   qt-mt323:qt-mt323.dll
 0001:0000d160       ?resizeEvent@QSpinBox@@MAEXPAVQResizeEvent@@@Z 1000e160 f   qt-mt323:qt-mt323.dll
 0001:0000d166       ?resizeEvent@QWidgetStack@@MAEXPAVQResizeEvent@@@Z 1000e166 f   qt-mt323:qt-mt323.dll
 0001:0000d16c       ?selectAll@QLineEdit@@UAEXXZ 1000e16c f   qt-mt323:qt-mt323.dll
 0001:0000d172       ?selectAll@QListView@@UAEX_N@Z 1000e172 f   qt-mt323:qt-mt323.dll
 0001:0000d178       ?selectAll@QSpinBox@@UAEXXZ 1000e178 f   qt-mt323:qt-mt323.dll
 0001:0000d17e       ?setAccel@QButton@@UAEXABVQKeySequence@@@Z 1000e17e f   qt-mt323:qt-mt323.dll
 0001:0000d184       ?setAlignment@QGroupBox@@UAEXH@Z 1000e184 f   qt-mt323:qt-mt323.dll
 0001:0000d18a       ?setAlignment@QLabel@@UAEXH@Z 1000e18a f   qt-mt323:qt-mt323.dll
 0001:0000d190       ?setAlignment@QLayoutItem@@UAEXH@Z 1000e190 f   qt-mt323:qt-mt323.dll
 0001:0000d196       ?setAlignment@QLineEdit@@UAEXH@Z 1000e196 f   qt-mt323:qt-mt323.dll
 0001:0000d19c       ?setAllColumnsShowFocus@QListView@@UAEX_N@Z 1000e19c f   qt-mt323:qt-mt323.dll
 0001:0000d1a2       ?setAutoAdd@QLayout@@UAEX_N@Z 1000e1a2 f   qt-mt323:qt-mt323.dll
 0001:0000d1a8       ?setAutoCompletion@QComboBox@@UAEX_N@Z 1000e1a8 f   qt-mt323:qt-mt323.dll
 0001:0000d1ae       ?setAutoDefault@QPushButton@@UAEX_N@Z 1000e1ae f   qt-mt323:qt-mt323.dll
 0001:0000d1b4       ?setAutoRepeat@QButton@@UAEX_N@Z 1000e1b4 f   qt-mt323:qt-mt323.dll
 0001:0000d1ba       ?setAutoResize@QComboBox@@UAEX_N@Z 1000e1ba f   qt-mt323:qt-mt323.dll
 0001:0000d1c0       ?setAutoResize@QLabel@@UAEX_N@Z 1000e1c0 f   qt-mt323:qt-mt323.dll
 0001:0000d1c6       ?setBuddy@QLabel@@UAEXPAVQWidget@@@Z 1000e1c6 f   qt-mt323:qt-mt323.dll
 0001:0000d1cc       ?setButtonSymbols@QSpinBox@@UAEXW4ButtonSymbols@1@@Z 1000e1cc f   qt-mt323:qt-mt323.dll
 0001:0000d1d2       ?setChildGeometries@QWidgetStack@@MAEXXZ 1000e1d2 f   qt-mt323:qt-mt323.dll
 0001:0000d1d8       ?setColStretch@QGridLayout@@UAEXHH@Z 1000e1d8 f   qt-mt323:qt-mt323.dll
 0001:0000d1de       ?setColumnAlignment@QListView@@UAEXHH@Z 1000e1de f   qt-mt323:qt-mt323.dll
 0001:0000d1e4       ?setColumnLayout@QGroupBox@@UAEXHW4Orientation@Qt@@@Z 1000e1e4 f   qt-mt323:qt-mt323.dll
 0001:0000d1ea       ?setColumnText@QListView@@UAEXHABVQIconSet@@ABVQString@@@Z 1000e1ea f   qt-mt323:qt-mt323.dll
 0001:0000d1f0       ?setColumnText@QListView@@UAEXHABVQString@@@Z 1000e1f0 f   qt-mt323:qt-mt323.dll
 0001:0000d1f6       ?setColumnWidth@QListView@@UAEXHH@Z 1000e1f6 f   qt-mt323:qt-mt323.dll
 0001:0000d1fc       ?setColumnWidthMode@QListView@@UAEXHW4WidthMode@1@@Z 1000e1fc f   qt-mt323:qt-mt323.dll
 0001:0000d202       ?setContentsPos@QListView@@UAEXHH@Z 1000e202 f   qt-mt323:qt-mt323.dll
 0001:0000d208       ?setCornerWidget@QScrollView@@UAEXPAVQWidget@@@Z 1000e208 f   qt-mt323:qt-mt323.dll
 0001:0000d20e       ?setCurrentItem@QComboBox@@UAEXH@Z 1000e20e f   qt-mt323:qt-mt323.dll
 0001:0000d214       ?setCurrentItem@QListView@@UAEXPAVQListViewItem@@@Z 1000e214 f   qt-mt323:qt-mt323.dll
 0001:0000d21a       ?setCurrentText@QComboBox@@UAEXABVQString@@@Z 1000e21a f   qt-mt323:qt-mt323.dll
 0001:0000d220       ?setCursorPosition@QLineEdit@@UAEXH@Z 1000e220 f   qt-mt323:qt-mt323.dll
 0001:0000d226       ?setDefault@QPushButton@@UAEX_N@Z 1000e226 f   qt-mt323:qt-mt323.dll
 0001:0000d22c       ?setDefaultRenameAction@QListView@@UAEXW4RenameAction@1@@Z 1000e22c f   qt-mt323:qt-mt323.dll
 0001:0000d232       ?setDown@QButton@@UAEX_N@Z 1000e232 f   qt-mt323:qt-mt323.dll
 0001:0000d238       ?setDragAutoScroll@QScrollView@@UAEX_N@Z 1000e238 f   qt-mt323:qt-mt323.dll
 0001:0000d23e       ?setDragEnabled@QLineEdit@@UAEX_N@Z 1000e23e f   qt-mt323:qt-mt323.dll
 0001:0000d244       ?setEchoMode@QLineEdit@@UAEXW4EchoMode@1@@Z 1000e244 f   qt-mt323:qt-mt323.dll
 0001:0000d24a       ?setEditText@QComboBox@@UAEXABVQString@@@Z 1000e24a f   qt-mt323:qt-mt323.dll
 0001:0000d250       ?setEnabled@QComboBox@@UAEX_N@Z 1000e250 f   qt-mt323:qt-mt323.dll
 0001:0000d256       ?setEnabled@QGroupBox@@UAEX_N@Z 1000e256 f   qt-mt323:qt-mt323.dll
 0001:0000d25c       ?setEnabled@QScrollView@@UAEX_N@Z 1000e25c f   qt-mt323:qt-mt323.dll
 0001:0000d262       ?setEnabled@QSpinBox@@UAEX_N@Z 1000e262 f   qt-mt323:qt-mt323.dll
 0001:0000d268       ?setFont@QComboBox@@UAEXABVQFont@@@Z 1000e268 f   qt-mt323:qt-mt323.dll
 0001:0000d26e       ?setFont@QLabel@@UAEXABVQFont@@@Z 1000e26e f   qt-mt323:qt-mt323.dll
 0001:0000d274       ?setFont@QLineEdit@@UAEXABVQFont@@@Z 1000e274 f   qt-mt323:qt-mt323.dll
 0001:0000d27a       ?setFont@QListView@@UAEXABVQFont@@@Z 1000e27a f   qt-mt323:qt-mt323.dll
 0001:0000d280       ?setFrame@QLineEdit@@UAEX_N@Z 1000e280 f   qt-mt323:qt-mt323.dll
 0001:0000d286       ?setFrameRect@QWidgetStack@@UAEXABVQRect@@@Z 1000e286 f   qt-mt323:qt-mt323.dll
 0001:0000d28c       ?setGeometry@QBoxLayout@@UAEXABVQRect@@@Z 1000e28c f   qt-mt323:qt-mt323.dll
 0001:0000d292       ?setGeometry@QGridLayout@@UAEXABVQRect@@@Z 1000e292 f   qt-mt323:qt-mt323.dll
 0001:0000d298       ?setGeometry@QPushButton@@UAEXABVQRect@@@Z 1000e298 f   qt-mt323:qt-mt323.dll
 0001:0000d29e       ?setGeometry@QPushButton@@UAEXHHHH@Z 1000e29e f   qt-mt323:qt-mt323.dll
 0001:0000d2a4       ?setGeometry@QSpacerItem@@UAEXABVQRect@@@Z 1000e2a4 f   qt-mt323:qt-mt323.dll
 0001:0000d2aa       ?setGroup@QButton@@EAEXPAVQButtonGroup@@@Z 1000e2aa f   qt-mt323:qt-mt323.dll
 0001:0000d2b0       ?setHBarGeometry@QScrollView@@MAEXAAVQScrollBar@@HHHH@Z 1000e2b0 f   qt-mt323:qt-mt323.dll
 0001:0000d2b6       ?setHScrollBarMode@QScrollView@@UAEXW4ScrollBarMode@1@@Z 1000e2b6 f   qt-mt323:qt-mt323.dll
 0001:0000d2bc       ?setInsertionPolicy@QComboBox@@UAEXW4Policy@1@@Z 1000e2bc f   qt-mt323:qt-mt323.dll
 0001:0000d2c2       ?setIsMenuButton@QPushButton@@UAEX_N@Z 1000e2c2 f   qt-mt323:qt-mt323.dll
 0001:0000d2c8       ?setItemMargin@QListView@@UAEXH@Z 1000e2c8 f   qt-mt323:qt-mt323.dll
 0001:0000d2ce       ?setLineEdit@QComboBox@@UAEXPAVQLineEdit@@@Z 1000e2ce f   qt-mt323:qt-mt323.dll
 0001:0000d2d4       ?setListBox@QComboBox@@UAEXPAVQListBox@@@Z 1000e2d4 f   qt-mt323:qt-mt323.dll
 0001:0000d2da       ?setMargin@QLayout@@UAEXH@Z 1000e2da f   qt-mt323:qt-mt323.dll
 0001:0000d2e0       ?setMargins@QScrollView@@MAEXHHHH@Z 1000e2e0 f   qt-mt323:qt-mt323.dll
 0001:0000d2e6       ?setMaxCount@QComboBox@@UAEXH@Z 1000e2e6 f   qt-mt323:qt-mt323.dll
 0001:0000d2ec       ?setMaxLength@QLineEdit@@UAEXH@Z 1000e2ec f   qt-mt323:qt-mt323.dll
 0001:0000d2f2       ?setMenuBar@QLayout@@UAEXPAVQMenuBar@@@Z 1000e2f2 f   qt-mt323:qt-mt323.dll
 0001:0000d2f8       ?setMovie@QLabel@@UAEXABVQMovie@@@Z 1000e2f8 f   qt-mt323:qt-mt323.dll
 0001:0000d2fe       ?setMultiSelection@QListView@@UAEX_N@Z 1000e2fe f   qt-mt323:qt-mt323.dll
 0001:0000d304       ?setNum@QLabel@@UAEXH@Z    1000e304 f   qt-mt323:qt-mt323.dll
 0001:0000d30a       ?setNum@QLabel@@UAEXN@Z    1000e30a f   qt-mt323:qt-mt323.dll
 0001:0000d310       ?setOn@QPushButton@@UAEX_N@Z 1000e310 f   qt-mt323:qt-mt323.dll
 0001:0000d316       ?setOpen@QListView@@UAEXPAVQListViewItem@@_N@Z 1000e316 f   qt-mt323:qt-mt323.dll
 0001:0000d31c       ?setPalette@QComboBox@@UAEXABVQPalette@@@Z 1000e31c f   qt-mt323:qt-mt323.dll
 0001:0000d322       ?setPalette@QLineEdit@@UAEXABVQPalette@@@Z 1000e322 f   qt-mt323:qt-mt323.dll
 0001:0000d328       ?setPalette@QListView@@UAEXABVQPalette@@@Z 1000e328 f   qt-mt323:qt-mt323.dll
 0001:0000d32e       ?setPicture@QLabel@@UAEXABVQPicture@@@Z 1000e32e f   qt-mt323:qt-mt323.dll
 0001:0000d334       ?setPixmap@QButton@@UAEXABVQPixmap@@@Z 1000e334 f   qt-mt323:qt-mt323.dll
 0001:0000d33a       ?setPixmap@QLabel@@UAEXABVQPixmap@@@Z 1000e33a f   qt-mt323:qt-mt323.dll
 0001:0000d340       ?setPrefix@QSpinBox@@UAEXABVQString@@@Z 1000e340 f   qt-mt323:qt-mt323.dll
 0001:0000d346       ?setReadOnly@QLineEdit@@UAEX_N@Z 1000e346 f   qt-mt323:qt-mt323.dll
 0001:0000d34c       ?setResizeMode@QListView@@UAEXW4ResizeMode@1@@Z 1000e34c f   qt-mt323:qt-mt323.dll
 0001:0000d352       ?setResizePolicy@QScrollView@@UAEXW4ResizePolicy@1@@Z 1000e352 f   qt-mt323:qt-mt323.dll
 0001:0000d358       ?setRootIsDecorated@QListView@@UAEX_N@Z 1000e358 f   qt-mt323:qt-mt323.dll
 0001:0000d35e       ?setRowStretch@QGridLayout@@UAEXHH@Z 1000e35e f   qt-mt323:qt-mt323.dll
 0001:0000d364       ?setSelected@QListView@@UAEXPAVQListViewItem@@_N@Z 1000e364 f   qt-mt323:qt-mt323.dll
 0001:0000d36a       ?setSelection@QLineEdit@@UAEXHH@Z 1000e36a f   qt-mt323:qt-mt323.dll
 0001:0000d370       ?setShowSortIndicator@QListView@@UAEX_N@Z 1000e370 f   qt-mt323:qt-mt323.dll
 0001:0000d376       ?setShowToolTips@QListView@@UAEX_N@Z 1000e376 f   qt-mt323:qt-mt323.dll
 0001:0000d37c       ?setSizeLimit@QComboBox@@UAEXH@Z 1000e37c f   qt-mt323:qt-mt323.dll
 0001:0000d382       ?setSorting@QListView@@UAEXH_N@Z 1000e382 f   qt-mt323:qt-mt323.dll
 0001:0000d388       ?setSpacing@QLayout@@UAEXH@Z 1000e388 f   qt-mt323:qt-mt323.dll
 0001:0000d38e       ?setSpecialValueText@QSpinBox@@UAEXABVQString@@@Z 1000e38e f   qt-mt323:qt-mt323.dll
 0001:0000d394       ?setState@QButton@@MAEXW4ToggleState@1@@Z 1000e394 f   qt-mt323:qt-mt323.dll
 0001:0000d39a       ?setSuffix@QSpinBox@@UAEXABVQString@@@Z 1000e39a f   qt-mt323:qt-mt323.dll
 0001:0000d3a0       ?setText@QButton@@UAEXABVQString@@@Z 1000e3a0 f   qt-mt323:qt-mt323.dll
 0001:0000d3a6       ?setText@QLabel@@UAEXABVQString@@@Z 1000e3a6 f   qt-mt323:qt-mt323.dll
 0001:0000d3ac       ?setText@QLineEdit@@UAEXABVQString@@@Z 1000e3ac f   qt-mt323:qt-mt323.dll
 0001:0000d3b2       ?setTitle@QGroupBox@@UAEXABVQString@@@Z 1000e3b2 f   qt-mt323:qt-mt323.dll
 0001:0000d3b8       ?setToggleType@QButton@@MAEXW4ToggleType@1@@Z 1000e3b8 f   qt-mt323:qt-mt323.dll
 0001:0000d3be       ?setTreeStepSize@QListView@@UAEXH@Z 1000e3be f   qt-mt323:qt-mt323.dll
 0001:0000d3c4       ?setVBarGeometry@QScrollView@@MAEXAAVQScrollBar@@HHHH@Z 1000e3c4 f   qt-mt323:qt-mt323.dll
 0001:0000d3ca       ?setVScrollBarMode@QScrollView@@UAEXW4ScrollBarMode@1@@Z 1000e3ca f   qt-mt323:qt-mt323.dll
 0001:0000d3d0       ?setValidator@QComboBox@@UAEXPBVQValidator@@@Z 1000e3d0 f   qt-mt323:qt-mt323.dll
 0001:0000d3d6       ?setValidator@QLineEdit@@UAEXPBVQValidator@@@Z 1000e3d6 f   qt-mt323:qt-mt323.dll
 0001:0000d3dc       ?setValidator@QSpinBox@@UAEXPBVQValidator@@@Z 1000e3dc f   qt-mt323:qt-mt323.dll
 0001:0000d3e2       ?setValue@QSpinBox@@UAEXH@Z 1000e3e2 f   qt-mt323:qt-mt323.dll
 0001:0000d3e8       ?setWrapping@QSpinBox@@UAEX_N@Z 1000e3e8 f   qt-mt323:qt-mt323.dll
 0001:0000d3ee       ?show@QListView@@UAEXXZ    1000e3ee f   qt-mt323:qt-mt323.dll
 0001:0000d3f4       ?show@QWidgetStack@@UAEXXZ 1000e3f4 f   qt-mt323:qt-mt323.dll
 0001:0000d3fa       ?showEvent@QListView@@MAEXPAVQShowEvent@@@Z 1000e3fa f   qt-mt323:qt-mt323.dll
 0001:0000d400       ?sizeHint@QBoxLayout@@UBE?AVQSize@@XZ 1000e400 f   qt-mt323:qt-mt323.dll
 0001:0000d406       ?sizeHint@QCheckBox@@UBE?AVQSize@@XZ 1000e406 f   qt-mt323:qt-mt323.dll
 0001:0000d40c       ?sizeHint@QComboBox@@UBE?AVQSize@@XZ 1000e40c f   qt-mt323:qt-mt323.dll
 0001:0000d412       ?sizeHint@QGridLayout@@UBE?AVQSize@@XZ 1000e412 f   qt-mt323:qt-mt323.dll
 0001:0000d418       ?sizeHint@QGroupBox@@UBE?AVQSize@@XZ 1000e418 f   qt-mt323:qt-mt323.dll
 0001:0000d41e       ?sizeHint@QLabel@@UBE?AVQSize@@XZ 1000e41e f   qt-mt323:qt-mt323.dll
 0001:0000d424       ?sizeHint@QLineEdit@@UBE?AVQSize@@XZ 1000e424 f   qt-mt323:qt-mt323.dll
 0001:0000d42a       ?sizeHint@QListView@@UBE?AVQSize@@XZ 1000e42a f   qt-mt323:qt-mt323.dll
 0001:0000d430       ?sizeHint@QPushButton@@UBE?AVQSize@@XZ 1000e430 f   qt-mt323:qt-mt323.dll
 0001:0000d436       ?sizeHint@QSpacerItem@@UBE?AVQSize@@XZ 1000e436 f   qt-mt323:qt-mt323.dll
 0001:0000d43c       ?sizeHint@QSpinBox@@UBE?AVQSize@@XZ 1000e43c f   qt-mt323:qt-mt323.dll
 0001:0000d442       ?sizeHint@QWidgetStack@@UBE?AVQSize@@XZ 1000e442 f   qt-mt323:qt-mt323.dll
 0001:0000d448       ?sort@QListView@@UAEXXZ    1000e448 f   qt-mt323:qt-mt323.dll
 0001:0000d44e       ?spacerItem@QLayoutItem@@UAEPAVQSpacerItem@@XZ 1000e44e f   qt-mt323:qt-mt323.dll
 0001:0000d454       ?spacerItem@QSpacerItem@@UAEPAV1@XZ 1000e454 f   qt-mt323:qt-mt323.dll
 0001:0000d45a       ?startDrag@QListView@@MAEXXZ 1000e45a f   qt-mt323:qt-mt323.dll
 0001:0000d460       ?stepChange@QRangeControl@@MAEXXZ 1000e460 f   qt-mt323:qt-mt323.dll
 0001:0000d466       ?stepDown@QSpinBox@@UAEXXZ 1000e466 f   qt-mt323:qt-mt323.dll
 0001:0000d46c       ?stepUp@QSpinBox@@UAEXXZ   1000e46c f   qt-mt323:qt-mt323.dll
 0001:0000d472       ?styleChange@QComboBox@@MAEXAAVQStyle@@@Z 1000e472 f   qt-mt323:qt-mt323.dll
 0001:0000d478       ?styleChange@QListView@@MAEXAAVQStyle@@@Z 1000e478 f   qt-mt323:qt-mt323.dll
 0001:0000d47e       ?styleChange@QSpinBox@@MAEXAAVQStyle@@@Z 1000e47e f   qt-mt323:qt-mt323.dll
 0001:0000d484       ?suffix@QSpinBox@@UBE?AVQString@@XZ 1000e484 f   qt-mt323:qt-mt323.dll
 0001:0000d48a       ?takeItem@QListView@@UAEXPAVQListViewItem@@@Z 1000e48a f   qt-mt323:qt-mt323.dll
 0001:0000d490       ?undo@QLineEdit@@UAEXXZ    1000e490 f   qt-mt323:qt-mt323.dll
 0001:0000d496       ?updateDisplay@QSpinBox@@MAEXXZ 1000e496 f   qt-mt323:qt-mt323.dll
 0001:0000d49c       ?updateMask@QCheckBox@@MAEXXZ 1000e49c f   qt-mt323:qt-mt323.dll
 0001:0000d4a2       ?updateMask@QComboBox@@MAEXXZ 1000e4a2 f   qt-mt323:qt-mt323.dll
 0001:0000d4a8       ?updateMask@QPushButton@@MAEXXZ 1000e4a8 f   qt-mt323:qt-mt323.dll
 0001:0000d4ae       ?valueChange@QSpinBox@@MAEXXZ 1000e4ae f   qt-mt323:qt-mt323.dll
 0001:0000d4b4       ?viewportContextMenuEvent@QScrollView@@MAEXPAVQContextMenuEvent@@@Z 1000e4b4 f   qt-mt323:qt-mt323.dll
 0001:0000d4ba       ?viewportDragEnterEvent@QScrollView@@MAEXPAVQDragEnterEvent@@@Z 1000e4ba f   qt-mt323:qt-mt323.dll
 0001:0000d4c0       ?viewportDragLeaveEvent@QScrollView@@MAEXPAVQDragLeaveEvent@@@Z 1000e4c0 f   qt-mt323:qt-mt323.dll
 0001:0000d4c6       ?viewportDragMoveEvent@QScrollView@@MAEXPAVQDragMoveEvent@@@Z 1000e4c6 f   qt-mt323:qt-mt323.dll
 0001:0000d4cc       ?viewportDropEvent@QScrollView@@MAEXPAVQDropEvent@@@Z 1000e4cc f   qt-mt323:qt-mt323.dll
 0001:0000d4d2       ?viewportMouseDoubleClickEvent@QScrollView@@MAEXPAVQMouseEvent@@@Z 1000e4d2 f   qt-mt323:qt-mt323.dll
 0001:0000d4d8       ?viewportMouseMoveEvent@QScrollView@@MAEXPAVQMouseEvent@@@Z 1000e4d8 f   qt-mt323:qt-mt323.dll
 0001:0000d4de       ?viewportMousePressEvent@QScrollView@@MAEXPAVQMouseEvent@@@Z 1000e4de f   qt-mt323:qt-mt323.dll
 0001:0000d4e4       ?viewportMouseReleaseEvent@QScrollView@@MAEXPAVQMouseEvent@@@Z 1000e4e4 f   qt-mt323:qt-mt323.dll
 0001:0000d4ea       ?viewportPaintEvent@QScrollView@@MAEXPAVQPaintEvent@@@Z 1000e4ea f   qt-mt323:qt-mt323.dll
 0001:0000d4f0       ?viewportResizeEvent@QListView@@MAEXPAVQResizeEvent@@@Z 1000e4f0 f   qt-mt323:qt-mt323.dll
 0001:0000d4f6       ?viewportWheelEvent@QScrollView@@MAEXPAVQWheelEvent@@@Z 1000e4f6 f   qt-mt323:qt-mt323.dll
 0001:0000d4fc       ?wheelEvent@QComboBox@@MAEXPAVQWheelEvent@@@Z 1000e4fc f   qt-mt323:qt-mt323.dll
 0001:0000d502       ?wheelEvent@QScrollView@@MAEXPAVQWheelEvent@@@Z 1000e502 f   qt-mt323:qt-mt323.dll
 0001:0000d508       ?wheelEvent@QSpinBox@@MAEXPAVQWheelEvent@@@Z 1000e508 f   qt-mt323:qt-mt323.dll
 0001:0000d50e       ?widget@QLayoutItem@@UAEPAVQWidget@@XZ 1000e50e f   qt-mt323:qt-mt323.dll
 0001:0000d514       ?windowActivationChange@QLineEdit@@MAEX_N@Z 1000e514 f   qt-mt323:qt-mt323.dll
 0001:0000d51a       ?windowActivationChange@QListView@@MAEX_N@Z 1000e51a f   qt-mt323:qt-mt323.dll
 0001:0000d520       ?addTab@QTabWidget@@UAEXPAVQWidget@@ABVQIconSet@@ABVQString@@@Z 1000e520 f   qt-mt323:qt-mt323.dll
 0001:0000d526       ?addTab@QTabWidget@@UAEXPAVQWidget@@ABVQString@@@Z 1000e526 f   qt-mt323:qt-mt323.dll
 0001:0000d52c       ?addTab@QTabWidget@@UAEXPAVQWidget@@PAVQTab@@@Z 1000e52c f   qt-mt323:qt-mt323.dll
 0001:0000d532       ?className@QTabWidget@@UBEPBDXZ 1000e532 f   qt-mt323:qt-mt323.dll
 0001:0000d538       ?eventFilter@QTabWidget@@MAE_NPAVQObject@@PAVQEvent@@@Z 1000e538 f   qt-mt323:qt-mt323.dll
 0001:0000d53e       ?insertTab@QTabWidget@@UAEXPAVQWidget@@ABVQIconSet@@ABVQString@@H@Z 1000e53e f   qt-mt323:qt-mt323.dll
 0001:0000d544       ?insertTab@QTabWidget@@UAEXPAVQWidget@@ABVQString@@H@Z 1000e544 f   qt-mt323:qt-mt323.dll
 0001:0000d54a       ?insertTab@QTabWidget@@UAEXPAVQWidget@@PAVQTab@@H@Z 1000e54a f   qt-mt323:qt-mt323.dll
 0001:0000d550       ?metaObject@QTabWidget@@UBEPAVQMetaObject@@XZ 1000e550 f   qt-mt323:qt-mt323.dll
 0001:0000d556       ?minimumSizeHint@QTabWidget@@UBE?AVQSize@@XZ 1000e556 f   qt-mt323:qt-mt323.dll
 0001:0000d55c       ?qt_cast@QTabWidget@@UAEPAXPBD@Z 1000e55c f   qt-mt323:qt-mt323.dll
 0001:0000d562       ?qt_emit@QTabWidget@@UAE_NHPAUQUObject@@@Z 1000e562 f   qt-mt323:qt-mt323.dll
 0001:0000d568       ?qt_invoke@QTabWidget@@UAE_NHPAUQUObject@@@Z 1000e568 f   qt-mt323:qt-mt323.dll
 0001:0000d56e       ?qt_property@QTabWidget@@UAE_NHHPAVQVariant@@@Z 1000e56e f   qt-mt323:qt-mt323.dll
 0001:0000d574       ?removePage@QTabWidget@@UAEXPAVQWidget@@@Z 1000e574 f   qt-mt323:qt-mt323.dll
 0001:0000d57a       ?resizeEvent@QTabWidget@@MAEXPAVQResizeEvent@@@Z 1000e57a f   qt-mt323:qt-mt323.dll
 0001:0000d580       ?showEvent@QTabWidget@@MAEXPAVQShowEvent@@@Z 1000e580 f   qt-mt323:qt-mt323.dll
 0001:0000d586       ?showPage@QTabWidget@@UAEXPAVQWidget@@@Z 1000e586 f   qt-mt323:qt-mt323.dll
 0001:0000d58c       ?sizeHint@QTabWidget@@UBE?AVQSize@@XZ 1000e58c f   qt-mt323:qt-mt323.dll
 0001:0000d592       ?styleChange@QTabWidget@@MAEXAAVQStyle@@@Z 1000e592 f   qt-mt323:qt-mt323.dll
 0001:0000d598       ?updateMask@QTabWidget@@MAEXXZ 1000e598 f   qt-mt323:qt-mt323.dll
 0001:0000d59e       ??0cfg_ListView@@QAE@ABV0@@Z 1000e59e f i cfg_widgets001:cfg_ListView.obj
 0001:0000d5e8       ??0cfg_ListView@@QAE@PAVQWidget@@PBD@Z 1000e5e8 f   cfg_widgets001:cfg_ListView.obj
 0001:0000d6a6       ??1cfg_ListView@@UAE@XZ    1000e6a6 f   cfg_widgets001:cfg_ListView.obj
 0001:0000d6fc       ??4cfg_ListView@@QAEAAV0@ABV0@@Z 1000e6fc f i cfg_widgets001:cfg_ListView.obj
 0001:0000d751       ??_Ecfg_ListView@@UAEPAXI@Z 1000e751 f i cfg_widgets001:cfg_ListView.obj
 0001:0000d79e       ??_Ecfg_ListView@@WCI@AEPAXI@Z 1000e79e f i cfg_widgets001:cfg_ListView.obj
 0001:0000d7a6       ??_Fcfg_ListView@@QAEXXZ   1000e7a6 f i cfg_widgets001:cfg_ListView.obj
 0001:0000d7b0       ?clearUndo@cfg_ListView@@AAEXXZ 1000e7b0 f   cfg_widgets001:cfg_ListView.obj
 0001:0000d7ee       ?clipBoardDataChanged@cfg_ListView@@IAEXXZ 1000e7ee f   cfg_widgets001:cfg_ListView.obj
 0001:0000d842       ?copyToClipboard@cfg_ListView@@QAEXXZ 1000e842 f   cfg_widgets001:cfg_ListView.obj
 0001:0000d971       ?deleteItems@cfg_ListView@@QAEXXZ 1000e971 f   cfg_widgets001:cfg_ListView.obj
 0001:0000da5c       ?insertData@cfg_ListView@@QAEXXZ 1000ea5c f   cfg_widgets001:cfg_ListView.obj
 0001:0000dbf7       ?metaObject@cfg_ListView@@UBEPAVQMetaObject@@XZ 1000ebf7 f i cfg_widgets001:cfg_ListView.obj
 0001:0000dbfc       ?newItem@cfg_ListView@@MAEPAVQListViewItem@@PAVQListView@@PAV2@@Z 1000ebfc f   cfg_widgets001:cfg_ListView.obj
 0001:0000dc3f       ?qObject@cfg_ListView@@QAEPAVQObject@@XZ 1000ec3f f i cfg_widgets001:cfg_ListView.obj
 0001:0000dc42       ?replaceData@cfg_ListView@@QAEXXZ 1000ec42 f   cfg_widgets001:cfg_ListView.obj
 0001:0000df80       ?undoPaste@cfg_ListView@@QAEXXZ 1000ef80 f   cfg_widgets001:cfg_ListView.obj
 0001:0000dfeb       ?updateEntry@cfg_ListView@@AAEPAVQListViewItem@@QAV2@ABVQString@@_N@Z 1000efeb f   cfg_widgets001:cfg_ListView.obj
 0001:0000e127       ?validateRow@cfg_ListView@@MAEHPAVQListViewItem@@@Z 1000f127 f   cfg_widgets001:cfg_ListView.obj
 0001:0000e139       ?className@cfg_ListView@@UBEPBDXZ 1000f139 f   cfg_widgets001:moc_cfg_ListView.obj
 0001:0000e13f       ?clipboardDataValid@cfg_ListView@@IAEX_N@Z 1000f13f f   cfg_widgets001:moc_cfg_ListView.obj
 0001:0000e15f       ?dataPasted@cfg_ListView@@IAEXXZ 1000f15f f   cfg_widgets001:moc_cfg_ListView.obj
 0001:0000e174       ?qt_cast@cfg_ListView@@UAEPAXPBD@Z 1000f174 f   cfg_widgets001:moc_cfg_ListView.obj
 0001:0000e1a2       ?qt_emit@cfg_ListView@@UAE_NHPAUQUObject@@@Z 1000f1a2 f   cfg_widgets001:moc_cfg_ListView.obj
 0001:0000e1e6       ?qt_invoke@cfg_ListView@@UAE_NHPAUQUObject@@@Z 1000f1e6 f   cfg_widgets001:moc_cfg_ListView.obj
 0001:0000e24a       ?qt_property@cfg_ListView@@UAE_NHHPAVQVariant@@@Z 1000f24a f   cfg_widgets001:moc_cfg_ListView.obj
 0001:0000e254       ?staticMetaObject@cfg_ListView@@SAPAVQMetaObject@@XZ 1000f254 f   cfg_widgets001:moc_cfg_ListView.obj
 0001:0000e2d3       ?tr@cfg_ListView@@SA?AVQString@@PBD0@Z 1000f2d3 f   cfg_widgets001:moc_cfg_ListView.obj
 0001:0000e316       ?trUtf8@cfg_ListView@@SA?AVQString@@PBD0@Z 1000f316 f   cfg_widgets001:moc_cfg_ListView.obj
 0001:0000e35a       ??2@YAPAXI@Z               1000f35a f   MSVCRT:MSVCR120.dll
 0001:0000e360       ??3@YAXPAX@Z               1000f360 f   MSVCRT:MSVCR120.dll
 0001:0000e366       @__security_check_cookie@4 1000f366 f   MSVCRT:secchk.obj
 0001:0000e375       __EH_epilog3               1000f375 f   MSVCRT:ehprolg3.obj
 0001:0000e389       __EH_epilog3_GS            1000f389 f   MSVCRT:ehprolg3.obj
 0001:0000e398       __EH_prolog3               1000f398 f   MSVCRT:ehprolg3.obj
 0001:0000e3cb       __EH_prolog3_GS            1000f3cb f   MSVCRT:ehprolg3.obj
 0001:0000e402       ___CxxFrameHandler3        1000f402 f   MSVCRT:MSVCR120.dll
 0001:0000e408       ??_Etype_info@@UAEPAXI@Z   1000f408 f i MSVCRT:ti_inst.obj
 0001:0000e460       __purecall                 1000f460 f   MSVCRT:MSVCR120.dll
 0001:0000e466       ??_L@YGXPAXIHP6EX0@Z1@Z    1000f466 f   MSVCRT:ehvecctr.obj
 0001:0000e4c8       ??_M@YGXPAXIHP6EX0@Z@Z     1000f4c8 f   MSVCRT:ehvecdtr.obj
 0001:0000e537       ?__ArrayUnwind@@YGXPAXIHP6EX0@Z@Z 1000f537 f   MSVCRT:ehvecdtr.obj
 0001:0000e595       ___atonexitinit            1000f595 f   MSVCRT:atonexit.obj
 0001:0000e5d1       __onexit                   1000f5d1 f   MSVCRT:atonexit.obj
 0001:0000e67a       _atexit                    1000f67a f   MSVCRT:atonexit.obj
 0001:0000e6db       __CRT_INIT@12              1000f6db f   MSVCRT:crtdll.obj
 0001:0000e8d2       __DllMainCRTStartup@12     1000f8d2 f   MSVCRT:crtdll.obj
 0001:0000ea28       ___raise_securityfailure   1000fa28 f   MSVCRT:gs_report.obj
 0001:0000ea65       ___report_gsfailure        1000fa65 f   MSVCRT:gs_report.obj
 0001:0000eb60       ??1type_info@@UAE@XZ       1000fb60 f   MSVCRT:MSVCR120.dll
 0001:0000eb70       __SEH_prolog4              1000fb70 f   MSVCRT:sehprolg4.obj
 0001:0000ebb5       __SEH_epilog4              1000fbb5 f   MSVCRT:sehprolg4.obj
 0001:0000ebc9       __except_handler4          1000fbc9 f   MSVCRT:chandler4gs.obj
 0001:0000ebec       ?terminate@@YAXXZ          1000fbec f   MSVCRT:MSVCR120.dll
 0001:0000ebf2       __lock                     1000fbf2 f   MSVCRT:MSVCR120.dll
 0001:0000ebf8       __unlock                   1000fbf8 f   MSVCRT:MSVCR120.dll
 0001:0000ebfe       ___dllonexit               1000fbfe f   MSVCRT:MSVCR120.dll
 0001:0000ec04       ___CppXcptFilter           1000fc04 f   MSVCRT:MSVCR120.dll
 0001:0000ec0a       __amsg_exit                1000fc0a f   MSVCRT:MSVCR120.dll
 0001:0000ec10       __FindPESection            1000fc10 f   MSVCRT:pesect.obj
 0001:0000ec60       __IsNonwritableInCurrentImage 1000fc60 f   MSVCRT:pesect.obj
 0001:0000ed20       __ValidateImageBase        1000fd20 f   MSVCRT:pesect.obj
 0001:0000ed51       ___security_init_cookie    1000fd51 f   MSVCRT:gs_support.obj
 0001:0000eded       _DllMain@12                1000fded f   MSVCRT:dllmain.obj
 0001:0000ee0f       __RTC_Initialize           1000fe0f f   MSVCRT:initsect.obj
 0001:0000ee2f       __RTC_Terminate            1000fe2f f   MSVCRT:initsect.obj
 0001:0000ee50       __initterm                 1000fe50 f   MSVCRT:MSVCR120.dll
 0001:0000ee56       __initterm_e               1000fe56 f   MSVCRT:MSVCR120.dll
 0001:0000ee5c       ___clean_type_info_names   1000fe5c f   MSVCRT:tncleanup.obj
 0001:0000ee68       __crt_debugger_hook        1000fe68 f   MSVCRT:MSVCR120.dll
 0001:0000ee6e       ___crtUnhandledException   1000fe6e f   MSVCRT:MSVCR120.dll
 0001:0000ee74       ___crtTerminateProcess     1000fe74 f   MSVCRT:MSVCR120.dll
 0001:0000ee7a       __except_handler4_common   1000fe7a f   MSVCRT:MSVCR120.dll
 0001:0000ee80       ___clean_type_info_names_internal 1000fe80 f   MSVCRT:MSVCR120.dll
 0001:0000ee86       _IsProcessorFeaturePresent@4 1000fe86 f   kernel32:KERNEL32.dll
 0002:00000000       __imp__DecodePointer@4     10013000     kernel32:KERNEL32.dll
 0002:00000004       __imp__DisableThreadLibraryCalls@4 10013004     kernel32:KERNEL32.dll
 0002:00000008       __imp__GetSystemTimeAsFileTime@4 10013008     kernel32:KERNEL32.dll
 0002:0000000c       __imp__GetCurrentThreadId@0 1001300c     kernel32:KERNEL32.dll
 0002:00000010       __imp__GetCurrentProcessId@0 10013010     kernel32:KERNEL32.dll
 0002:00000014       __imp__QueryPerformanceCounter@4 10013014     kernel32:KERNEL32.dll
 0002:00000018       __imp__IsProcessorFeaturePresent@4 10013018     kernel32:KERNEL32.dll
 0002:0000001c       __imp__IsDebuggerPresent@0 1001301c     kernel32:KERNEL32.dll
 0002:00000020       __imp__EncodePointer@4     10013020     kernel32:KERNEL32.dll
 0002:00000024       \177KERNEL32_NULL_THUNK_DATA 10013024     kernel32:KERNEL32.dll
 0002:00000028       __imp_??3@YAXPAX@Z         10013028     MSVCRT:MSVCR120.dll
 0002:0000002c       __imp____clean_type_info_names_internal 1001302c     MSVCRT:MSVCR120.dll
 0002:00000030       __imp___except_handler4_common 10013030     MSVCRT:MSVCR120.dll
 0002:00000034       __imp____crtTerminateProcess 10013034     MSVCRT:MSVCR120.dll
 0002:00000038       __imp____crtUnhandledException 10013038     MSVCRT:MSVCR120.dll
 0002:0000003c       __imp___crt_debugger_hook  1001303c     MSVCRT:MSVCR120.dll
 0002:00000040       __imp___initterm_e         10013040     MSVCRT:MSVCR120.dll
 0002:00000044       __imp___initterm           10013044     MSVCRT:MSVCR120.dll
 0002:00000048       __imp___malloc_crt         10013048     MSVCRT:MSVCR120.dll
 0002:0000004c       __imp__free                1001304c     MSVCRT:MSVCR120.dll
 0002:00000050       __imp___amsg_exit          10013050     MSVCRT:MSVCR120.dll
 0002:00000054       __imp____CppXcptFilter     10013054     MSVCRT:MSVCR120.dll
 0002:00000058       __imp___onexit             10013058     MSVCRT:MSVCR120.dll
 0002:0000005c       __imp____dllonexit         1001305c     MSVCRT:MSVCR120.dll
 0002:00000060       __imp___calloc_crt         10013060     MSVCRT:MSVCR120.dll
 0002:00000064       __imp___unlock             10013064     MSVCRT:MSVCR120.dll
 0002:00000068       __imp___lock               10013068     MSVCRT:MSVCR120.dll
 0002:0000006c       __imp_?terminate@@YAXXZ    1001306c     MSVCRT:MSVCR120.dll
 0002:00000070       __imp_??1type_info@@UAE@XZ 10013070     MSVCRT:MSVCR120.dll
 0002:00000074       __imp___purecall           10013074     MSVCRT:MSVCR120.dll
 0002:00000078       __imp____CxxFrameHandler3  10013078     MSVCRT:MSVCR120.dll
 0002:0000007c       __imp_??2@YAPAXI@Z         1001307c     MSVCRT:MSVCR120.dll
 0002:00000080       \177MSVCR120_NULL_THUNK_DATA 10013080     MSVCRT:MSVCR120.dll
 0002:00000084       __imp_?fnConfig_icons@@YAPAPBDPBD@Z 10013084     config_icons:config_icons.dll
 0002:00000088       \177config_icons_NULL_THUNK_DATA 10013088     config_icons:config_icons.dll
 0002:0000008c       __imp_?rect@QWidget@@QBE?AVQRect@@XZ 1001308c     qt-mt323:qt-mt323.dll
 0002:00000090       __imp_?closeEvent@QWidget@@MAEXPAVQCloseEvent@@@Z 10013090     qt-mt323:qt-mt323.dll
 0002:00000094       __imp_?information@QMessageBox@@SAHPAVQWidget@@ABVQString@@1111HH@Z 10013094     qt-mt323:qt-mt323.dll
 0002:00000098       __imp_?critical@QMessageBox@@SAHPAVQWidget@@ABVQString@@1111HH@Z 10013098     qt-mt323:qt-mt323.dll
 0002:0000009c       __imp_??0QKeySequence@@QAE@H@Z 1001309c     qt-mt323:qt-mt323.dll
 0002:000000a0       __imp_??0QPixmap@@QAE@QAPBD@Z 100130a0     qt-mt323:qt-mt323.dll
 0002:000000a4       __imp_??1QPixmap@@UAE@XZ   100130a4     qt-mt323:qt-mt323.dll
 0002:000000a8       __imp_??0QIconSet@@QAE@ABVQPixmap@@W4Size@0@@Z 100130a8     qt-mt323:qt-mt323.dll
 0002:000000ac       __imp_??1QIconSet@@UAE@XZ  100130ac     qt-mt323:qt-mt323.dll
 0002:000000b0       __imp_??0QAction@@QAE@ABVQString@@ABVQIconSet@@0VQKeySequence@@PAVQObject@@PBD_N@Z 100130b0     qt-mt323:qt-mt323.dll
 0002:000000b4       __imp_??1QAction@@UAE@XZ   100130b4     qt-mt323:qt-mt323.dll
 0002:000000b8       __imp_??0QDockWindow@@QAE@PAVQWidget@@PBDI@Z 100130b8     qt-mt323:qt-mt323.dll
 0002:000000bc       __imp_??1QDockWindow@@UAE@XZ 100130bc     qt-mt323:qt-mt323.dll
 0002:000000c0       __imp_??1?$QPtrList@VQDockWindow@@@@UAE@XZ 100130c0     qt-mt323:qt-mt323.dll
 0002:000000c4       __imp_??0QToolBar@@QAE@PAVQMainWindow@@PBD@Z 100130c4     qt-mt323:qt-mt323.dll
 0002:000000c8       __imp_??1QToolBar@@UAE@XZ  100130c8     qt-mt323:qt-mt323.dll
 0002:000000cc       __imp_??0QFile@@QAE@ABVQString@@@Z 100130cc     qt-mt323:qt-mt323.dll
 0002:000000d0       __imp_??1QFile@@UAE@XZ     100130d0     qt-mt323:qt-mt323.dll
 0002:000000d4       __imp_?exists@QFile@@QBE_NXZ 100130d4     qt-mt323:qt-mt323.dll
 0002:000000d8       __imp_?remove@QFile@@QAE_NXZ 100130d8     qt-mt323:qt-mt323.dll
 0002:000000dc       __imp_??9QDateTime@@QBE_NABV0@@Z 100130dc     qt-mt323:qt-mt323.dll
 0002:000000e0       __imp_??0QFileInfo@@QAE@ABVQString@@@Z 100130e0     qt-mt323:qt-mt323.dll
 0002:000000e4       __imp_??1QFileInfo@@QAE@XZ 100130e4     qt-mt323:qt-mt323.dll
 0002:000000e8       __imp_?lastModified@QFileInfo@@QBE?AVQDateTime@@XZ 100130e8     qt-mt323:qt-mt323.dll
 0002:000000ec       __imp_??0QDir@@QAE@XZ      100130ec     qt-mt323:qt-mt323.dll
 0002:000000f0       __imp_??1QDir@@UAE@XZ      100130f0     qt-mt323:qt-mt323.dll
 0002:000000f4       __imp_?setPath@QDir@@UAEXABVQString@@@Z 100130f4     qt-mt323:qt-mt323.dll
 0002:000000f8       __imp_?mkdir@QDir@@UBE_NABVQString@@_N@Z 100130f8     qt-mt323:qt-mt323.dll
 0002:000000fc       __imp_?exists@QDir@@UBE_NXZ 100130fc     qt-mt323:qt-mt323.dll
 0002:00000100       __imp_??0QGuardedPtrPrivate@@QAE@PAVQObject@@@Z 10013100     qt-mt323:qt-mt323.dll
 0002:00000104       __imp_??1QGuardedPtrPrivate@@UAE@XZ 10013104     qt-mt323:qt-mt323.dll
 0002:00000108       __imp_?reconnect@QGuardedPtrPrivate@@QAEXPAVQObject@@@Z 10013108     qt-mt323:qt-mt323.dll
 0002:0000010c       __imp_??0QPopupMenu@@QAE@PAVQWidget@@PBD@Z 1001310c     qt-mt323:qt-mt323.dll
 0002:00000110       __imp_??1QPopupMenu@@UAE@XZ 10013110     qt-mt323:qt-mt323.dll
 0002:00000114       __imp_?look_string@QGDict@@QAEPAXABVQString@@PAXH@Z 10013114     qt-mt323:qt-mt323.dll
 0002:00000118       __imp_??0QGDict@@IAE@IW4KeyType@0@_N1@Z 10013118     qt-mt323:qt-mt323.dll
 0002:0000011c       __imp_??1QGDict@@MAE@XZ    1001311c     qt-mt323:qt-mt323.dll
 0002:00000120       __imp_?clear@QGDict@@MAEXXZ 10013120     qt-mt323:qt-mt323.dll
 0002:00000124       __imp_?activateItemAt@QPopupMenu@@UAEXH@Z 10013124     qt-mt323:qt-mt323.dll
 0002:00000128       __imp_?addTo@QAction@@UAE_NPAVQWidget@@@Z 10013128     qt-mt323:qt-mt323.dll
 0002:0000012c       __imp_?addedTo@QAction@@MAEXHPAVQPopupMenu@@@Z 1001312c     qt-mt323:qt-mt323.dll
 0002:00000130       __imp_?addedTo@QAction@@MAEXPAVQWidget@@0@Z 10013130     qt-mt323:qt-mt323.dll
 0002:00000134       __imp_?adjustSize@QWidget@@UAEXXZ 10013134     qt-mt323:qt-mt323.dll
 0002:00000138       __imp_?checkConnectArgs@QObject@@MAE_NPBDPBV1@0@Z 10013138     qt-mt323:qt-mt323.dll
 0002:0000013c       __imp_?childEvent@QObject@@MAEXPAVQChildEvent@@@Z 1001313c     qt-mt323:qt-mt323.dll
 0002:00000140       __imp_?className@QAction@@UBEPBDXZ 10013140     qt-mt323:qt-mt323.dll
 0002:00000144       __imp_?className@QDockWindow@@UBEPBDXZ 10013144     qt-mt323:qt-mt323.dll
 0002:00000148       __imp_?className@QGuardedPtrPrivate@@UBEPBDXZ 10013148     qt-mt323:qt-mt323.dll
 0002:0000014c       __imp_?className@QPopupMenu@@UBEPBDXZ 1001314c     qt-mt323:qt-mt323.dll
 0002:00000150       __imp_?className@QToolBar@@UBEPBDXZ 10013150     qt-mt323:qt-mt323.dll
 0002:00000154       __imp_?className@QWidget@@UBEPBDXZ 10013154     qt-mt323:qt-mt323.dll
 0002:00000158       __imp_?clear@?$QPtrList@VQDockWindow@@@@UAEXXZ 10013158     qt-mt323:qt-mt323.dll
 0002:0000015c       __imp_?clear@QToolBar@@UAEXXZ 1001315c     qt-mt323:qt-mt323.dll
 0002:00000160       __imp_?close@QWidget@@UAE_N_N@Z 10013160     qt-mt323:qt-mt323.dll
 0002:00000164       __imp_?closeEvent@QPopupMenu@@MAEXPAVQCloseEvent@@@Z 10013164     qt-mt323:qt-mt323.dll
 0002:00000168       __imp_?cmd@QPaintDevice@@MAE_NHPAVQPainter@@PATQPDevCmdParam@@@Z 10013168     qt-mt323:qt-mt323.dll
 0002:0000016c       __imp_?compareItems@QGList@@MAEHPAX0@Z 1001316c     qt-mt323:qt-mt323.dll
 0002:00000170       __imp_?connectNotify@QObject@@MAEXPBD@Z 10013170     qt-mt323:qt-mt323.dll
 0002:00000174       __imp_?contextMenuEvent@QDockWindow@@MAEXPAVQContextMenuEvent@@@Z 10013174     qt-mt323:qt-mt323.dll
 0002:00000178       __imp_?contextMenuEvent@QWidget@@MAEXPAVQContextMenuEvent@@@Z 10013178     qt-mt323:qt-mt323.dll
 0002:0000017c       __imp_?count@?$QPtrList@VQDockWindow@@@@UBEIXZ 1001317c     qt-mt323:qt-mt323.dll
 0002:00000180       __imp_?create@QWidget@@MAEXPAUHWND__@@_N1@Z 10013180     qt-mt323:qt-mt323.dll
 0002:00000184       __imp_?customEvent@QObject@@MAEXPAVQCustomEvent@@@Z 10013184     qt-mt323:qt-mt323.dll
 0002:00000188       __imp_?customWhatsThis@QPopupMenu@@UBE_NXZ 10013188     qt-mt323:qt-mt323.dll
 0002:0000018c       __imp_?customWhatsThis@QWidget@@UBE_NXZ 1001318c     qt-mt323:qt-mt323.dll
 0002:00000190       __imp_?deleteItem@?$QPtrList@VQDockWindow@@@@EAEXPAX@Z 10013190     qt-mt323:qt-mt323.dll
 0002:00000194       __imp_?destroy@QWidget@@MAEX_N0@Z 10013194     qt-mt323:qt-mt323.dll
 0002:00000198       __imp_?disconnectNotify@QObject@@MAEXPBD@Z 10013198     qt-mt323:qt-mt323.dll
 0002:0000019c       __imp_?dock@QDockWindow@@UAEXXZ 1001319c     qt-mt323:qt-mt323.dll
 0002:000001a0       __imp_?dragEnterEvent@QWidget@@MAEXPAVQDragEnterEvent@@@Z 100131a0     qt-mt323:qt-mt323.dll
 0002:000001a4       __imp_?dragLeaveEvent@QWidget@@MAEXPAVQDragLeaveEvent@@@Z 100131a4     qt-mt323:qt-mt323.dll
 0002:000001a8       __imp_?dragMoveEvent@QWidget@@MAEXPAVQDragMoveEvent@@@Z 100131a8     qt-mt323:qt-mt323.dll
 0002:000001ac       __imp_?drawContents@QDockWindow@@MAEXPAVQPainter@@@Z 100131ac     qt-mt323:qt-mt323.dll
 0002:000001b0       __imp_?drawContents@QPopupMenu@@MAEXPAVQPainter@@@Z 100131b0     qt-mt323:qt-mt323.dll
 0002:000001b4       __imp_?drawFrame@QDockWindow@@MAEXPAVQPainter@@@Z 100131b4     qt-mt323:qt-mt323.dll
 0002:000001b8       __imp_?drawFrame@QFrame@@MAEXPAVQPainter@@@Z 100131b8     qt-mt323:qt-mt323.dll
 0002:000001bc       __imp_?dropEvent@QWidget@@MAEXPAVQDropEvent@@@Z 100131bc     qt-mt323:qt-mt323.dll
 0002:000001c0       __imp_?enabledChange@QPopupMenu@@MAEX_N@Z 100131c0     qt-mt323:qt-mt323.dll
 0002:000001c4       __imp_?enabledChange@QWidget@@MAEX_N@Z 100131c4     qt-mt323:qt-mt323.dll
 0002:000001c8       __imp_?enterEvent@QWidget@@MAEXPAVQEvent@@@Z 100131c8     qt-mt323:qt-mt323.dll
 0002:000001cc       __imp_?event@QDockWindow@@MAE_NPAVQEvent@@@Z 100131cc     qt-mt323:qt-mt323.dll
 0002:000001d0       __imp_?event@QObject@@UAE_NPAVQEvent@@@Z 100131d0     qt-mt323:qt-mt323.dll
 0002:000001d4       __imp_?event@QToolBar@@UAE_NPAVQEvent@@@Z 100131d4     qt-mt323:qt-mt323.dll
 0002:000001d8       __imp_?event@QWidget@@MAE_NPAVQEvent@@@Z 100131d8     qt-mt323:qt-mt323.dll
 0002:000001dc       __imp_?eventFilter@QDockWindow@@UAE_NPAVQObject@@PAVQEvent@@@Z 100131dc     qt-mt323:qt-mt323.dll
 0002:000001e0       __imp_?eventFilter@QObject@@UAE_NPAV1@PAVQEvent@@@Z 100131e0     qt-mt323:qt-mt323.dll
 0002:000001e4       __imp_?focusInEvent@QPopupMenu@@MAEXPAVQFocusEvent@@@Z 100131e4     qt-mt323:qt-mt323.dll
 0002:000001e8       __imp_?focusInEvent@QWidget@@MAEXPAVQFocusEvent@@@Z 100131e8     qt-mt323:qt-mt323.dll
 0002:000001ec       __imp_?focusNextPrevChild@QPopupMenu@@MAE_N_N@Z 100131ec     qt-mt323:qt-mt323.dll
 0002:000001f0       __imp_?focusNextPrevChild@QWidget@@MAE_N_N@Z 100131f0     qt-mt323:qt-mt323.dll
 0002:000001f4       __imp_?focusOutEvent@QPopupMenu@@MAEXPAVQFocusEvent@@@Z 100131f4     qt-mt323:qt-mt323.dll
 0002:000001f8       __imp_?focusOutEvent@QWidget@@MAEXPAVQFocusEvent@@@Z 100131f8     qt-mt323:qt-mt323.dll
 0002:000001fc       __imp_?fontChange@QWidget@@MAEXABVQFont@@@Z 100131fc     qt-mt323:qt-mt323.dll
 0002:00000200       __imp_?fontInf@QPaintDevice@@MBEHPAVQFont@@H@Z 10013200     qt-mt323:qt-mt323.dll
 0002:00000204       __imp_?fontMet@QPaintDevice@@MBEHPAVQFont@@HPBDH@Z 10013204     qt-mt323:qt-mt323.dll
 0002:00000208       __imp_?frameChanged@QFrame@@MAEXXZ 10013208     qt-mt323:qt-mt323.dll
 0002:0000020c       __imp_?frameChanged@QPopupMenu@@EAEXXZ 1001320c     qt-mt323:qt-mt323.dll
 0002:00000210       __imp_?handle@QPaintDevice@@UBEPAUHDC__@@XZ 10013210     qt-mt323:qt-mt323.dll
 0002:00000214       __imp_?heightForWidth@QWidget@@UBEHH@Z 10013214     qt-mt323:qt-mt323.dll
 0002:00000218       __imp_?hide@QPopupMenu@@UAEXXZ 10013218     qt-mt323:qt-mt323.dll
 0002:0000021c       __imp_?hide@QToolBar@@UAEXXZ 1001321c     qt-mt323:qt-mt323.dll
 0002:00000220       __imp_?hide@QWidget@@UAEXXZ 10013220     qt-mt323:qt-mt323.dll
 0002:00000224       __imp_?hideEvent@QDockWindow@@MAEXPAVQHideEvent@@@Z 10013224     qt-mt323:qt-mt323.dll
 0002:00000228       __imp_?hideEvent@QWidget@@MAEXPAVQHideEvent@@@Z 10013228     qt-mt323:qt-mt323.dll
 0002:0000022c       __imp_?imComposeEvent@QWidget@@MAEXPAVQIMEvent@@@Z 1001322c     qt-mt323:qt-mt323.dll
 0002:00000230       __imp_?imEndEvent@QWidget@@MAEXPAVQIMEvent@@@Z 10013230     qt-mt323:qt-mt323.dll
 0002:00000234       __imp_?imStartEvent@QWidget@@MAEXPAVQIMEvent@@@Z 10013234     qt-mt323:qt-mt323.dll
 0002:00000238       __imp_?insertChild@QObject@@UAEXPAV1@@Z 10013238     qt-mt323:qt-mt323.dll
 0002:0000023c       __imp_?keyPressEvent@QPopupMenu@@MAEXPAVQKeyEvent@@@Z 1001323c     qt-mt323:qt-mt323.dll
 0002:00000240       __imp_?keyPressEvent@QWidget@@MAEXPAVQKeyEvent@@@Z 10013240     qt-mt323:qt-mt323.dll
 0002:00000244       __imp_?keyReleaseEvent@QWidget@@MAEXPAVQKeyEvent@@@Z 10013244     qt-mt323:qt-mt323.dll
 0002:00000248       __imp_?leaveEvent@QPopupMenu@@MAEXPAVQEvent@@@Z 10013248     qt-mt323:qt-mt323.dll
 0002:0000024c       __imp_?leaveEvent@QWidget@@MAEXPAVQEvent@@@Z 1001324c     qt-mt323:qt-mt323.dll
 0002:00000250       __imp_?menuContentsChanged@QPopupMenu@@EAEXXZ 10013250     qt-mt323:qt-mt323.dll
 0002:00000254       __imp_?menuDelPopup@QPopupMenu@@EAEXPAV1@@Z 10013254     qt-mt323:qt-mt323.dll
 0002:00000258       __imp_?menuInsPopup@QPopupMenu@@EAEXPAV1@@Z 10013258     qt-mt323:qt-mt323.dll
 0002:0000025c       __imp_?menuStateChanged@QPopupMenu@@EAEXXZ 1001325c     qt-mt323:qt-mt323.dll
 0002:00000260       __imp_?metaObject@QAction@@UBEPAVQMetaObject@@XZ 10013260     qt-mt323:qt-mt323.dll
 0002:00000264       __imp_?metaObject@QDockWindow@@UBEPAVQMetaObject@@XZ 10013264     qt-mt323:qt-mt323.dll
 0002:00000268       __imp_?metaObject@QGuardedPtrPrivate@@UBEPAVQMetaObject@@XZ 10013268     qt-mt323:qt-mt323.dll
 0002:0000026c       __imp_?metaObject@QPopupMenu@@UBEPAVQMetaObject@@XZ 1001326c     qt-mt323:qt-mt323.dll
 0002:00000270       __imp_?metaObject@QToolBar@@UBEPAVQMetaObject@@XZ 10013270     qt-mt323:qt-mt323.dll
 0002:00000274       __imp_?metaObject@QWidget@@UBEPAVQMetaObject@@XZ 10013274     qt-mt323:qt-mt323.dll
 0002:00000278       __imp_?metric@QWidget@@MBEHH@Z 10013278     qt-mt323:qt-mt323.dll
 0002:0000027c       __imp_?minimumSizeHint@QDockWindow@@UBE?AVQSize@@XZ 1001327c     qt-mt323:qt-mt323.dll
 0002:00000280       __imp_?minimumSizeHint@QToolBar@@UBE?AVQSize@@XZ 10013280     qt-mt323:qt-mt323.dll
 0002:00000284       __imp_?minimumSizeHint@QWidget@@UBE?AVQSize@@XZ 10013284     qt-mt323:qt-mt323.dll
 0002:00000288       __imp_?mouseDoubleClickEvent@QWidget@@MAEXPAVQMouseEvent@@@Z 10013288     qt-mt323:qt-mt323.dll
 0002:0000028c       __imp_?mouseMoveEvent@QPopupMenu@@MAEXPAVQMouseEvent@@@Z 1001328c     qt-mt323:qt-mt323.dll
 0002:00000290       __imp_?mouseMoveEvent@QWidget@@MAEXPAVQMouseEvent@@@Z 10013290     qt-mt323:qt-mt323.dll
 0002:00000294       __imp_?mousePressEvent@QPopupMenu@@MAEXPAVQMouseEvent@@@Z 10013294     qt-mt323:qt-mt323.dll
 0002:00000298       __imp_?mousePressEvent@QWidget@@MAEXPAVQMouseEvent@@@Z 10013298     qt-mt323:qt-mt323.dll
 0002:0000029c       __imp_?mouseReleaseEvent@QPopupMenu@@MAEXPAVQMouseEvent@@@Z 1001329c     qt-mt323:qt-mt323.dll
 0002:000002a0       __imp_?mouseReleaseEvent@QWidget@@MAEXPAVQMouseEvent@@@Z 100132a0     qt-mt323:qt-mt323.dll
 0002:000002a4       __imp_?move@QWidget@@UAEXHH@Z 100132a4     qt-mt323:qt-mt323.dll
 0002:000002a8       __imp_?moveEvent@QWidget@@MAEXPAVQMoveEvent@@@Z 100132a8     qt-mt323:qt-mt323.dll
 0002:000002ac       __imp_?newItem@QPtrCollection@@MAEPAXPAX@Z 100132ac     qt-mt323:qt-mt323.dll
 0002:000002b0       __imp_?paintEvent@QFrame@@MAEXPAVQPaintEvent@@@Z 100132b0     qt-mt323:qt-mt323.dll
 0002:000002b4       __imp_?paintEvent@QPopupMenu@@MAEXPAVQPaintEvent@@@Z 100132b4     qt-mt323:qt-mt323.dll
 0002:000002b8       __imp_?paintEvent@QWidget@@MAEXPAVQPaintEvent@@@Z 100132b8     qt-mt323:qt-mt323.dll
 0002:000002bc       __imp_?paletteChange@QWidget@@MAEXABVQPalette@@@Z 100132bc     qt-mt323:qt-mt323.dll
 0002:000002c0       __imp_?polish@QWidget@@UAEXXZ 100132c0     qt-mt323:qt-mt323.dll
 0002:000002c4       __imp_?property@QObject@@UBE?AVQVariant@@PBD@Z 100132c4     qt-mt323:qt-mt323.dll
 0002:000002c8       __imp_?qt_cast@QAction@@UAEPAXPBD@Z 100132c8     qt-mt323:qt-mt323.dll
 0002:000002cc       __imp_?qt_cast@QDockWindow@@UAEPAXPBD@Z 100132cc     qt-mt323:qt-mt323.dll
 0002:000002d0       __imp_?qt_cast@QGuardedPtrPrivate@@UAEPAXPBD@Z 100132d0     qt-mt323:qt-mt323.dll
 0002:000002d4       __imp_?qt_cast@QPopupMenu@@UAEPAXPBD@Z 100132d4     qt-mt323:qt-mt323.dll
 0002:000002d8       __imp_?qt_cast@QToolBar@@UAEPAXPBD@Z 100132d8     qt-mt323:qt-mt323.dll
 0002:000002dc       __imp_?qt_cast@QWidget@@UAEPAXPBD@Z 100132dc     qt-mt323:qt-mt323.dll
 0002:000002e0       __imp_?qt_emit@QAction@@UAE_NHPAUQUObject@@@Z 100132e0     qt-mt323:qt-mt323.dll
 0002:000002e4       __imp_?qt_emit@QDockWindow@@UAE_NHPAUQUObject@@@Z 100132e4     qt-mt323:qt-mt323.dll
 0002:000002e8       __imp_?qt_emit@QGuardedPtrPrivate@@UAE_NHPAUQUObject@@@Z 100132e8     qt-mt323:qt-mt323.dll
 0002:000002ec       __imp_?qt_emit@QPopupMenu@@UAE_NHPAUQUObject@@@Z 100132ec     qt-mt323:qt-mt323.dll
 0002:000002f0       __imp_?qt_emit@QToolBar@@UAE_NHPAUQUObject@@@Z 100132f0     qt-mt323:qt-mt323.dll
 0002:000002f4       __imp_?qt_emit@QWidget@@UAE_NHPAUQUObject@@@Z 100132f4     qt-mt323:qt-mt323.dll
 0002:000002f8       __imp_?qt_invoke@QAction@@UAE_NHPAUQUObject@@@Z 100132f8     qt-mt323:qt-mt323.dll
 0002:000002fc       __imp_?qt_invoke@QDockWindow@@UAE_NHPAUQUObject@@@Z 100132fc     qt-mt323:qt-mt323.dll
 0002:00000300       __imp_?qt_invoke@QGuardedPtrPrivate@@UAE_NHPAUQUObject@@@Z 10013300     qt-mt323:qt-mt323.dll
 0002:00000304       __imp_?qt_invoke@QPopupMenu@@UAE_NHPAUQUObject@@@Z 10013304     qt-mt323:qt-mt323.dll
 0002:00000308       __imp_?qt_invoke@QToolBar@@UAE_NHPAUQUObject@@@Z 10013308     qt-mt323:qt-mt323.dll
 0002:0000030c       __imp_?qt_invoke@QWidget@@UAE_NHPAUQUObject@@@Z 1001330c     qt-mt323:qt-mt323.dll
 0002:00000310       __imp_?qt_property@QAction@@UAE_NHHPAVQVariant@@@Z 10013310     qt-mt323:qt-mt323.dll
 0002:00000314       __imp_?qt_property@QDockWindow@@UAE_NHHPAVQVariant@@@Z 10013314     qt-mt323:qt-mt323.dll
 0002:00000318       __imp_?qt_property@QGuardedPtrPrivate@@UAE_NHHPAVQVariant@@@Z 10013318     qt-mt323:qt-mt323.dll
 0002:0000031c       __imp_?qt_property@QPopupMenu@@UAE_NHHPAVQVariant@@@Z 1001331c     qt-mt323:qt-mt323.dll
 0002:00000320       __imp_?qt_property@QToolBar@@UAE_NHHPAVQVariant@@@Z 10013320     qt-mt323:qt-mt323.dll
 0002:00000324       __imp_?qt_property@QWidget@@UAE_NHHPAVQVariant@@@Z 10013324     qt-mt323:qt-mt323.dll
 0002:00000328       __imp_?read@QGDict@@MAEAAVQDataStream@@AAV2@AAPAX@Z 10013328     qt-mt323:qt-mt323.dll
 0002:0000032c       __imp_?read@QGList@@MAEAAVQDataStream@@AAV2@AAPAX@Z 1001332c     qt-mt323:qt-mt323.dll
 0002:00000330       __imp_?removeChild@QObject@@UAEXPAV1@@Z 10013330     qt-mt323:qt-mt323.dll
 0002:00000334       __imp_?removeFrom@QAction@@UAE_NPAVQWidget@@@Z 10013334     qt-mt323:qt-mt323.dll
 0002:00000338       __imp_?reparent@QWidget@@UAEXPAV1@IABVQPoint@@_N@Z 10013338     qt-mt323:qt-mt323.dll
 0002:0000033c       __imp_?resize@QWidget@@UAEXHH@Z 1001333c     qt-mt323:qt-mt323.dll
 0002:00000340       __imp_?resizeEvent@QDockWindow@@MAEXPAVQResizeEvent@@@Z 10013340     qt-mt323:qt-mt323.dll
 0002:00000344       __imp_?resizeEvent@QFrame@@MAEXPAVQResizeEvent@@@Z 10013344     qt-mt323:qt-mt323.dll
 0002:00000348       __imp_?resizeEvent@QToolBar@@MAEXPAVQResizeEvent@@@Z 10013348     qt-mt323:qt-mt323.dll
 0002:0000034c       __imp_?resizeEvent@QWidget@@MAEXPAVQResizeEvent@@@Z 1001334c     qt-mt323:qt-mt323.dll
 0002:00000350       __imp_?resolution@QPaintDevice@@UBEHXZ 10013350     qt-mt323:qt-mt323.dll
 0002:00000354       __imp_?setAccel@QAction@@UAEXABVQKeySequence@@@Z 10013354     qt-mt323:qt-mt323.dll
 0002:00000358       __imp_?setAcceptDrops@QWidget@@UAEX_N@Z 10013358     qt-mt323:qt-mt323.dll
 0002:0000035c       __imp_?setActiveItem@QPopupMenu@@UAEXH@Z 1001335c     qt-mt323:qt-mt323.dll
 0002:00000360       __imp_?setActiveWindow@QWidget@@UAEXXZ 10013360     qt-mt323:qt-mt323.dll
 0002:00000364       __imp_?setAutoMask@QWidget@@UAEX_N@Z 10013364     qt-mt323:qt-mt323.dll
 0002:00000368       __imp_?setBackgroundColor@QWidget@@UAEXABVQColor@@@Z 10013368     qt-mt323:qt-mt323.dll
 0002:0000036c       __imp_?setBackgroundMode@QWidget@@UAEXW4BackgroundMode@Qt@@@Z 1001336c     qt-mt323:qt-mt323.dll
 0002:00000370       __imp_?setBackgroundOrigin@QWidget@@UAEXW4BackgroundOrigin@1@@Z 10013370     qt-mt323:qt-mt323.dll
 0002:00000374       __imp_?setBackgroundPixmap@QWidget@@UAEXABVQPixmap@@@Z 10013374     qt-mt323:qt-mt323.dll
 0002:00000378       __imp_?setCaption@QDockWindow@@UAEXABVQString@@@Z 10013378     qt-mt323:qt-mt323.dll
 0002:0000037c       __imp_?setCaption@QWidget@@UAEXABVQString@@@Z 1001337c     qt-mt323:qt-mt323.dll
 0002:00000380       __imp_?setCheckable@QPopupMenu@@UAEX_N@Z 10013380     qt-mt323:qt-mt323.dll
 0002:00000384       __imp_?setCloseMode@QDockWindow@@UAEXH@Z 10013384     qt-mt323:qt-mt323.dll
 0002:00000388       __imp_?setCursor@QWidget@@UAEXABVQCursor@@@Z 10013388     qt-mt323:qt-mt323.dll
 0002:0000038c       __imp_?setEnabled@QAction@@UAEX_N@Z 1001338c     qt-mt323:qt-mt323.dll
 0002:00000390       __imp_?setEnabled@QWidget@@UAEX_N@Z 10013390     qt-mt323:qt-mt323.dll
 0002:00000394       __imp_?setEraseColor@QWidget@@UAEXABVQColor@@@Z 10013394     qt-mt323:qt-mt323.dll
 0002:00000398       __imp_?setErasePixmap@QWidget@@UAEXABVQPixmap@@@Z 10013398     qt-mt323:qt-mt323.dll
 0002:0000039c       __imp_?setFirstItemActive@QPopupMenu@@EAEXXZ 1001339c     qt-mt323:qt-mt323.dll
 0002:000003a0       __imp_?setFixedExtentHeight@QDockWindow@@UAEXH@Z 100133a0     qt-mt323:qt-mt323.dll
 0002:000003a4       __imp_?setFixedExtentWidth@QDockWindow@@UAEXH@Z 100133a4     qt-mt323:qt-mt323.dll
 0002:000003a8       __imp_?setFocus@QWidget@@UAEXXZ 100133a8     qt-mt323:qt-mt323.dll
 0002:000003ac       __imp_?setFocusPolicy@QWidget@@UAEXW4FocusPolicy@1@@Z 100133ac     qt-mt323:qt-mt323.dll
 0002:000003b0       __imp_?setFocusProxy@QWidget@@UAEXPAV1@@Z 100133b0     qt-mt323:qt-mt323.dll
 0002:000003b4       __imp_?setFont@QPopupMenu@@UAEXABVQFont@@@Z 100133b4     qt-mt323:qt-mt323.dll
 0002:000003b8       __imp_?setFont@QWidget@@UAEXABVQFont@@@Z 100133b8     qt-mt323:qt-mt323.dll
 0002:000003bc       __imp_?setFrameRect@QFrame@@UAEXABVQRect@@@Z 100133bc     qt-mt323:qt-mt323.dll
 0002:000003c0       __imp_?setFrameStyle@QFrame@@UAEXH@Z 100133c0     qt-mt323:qt-mt323.dll
 0002:000003c4       __imp_?setGeometry@QWidget@@UAEXABVQRect@@@Z 100133c4     qt-mt323:qt-mt323.dll
 0002:000003c8       __imp_?setGeometry@QWidget@@UAEXHHHH@Z 100133c8     qt-mt323:qt-mt323.dll
 0002:000003cc       __imp_?setHorizontallyStretchable@QDockWindow@@UAEX_N@Z 100133cc     qt-mt323:qt-mt323.dll
 0002:000003d0       __imp_?setIcon@QWidget@@UAEXABVQPixmap@@@Z 100133d0     qt-mt323:qt-mt323.dll
 0002:000003d4       __imp_?setIconSet@QAction@@UAEXABVQIconSet@@@Z 100133d4     qt-mt323:qt-mt323.dll
 0002:000003d8       __imp_?setIconText@QWidget@@UAEXABVQString@@@Z 100133d8     qt-mt323:qt-mt323.dll
 0002:000003dc       __imp_?setId@QMenuData@@UAEXHH@Z 100133dc     qt-mt323:qt-mt323.dll
 0002:000003e0       __imp_?setKeyCompression@QWidget@@MAEX_N@Z 100133e0     qt-mt323:qt-mt323.dll
 0002:000003e4       __imp_?setLabel@QToolBar@@UAEXABVQString@@@Z 100133e4     qt-mt323:qt-mt323.dll
 0002:000003e8       __imp_?setLineWidth@QFrame@@UAEXH@Z 100133e8     qt-mt323:qt-mt323.dll
 0002:000003ec       __imp_?setMargin@QFrame@@UAEXH@Z 100133ec     qt-mt323:qt-mt323.dll
 0002:000003f0       __imp_?setMask@QWidget@@UAEXABVQBitmap@@@Z 100133f0     qt-mt323:qt-mt323.dll
 0002:000003f4       __imp_?setMask@QWidget@@UAEXABVQRegion@@@Z 100133f4     qt-mt323:qt-mt323.dll
 0002:000003f8       __imp_?setMaximumSize@QWidget@@UAEXHH@Z 100133f8     qt-mt323:qt-mt323.dll
 0002:000003fc       __imp_?setMenuText@QAction@@UAEXABVQString@@@Z 100133fc     qt-mt323:qt-mt323.dll
 0002:00000400       __imp_?setMicroFocusHint@QWidget@@MAEXHHHH_NPAVQFont@@@Z 10013400     qt-mt323:qt-mt323.dll
 0002:00000404       __imp_?setMidLineWidth@QFrame@@UAEXH@Z 10013404     qt-mt323:qt-mt323.dll
 0002:00000408       __imp_?setMinimumSize@QToolBar@@UAEXHH@Z 10013408     qt-mt323:qt-mt323.dll
 0002:0000040c       __imp_?setMinimumSize@QWidget@@UAEXHH@Z 1001340c     qt-mt323:qt-mt323.dll
 0002:00000410       __imp_?setMouseTracking@QWidget@@UAEX_N@Z 10013410     qt-mt323:qt-mt323.dll
 0002:00000414       __imp_?setMovingEnabled@QDockWindow@@UAEX_N@Z 10013414     qt-mt323:qt-mt323.dll
 0002:00000418       __imp_?setName@QObject@@UAEXPBD@Z 10013418     qt-mt323:qt-mt323.dll
 0002:0000041c       __imp_?setNewLine@QDockWindow@@UAEX_N@Z 1001341c     qt-mt323:qt-mt323.dll
 0002:00000420       __imp_?setOffset@QDockWindow@@UAEXH@Z 10013420     qt-mt323:qt-mt323.dll
 0002:00000424       __imp_?setOn@QAction@@UAEX_N@Z 10013424     qt-mt323:qt-mt323.dll
 0002:00000428       __imp_?setOpaqueMoving@QDockWindow@@UAEX_N@Z 10013428     qt-mt323:qt-mt323.dll
 0002:0000042c       __imp_?setOrientation@QDockWindow@@UAEXW4Orientation@Qt@@@Z 1001342c     qt-mt323:qt-mt323.dll
 0002:00000430       __imp_?setOrientation@QToolBar@@UAEXW4Orientation@Qt@@@Z 10013430     qt-mt323:qt-mt323.dll
 0002:00000434       __imp_?setPalette@QWidget@@UAEXABVQPalette@@@Z 10013434     qt-mt323:qt-mt323.dll
 0002:00000438       __imp_?setPaletteBackgroundColor@QWidget@@UAEXABVQColor@@@Z 10013438     qt-mt323:qt-mt323.dll
 0002:0000043c       __imp_?setPaletteBackgroundPixmap@QWidget@@UAEXABVQPixmap@@@Z 1001343c     qt-mt323:qt-mt323.dll
 0002:00000440       __imp_?setProperty@QObject@@UAE_NPBDABVQVariant@@@Z 10013440     qt-mt323:qt-mt323.dll
 0002:00000444       __imp_?setResizeEnabled@QDockWindow@@UAEX_N@Z 10013444     qt-mt323:qt-mt323.dll
 0002:00000448       __imp_?setResolution@QPaintDevice@@UAEXH@Z 10013448     qt-mt323:qt-mt323.dll
 0002:0000044c       __imp_?setSizeIncrement@QWidget@@UAEXHH@Z 1001344c     qt-mt323:qt-mt323.dll
 0002:00000450       __imp_?setSizePolicy@QWidget@@UAEXVQSizePolicy@@@Z 10013450     qt-mt323:qt-mt323.dll
 0002:00000454       __imp_?setStatusTip@QAction@@UAEXABVQString@@@Z 10013454     qt-mt323:qt-mt323.dll
 0002:00000458       __imp_?setStretchableWidget@QToolBar@@UAEXPAVQWidget@@@Z 10013458     qt-mt323:qt-mt323.dll
 0002:0000045c       __imp_?setText@QAction@@UAEXABVQString@@@Z 1001345c     qt-mt323:qt-mt323.dll
 0002:00000460       __imp_?setToggleAction@QAction@@UAEX_N@Z 10013460     qt-mt323:qt-mt323.dll
 0002:00000464       __imp_?setToolTip@QAction@@UAEXABVQString@@@Z 10013464     qt-mt323:qt-mt323.dll
 0002:00000468       __imp_?setUpdatesEnabled@QWidget@@UAEX_N@Z 10013468     qt-mt323:qt-mt323.dll
 0002:0000046c       __imp_?setVerticallyStretchable@QDockWindow@@UAEX_N@Z 1001346c     qt-mt323:qt-mt323.dll
 0002:00000470       __imp_?setWFlags@QWidget@@MAEXI@Z 10013470     qt-mt323:qt-mt323.dll
 0002:00000474       __imp_?setWState@QWidget@@MAEXI@Z 10013474     qt-mt323:qt-mt323.dll
 0002:00000478       __imp_?setWhatsThis@QAction@@UAEXABVQString@@@Z 10013478     qt-mt323:qt-mt323.dll
 0002:0000047c       __imp_?setWidget@QDockWindow@@UAEXPAVQWidget@@@Z 1001347c     qt-mt323:qt-mt323.dll
 0002:00000480       __imp_?show@QPopupMenu@@UAEXXZ 10013480     qt-mt323:qt-mt323.dll
 0002:00000484       __imp_?show@QToolBar@@UAEXXZ 10013484     qt-mt323:qt-mt323.dll
 0002:00000488       __imp_?show@QWidget@@UAEXXZ 10013488     qt-mt323:qt-mt323.dll
 0002:0000048c       __imp_?showEvent@QDockWindow@@MAEXPAVQShowEvent@@@Z 1001348c     qt-mt323:qt-mt323.dll
 0002:00000490       __imp_?showEvent@QWidget@@MAEXPAVQShowEvent@@@Z 10013490     qt-mt323:qt-mt323.dll
 0002:00000494       __imp_?showMaximized@QWidget@@UAEXXZ 10013494     qt-mt323:qt-mt323.dll
 0002:00000498       __imp_?showMinimized@QWidget@@UAEXXZ 10013498     qt-mt323:qt-mt323.dll
 0002:0000049c       __imp_?showNormal@QWidget@@UAEXXZ 1001349c     qt-mt323:qt-mt323.dll
 0002:000004a0       __imp_?sizeHint@QDockWindow@@UBE?AVQSize@@XZ 100134a0     qt-mt323:qt-mt323.dll
 0002:000004a4       __imp_?sizeHint@QPopupMenu@@UBE?AVQSize@@XZ 100134a4     qt-mt323:qt-mt323.dll
 0002:000004a8       __imp_?sizeHint@QWidget@@UBE?AVQSize@@XZ 100134a8     qt-mt323:qt-mt323.dll
 0002:000004ac       __imp_?sizePolicy@QWidget@@UBE?AVQSizePolicy@@XZ 100134ac     qt-mt323:qt-mt323.dll
 0002:000004b0       __imp_?styleChange@QFrame@@MAEXAAVQStyle@@@Z 100134b0     qt-mt323:qt-mt323.dll
 0002:000004b4       __imp_?styleChange@QPopupMenu@@MAEXAAVQStyle@@@Z 100134b4     qt-mt323:qt-mt323.dll
 0002:000004b8       __imp_?styleChange@QToolBar@@MAEXAAVQStyle@@@Z 100134b8     qt-mt323:qt-mt323.dll
 0002:000004bc       __imp_?styleChange@QWidget@@MAEXAAVQStyle@@@Z 100134bc     qt-mt323:qt-mt323.dll
 0002:000004c0       __imp_?tabletEvent@QWidget@@MAEXPAVQTabletEvent@@@Z 100134c0     qt-mt323:qt-mt323.dll
 0002:000004c4       __imp_?timerEvent@QObject@@MAEXPAVQTimerEvent@@@Z 100134c4     qt-mt323:qt-mt323.dll
 0002:000004c8       __imp_?timerEvent@QPopupMenu@@MAEXPAVQTimerEvent@@@Z 100134c8     qt-mt323:qt-mt323.dll
 0002:000004cc       __imp_?undock@QDockWindow@@UAEXPAVQWidget@@@Z 100134cc     qt-mt323:qt-mt323.dll
 0002:000004d0       __imp_?undock@QDockWindow@@UAEXXZ 100134d0     qt-mt323:qt-mt323.dll
 0002:000004d4       __imp_?unsetCursor@QWidget@@UAEXXZ 100134d4     qt-mt323:qt-mt323.dll
 0002:000004d8       __imp_?updateItem@QPopupMenu@@UAEXH@Z 100134d8     qt-mt323:qt-mt323.dll
 0002:000004dc       __imp_?updateMask@QWidget@@MAEXXZ 100134dc     qt-mt323:qt-mt323.dll
 0002:000004e0       __imp_?wheelEvent@QWidget@@MAEXPAVQWheelEvent@@@Z 100134e0     qt-mt323:qt-mt323.dll
 0002:000004e4       __imp_?winEvent@QWidget@@MAE_NPAUtagMSG@@@Z 100134e4     qt-mt323:qt-mt323.dll
 0002:000004e8       __imp_?windowActivationChange@QWidget@@MAEX_N@Z 100134e8     qt-mt323:qt-mt323.dll
 0002:000004ec       __imp_?write@QGDict@@MBEAAVQDataStream@@AAV2@PAX@Z 100134ec     qt-mt323:qt-mt323.dll
 0002:000004f0       __imp_?write@QGList@@MBEAAVQDataStream@@AAV2@PAX@Z 100134f0     qt-mt323:qt-mt323.dll
 0002:000004f4       __imp_?null@QString@@2V1@A 100134f4     qt-mt323:qt-mt323.dll
 0002:000004f8       __imp_??_7?$QPtrList@VQDockWindow@@@@6B@ 100134f8     qt-mt323:qt-mt323.dll
 0002:000004fc       __imp_??4QString@@QAEAAV0@PBD@Z 100134fc     qt-mt323:qt-mt323.dll
 0002:00000500       __imp_?arg@QString@@QBE?AV1@HHH@Z 10013500     qt-mt323:qt-mt323.dll
 0002:00000504       __imp_?remove@QString@@QAEAAV1@D@Z 10013504     qt-mt323:qt-mt323.dll
 0002:00000508       __imp_?toInt@QString@@QBEHPA_NH@Z 10013508     qt-mt323:qt-mt323.dll
 0002:0000050c       __imp_?toFloat@QString@@QBEMPA_N@Z 1001350c     qt-mt323:qt-mt323.dll
 0002:00000510       __imp_??9@YA_NABVQString@@0@Z 10013510     qt-mt323:qt-mt323.dll
 0002:00000514       __imp_??9@YA_NABVQString@@PBD@Z 10013514     qt-mt323:qt-mt323.dll
 0002:00000518       __imp_??0QTextStream@@QAE@PAVQIODevice@@@Z 10013518     qt-mt323:qt-mt323.dll
 0002:0000051c       __imp_??1QTextStream@@UAE@XZ 1001351c     qt-mt323:qt-mt323.dll
 0002:00000520       __imp_??6QTextStream@@QAEAAV0@ABVQString@@@Z 10013520     qt-mt323:qt-mt323.dll
 0002:00000524       __imp_??A?$QValueList@VQString@@@@QAEAAVQString@@I@Z 10013524     qt-mt323:qt-mt323.dll
 0002:00000528       __imp_?remove@QGList@@IAE_NPAX@Z 10013528     qt-mt323:qt-mt323.dll
 0002:0000052c       __imp_?first@QGList@@IAEPAXXZ 1001352c     qt-mt323:qt-mt323.dll
 0002:00000530       __imp_??0QGListIterator@@IAE@ABVQGList@@@Z 10013530     qt-mt323:qt-mt323.dll
 0002:00000534       __imp_??1QGListIterator@@IAE@XZ 10013534     qt-mt323:qt-mt323.dll
 0002:00000538       __imp_??EQGListIterator@@IAEPAXXZ 10013538     qt-mt323:qt-mt323.dll
 0002:0000053c       __imp_?split@QStringList@@SA?AV1@ABVQChar@@ABVQString@@_N@Z 1001353c     qt-mt323:qt-mt323.dll
 0002:00000540       __imp_??4QStringList@@QAEAAV0@ABV0@@Z 10013540     qt-mt323:qt-mt323.dll
 0002:00000544       __imp_?setDisabled@QWidget@@QAEX_N@Z 10013544     qt-mt323:qt-mt323.dll
 0002:00000548       __imp_?clearMask@QWidget@@QAEXXZ 10013548     qt-mt323:qt-mt323.dll
 0002:0000054c       __imp_?open@QFile@@UAE_NH@Z 1001354c     qt-mt323:qt-mt323.dll
 0002:00000550       __imp_?close@QFile@@UAEXXZ 10013550     qt-mt323:qt-mt323.dll
 0002:00000554       __imp_??4QDomNode@@QAEAAV0@ABV0@@Z 10013554     qt-mt323:qt-mt323.dll
 0002:00000558       __imp_??1QDomNode@@UAE@XZ  10013558     qt-mt323:qt-mt323.dll
 0002:0000055c       __imp_?replaceChild@QDomNode@@UAE?AV1@ABV1@0@Z 1001355c     qt-mt323:qt-mt323.dll
 0002:00000560       __imp_?removeChild@QDomNode@@UAE?AV1@ABV1@@Z 10013560     qt-mt323:qt-mt323.dll
 0002:00000564       __imp_?appendChild@QDomNode@@UAE?AV1@ABV1@@Z 10013564     qt-mt323:qt-mt323.dll
 0002:00000568       __imp_?cloneNode@QDomNode@@UBE?AV1@_N@Z 10013568     qt-mt323:qt-mt323.dll
 0002:0000056c       __imp_?firstChild@QDomNode@@UBE?AV1@XZ 1001356c     qt-mt323:qt-mt323.dll
 0002:00000570       __imp_?nextSibling@QDomNode@@UBE?AV1@XZ 10013570     qt-mt323:qt-mt323.dll
 0002:00000574       __imp_?namedItem@QDomNode@@QBE?AV1@ABVQString@@@Z 10013574     qt-mt323:qt-mt323.dll
 0002:00000578       __imp_?isNull@QDomNode@@QBE_NXZ 10013578     qt-mt323:qt-mt323.dll
 0002:0000057c       __imp_?toElement@QDomNode@@QAE?AVQDomElement@@XZ 1001357c     qt-mt323:qt-mt323.dll
 0002:00000580       __imp_??0QDomDocument@@QAE@XZ 10013580     qt-mt323:qt-mt323.dll
 0002:00000584       __imp_??0QDomDocument@@QAE@ABVQString@@@Z 10013584     qt-mt323:qt-mt323.dll
 0002:00000588       __imp_??1QDomDocument@@UAE@XZ 10013588     qt-mt323:qt-mt323.dll
 0002:0000058c       __imp_?createElement@QDomDocument@@QAE?AVQDomElement@@ABVQString@@@Z 1001358c     qt-mt323:qt-mt323.dll
 0002:00000590       __imp_?documentElement@QDomDocument@@QBE?AVQDomElement@@XZ 10013590     qt-mt323:qt-mt323.dll
 0002:00000594       __imp_?setContent@QDomDocument@@QAE_NABVQString@@_NPAV2@PAH3@Z 10013594     qt-mt323:qt-mt323.dll
 0002:00000598       __imp_?setContent@QDomDocument@@QAE_NPAVQIODevice@@PAVQString@@PAH2@Z 10013598     qt-mt323:qt-mt323.dll
 0002:0000059c       __imp_?toString@QDomDocument@@QBE?AVQString@@XZ 1001359c     qt-mt323:qt-mt323.dll
 0002:000005a0       __imp_?toString@QDomDocument@@QBE?AVQString@@H@Z 100135a0     qt-mt323:qt-mt323.dll
 0002:000005a4       __imp_??0QDomElement@@QAE@ABV0@@Z 100135a4     qt-mt323:qt-mt323.dll
 0002:000005a8       __imp_??4QDomElement@@QAEAAV0@ABV0@@Z 100135a8     qt-mt323:qt-mt323.dll
 0002:000005ac       __imp_??1QDomElement@@UAE@XZ 100135ac     qt-mt323:qt-mt323.dll
 0002:000005b0       __imp_?attribute@QDomElement@@QBE?AVQString@@ABV2@0@Z 100135b0     qt-mt323:qt-mt323.dll
 0002:000005b4       __imp_?setAttribute@QDomElement@@QAEXABVQString@@0@Z 100135b4     qt-mt323:qt-mt323.dll
 0002:000005b8       __imp_?setAttribute@QDomElement@@QAEXABVQString@@H@Z 100135b8     qt-mt323:qt-mt323.dll
 0002:000005bc       __imp_?removeAttribute@QDomElement@@QAEXABVQString@@@Z 100135bc     qt-mt323:qt-mt323.dll
 0002:000005c0       __imp_?tagName@QDomElement@@QBE?AVQString@@XZ 100135c0     qt-mt323:qt-mt323.dll
 0002:000005c4       __imp_??0QListViewItem@@QAE@PAVQListView@@VQString@@1111111@Z 100135c4     qt-mt323:qt-mt323.dll
 0002:000005c8       __imp_??1QListViewItem@@UAE@XZ 100135c8     qt-mt323:qt-mt323.dll
 0002:000005cc       __imp_?columns@QListView@@QBEHXZ 100135cc     qt-mt323:qt-mt323.dll
 0002:000005d0       __imp_?setSelectionMode@QListView@@QAEXW4SelectionMode@1@@Z 100135d0     qt-mt323:qt-mt323.dll
 0002:000005d4       __imp_?currentItem@QListView@@QBEPAVQListViewItem@@XZ 100135d4     qt-mt323:qt-mt323.dll
 0002:000005d8       __imp_?firstChild@QListView@@QBEPAVQListViewItem@@XZ 100135d8     qt-mt323:qt-mt323.dll
 0002:000005dc       __imp_?childCount@QListView@@QBEHXZ 100135dc     qt-mt323:qt-mt323.dll
 0002:000005e0       __imp_?findItem@QListView@@QBEPAVQListViewItem@@ABVQString@@HI@Z 100135e0     qt-mt323:qt-mt323.dll
 0002:000005e4       __imp_??0QListViewItemIterator@@QAE@PAVQListView@@@Z 100135e4     qt-mt323:qt-mt323.dll
 0002:000005e8       __imp_??1QListViewItemIterator@@QAE@XZ 100135e8     qt-mt323:qt-mt323.dll
 0002:000005ec       __imp_??EQListViewItemIterator@@QAEAAV0@XZ 100135ec     qt-mt323:qt-mt323.dll
 0002:000005f0       __imp_?current@QListViewItemIterator@@QBEPAVQListViewItem@@XZ 100135f0     qt-mt323:qt-mt323.dll
 0002:000005f4       __imp_?insertItem@QComboBox@@QAEXABVQString@@H@Z 100135f4     qt-mt323:qt-mt323.dll
 0002:000005f8       __imp_?currentItem@QComboBox@@QBEHXZ 100135f8     qt-mt323:qt-mt323.dll
 0002:000005fc       __imp_?currentText@QComboBox@@QBE?AVQString@@XZ 100135fc     qt-mt323:qt-mt323.dll
 0002:00000600       __imp_?setChecked@QCheckBox@@QAEX_N@Z 10013600     qt-mt323:qt-mt323.dll
 0002:00000604       __imp_?value@QSpinBox@@QBEHXZ 10013604     qt-mt323:qt-mt323.dll
 0002:00000608       __imp_?raiseWidget@QWidgetStack@@QAEXH@Z 10013608     qt-mt323:qt-mt323.dll
 0002:0000060c       __imp_?text@QLineEdit@@QBE?AVQString@@XZ 1001360c     qt-mt323:qt-mt323.dll
 0002:00000610       __imp_?getText@QInputDialog@@SA?AVQString@@ABV2@0W4EchoMode@QLineEdit@@0PA_NPAVQWidget@@PBD@Z 10013610     qt-mt323:qt-mt323.dll
 0002:00000614       __imp_?warning@QMessageBox@@SAHPAVQWidget@@ABVQString@@1111HH@Z 10013614     qt-mt323:qt-mt323.dll
 0002:00000618       __imp_?clipboard@QApplication@@SAPAVQClipboard@@XZ 10013618     qt-mt323:qt-mt323.dll
 0002:0000061c       __imp_?text@QClipboard@@QBE?AVQString@@XZ 1001361c     qt-mt323:qt-mt323.dll
 0002:00000620       __imp_?setText@QClipboard@@QAEXABVQString@@@Z 10013620     qt-mt323:qt-mt323.dll
 0002:00000624       __imp_?baseName@QFileInfo@@QBE?AVQString@@_N@Z 10013624     qt-mt323:qt-mt323.dll
 0002:00000628       __imp_??0QDir@@QAE@ABVQString@@0HH@Z 10013628     qt-mt323:qt-mt323.dll
 0002:0000062c       __imp_?setNameFilter@QDir@@UAEXABVQString@@@Z 1001362c     qt-mt323:qt-mt323.dll
 0002:00000630       __imp_?setFilter@QDir@@UAEXH@Z 10013630     qt-mt323:qt-mt323.dll
 0002:00000634       __imp_?setSorting@QDir@@UAEXH@Z 10013634     qt-mt323:qt-mt323.dll
 0002:00000638       __imp_?entryInfoList@QDir@@UBEPBV?$QPtrList@VQFileInfo@@@@HH@Z 10013638     qt-mt323:qt-mt323.dll
 0002:0000063c       __imp_?acceptDrop@QListViewItem@@UBE_NPBVQMimeSource@@@Z 1001363c     qt-mt323:qt-mt323.dll
 0002:00000640       __imp_?activate@QListViewItem@@MAEXXZ 10013640     qt-mt323:qt-mt323.dll
 0002:00000644       __imp_?attributes@QDomElement@@UBE?AVQDomNamedNodeMap@@XZ 10013644     qt-mt323:qt-mt323.dll
 0002:00000648       __imp_?attributes@QDomNode@@UBE?AVQDomNamedNodeMap@@XZ 10013648     qt-mt323:qt-mt323.dll
 0002:0000064c       __imp_?cancelRename@QListViewItem@@MAEXH@Z 1001364c     qt-mt323:qt-mt323.dll
 0002:00000650       __imp_?childNodes@QDomNode@@UBE?AVQDomNodeList@@XZ 10013650     qt-mt323:qt-mt323.dll
 0002:00000654       __imp_?compare@QListViewItem@@UBEHPAV1@H_N@Z 10013654     qt-mt323:qt-mt323.dll
 0002:00000658       __imp_?dragEntered@QListViewItem@@MAEXXZ 10013658     qt-mt323:qt-mt323.dll
 0002:0000065c       __imp_?dragLeft@QListViewItem@@MAEXXZ 1001365c     qt-mt323:qt-mt323.dll
 0002:00000660       __imp_?dropped@QListViewItem@@MAEXPAVQDropEvent@@@Z 10013660     qt-mt323:qt-mt323.dll
 0002:00000664       __imp_?elementsByTagName@QDomElement@@UBE?AVQDomNodeList@@ABVQString@@@Z 10013664     qt-mt323:qt-mt323.dll
 0002:00000668       __imp_?elementsByTagNameNS@QDomElement@@UBE?AVQDomNodeList@@ABVQString@@0@Z 10013668     qt-mt323:qt-mt323.dll
 0002:0000066c       __imp_?enforceSortOrder@QListViewItem@@MBEXXZ 1001366c     qt-mt323:qt-mt323.dll
 0002:00000670       __imp_?hasAttributes@QDomNode@@UBE_NXZ 10013670     qt-mt323:qt-mt323.dll
 0002:00000674       __imp_?hasChildNodes@QDomNode@@UBE_NXZ 10013674     qt-mt323:qt-mt323.dll
 0002:00000678       __imp_?insertAfter@QDomNode@@UAE?AV1@ABV1@0@Z 10013678     qt-mt323:qt-mt323.dll
 0002:0000067c       __imp_?insertBefore@QDomNode@@UAE?AV1@ABV1@0@Z 1001367c     qt-mt323:qt-mt323.dll
 0002:00000680       __imp_?insertItem@QListViewItem@@UAEXPAV1@@Z 10013680     qt-mt323:qt-mt323.dll
 0002:00000684       __imp_?invalidateHeight@QListViewItem@@UAEXXZ 10013684     qt-mt323:qt-mt323.dll
 0002:00000688       __imp_?isAttr@QDomNode@@UBE_NXZ 10013688     qt-mt323:qt-mt323.dll
 0002:0000068c       __imp_?isCDATASection@QDomNode@@UBE_NXZ 1001368c     qt-mt323:qt-mt323.dll
 0002:00000690       __imp_?isCharacterData@QDomNode@@UBE_NXZ 10013690     qt-mt323:qt-mt323.dll
 0002:00000694       __imp_?isComment@QDomNode@@UBE_NXZ 10013694     qt-mt323:qt-mt323.dll
 0002:00000698       __imp_?isDocument@QDomDocument@@UBE_NXZ 10013698     qt-mt323:qt-mt323.dll
 0002:0000069c       __imp_?isDocument@QDomNode@@UBE_NXZ 1001369c     qt-mt323:qt-mt323.dll
 0002:000006a0       __imp_?isDocumentFragment@QDomNode@@UBE_NXZ 100136a0     qt-mt323:qt-mt323.dll
 0002:000006a4       __imp_?isDocumentType@QDomNode@@UBE_NXZ 100136a4     qt-mt323:qt-mt323.dll
 0002:000006a8       __imp_?isElement@QDomElement@@UBE_NXZ 100136a8     qt-mt323:qt-mt323.dll
 0002:000006ac       __imp_?isElement@QDomNode@@UBE_NXZ 100136ac     qt-mt323:qt-mt323.dll
 0002:000006b0       __imp_?isEntity@QDomNode@@UBE_NXZ 100136b0     qt-mt323:qt-mt323.dll
 0002:000006b4       __imp_?isEntityReference@QDomNode@@UBE_NXZ 100136b4     qt-mt323:qt-mt323.dll
 0002:000006b8       __imp_?isNotation@QDomNode@@UBE_NXZ 100136b8     qt-mt323:qt-mt323.dll
 0002:000006bc       __imp_?isProcessingInstruction@QDomNode@@UBE_NXZ 100136bc     qt-mt323:qt-mt323.dll
 0002:000006c0       __imp_?isSupported@QDomNode@@UBE_NABVQString@@0@Z 100136c0     qt-mt323:qt-mt323.dll
 0002:000006c4       __imp_?isText@QDomNode@@UBE_NXZ 100136c4     qt-mt323:qt-mt323.dll
 0002:000006c8       __imp_?key@QListViewItem@@UBE?AVQString@@H_N@Z 100136c8     qt-mt323:qt-mt323.dll
 0002:000006cc       __imp_?lastChild@QDomNode@@UBE?AV1@XZ 100136cc     qt-mt323:qt-mt323.dll
 0002:000006d0       __imp_?localName@QDomNode@@UBE?AVQString@@XZ 100136d0     qt-mt323:qt-mt323.dll
 0002:000006d4       __imp_?namespaceURI@QDomNode@@UBE?AVQString@@XZ 100136d4     qt-mt323:qt-mt323.dll
 0002:000006d8       __imp_?nodeName@QDomNode@@UBE?AVQString@@XZ 100136d8     qt-mt323:qt-mt323.dll
 0002:000006dc       __imp_?nodeType@QDomDocument@@UBE?AW4NodeType@QDomNode@@XZ 100136dc     qt-mt323:qt-mt323.dll
 0002:000006e0       __imp_?nodeType@QDomElement@@UBE?AW4NodeType@QDomNode@@XZ 100136e0     qt-mt323:qt-mt323.dll
 0002:000006e4       __imp_?nodeValue@QDomNode@@UBE?AVQString@@XZ 100136e4     qt-mt323:qt-mt323.dll
 0002:000006e8       __imp_?normalize@QDomNode@@UAEXXZ 100136e8     qt-mt323:qt-mt323.dll
 0002:000006ec       __imp_?okRename@QListViewItem@@MAEXH@Z 100136ec     qt-mt323:qt-mt323.dll
 0002:000006f0       __imp_?ownerDocument@QDomNode@@UBE?AVQDomDocument@@XZ 100136f0     qt-mt323:qt-mt323.dll
 0002:000006f4       __imp_?paintBranches@QListViewItem@@UAEXPAVQPainter@@ABVQColorGroup@@HHH@Z 100136f4     qt-mt323:qt-mt323.dll
 0002:000006f8       __imp_?paintCell@QListViewItem@@UAEXPAVQPainter@@ABVQColorGroup@@HHH@Z 100136f8     qt-mt323:qt-mt323.dll
 0002:000006fc       __imp_?paintFocus@QListViewItem@@UAEXPAVQPainter@@ABVQColorGroup@@ABVQRect@@@Z 100136fc     qt-mt323:qt-mt323.dll
 0002:00000700       __imp_?parentNode@QDomNode@@UBE?AV1@XZ 10013700     qt-mt323:qt-mt323.dll
 0002:00000704       __imp_?pixmap@QListViewItem@@UBEPBVQPixmap@@H@Z 10013704     qt-mt323:qt-mt323.dll
 0002:00000708       __imp_?prefix@QDomNode@@UBE?AVQString@@XZ 10013708     qt-mt323:qt-mt323.dll
 0002:0000070c       __imp_?previousSibling@QDomNode@@UBE?AV1@XZ 1001370c     qt-mt323:qt-mt323.dll
 0002:00000710       __imp_?removeItem@QListViewItem@@UAEXPAV1@@Z 10013710     qt-mt323:qt-mt323.dll
 0002:00000714       __imp_?rtti@QListViewItem@@UBEHXZ 10013714     qt-mt323:qt-mt323.dll
 0002:00000718       __imp_?setDragEnabled@QListViewItem@@UAEX_N@Z 10013718     qt-mt323:qt-mt323.dll
 0002:0000071c       __imp_?setDropEnabled@QListViewItem@@UAEX_N@Z 1001371c     qt-mt323:qt-mt323.dll
 0002:00000720       __imp_?setEnabled@QListViewItem@@UAEX_N@Z 10013720     qt-mt323:qt-mt323.dll
 0002:00000724       __imp_?setExpandable@QListViewItem@@UAEX_N@Z 10013724     qt-mt323:qt-mt323.dll
 0002:00000728       __imp_?setHeight@QListViewItem@@MAEXH@Z 10013728     qt-mt323:qt-mt323.dll
 0002:0000072c       __imp_?setMultiLinesEnabled@QListViewItem@@UAEX_N@Z 1001372c     qt-mt323:qt-mt323.dll
 0002:00000730       __imp_?setNodeValue@QDomNode@@UAEXABVQString@@@Z 10013730     qt-mt323:qt-mt323.dll
 0002:00000734       __imp_?setOpen@QListViewItem@@UAEX_N@Z 10013734     qt-mt323:qt-mt323.dll
 0002:00000738       __imp_?setPixmap@QListViewItem@@UAEXHABVQPixmap@@@Z 10013738     qt-mt323:qt-mt323.dll
 0002:0000073c       __imp_?setPrefix@QDomNode@@UAEXABVQString@@@Z 1001373c     qt-mt323:qt-mt323.dll
 0002:00000740       __imp_?setRenameEnabled@QListViewItem@@UAEXH_N@Z 10013740     qt-mt323:qt-mt323.dll
 0002:00000744       __imp_?setSelectable@QListViewItem@@UAEX_N@Z 10013744     qt-mt323:qt-mt323.dll
 0002:00000748       __imp_?setSelected@QListViewItem@@UAEX_N@Z 10013748     qt-mt323:qt-mt323.dll
 0002:0000074c       __imp_?setText@QListViewItem@@UAEXHABVQString@@@Z 1001374c     qt-mt323:qt-mt323.dll
 0002:00000750       __imp_?setup@QListViewItem@@UAEXXZ 10013750     qt-mt323:qt-mt323.dll
 0002:00000754       __imp_?sort@QListViewItem@@UAEXXZ 10013754     qt-mt323:qt-mt323.dll
 0002:00000758       __imp_?sortChildItems@QListViewItem@@UAEXH_N@Z 10013758     qt-mt323:qt-mt323.dll
 0002:0000075c       __imp_?startRename@QListViewItem@@UAEXH@Z 1001375c     qt-mt323:qt-mt323.dll
 0002:00000760       __imp_?takeItem@QListViewItem@@UAEXPAV1@@Z 10013760     qt-mt323:qt-mt323.dll
 0002:00000764       __imp_?text@QListViewItem@@UBE?AVQString@@H@Z 10013764     qt-mt323:qt-mt323.dll
 0002:00000768       __imp_?width@QListViewItem@@UBEHABVQFontMetrics@@PBVQListView@@H@Z 10013768     qt-mt323:qt-mt323.dll
 0002:0000076c       __imp_?isDigit@QChar@@QBE_NXZ 1001376c     qt-mt323:qt-mt323.dll
 0002:00000770       __imp_?remove@QString@@QAEAAV1@II@Z 10013770     qt-mt323:qt-mt323.dll
 0002:00000774       __imp_?upper@QCharRef@@QBE?AVQChar@@XZ 10013774     qt-mt323:qt-mt323.dll
 0002:00000778       __imp_??0QListViewItem@@QAE@PAVQListView@@@Z 10013778     qt-mt323:qt-mt323.dll
 0002:0000077c       __imp_??6?$QValueList@VQString@@@@QAEAAV0@ABVQString@@@Z 1001377c     qt-mt323:qt-mt323.dll
 0002:00000780       __imp_?findIndex@?$QValueList@VQString@@@@QBEHABVQString@@@Z 10013780     qt-mt323:qt-mt323.dll
 0002:00000784       __imp_?sort@QStringList@@QAEXXZ 10013784     qt-mt323:qt-mt323.dll
 0002:00000788       __imp_?selectedItem@QListView@@QBEPAVQListViewItem@@XZ 10013788     qt-mt323:qt-mt323.dll
 0002:0000078c       __imp_?flush@QFile@@UAEXXZ 1001378c     qt-mt323:qt-mt323.dll
 0002:00000790       __imp_?getItem@QInputDialog@@SA?AVQString@@ABV2@0ABVQStringList@@H_NPA_NPAVQWidget@@PBD@Z 10013790     qt-mt323:qt-mt323.dll
 0002:00000794       __imp_??0QPixmap@@QAE@XZ   10013794     qt-mt323:qt-mt323.dll
 0002:00000798       __imp_?setTabOrder@QWidget@@SAXPAV1@0@Z 10013798     qt-mt323:qt-mt323.dll
 0002:0000079c       __imp_?resize@QWidget@@QAEXABVQSize@@@Z 1001379c     qt-mt323:qt-mt323.dll
 0002:000007a0       __imp_?setFrameShape@QFrame@@QAEXW4Shape@1@@Z 100137a0     qt-mt323:qt-mt323.dll
 0002:000007a4       __imp_?setFrameShadow@QFrame@@QAEXW4Shadow@1@@Z 100137a4     qt-mt323:qt-mt323.dll
 0002:000007a8       __imp_??0QListView@@QAE@PAVQWidget@@PBDI@Z 100137a8     qt-mt323:qt-mt323.dll
 0002:000007ac       __imp_??1QListView@@UAE@XZ 100137ac     qt-mt323:qt-mt323.dll
 0002:000007b0       __imp_?header@QListView@@QBEPAVQHeader@@XZ 100137b0     qt-mt323:qt-mt323.dll
 0002:000007b4       __imp_??1QButton@@UAE@XZ   100137b4     qt-mt323:qt-mt323.dll
 0002:000007b8       __imp_??0QPushButton@@QAE@PAVQWidget@@PBD@Z 100137b8     qt-mt323:qt-mt323.dll
 0002:000007bc       __imp_??1QPushButton@@UAE@XZ 100137bc     qt-mt323:qt-mt323.dll
 0002:000007c0       __imp_??0QLabel@@QAE@PAVQWidget@@PBDI@Z 100137c0     qt-mt323:qt-mt323.dll
 0002:000007c4       __imp_??1QLabel@@UAE@XZ    100137c4     qt-mt323:qt-mt323.dll
 0002:000007c8       __imp_??0QComboBox@@QAE@_NPAVQWidget@@PBD@Z 100137c8     qt-mt323:qt-mt323.dll
 0002:000007cc       __imp_??1QComboBox@@UAE@XZ 100137cc     qt-mt323:qt-mt323.dll
 0002:000007d0       __imp_?setEditable@QComboBox@@QAEX_N@Z 100137d0     qt-mt323:qt-mt323.dll
 0002:000007d4       __imp_?clear@QComboBox@@QAEXXZ 100137d4     qt-mt323:qt-mt323.dll
 0002:000007d8       __imp_??0QGroupBox@@QAE@PAVQWidget@@PBD@Z 100137d8     qt-mt323:qt-mt323.dll
 0002:000007dc       __imp_?setName@QWidget@@UAEXPBD@Z 100137dc     qt-mt323:qt-mt323.dll
 0002:000007e0       __imp_??0QSpinBox@@QAE@PAVQWidget@@PBD@Z 100137e0     qt-mt323:qt-mt323.dll
 0002:000007e4       __imp_??1QSpinBox@@UAE@XZ  100137e4     qt-mt323:qt-mt323.dll
 0002:000007e8       __imp_?setMinValue@QSpinBox@@QAEXH@Z 100137e8     qt-mt323:qt-mt323.dll
 0002:000007ec       __imp_?setMaxValue@QSpinBox@@QAEXH@Z 100137ec     qt-mt323:qt-mt323.dll
 0002:000007f0       __imp_??0QLineEdit@@QAE@PAVQWidget@@PBD@Z 100137f0     qt-mt323:qt-mt323.dll
 0002:000007f4       __imp_??1QLineEdit@@UAE@XZ 100137f4     qt-mt323:qt-mt323.dll
 0002:000007f8       __imp_??0QWidgetStack@@QAE@PAVQWidget@@PBD@Z 100137f8     qt-mt323:qt-mt323.dll
 0002:000007fc       __imp_??1QWidgetStack@@UAE@XZ 100137fc     qt-mt323:qt-mt323.dll
 0002:00000800       __imp_?addWidget@QWidgetStack@@QAEHPAVQWidget@@H@Z 10013800     qt-mt323:qt-mt323.dll
 0002:00000804       __imp_??0QCheckBox@@QAE@PAVQWidget@@PBD@Z 10013804     qt-mt323:qt-mt323.dll
 0002:00000808       __imp_??1QLayoutItem@@UAE@XZ 10013808     qt-mt323:qt-mt323.dll
 0002:0000080c       __imp_??0QSpacerItem@@QAE@HHW4SizeType@QSizePolicy@@0@Z 1001380c     qt-mt323:qt-mt323.dll
 0002:00000810       __imp_??0QGridLayout@@QAE@PAVQWidget@@HHHHPBD@Z 10013810     qt-mt323:qt-mt323.dll
 0002:00000814       __imp_??0QGridLayout@@QAE@PAVQLayout@@HHHPBD@Z 10013814     qt-mt323:qt-mt323.dll
 0002:00000818       __imp_??1QGridLayout@@UAE@XZ 10013818     qt-mt323:qt-mt323.dll
 0002:0000081c       __imp_?addItem@QGridLayout@@QAEXPAVQLayoutItem@@HH@Z 1001381c     qt-mt323:qt-mt323.dll
 0002:00000820       __imp_?addWidget@QGridLayout@@QAEXPAVQWidget@@HHH@Z 10013820     qt-mt323:qt-mt323.dll
 0002:00000824       __imp_?addMultiCellWidget@QGridLayout@@QAEXPAVQWidget@@HHHHH@Z 10013824     qt-mt323:qt-mt323.dll
 0002:00000828       __imp_?addWidget@QBoxLayout@@QAEXPAVQWidget@@HH@Z 10013828     qt-mt323:qt-mt323.dll
 0002:0000082c       __imp_?addLayout@QBoxLayout@@QAEXPAVQLayout@@H@Z 1001382c     qt-mt323:qt-mt323.dll
 0002:00000830       __imp_??0QHBoxLayout@@QAE@PAVQWidget@@HHPBD@Z 10013830     qt-mt323:qt-mt323.dll
 0002:00000834       __imp_??1QHBoxLayout@@UAE@XZ 10013834     qt-mt323:qt-mt323.dll
 0002:00000838       __imp_??0QVBoxLayout@@QAE@PAVQWidget@@HHPBD@Z 10013838     qt-mt323:qt-mt323.dll
 0002:0000083c       __imp_??0QVBoxLayout@@QAE@PAVQLayout@@HPBD@Z 1001383c     qt-mt323:qt-mt323.dll
 0002:00000840       __imp_??1QVBoxLayout@@UAE@XZ 10013840     qt-mt323:qt-mt323.dll
 0002:00000844       __imp_?add@QToolTip@@SAXPAVQWidget@@ABVQString@@@Z 10013844     qt-mt323:qt-mt323.dll
 0002:00000848       __imp_?addChild@QScrollView@@UAEXPAVQWidget@@HH@Z 10013848     qt-mt323:qt-mt323.dll
 0002:0000084c       __imp_?addColumn@QListView@@UAEHABVQIconSet@@ABVQString@@H@Z 1001384c     qt-mt323:qt-mt323.dll
 0002:00000850       __imp_?addColumn@QListView@@UAEHABVQString@@H@Z 10013850     qt-mt323:qt-mt323.dll
 0002:00000854       __imp_?addItem@QBoxLayout@@UAEXPAVQLayoutItem@@@Z 10013854     qt-mt323:qt-mt323.dll
 0002:00000858       __imp_?addItem@QGridLayout@@UAEXPAVQLayoutItem@@@Z 10013858     qt-mt323:qt-mt323.dll
 0002:0000085c       __imp_?childEvent@QGroupBox@@MAEXPAVQChildEvent@@@Z 1001385c     qt-mt323:qt-mt323.dll
 0002:00000860       __imp_?childEvent@QLayout@@MAEXPAVQChildEvent@@@Z 10013860     qt-mt323:qt-mt323.dll
 0002:00000864       __imp_?childEvent@QWidgetStack@@MAEXPAVQChildEvent@@@Z 10013864     qt-mt323:qt-mt323.dll
 0002:00000868       __imp_?className@QCheckBox@@UBEPBDXZ 10013868     qt-mt323:qt-mt323.dll
 0002:0000086c       __imp_?className@QComboBox@@UBEPBDXZ 1001386c     qt-mt323:qt-mt323.dll
 0002:00000870       __imp_?className@QGridLayout@@UBEPBDXZ 10013870     qt-mt323:qt-mt323.dll
 0002:00000874       __imp_?className@QGroupBox@@UBEPBDXZ 10013874     qt-mt323:qt-mt323.dll
 0002:00000878       __imp_?className@QHBoxLayout@@UBEPBDXZ 10013878     qt-mt323:qt-mt323.dll
 0002:0000087c       __imp_?className@QLabel@@UBEPBDXZ 1001387c     qt-mt323:qt-mt323.dll
 0002:00000880       __imp_?className@QLineEdit@@UBEPBDXZ 10013880     qt-mt323:qt-mt323.dll
 0002:00000884       __imp_?className@QListView@@UBEPBDXZ 10013884     qt-mt323:qt-mt323.dll
 0002:00000888       __imp_?className@QPushButton@@UBEPBDXZ 10013888     qt-mt323:qt-mt323.dll
 0002:0000088c       __imp_?className@QSpinBox@@UBEPBDXZ 1001388c     qt-mt323:qt-mt323.dll
 0002:00000890       __imp_?className@QVBoxLayout@@UBEPBDXZ 10013890     qt-mt323:qt-mt323.dll
 0002:00000894       __imp_?className@QWidgetStack@@UBEPBDXZ 10013894     qt-mt323:qt-mt323.dll
 0002:00000898       __imp_?cleanText@QSpinBox@@UBE?AVQString@@XZ 10013898     qt-mt323:qt-mt323.dll
 0002:0000089c       __imp_?clear@QLineEdit@@UAEXXZ 1001389c     qt-mt323:qt-mt323.dll
 0002:000008a0       __imp_?clear@QListView@@UAEXXZ 100138a0     qt-mt323:qt-mt323.dll
 0002:000008a4       __imp_?clearSelection@QListView@@UAEXXZ 100138a4     qt-mt323:qt-mt323.dll
 0002:000008a8       __imp_?clearValidator@QLineEdit@@UAEXXZ 100138a8     qt-mt323:qt-mt323.dll
 0002:000008ac       __imp_?contentsContextMenuEvent@QListView@@MAEXPAVQContextMenuEvent@@@Z 100138ac     qt-mt323:qt-mt323.dll
 0002:000008b0       __imp_?contentsDragEnterEvent@QListView@@MAEXPAVQDragEnterEvent@@@Z 100138b0     qt-mt323:qt-mt323.dll
 0002:000008b4       __imp_?contentsDragLeaveEvent@QListView@@MAEXPAVQDragLeaveEvent@@@Z 100138b4     qt-mt323:qt-mt323.dll
 0002:000008b8       __imp_?contentsDragMoveEvent@QListView@@MAEXPAVQDragMoveEvent@@@Z 100138b8     qt-mt323:qt-mt323.dll
 0002:000008bc       __imp_?contentsDropEvent@QListView@@MAEXPAVQDropEvent@@@Z 100138bc     qt-mt323:qt-mt323.dll
 0002:000008c0       __imp_?contentsMouseDoubleClickEvent@QListView@@MAEXPAVQMouseEvent@@@Z 100138c0     qt-mt323:qt-mt323.dll
 0002:000008c4       __imp_?contentsMouseMoveEvent@QListView@@MAEXPAVQMouseEvent@@@Z 100138c4     qt-mt323:qt-mt323.dll
 0002:000008c8       __imp_?contentsMousePressEvent@QListView@@MAEXPAVQMouseEvent@@@Z 100138c8     qt-mt323:qt-mt323.dll
 0002:000008cc       __imp_?contentsMouseReleaseEvent@QListView@@MAEXPAVQMouseEvent@@@Z 100138cc     qt-mt323:qt-mt323.dll
 0002:000008d0       __imp_?contentsWheelEvent@QScrollView@@MAEXPAVQWheelEvent@@@Z 100138d0     qt-mt323:qt-mt323.dll
 0002:000008d4       __imp_?contextMenuEvent@QLineEdit@@MAEXPAVQContextMenuEvent@@@Z 100138d4     qt-mt323:qt-mt323.dll
 0002:000008d8       __imp_?contextMenuEvent@QScrollView@@MAEXPAVQContextMenuEvent@@@Z 100138d8     qt-mt323:qt-mt323.dll
 0002:000008dc       __imp_?copy@QLineEdit@@UBEXXZ 100138dc     qt-mt323:qt-mt323.dll
 0002:000008e0       __imp_?createPopupMenu@QLineEdit@@MAEPAVQPopupMenu@@XZ 100138e0     qt-mt323:qt-mt323.dll
 0002:000008e4       __imp_?cut@QLineEdit@@UAEXXZ 100138e4     qt-mt323:qt-mt323.dll
 0002:000008e8       __imp_?deselect@QLineEdit@@UAEXXZ 100138e8     qt-mt323:qt-mt323.dll
 0002:000008ec       __imp_?dragEnterEvent@QLineEdit@@MAEXPAVQDragEnterEvent@@@Z 100138ec     qt-mt323:qt-mt323.dll
 0002:000008f0       __imp_?dragLeaveEvent@QLineEdit@@MAEXPAVQDragLeaveEvent@@@Z 100138f0     qt-mt323:qt-mt323.dll
 0002:000008f4       __imp_?dragMoveEvent@QLineEdit@@MAEXPAVQDragMoveEvent@@@Z 100138f4     qt-mt323:qt-mt323.dll
 0002:000008f8       __imp_?dragObject@QListView@@MAEPAVQDragObject@@XZ 100138f8     qt-mt323:qt-mt323.dll
 0002:000008fc       __imp_?drawButton@QCheckBox@@MAEXPAVQPainter@@@Z 100138fc     qt-mt323:qt-mt323.dll
 0002:00000900       __imp_?drawButton@QPushButton@@MAEXPAVQPainter@@@Z 10013900     qt-mt323:qt-mt323.dll
 0002:00000904       __imp_?drawButtonLabel@QCheckBox@@MAEXPAVQPainter@@@Z 10013904     qt-mt323:qt-mt323.dll
 0002:00000908       __imp_?drawButtonLabel@QPushButton@@MAEXPAVQPainter@@@Z 10013908     qt-mt323:qt-mt323.dll
 0002:0000090c       __imp_?drawContents@QFrame@@MAEXPAVQPainter@@@Z 1001390c     qt-mt323:qt-mt323.dll
 0002:00000910       __imp_?drawContents@QLabel@@MAEXPAVQPainter@@@Z 10013910     qt-mt323:qt-mt323.dll
 0002:00000914       __imp_?drawContents@QLineEdit@@MAEXPAVQPainter@@@Z 10013914     qt-mt323:qt-mt323.dll
 0002:00000918       __imp_?drawContents@QScrollView@@EAEXPAVQPainter@@@Z 10013918     qt-mt323:qt-mt323.dll
 0002:0000091c       __imp_?drawContents@QScrollView@@MAEXPAVQPainter@@HHHH@Z 1001391c     qt-mt323:qt-mt323.dll
 0002:00000920       __imp_?drawContentsOffset@QListView@@MAEXPAVQPainter@@HHHHHH@Z 10013920     qt-mt323:qt-mt323.dll
 0002:00000924       __imp_?dropEvent@QLineEdit@@MAEXPAVQDropEvent@@@Z 10013924     qt-mt323:qt-mt323.dll
 0002:00000928       __imp_?enabledChange@QButton@@MAEX_N@Z 10013928     qt-mt323:qt-mt323.dll
 0002:0000092c       __imp_?event@QGroupBox@@MAE_NPAVQEvent@@@Z 1001392c     qt-mt323:qt-mt323.dll
 0002:00000930       __imp_?event@QLineEdit@@MAE_NPAVQEvent@@@Z 10013930     qt-mt323:qt-mt323.dll
 0002:00000934       __imp_?eventFilter@QComboBox@@UAE_NPAVQObject@@PAVQEvent@@@Z 10013934     qt-mt323:qt-mt323.dll
 0002:00000938       __imp_?eventFilter@QLayout@@MAE_NPAVQObject@@PAVQEvent@@@Z 10013938     qt-mt323:qt-mt323.dll
 0002:0000093c       __imp_?eventFilter@QListView@@UAE_NPAVQObject@@PAVQEvent@@@Z 1001393c     qt-mt323:qt-mt323.dll
 0002:00000940       __imp_?eventFilter@QSpinBox@@MAE_NPAVQObject@@PAVQEvent@@@Z 10013940     qt-mt323:qt-mt323.dll
 0002:00000944       __imp_?expanding@QBoxLayout@@UBE?AW4ExpandData@QSizePolicy@@XZ 10013944     qt-mt323:qt-mt323.dll
 0002:00000948       __imp_?expanding@QGridLayout@@UBE?AW4ExpandData@QSizePolicy@@XZ 10013948     qt-mt323:qt-mt323.dll
 0002:0000094c       __imp_?expanding@QSpacerItem@@UBE?AW4ExpandData@QSizePolicy@@XZ 1001394c     qt-mt323:qt-mt323.dll
 0002:00000950       __imp_?focusInEvent@QButton@@MAEXPAVQFocusEvent@@@Z 10013950     qt-mt323:qt-mt323.dll
 0002:00000954       __imp_?focusInEvent@QComboBox@@MAEXPAVQFocusEvent@@@Z 10013954     qt-mt323:qt-mt323.dll
 0002:00000958       __imp_?focusInEvent@QGroupBox@@MAEXPAVQFocusEvent@@@Z 10013958     qt-mt323:qt-mt323.dll
 0002:0000095c       __imp_?focusInEvent@QLineEdit@@MAEXPAVQFocusEvent@@@Z 1001395c     qt-mt323:qt-mt323.dll
 0002:00000960       __imp_?focusInEvent@QListView@@MAEXPAVQFocusEvent@@@Z 10013960     qt-mt323:qt-mt323.dll
 0002:00000964       __imp_?focusInEvent@QPushButton@@MAEXPAVQFocusEvent@@@Z 10013964     qt-mt323:qt-mt323.dll
 0002:00000968       __imp_?focusNextPrevChild@QScrollView@@MAE_N_N@Z 10013968     qt-mt323:qt-mt323.dll
 0002:0000096c       __imp_?focusOutEvent@QButton@@MAEXPAVQFocusEvent@@@Z 1001396c     qt-mt323:qt-mt323.dll
 0002:00000970       __imp_?focusOutEvent@QComboBox@@MAEXPAVQFocusEvent@@@Z 10013970     qt-mt323:qt-mt323.dll
 0002:00000974       __imp_?focusOutEvent@QLineEdit@@MAEXPAVQFocusEvent@@@Z 10013974     qt-mt323:qt-mt323.dll
 0002:00000978       __imp_?focusOutEvent@QListView@@MAEXPAVQFocusEvent@@@Z 10013978     qt-mt323:qt-mt323.dll
 0002:0000097c       __imp_?focusOutEvent@QPushButton@@MAEXPAVQFocusEvent@@@Z 1001397c     qt-mt323:qt-mt323.dll
 0002:00000980       __imp_?fontChange@QGroupBox@@MAEXABVQFont@@@Z 10013980     qt-mt323:qt-mt323.dll
 0002:00000984       __imp_?fontChange@QLabel@@MAEXABVQFont@@@Z 10013984     qt-mt323:qt-mt323.dll
 0002:00000988       __imp_?fontChange@QScrollView@@MAEXABVQFont@@@Z 10013988     qt-mt323:qt-mt323.dll
 0002:0000098c       __imp_?frameChanged@QScrollView@@MAEXXZ 1001398c     qt-mt323:qt-mt323.dll
 0002:00000990       __imp_?frameChanged@QWidgetStack@@MAEXXZ 10013990     qt-mt323:qt-mt323.dll
 0002:00000994       __imp_?geometry@QLayout@@UBE?AVQRect@@XZ 10013994     qt-mt323:qt-mt323.dll
 0002:00000998       __imp_?geometry@QSpacerItem@@UBE?AVQRect@@XZ 10013998     qt-mt323:qt-mt323.dll
 0002:0000099c       __imp_?hasHeightForWidth@QBoxLayout@@UBE_NXZ 1001399c     qt-mt323:qt-mt323.dll
 0002:000009a0       __imp_?hasHeightForWidth@QGridLayout@@UBE_NXZ 100139a0     qt-mt323:qt-mt323.dll
 0002:000009a4       __imp_?hasHeightForWidth@QLayoutItem@@UBE_NXZ 100139a4     qt-mt323:qt-mt323.dll
 0002:000009a8       __imp_?heightForWidth@QBoxLayout@@UBEHH@Z 100139a8     qt-mt323:qt-mt323.dll
 0002:000009ac       __imp_?heightForWidth@QGridLayout@@UBEHH@Z 100139ac     qt-mt323:qt-mt323.dll
 0002:000009b0       __imp_?heightForWidth@QLabel@@UBEHH@Z 100139b0     qt-mt323:qt-mt323.dll
 0002:000009b4       __imp_?heightForWidth@QLayoutItem@@UBEHH@Z 100139b4     qt-mt323:qt-mt323.dll
 0002:000009b8       __imp_?hitButton@QButton@@MBE_NABVQPoint@@@Z 100139b8     qt-mt323:qt-mt323.dll
 0002:000009bc       __imp_?hitButton@QCheckBox@@MBE_NABVQPoint@@@Z 100139bc     qt-mt323:qt-mt323.dll
 0002:000009c0       __imp_?imComposeEvent@QLineEdit@@MAEXPAVQIMEvent@@@Z 100139c0     qt-mt323:qt-mt323.dll
 0002:000009c4       __imp_?imEndEvent@QLineEdit@@MAEXPAVQIMEvent@@@Z 100139c4     qt-mt323:qt-mt323.dll
 0002:000009c8       __imp_?imStartEvent@QLineEdit@@MAEXPAVQIMEvent@@@Z 100139c8     qt-mt323:qt-mt323.dll
 0002:000009cc       __imp_?insert@QLineEdit@@UAEXABVQString@@@Z 100139cc     qt-mt323:qt-mt323.dll
 0002:000009d0       __imp_?insertItem@QListView@@UAEXPAVQListViewItem@@@Z 100139d0     qt-mt323:qt-mt323.dll
 0002:000009d4       __imp_?interpretText@QSpinBox@@MAEXXZ 100139d4     qt-mt323:qt-mt323.dll
 0002:000009d8       __imp_?invalidate@QBoxLayout@@UAEXXZ 100139d8     qt-mt323:qt-mt323.dll
 0002:000009dc       __imp_?invalidate@QGridLayout@@UAEXXZ 100139dc     qt-mt323:qt-mt323.dll
 0002:000009e0       __imp_?invalidate@QLayoutItem@@UAEXXZ 100139e0     qt-mt323:qt-mt323.dll
 0002:000009e4       __imp_?invertSelection@QListView@@UAEXXZ 100139e4     qt-mt323:qt-mt323.dll
 0002:000009e8       __imp_?isEmpty@QLayout@@UBE_NXZ 100139e8     qt-mt323:qt-mt323.dll
 0002:000009ec       __imp_?isEmpty@QSpacerItem@@UBE_NXZ 100139ec     qt-mt323:qt-mt323.dll
 0002:000009f0       __imp_?iterator@QBoxLayout@@UAE?AVQLayoutIterator@@XZ 100139f0     qt-mt323:qt-mt323.dll
 0002:000009f4       __imp_?iterator@QGridLayout@@UAE?AVQLayoutIterator@@XZ 100139f4     qt-mt323:qt-mt323.dll
 0002:000009f8       __imp_?iterator@QLayoutItem@@UAE?AVQLayoutIterator@@XZ 100139f8     qt-mt323:qt-mt323.dll
 0002:000009fc       __imp_?keyPressEvent@QButton@@MAEXPAVQKeyEvent@@@Z 100139fc     qt-mt323:qt-mt323.dll
 0002:00000a00       __imp_?keyPressEvent@QComboBox@@MAEXPAVQKeyEvent@@@Z 10013a00     qt-mt323:qt-mt323.dll
 0002:00000a04       __imp_?keyPressEvent@QLineEdit@@MAEXPAVQKeyEvent@@@Z 10013a04     qt-mt323:qt-mt323.dll
 0002:00000a08       __imp_?keyPressEvent@QListView@@MAEXPAVQKeyEvent@@@Z 10013a08     qt-mt323:qt-mt323.dll
 0002:00000a0c       __imp_?keyReleaseEvent@QButton@@MAEXPAVQKeyEvent@@@Z 10013a0c     qt-mt323:qt-mt323.dll
 0002:00000a10       __imp_?layout@QLayout@@UAEPAV1@XZ 10013a10     qt-mt323:qt-mt323.dll
 0002:00000a14       __imp_?layout@QLayoutItem@@UAEPAVQLayout@@XZ 10013a14     qt-mt323:qt-mt323.dll
 0002:00000a18       __imp_?leaveEvent@QSpinBox@@MAEXPAVQEvent@@@Z 10013a18     qt-mt323:qt-mt323.dll
 0002:00000a1c       __imp_?mapTextToValue@QSpinBox@@MAEHPA_N@Z 10013a1c     qt-mt323:qt-mt323.dll
 0002:00000a20       __imp_?mapValueToText@QSpinBox@@MAE?AVQString@@H@Z 10013a20     qt-mt323:qt-mt323.dll
 0002:00000a24       __imp_?maximumSize@QBoxLayout@@UBE?AVQSize@@XZ 10013a24     qt-mt323:qt-mt323.dll
 0002:00000a28       __imp_?maximumSize@QGridLayout@@UBE?AVQSize@@XZ 10013a28     qt-mt323:qt-mt323.dll
 0002:00000a2c       __imp_?maximumSize@QSpacerItem@@UBE?AVQSize@@XZ 10013a2c     qt-mt323:qt-mt323.dll
 0002:00000a30       __imp_?metaObject@QCheckBox@@UBEPAVQMetaObject@@XZ 10013a30     qt-mt323:qt-mt323.dll
 0002:00000a34       __imp_?metaObject@QComboBox@@UBEPAVQMetaObject@@XZ 10013a34     qt-mt323:qt-mt323.dll
 0002:00000a38       __imp_?metaObject@QGridLayout@@UBEPAVQMetaObject@@XZ 10013a38     qt-mt323:qt-mt323.dll
 0002:00000a3c       __imp_?metaObject@QGroupBox@@UBEPAVQMetaObject@@XZ 10013a3c     qt-mt323:qt-mt323.dll
 0002:00000a40       __imp_?metaObject@QHBoxLayout@@UBEPAVQMetaObject@@XZ 10013a40     qt-mt323:qt-mt323.dll
 0002:00000a44       __imp_?metaObject@QLabel@@UBEPAVQMetaObject@@XZ 10013a44     qt-mt323:qt-mt323.dll
 0002:00000a48       __imp_?metaObject@QLineEdit@@UBEPAVQMetaObject@@XZ 10013a48     qt-mt323:qt-mt323.dll
 0002:00000a4c       __imp_?metaObject@QListView@@UBEPAVQMetaObject@@XZ 10013a4c     qt-mt323:qt-mt323.dll
 0002:00000a50       __imp_?metaObject@QPushButton@@UBEPAVQMetaObject@@XZ 10013a50     qt-mt323:qt-mt323.dll
 0002:00000a54       __imp_?metaObject@QSpinBox@@UBEPAVQMetaObject@@XZ 10013a54     qt-mt323:qt-mt323.dll
 0002:00000a58       __imp_?metaObject@QVBoxLayout@@UBEPAVQMetaObject@@XZ 10013a58     qt-mt323:qt-mt323.dll
 0002:00000a5c       __imp_?metaObject@QWidgetStack@@UBEPAVQMetaObject@@XZ 10013a5c     qt-mt323:qt-mt323.dll
 0002:00000a60       __imp_?minimumSize@QBoxLayout@@UBE?AVQSize@@XZ 10013a60     qt-mt323:qt-mt323.dll
 0002:00000a64       __imp_?minimumSize@QGridLayout@@UBE?AVQSize@@XZ 10013a64     qt-mt323:qt-mt323.dll
 0002:00000a68       __imp_?minimumSize@QSpacerItem@@UBE?AVQSize@@XZ 10013a68     qt-mt323:qt-mt323.dll
 0002:00000a6c       __imp_?minimumSizeHint@QLabel@@UBE?AVQSize@@XZ 10013a6c     qt-mt323:qt-mt323.dll
 0002:00000a70       __imp_?minimumSizeHint@QLineEdit@@UBE?AVQSize@@XZ 10013a70     qt-mt323:qt-mt323.dll
 0002:00000a74       __imp_?minimumSizeHint@QListView@@UBE?AVQSize@@XZ 10013a74     qt-mt323:qt-mt323.dll
 0002:00000a78       __imp_?minimumSizeHint@QSpinBox@@UBE?AVQSize@@XZ 10013a78     qt-mt323:qt-mt323.dll
 0002:00000a7c       __imp_?minimumSizeHint@QWidgetStack@@UBE?AVQSize@@XZ 10013a7c     qt-mt323:qt-mt323.dll
 0002:00000a80       __imp_?mouseDoubleClickEvent@QComboBox@@MAEXPAVQMouseEvent@@@Z 10013a80     qt-mt323:qt-mt323.dll
 0002:00000a84       __imp_?mouseDoubleClickEvent@QLineEdit@@MAEXPAVQMouseEvent@@@Z 10013a84     qt-mt323:qt-mt323.dll
 0002:00000a88       __imp_?mouseDoubleClickEvent@QScrollView@@MAEXPAVQMouseEvent@@@Z 10013a88     qt-mt323:qt-mt323.dll
 0002:00000a8c       __imp_?mouseMoveEvent@QButton@@MAEXPAVQMouseEvent@@@Z 10013a8c     qt-mt323:qt-mt323.dll
 0002:00000a90       __imp_?mouseMoveEvent@QComboBox@@MAEXPAVQMouseEvent@@@Z 10013a90     qt-mt323:qt-mt323.dll
 0002:00000a94       __imp_?mouseMoveEvent@QLineEdit@@MAEXPAVQMouseEvent@@@Z 10013a94     qt-mt323:qt-mt323.dll
 0002:00000a98       __imp_?mouseMoveEvent@QScrollView@@MAEXPAVQMouseEvent@@@Z 10013a98     qt-mt323:qt-mt323.dll
 0002:00000a9c       __imp_?mousePressEvent@QButton@@MAEXPAVQMouseEvent@@@Z 10013a9c     qt-mt323:qt-mt323.dll
 0002:00000aa0       __imp_?mousePressEvent@QComboBox@@MAEXPAVQMouseEvent@@@Z 10013aa0     qt-mt323:qt-mt323.dll
 0002:00000aa4       __imp_?mousePressEvent@QLineEdit@@MAEXPAVQMouseEvent@@@Z 10013aa4     qt-mt323:qt-mt323.dll
 0002:00000aa8       __imp_?mousePressEvent@QScrollView@@MAEXPAVQMouseEvent@@@Z 10013aa8     qt-mt323:qt-mt323.dll
 0002:00000aac       __imp_?mouseReleaseEvent@QButton@@MAEXPAVQMouseEvent@@@Z 10013aac     qt-mt323:qt-mt323.dll
 0002:00000ab0       __imp_?mouseReleaseEvent@QComboBox@@MAEXPAVQMouseEvent@@@Z 10013ab0     qt-mt323:qt-mt323.dll
 0002:00000ab4       __imp_?mouseReleaseEvent@QLineEdit@@MAEXPAVQMouseEvent@@@Z 10013ab4     qt-mt323:qt-mt323.dll
 0002:00000ab8       __imp_?mouseReleaseEvent@QScrollView@@MAEXPAVQMouseEvent@@@Z 10013ab8     qt-mt323:qt-mt323.dll
 0002:00000abc       __imp_?move@QPushButton@@UAEXHH@Z 10013abc     qt-mt323:qt-mt323.dll
 0002:00000ac0       __imp_?moveChild@QScrollView@@UAEXPAVQWidget@@HH@Z 10013ac0     qt-mt323:qt-mt323.dll
 0002:00000ac4       __imp_?paintEmptyArea@QListView@@MAEXPAVQPainter@@ABVQRect@@@Z 10013ac4     qt-mt323:qt-mt323.dll
 0002:00000ac8       __imp_?paintEvent@QButton@@MAEXPAVQPaintEvent@@@Z 10013ac8     qt-mt323:qt-mt323.dll
 0002:00000acc       __imp_?paintEvent@QComboBox@@MAEXPAVQPaintEvent@@@Z 10013acc     qt-mt323:qt-mt323.dll
 0002:00000ad0       __imp_?paintEvent@QGroupBox@@MAEXPAVQPaintEvent@@@Z 10013ad0     qt-mt323:qt-mt323.dll
 0002:00000ad4       __imp_?paste@QLineEdit@@UAEXXZ 10013ad4     qt-mt323:qt-mt323.dll
 0002:00000ad8       __imp_?popup@QComboBox@@UAEXXZ 10013ad8     qt-mt323:qt-mt323.dll
 0002:00000adc       __imp_?prefix@QSpinBox@@UBE?AVQString@@XZ 10013adc     qt-mt323:qt-mt323.dll
 0002:00000ae0       __imp_?qt_cast@QCheckBox@@UAEPAXPBD@Z 10013ae0     qt-mt323:qt-mt323.dll
 0002:00000ae4       __imp_?qt_cast@QComboBox@@UAEPAXPBD@Z 10013ae4     qt-mt323:qt-mt323.dll
 0002:00000ae8       __imp_?qt_cast@QGridLayout@@UAEPAXPBD@Z 10013ae8     qt-mt323:qt-mt323.dll
 0002:00000aec       __imp_?qt_cast@QGroupBox@@UAEPAXPBD@Z 10013aec     qt-mt323:qt-mt323.dll
 0002:00000af0       __imp_?qt_cast@QHBoxLayout@@UAEPAXPBD@Z 10013af0     qt-mt323:qt-mt323.dll
 0002:00000af4       __imp_?qt_cast@QLabel@@UAEPAXPBD@Z 10013af4     qt-mt323:qt-mt323.dll
 0002:00000af8       __imp_?qt_cast@QLineEdit@@UAEPAXPBD@Z 10013af8     qt-mt323:qt-mt323.dll
 0002:00000afc       __imp_?qt_cast@QListView@@UAEPAXPBD@Z 10013afc     qt-mt323:qt-mt323.dll
 0002:00000b00       __imp_?qt_cast@QPushButton@@UAEPAXPBD@Z 10013b00     qt-mt323:qt-mt323.dll
 0002:00000b04       __imp_?qt_cast@QSpinBox@@UAEPAXPBD@Z 10013b04     qt-mt323:qt-mt323.dll
 0002:00000b08       __imp_?qt_cast@QVBoxLayout@@UAEPAXPBD@Z 10013b08     qt-mt323:qt-mt323.dll
 0002:00000b0c       __imp_?qt_cast@QWidgetStack@@UAEPAXPBD@Z 10013b0c     qt-mt323:qt-mt323.dll
 0002:00000b10       __imp_?qt_emit@QCheckBox@@UAE_NHPAUQUObject@@@Z 10013b10     qt-mt323:qt-mt323.dll
 0002:00000b14       __imp_?qt_emit@QComboBox@@UAE_NHPAUQUObject@@@Z 10013b14     qt-mt323:qt-mt323.dll
 0002:00000b18       __imp_?qt_emit@QGridLayout@@UAE_NHPAUQUObject@@@Z 10013b18     qt-mt323:qt-mt323.dll
 0002:00000b1c       __imp_?qt_emit@QGroupBox@@UAE_NHPAUQUObject@@@Z 10013b1c     qt-mt323:qt-mt323.dll
 0002:00000b20       __imp_?qt_emit@QHBoxLayout@@UAE_NHPAUQUObject@@@Z 10013b20     qt-mt323:qt-mt323.dll
 0002:00000b24       __imp_?qt_emit@QLabel@@UAE_NHPAUQUObject@@@Z 10013b24     qt-mt323:qt-mt323.dll
 0002:00000b28       __imp_?qt_emit@QLineEdit@@UAE_NHPAUQUObject@@@Z 10013b28     qt-mt323:qt-mt323.dll
 0002:00000b2c       __imp_?qt_emit@QListView@@UAE_NHPAUQUObject@@@Z 10013b2c     qt-mt323:qt-mt323.dll
 0002:00000b30       __imp_?qt_emit@QPushButton@@UAE_NHPAUQUObject@@@Z 10013b30     qt-mt323:qt-mt323.dll
 0002:00000b34       __imp_?qt_emit@QSpinBox@@UAE_NHPAUQUObject@@@Z 10013b34     qt-mt323:qt-mt323.dll
 0002:00000b38       __imp_?qt_emit@QVBoxLayout@@UAE_NHPAUQUObject@@@Z 10013b38     qt-mt323:qt-mt323.dll
 0002:00000b3c       __imp_?qt_emit@QWidgetStack@@UAE_NHPAUQUObject@@@Z 10013b3c     qt-mt323:qt-mt323.dll
 0002:00000b40       __imp_?qt_invoke@QCheckBox@@UAE_NHPAUQUObject@@@Z 10013b40     qt-mt323:qt-mt323.dll
 0002:00000b44       __imp_?qt_invoke@QComboBox@@UAE_NHPAUQUObject@@@Z 10013b44     qt-mt323:qt-mt323.dll
 0002:00000b48       __imp_?qt_invoke@QGridLayout@@UAE_NHPAUQUObject@@@Z 10013b48     qt-mt323:qt-mt323.dll
 0002:00000b4c       __imp_?qt_invoke@QGroupBox@@UAE_NHPAUQUObject@@@Z 10013b4c     qt-mt323:qt-mt323.dll
 0002:00000b50       __imp_?qt_invoke@QHBoxLayout@@UAE_NHPAUQUObject@@@Z 10013b50     qt-mt323:qt-mt323.dll
 0002:00000b54       __imp_?qt_invoke@QLabel@@UAE_NHPAUQUObject@@@Z 10013b54     qt-mt323:qt-mt323.dll
 0002:00000b58       __imp_?qt_invoke@QLineEdit@@UAE_NHPAUQUObject@@@Z 10013b58     qt-mt323:qt-mt323.dll
 0002:00000b5c       __imp_?qt_invoke@QListView@@UAE_NHPAUQUObject@@@Z 10013b5c     qt-mt323:qt-mt323.dll
 0002:00000b60       __imp_?qt_invoke@QPushButton@@UAE_NHPAUQUObject@@@Z 10013b60     qt-mt323:qt-mt323.dll
 0002:00000b64       __imp_?qt_invoke@QSpinBox@@UAE_NHPAUQUObject@@@Z 10013b64     qt-mt323:qt-mt323.dll
 0002:00000b68       __imp_?qt_invoke@QVBoxLayout@@UAE_NHPAUQUObject@@@Z 10013b68     qt-mt323:qt-mt323.dll
 0002:00000b6c       __imp_?qt_invoke@QWidgetStack@@UAE_NHPAUQUObject@@@Z 10013b6c     qt-mt323:qt-mt323.dll
 0002:00000b70       __imp_?qt_property@QCheckBox@@UAE_NHHPAVQVariant@@@Z 10013b70     qt-mt323:qt-mt323.dll
 0002:00000b74       __imp_?qt_property@QComboBox@@UAE_NHHPAVQVariant@@@Z 10013b74     qt-mt323:qt-mt323.dll
 0002:00000b78       __imp_?qt_property@QGridLayout@@UAE_NHHPAVQVariant@@@Z 10013b78     qt-mt323:qt-mt323.dll
 0002:00000b7c       __imp_?qt_property@QGroupBox@@UAE_NHHPAVQVariant@@@Z 10013b7c     qt-mt323:qt-mt323.dll
 0002:00000b80       __imp_?qt_property@QHBoxLayout@@UAE_NHHPAVQVariant@@@Z 10013b80     qt-mt323:qt-mt323.dll
 0002:00000b84       __imp_?qt_property@QLabel@@UAE_NHHPAVQVariant@@@Z 10013b84     qt-mt323:qt-mt323.dll
 0002:00000b88       __imp_?qt_property@QLineEdit@@UAE_NHHPAVQVariant@@@Z 10013b88     qt-mt323:qt-mt323.dll
 0002:00000b8c       __imp_?qt_property@QListView@@UAE_NHHPAVQVariant@@@Z 10013b8c     qt-mt323:qt-mt323.dll
 0002:00000b90       __imp_?qt_property@QPushButton@@UAE_NHHPAVQVariant@@@Z 10013b90     qt-mt323:qt-mt323.dll
 0002:00000b94       __imp_?qt_property@QSpinBox@@UAE_NHHPAVQVariant@@@Z 10013b94     qt-mt323:qt-mt323.dll
 0002:00000b98       __imp_?qt_property@QVBoxLayout@@UAE_NHHPAVQVariant@@@Z 10013b98     qt-mt323:qt-mt323.dll
 0002:00000b9c       __imp_?qt_property@QWidgetStack@@UAE_NHHPAVQVariant@@@Z 10013b9c     qt-mt323:qt-mt323.dll
 0002:00000ba0       __imp_?rangeChange@QSpinBox@@MAEXXZ 10013ba0     qt-mt323:qt-mt323.dll
 0002:00000ba4       __imp_?redo@QLineEdit@@UAEXXZ 10013ba4     qt-mt323:qt-mt323.dll
 0002:00000ba8       __imp_?removeChild@QScrollView@@UAEXPAVQObject@@@Z 10013ba8     qt-mt323:qt-mt323.dll
 0002:00000bac       __imp_?removeColumn@QListView@@UAEXH@Z 10013bac     qt-mt323:qt-mt323.dll
 0002:00000bb0       __imp_?removeItem@QListView@@UAEXPAVQListViewItem@@@Z 10013bb0     qt-mt323:qt-mt323.dll
 0002:00000bb4       __imp_?resize@QPushButton@@UAEXHH@Z 10013bb4     qt-mt323:qt-mt323.dll
 0002:00000bb8       __imp_?resize@QScrollView@@UAEXHH@Z 10013bb8     qt-mt323:qt-mt323.dll
 0002:00000bbc       __imp_?resizeContents@QScrollView@@UAEXHH@Z 10013bbc     qt-mt323:qt-mt323.dll
 0002:00000bc0       __imp_?resizeEvent@QCheckBox@@MAEXPAVQResizeEvent@@@Z 10013bc0     qt-mt323:qt-mt323.dll
 0002:00000bc4       __imp_?resizeEvent@QComboBox@@MAEXPAVQResizeEvent@@@Z 10013bc4     qt-mt323:qt-mt323.dll
 0002:00000bc8       __imp_?resizeEvent@QGroupBox@@MAEXPAVQResizeEvent@@@Z 10013bc8     qt-mt323:qt-mt323.dll
 0002:00000bcc       __imp_?resizeEvent@QLabel@@MAEXPAVQResizeEvent@@@Z 10013bcc     qt-mt323:qt-mt323.dll
 0002:00000bd0       __imp_?resizeEvent@QLineEdit@@MAEXPAVQResizeEvent@@@Z 10013bd0     qt-mt323:qt-mt323.dll
 0002:00000bd4       __imp_?resizeEvent@QListView@@MAEXPAVQResizeEvent@@@Z 10013bd4     qt-mt323:qt-mt323.dll
 0002:00000bd8       __imp_?resizeEvent@QPushButton@@MAEXPAVQResizeEvent@@@Z 10013bd8     qt-mt323:qt-mt323.dll
 0002:00000bdc       __imp_?resizeEvent@QSpinBox@@MAEXPAVQResizeEvent@@@Z 10013bdc     qt-mt323:qt-mt323.dll
 0002:00000be0       __imp_?resizeEvent@QWidgetStack@@MAEXPAVQResizeEvent@@@Z 10013be0     qt-mt323:qt-mt323.dll
 0002:00000be4       __imp_?selectAll@QLineEdit@@UAEXXZ 10013be4     qt-mt323:qt-mt323.dll
 0002:00000be8       __imp_?selectAll@QListView@@UAEX_N@Z 10013be8     qt-mt323:qt-mt323.dll
 0002:00000bec       __imp_?selectAll@QSpinBox@@UAEXXZ 10013bec     qt-mt323:qt-mt323.dll
 0002:00000bf0       __imp_?setAccel@QButton@@UAEXABVQKeySequence@@@Z 10013bf0     qt-mt323:qt-mt323.dll
 0002:00000bf4       __imp_?setAlignment@QGroupBox@@UAEXH@Z 10013bf4     qt-mt323:qt-mt323.dll
 0002:00000bf8       __imp_?setAlignment@QLabel@@UAEXH@Z 10013bf8     qt-mt323:qt-mt323.dll
 0002:00000bfc       __imp_?setAlignment@QLayoutItem@@UAEXH@Z 10013bfc     qt-mt323:qt-mt323.dll
 0002:00000c00       __imp_?setAlignment@QLineEdit@@UAEXH@Z 10013c00     qt-mt323:qt-mt323.dll
 0002:00000c04       __imp_?setAllColumnsShowFocus@QListView@@UAEX_N@Z 10013c04     qt-mt323:qt-mt323.dll
 0002:00000c08       __imp_?setAutoAdd@QLayout@@UAEX_N@Z 10013c08     qt-mt323:qt-mt323.dll
 0002:00000c0c       __imp_?setAutoCompletion@QComboBox@@UAEX_N@Z 10013c0c     qt-mt323:qt-mt323.dll
 0002:00000c10       __imp_?setAutoDefault@QPushButton@@UAEX_N@Z 10013c10     qt-mt323:qt-mt323.dll
 0002:00000c14       __imp_?setAutoRepeat@QButton@@UAEX_N@Z 10013c14     qt-mt323:qt-mt323.dll
 0002:00000c18       __imp_?setAutoResize@QComboBox@@UAEX_N@Z 10013c18     qt-mt323:qt-mt323.dll
 0002:00000c1c       __imp_?setAutoResize@QLabel@@UAEX_N@Z 10013c1c     qt-mt323:qt-mt323.dll
 0002:00000c20       __imp_?setBuddy@QLabel@@UAEXPAVQWidget@@@Z 10013c20     qt-mt323:qt-mt323.dll
 0002:00000c24       __imp_?setButtonSymbols@QSpinBox@@UAEXW4ButtonSymbols@1@@Z 10013c24     qt-mt323:qt-mt323.dll
 0002:00000c28       __imp_?setChildGeometries@QWidgetStack@@MAEXXZ 10013c28     qt-mt323:qt-mt323.dll
 0002:00000c2c       __imp_?setColStretch@QGridLayout@@UAEXHH@Z 10013c2c     qt-mt323:qt-mt323.dll
 0002:00000c30       __imp_?setColumnAlignment@QListView@@UAEXHH@Z 10013c30     qt-mt323:qt-mt323.dll
 0002:00000c34       __imp_?setColumnLayout@QGroupBox@@UAEXHW4Orientation@Qt@@@Z 10013c34     qt-mt323:qt-mt323.dll
 0002:00000c38       __imp_?setColumnText@QListView@@UAEXHABVQIconSet@@ABVQString@@@Z 10013c38     qt-mt323:qt-mt323.dll
 0002:00000c3c       __imp_?setColumnText@QListView@@UAEXHABVQString@@@Z 10013c3c     qt-mt323:qt-mt323.dll
 0002:00000c40       __imp_?setColumnWidth@QListView@@UAEXHH@Z 10013c40     qt-mt323:qt-mt323.dll
 0002:00000c44       __imp_?setColumnWidthMode@QListView@@UAEXHW4WidthMode@1@@Z 10013c44     qt-mt323:qt-mt323.dll
 0002:00000c48       __imp_?setContentsPos@QListView@@UAEXHH@Z 10013c48     qt-mt323:qt-mt323.dll
 0002:00000c4c       __imp_?setCornerWidget@QScrollView@@UAEXPAVQWidget@@@Z 10013c4c     qt-mt323:qt-mt323.dll
 0002:00000c50       __imp_?setCurrentItem@QComboBox@@UAEXH@Z 10013c50     qt-mt323:qt-mt323.dll
 0002:00000c54       __imp_?setCurrentItem@QListView@@UAEXPAVQListViewItem@@@Z 10013c54     qt-mt323:qt-mt323.dll
 0002:00000c58       __imp_?setCurrentText@QComboBox@@UAEXABVQString@@@Z 10013c58     qt-mt323:qt-mt323.dll
 0002:00000c5c       __imp_?setCursorPosition@QLineEdit@@UAEXH@Z 10013c5c     qt-mt323:qt-mt323.dll
 0002:00000c60       __imp_?setDefault@QPushButton@@UAEX_N@Z 10013c60     qt-mt323:qt-mt323.dll
 0002:00000c64       __imp_?setDefaultRenameAction@QListView@@UAEXW4RenameAction@1@@Z 10013c64     qt-mt323:qt-mt323.dll
 0002:00000c68       __imp_?setDown@QButton@@UAEX_N@Z 10013c68     qt-mt323:qt-mt323.dll
 0002:00000c6c       __imp_?setDragAutoScroll@QScrollView@@UAEX_N@Z 10013c6c     qt-mt323:qt-mt323.dll
 0002:00000c70       __imp_?setDragEnabled@QLineEdit@@UAEX_N@Z 10013c70     qt-mt323:qt-mt323.dll
 0002:00000c74       __imp_?setEchoMode@QLineEdit@@UAEXW4EchoMode@1@@Z 10013c74     qt-mt323:qt-mt323.dll
 0002:00000c78       __imp_?setEditText@QComboBox@@UAEXABVQString@@@Z 10013c78     qt-mt323:qt-mt323.dll
 0002:00000c7c       __imp_?setEnabled@QComboBox@@UAEX_N@Z 10013c7c     qt-mt323:qt-mt323.dll
 0002:00000c80       __imp_?setEnabled@QGroupBox@@UAEX_N@Z 10013c80     qt-mt323:qt-mt323.dll
 0002:00000c84       __imp_?setEnabled@QScrollView@@UAEX_N@Z 10013c84     qt-mt323:qt-mt323.dll
 0002:00000c88       __imp_?setEnabled@QSpinBox@@UAEX_N@Z 10013c88     qt-mt323:qt-mt323.dll
 0002:00000c8c       __imp_?setFont@QComboBox@@UAEXABVQFont@@@Z 10013c8c     qt-mt323:qt-mt323.dll
 0002:00000c90       __imp_?setFont@QLabel@@UAEXABVQFont@@@Z 10013c90     qt-mt323:qt-mt323.dll
 0002:00000c94       __imp_?setFont@QLineEdit@@UAEXABVQFont@@@Z 10013c94     qt-mt323:qt-mt323.dll
 0002:00000c98       __imp_?setFont@QListView@@UAEXABVQFont@@@Z 10013c98     qt-mt323:qt-mt323.dll
 0002:00000c9c       __imp_?setFrame@QLineEdit@@UAEX_N@Z 10013c9c     qt-mt323:qt-mt323.dll
 0002:00000ca0       __imp_?setFrameRect@QWidgetStack@@UAEXABVQRect@@@Z 10013ca0     qt-mt323:qt-mt323.dll
 0002:00000ca4       __imp_?setGeometry@QBoxLayout@@UAEXABVQRect@@@Z 10013ca4     qt-mt323:qt-mt323.dll
 0002:00000ca8       __imp_?setGeometry@QGridLayout@@UAEXABVQRect@@@Z 10013ca8     qt-mt323:qt-mt323.dll
 0002:00000cac       __imp_?setGeometry@QPushButton@@UAEXABVQRect@@@Z 10013cac     qt-mt323:qt-mt323.dll
 0002:00000cb0       __imp_?setGeometry@QPushButton@@UAEXHHHH@Z 10013cb0     qt-mt323:qt-mt323.dll
 0002:00000cb4       __imp_?setGeometry@QSpacerItem@@UAEXABVQRect@@@Z 10013cb4     qt-mt323:qt-mt323.dll
 0002:00000cb8       __imp_?setGroup@QButton@@EAEXPAVQButtonGroup@@@Z 10013cb8     qt-mt323:qt-mt323.dll
 0002:00000cbc       __imp_?setHBarGeometry@QScrollView@@MAEXAAVQScrollBar@@HHHH@Z 10013cbc     qt-mt323:qt-mt323.dll
 0002:00000cc0       __imp_?setHScrollBarMode@QScrollView@@UAEXW4ScrollBarMode@1@@Z 10013cc0     qt-mt323:qt-mt323.dll
 0002:00000cc4       __imp_?setInsertionPolicy@QComboBox@@UAEXW4Policy@1@@Z 10013cc4     qt-mt323:qt-mt323.dll
 0002:00000cc8       __imp_?setIsMenuButton@QPushButton@@UAEX_N@Z 10013cc8     qt-mt323:qt-mt323.dll
 0002:00000ccc       __imp_?setItemMargin@QListView@@UAEXH@Z 10013ccc     qt-mt323:qt-mt323.dll
 0002:00000cd0       __imp_?setLineEdit@QComboBox@@UAEXPAVQLineEdit@@@Z 10013cd0     qt-mt323:qt-mt323.dll
 0002:00000cd4       __imp_?setListBox@QComboBox@@UAEXPAVQListBox@@@Z 10013cd4     qt-mt323:qt-mt323.dll
 0002:00000cd8       __imp_?setMargin@QLayout@@UAEXH@Z 10013cd8     qt-mt323:qt-mt323.dll
 0002:00000cdc       __imp_?setMargins@QScrollView@@MAEXHHHH@Z 10013cdc     qt-mt323:qt-mt323.dll
 0002:00000ce0       __imp_?setMaxCount@QComboBox@@UAEXH@Z 10013ce0     qt-mt323:qt-mt323.dll
 0002:00000ce4       __imp_?setMaxLength@QLineEdit@@UAEXH@Z 10013ce4     qt-mt323:qt-mt323.dll
 0002:00000ce8       __imp_?setMenuBar@QLayout@@UAEXPAVQMenuBar@@@Z 10013ce8     qt-mt323:qt-mt323.dll
 0002:00000cec       __imp_?setMovie@QLabel@@UAEXABVQMovie@@@Z 10013cec     qt-mt323:qt-mt323.dll
 0002:00000cf0       __imp_?setMultiSelection@QListView@@UAEX_N@Z 10013cf0     qt-mt323:qt-mt323.dll
 0002:00000cf4       __imp_?setNum@QLabel@@UAEXH@Z 10013cf4     qt-mt323:qt-mt323.dll
 0002:00000cf8       __imp_?setNum@QLabel@@UAEXN@Z 10013cf8     qt-mt323:qt-mt323.dll
 0002:00000cfc       __imp_?setOn@QPushButton@@UAEX_N@Z 10013cfc     qt-mt323:qt-mt323.dll
 0002:00000d00       __imp_?setOpen@QListView@@UAEXPAVQListViewItem@@_N@Z 10013d00     qt-mt323:qt-mt323.dll
 0002:00000d04       __imp_?setPalette@QComboBox@@UAEXABVQPalette@@@Z 10013d04     qt-mt323:qt-mt323.dll
 0002:00000d08       __imp_?setPalette@QLineEdit@@UAEXABVQPalette@@@Z 10013d08     qt-mt323:qt-mt323.dll
 0002:00000d0c       __imp_?setPalette@QListView@@UAEXABVQPalette@@@Z 10013d0c     qt-mt323:qt-mt323.dll
 0002:00000d10       __imp_?setPicture@QLabel@@UAEXABVQPicture@@@Z 10013d10     qt-mt323:qt-mt323.dll
 0002:00000d14       __imp_?setPixmap@QButton@@UAEXABVQPixmap@@@Z 10013d14     qt-mt323:qt-mt323.dll
 0002:00000d18       __imp_?setPixmap@QLabel@@UAEXABVQPixmap@@@Z 10013d18     qt-mt323:qt-mt323.dll
 0002:00000d1c       __imp_?setPrefix@QSpinBox@@UAEXABVQString@@@Z 10013d1c     qt-mt323:qt-mt323.dll
 0002:00000d20       __imp_?setReadOnly@QLineEdit@@UAEX_N@Z 10013d20     qt-mt323:qt-mt323.dll
 0002:00000d24       __imp_?setResizeMode@QListView@@UAEXW4ResizeMode@1@@Z 10013d24     qt-mt323:qt-mt323.dll
 0002:00000d28       __imp_?setResizePolicy@QScrollView@@UAEXW4ResizePolicy@1@@Z 10013d28     qt-mt323:qt-mt323.dll
 0002:00000d2c       __imp_?setRootIsDecorated@QListView@@UAEX_N@Z 10013d2c     qt-mt323:qt-mt323.dll
 0002:00000d30       __imp_?setRowStretch@QGridLayout@@UAEXHH@Z 10013d30     qt-mt323:qt-mt323.dll
 0002:00000d34       __imp_?setSelected@QListView@@UAEXPAVQListViewItem@@_N@Z 10013d34     qt-mt323:qt-mt323.dll
 0002:00000d38       __imp_?setSelection@QLineEdit@@UAEXHH@Z 10013d38     qt-mt323:qt-mt323.dll
 0002:00000d3c       __imp_?setShowSortIndicator@QListView@@UAEX_N@Z 10013d3c     qt-mt323:qt-mt323.dll
 0002:00000d40       __imp_?setShowToolTips@QListView@@UAEX_N@Z 10013d40     qt-mt323:qt-mt323.dll
 0002:00000d44       __imp_?setSizeLimit@QComboBox@@UAEXH@Z 10013d44     qt-mt323:qt-mt323.dll
 0002:00000d48       __imp_?setSorting@QListView@@UAEXH_N@Z 10013d48     qt-mt323:qt-mt323.dll
 0002:00000d4c       __imp_?setSpacing@QLayout@@UAEXH@Z 10013d4c     qt-mt323:qt-mt323.dll
 0002:00000d50       __imp_?setSpecialValueText@QSpinBox@@UAEXABVQString@@@Z 10013d50     qt-mt323:qt-mt323.dll
 0002:00000d54       __imp_?setState@QButton@@MAEXW4ToggleState@1@@Z 10013d54     qt-mt323:qt-mt323.dll
 0002:00000d58       __imp_?setSuffix@QSpinBox@@UAEXABVQString@@@Z 10013d58     qt-mt323:qt-mt323.dll
 0002:00000d5c       __imp_?setText@QButton@@UAEXABVQString@@@Z 10013d5c     qt-mt323:qt-mt323.dll
 0002:00000d60       __imp_?setText@QLabel@@UAEXABVQString@@@Z 10013d60     qt-mt323:qt-mt323.dll
 0002:00000d64       __imp_?setText@QLineEdit@@UAEXABVQString@@@Z 10013d64     qt-mt323:qt-mt323.dll
 0002:00000d68       __imp_?setTitle@QGroupBox@@UAEXABVQString@@@Z 10013d68     qt-mt323:qt-mt323.dll
 0002:00000d6c       __imp_?setToggleType@QButton@@MAEXW4ToggleType@1@@Z 10013d6c     qt-mt323:qt-mt323.dll
 0002:00000d70       __imp_?setTreeStepSize@QListView@@UAEXH@Z 10013d70     qt-mt323:qt-mt323.dll
 0002:00000d74       __imp_?setVBarGeometry@QScrollView@@MAEXAAVQScrollBar@@HHHH@Z 10013d74     qt-mt323:qt-mt323.dll
 0002:00000d78       __imp_?setVScrollBarMode@QScrollView@@UAEXW4ScrollBarMode@1@@Z 10013d78     qt-mt323:qt-mt323.dll
 0002:00000d7c       __imp_?setValidator@QComboBox@@UAEXPBVQValidator@@@Z 10013d7c     qt-mt323:qt-mt323.dll
 0002:00000d80       __imp_?setValidator@QLineEdit@@UAEXPBVQValidator@@@Z 10013d80     qt-mt323:qt-mt323.dll
 0002:00000d84       __imp_?setValidator@QSpinBox@@UAEXPBVQValidator@@@Z 10013d84     qt-mt323:qt-mt323.dll
 0002:00000d88       __imp_?setValue@QSpinBox@@UAEXH@Z 10013d88     qt-mt323:qt-mt323.dll
 0002:00000d8c       __imp_?setWrapping@QSpinBox@@UAEX_N@Z 10013d8c     qt-mt323:qt-mt323.dll
 0002:00000d90       __imp_?show@QListView@@UAEXXZ 10013d90     qt-mt323:qt-mt323.dll
 0002:00000d94       __imp_?show@QWidgetStack@@UAEXXZ 10013d94     qt-mt323:qt-mt323.dll
 0002:00000d98       __imp_?showEvent@QListView@@MAEXPAVQShowEvent@@@Z 10013d98     qt-mt323:qt-mt323.dll
 0002:00000d9c       __imp_?sizeHint@QBoxLayout@@UBE?AVQSize@@XZ 10013d9c     qt-mt323:qt-mt323.dll
 0002:00000da0       __imp_?sizeHint@QCheckBox@@UBE?AVQSize@@XZ 10013da0     qt-mt323:qt-mt323.dll
 0002:00000da4       __imp_?sizeHint@QComboBox@@UBE?AVQSize@@XZ 10013da4     qt-mt323:qt-mt323.dll
 0002:00000da8       __imp_?sizeHint@QGridLayout@@UBE?AVQSize@@XZ 10013da8     qt-mt323:qt-mt323.dll
 0002:00000dac       __imp_?sizeHint@QGroupBox@@UBE?AVQSize@@XZ 10013dac     qt-mt323:qt-mt323.dll
 0002:00000db0       __imp_?sizeHint@QLabel@@UBE?AVQSize@@XZ 10013db0     qt-mt323:qt-mt323.dll
 0002:00000db4       __imp_?sizeHint@QLineEdit@@UBE?AVQSize@@XZ 10013db4     qt-mt323:qt-mt323.dll
 0002:00000db8       __imp_?sizeHint@QListView@@UBE?AVQSize@@XZ 10013db8     qt-mt323:qt-mt323.dll
 0002:00000dbc       __imp_?sizeHint@QPushButton@@UBE?AVQSize@@XZ 10013dbc     qt-mt323:qt-mt323.dll
 0002:00000dc0       __imp_?sizeHint@QSpacerItem@@UBE?AVQSize@@XZ 10013dc0     qt-mt323:qt-mt323.dll
 0002:00000dc4       __imp_?sizeHint@QSpinBox@@UBE?AVQSize@@XZ 10013dc4     qt-mt323:qt-mt323.dll
 0002:00000dc8       __imp_?sizeHint@QWidgetStack@@UBE?AVQSize@@XZ 10013dc8     qt-mt323:qt-mt323.dll
 0002:00000dcc       __imp_?sort@QListView@@UAEXXZ 10013dcc     qt-mt323:qt-mt323.dll
 0002:00000dd0       __imp_?spacerItem@QLayoutItem@@UAEPAVQSpacerItem@@XZ 10013dd0     qt-mt323:qt-mt323.dll
 0002:00000dd4       __imp_?spacerItem@QSpacerItem@@UAEPAV1@XZ 10013dd4     qt-mt323:qt-mt323.dll
 0002:00000dd8       __imp_?startDrag@QListView@@MAEXXZ 10013dd8     qt-mt323:qt-mt323.dll
 0002:00000ddc       __imp_?stepChange@QRangeControl@@MAEXXZ 10013ddc     qt-mt323:qt-mt323.dll
 0002:00000de0       __imp_?stepDown@QSpinBox@@UAEXXZ 10013de0     qt-mt323:qt-mt323.dll
 0002:00000de4       __imp_?stepUp@QSpinBox@@UAEXXZ 10013de4     qt-mt323:qt-mt323.dll
 0002:00000de8       __imp_?styleChange@QComboBox@@MAEXAAVQStyle@@@Z 10013de8     qt-mt323:qt-mt323.dll
 0002:00000dec       __imp_?styleChange@QListView@@MAEXAAVQStyle@@@Z 10013dec     qt-mt323:qt-mt323.dll
 0002:00000df0       __imp_?styleChange@QSpinBox@@MAEXAAVQStyle@@@Z 10013df0     qt-mt323:qt-mt323.dll
 0002:00000df4       __imp_?suffix@QSpinBox@@UBE?AVQString@@XZ 10013df4     qt-mt323:qt-mt323.dll
 0002:00000df8       __imp_?takeItem@QListView@@UAEXPAVQListViewItem@@@Z 10013df8     qt-mt323:qt-mt323.dll
 0002:00000dfc       __imp_?undo@QLineEdit@@UAEXXZ 10013dfc     qt-mt323:qt-mt323.dll
 0002:00000e00       __imp_?updateDisplay@QSpinBox@@MAEXXZ 10013e00     qt-mt323:qt-mt323.dll
 0002:00000e04       __imp_?updateMask@QCheckBox@@MAEXXZ 10013e04     qt-mt323:qt-mt323.dll
 0002:00000e08       __imp_?updateMask@QComboBox@@MAEXXZ 10013e08     qt-mt323:qt-mt323.dll
 0002:00000e0c       __imp_?updateMask@QPushButton@@MAEXXZ 10013e0c     qt-mt323:qt-mt323.dll
 0002:00000e10       __imp_?valueChange@QSpinBox@@MAEXXZ 10013e10     qt-mt323:qt-mt323.dll
 0002:00000e14       __imp_?viewportContextMenuEvent@QScrollView@@MAEXPAVQContextMenuEvent@@@Z 10013e14     qt-mt323:qt-mt323.dll
 0002:00000e18       __imp_?viewportDragEnterEvent@QScrollView@@MAEXPAVQDragEnterEvent@@@Z 10013e18     qt-mt323:qt-mt323.dll
 0002:00000e1c       __imp_?viewportDragLeaveEvent@QScrollView@@MAEXPAVQDragLeaveEvent@@@Z 10013e1c     qt-mt323:qt-mt323.dll
 0002:00000e20       __imp_?viewportDragMoveEvent@QScrollView@@MAEXPAVQDragMoveEvent@@@Z 10013e20     qt-mt323:qt-mt323.dll
 0002:00000e24       __imp_?viewportDropEvent@QScrollView@@MAEXPAVQDropEvent@@@Z 10013e24     qt-mt323:qt-mt323.dll
 0002:00000e28       __imp_?viewportMouseDoubleClickEvent@QScrollView@@MAEXPAVQMouseEvent@@@Z 10013e28     qt-mt323:qt-mt323.dll
 0002:00000e2c       __imp_?viewportMouseMoveEvent@QScrollView@@MAEXPAVQMouseEvent@@@Z 10013e2c     qt-mt323:qt-mt323.dll
 0002:00000e30       __imp_?viewportMousePressEvent@QScrollView@@MAEXPAVQMouseEvent@@@Z 10013e30     qt-mt323:qt-mt323.dll
 0002:00000e34       __imp_?viewportMouseReleaseEvent@QScrollView@@MAEXPAVQMouseEvent@@@Z 10013e34     qt-mt323:qt-mt323.dll
 0002:00000e38       __imp_?viewportPaintEvent@QScrollView@@MAEXPAVQPaintEvent@@@Z 10013e38     qt-mt323:qt-mt323.dll
 0002:00000e3c       __imp_?viewportResizeEvent@QListView@@MAEXPAVQResizeEvent@@@Z 10013e3c     qt-mt323:qt-mt323.dll
 0002:00000e40       __imp_?viewportWheelEvent@QScrollView@@MAEXPAVQWheelEvent@@@Z 10013e40     qt-mt323:qt-mt323.dll
 0002:00000e44       __imp_?wheelEvent@QComboBox@@MAEXPAVQWheelEvent@@@Z 10013e44     qt-mt323:qt-mt323.dll
 0002:00000e48       __imp_?wheelEvent@QScrollView@@MAEXPAVQWheelEvent@@@Z 10013e48     qt-mt323:qt-mt323.dll
 0002:00000e4c       __imp_?wheelEvent@QSpinBox@@MAEXPAVQWheelEvent@@@Z 10013e4c     qt-mt323:qt-mt323.dll
 0002:00000e50       __imp_?widget@QLayoutItem@@UAEPAVQWidget@@XZ 10013e50     qt-mt323:qt-mt323.dll
 0002:00000e54       __imp_?windowActivationChange@QLineEdit@@MAEX_N@Z 10013e54     qt-mt323:qt-mt323.dll
 0002:00000e58       __imp_?windowActivationChange@QListView@@MAEX_N@Z 10013e58     qt-mt323:qt-mt323.dll
 0002:00000e5c       __imp_?qstrcmp@@YAHPBD0@Z  10013e5c     qt-mt323:qt-mt323.dll
 0002:00000e60       __imp_?fromLatin1@QString@@SA?AV1@PBDH@Z 10013e60     qt-mt323:qt-mt323.dll
 0002:00000e64       __imp_?fromUtf8@QString@@SA?AV1@PBDH@Z 10013e64     qt-mt323:qt-mt323.dll
 0002:00000e68       __imp_?receivers@QObject@@IBEPAVQConnectionList@@H@Z 10013e68     qt-mt323:qt-mt323.dll
 0002:00000e6c       __imp_?activate_signal@QObject@@IAEXPAVQConnectionList@@PAUQUObject@@@Z 10013e6c     qt-mt323:qt-mt323.dll
 0002:00000e70       __imp_?staticMetaObject@QWidget@@SAPAVQMetaObject@@XZ 10013e70     qt-mt323:qt-mt323.dll
 0002:00000e74       __imp_?new_metaobject@QMetaObject@@SAPAV1@PBDPAV1@QBUQMetaData@@H2HQBVQMetaProperty@@HQBUQMetaEnum@@HQBUQClassInfo@@H@Z 10013e74     qt-mt323:qt-mt323.dll
 0002:00000e78       __imp_??0QMetaObjectCleanUp@@QAE@PBDP6APAVQMetaObject@@XZ@Z 10013e78     qt-mt323:qt-mt323.dll
 0002:00000e7c       __imp_??1QMetaObjectCleanUp@@QAE@XZ 10013e7c     qt-mt323:qt-mt323.dll
 0002:00000e80       __imp_?setMetaObject@QMetaObjectCleanUp@@QAEXAAPAVQMetaObject@@@Z 10013e80     qt-mt323:qt-mt323.dll
 0002:00000e84       __imp_?translate@QApplication@@QBE?AVQString@@PBD00W4Encoding@1@@Z 10013e84     qt-mt323:qt-mt323.dll
 0002:00000e88       __imp_??0QUObject@@QAE@XZ  10013e88     qt-mt323:qt-mt323.dll
 0002:00000e8c       __imp_??1QUObject@@QAE@XZ  10013e8c     qt-mt323:qt-mt323.dll
 0002:00000e90       __imp_?set@QUType_QString@@QAEXPAUQUObject@@ABVQString@@@Z 10013e90     qt-mt323:qt-mt323.dll
 0002:00000e94       __imp_?qApp@@3PAVQApplication@@A 10013e94     qt-mt323:qt-mt323.dll
 0002:00000e98       __imp_?static_QUType_QString@@3UQUType_QString@@A 10013e98     qt-mt323:qt-mt323.dll
 0002:00000e9c       __imp_?activate_signal@QObject@@IAEXH@Z 10013e9c     qt-mt323:qt-mt323.dll
 0002:00000ea0       __imp_?static_QUType_ptr@@3UQUType_ptr@@A 10013ea0     qt-mt323:qt-mt323.dll
 0002:00000ea4       __imp_?static_QUType_int@@3UQUType_int@@A 10013ea4     qt-mt323:qt-mt323.dll
 0002:00000ea8       __imp_?static_QUType_varptr@@3UQUType_varptr@@A 10013ea8     qt-mt323:qt-mt323.dll
 0002:00000eac       __imp_?activate_signal@QObject@@IAEXHVQString@@@Z 10013eac     qt-mt323:qt-mt323.dll
 0002:00000eb0       __imp_??0QTabWidget@@QAE@PAVQWidget@@PBDI@Z 10013eb0     qt-mt323:qt-mt323.dll
 0002:00000eb4       __imp_??1QTabWidget@@UAE@XZ 10013eb4     qt-mt323:qt-mt323.dll
 0002:00000eb8       __imp_?changeTab@QTabWidget@@QAEXPAVQWidget@@ABVQString@@@Z 10013eb8     qt-mt323:qt-mt323.dll
 0002:00000ebc       __imp_?addTab@QTabWidget@@UAEXPAVQWidget@@ABVQIconSet@@ABVQString@@@Z 10013ebc     qt-mt323:qt-mt323.dll
 0002:00000ec0       __imp_?addTab@QTabWidget@@UAEXPAVQWidget@@ABVQString@@@Z 10013ec0     qt-mt323:qt-mt323.dll
 0002:00000ec4       __imp_?addTab@QTabWidget@@UAEXPAVQWidget@@PAVQTab@@@Z 10013ec4     qt-mt323:qt-mt323.dll
 0002:00000ec8       __imp_?className@QTabWidget@@UBEPBDXZ 10013ec8     qt-mt323:qt-mt323.dll
 0002:00000ecc       __imp_?eventFilter@QTabWidget@@MAE_NPAVQObject@@PAVQEvent@@@Z 10013ecc     qt-mt323:qt-mt323.dll
 0002:00000ed0       __imp_?insertTab@QTabWidget@@UAEXPAVQWidget@@ABVQIconSet@@ABVQString@@H@Z 10013ed0     qt-mt323:qt-mt323.dll
 0002:00000ed4       __imp_?insertTab@QTabWidget@@UAEXPAVQWidget@@ABVQString@@H@Z 10013ed4     qt-mt323:qt-mt323.dll
 0002:00000ed8       __imp_?insertTab@QTabWidget@@UAEXPAVQWidget@@PAVQTab@@H@Z 10013ed8     qt-mt323:qt-mt323.dll
 0002:00000edc       __imp_?metaObject@QTabWidget@@UBEPAVQMetaObject@@XZ 10013edc     qt-mt323:qt-mt323.dll
 0002:00000ee0       __imp_?minimumSizeHint@QTabWidget@@UBE?AVQSize@@XZ 10013ee0     qt-mt323:qt-mt323.dll
 0002:00000ee4       __imp_?qt_cast@QTabWidget@@UAEPAXPBD@Z 10013ee4     qt-mt323:qt-mt323.dll
 0002:00000ee8       __imp_?qt_emit@QTabWidget@@UAE_NHPAUQUObject@@@Z 10013ee8     qt-mt323:qt-mt323.dll
 0002:00000eec       __imp_?qt_invoke@QTabWidget@@UAE_NHPAUQUObject@@@Z 10013eec     qt-mt323:qt-mt323.dll
 0002:00000ef0       __imp_?qt_property@QTabWidget@@UAE_NHHPAVQVariant@@@Z 10013ef0     qt-mt323:qt-mt323.dll
 0002:00000ef4       __imp_?removePage@QTabWidget@@UAEXPAVQWidget@@@Z 10013ef4     qt-mt323:qt-mt323.dll
 0002:00000ef8       __imp_?resizeEvent@QTabWidget@@MAEXPAVQResizeEvent@@@Z 10013ef8     qt-mt323:qt-mt323.dll
 0002:00000efc       __imp_?showEvent@QTabWidget@@MAEXPAVQShowEvent@@@Z 10013efc     qt-mt323:qt-mt323.dll
 0002:00000f00       __imp_?showPage@QTabWidget@@UAEXPAVQWidget@@@Z 10013f00     qt-mt323:qt-mt323.dll
 0002:00000f04       __imp_?sizeHint@QTabWidget@@UBE?AVQSize@@XZ 10013f04     qt-mt323:qt-mt323.dll
 0002:00000f08       __imp_?styleChange@QTabWidget@@MAEXAAVQStyle@@@Z 10013f08     qt-mt323:qt-mt323.dll
 0002:00000f0c       __imp_?updateMask@QTabWidget@@MAEXXZ 10013f0c     qt-mt323:qt-mt323.dll
 0002:00000f10       __imp_??1QWidget@@UAE@XZ   10013f10     qt-mt323:qt-mt323.dll
 0002:00000f14       __imp_??0QWidget@@QAE@PAV0@PBDI@Z 10013f14     qt-mt323:qt-mt323.dll
 0002:00000f18       __imp_??1QStringList@@QAE@XZ 10013f18     qt-mt323:qt-mt323.dll
 0002:00000f1c       __imp_?split@QStringList@@SA?AV1@ABVQString@@0_N@Z 10013f1c     qt-mt323:qt-mt323.dll
 0002:00000f20       __imp_??0QStringList@@QAE@XZ 10013f20     qt-mt323:qt-mt323.dll
 0002:00000f24       __imp_?connect@QObject@@SA_NPBV1@PBD01@Z 10013f24     qt-mt323:qt-mt323.dll
 0002:00000f28       __imp_?clear@QGList@@MAEXXZ 10013f28     qt-mt323:qt-mt323.dll
 0002:00000f2c       __imp_?append@QGList@@IAEXPAX@Z 10013f2c     qt-mt323:qt-mt323.dll
 0002:00000f30       __imp_??1QGList@@MAE@XZ    10013f30     qt-mt323:qt-mt323.dll
 0002:00000f34       __imp_??0QGList@@IAE@XZ    10013f34     qt-mt323:qt-mt323.dll
 0002:00000f38       __imp_?detachInternal@?$QValueList@VQString@@@@AAEXXZ 10013f38     qt-mt323:qt-mt323.dll
 0002:00000f3c       __imp_?contains@?$QValueList@VQString@@@@QBEIABVQString@@@Z 10013f3c     qt-mt323:qt-mt323.dll
 0002:00000f40       __imp_?append@?$QValueList@VQString@@@@QAE?AV?$QValueListIterator@VQString@@@@ABVQString@@@Z 10013f40     qt-mt323:qt-mt323.dll
 0002:00000f44       __imp_?remove@?$QValueList@VQString@@@@QAEIABVQString@@@Z 10013f44     qt-mt323:qt-mt323.dll
 0002:00000f48       __imp_?begin@?$QValueList@VQString@@@@QAE?AV?$QValueListIterator@VQString@@@@XZ 10013f48     qt-mt323:qt-mt323.dll
 0002:00000f4c       __imp_??H@YA?BVQString@@PBDABV0@@Z 10013f4c     qt-mt323:qt-mt323.dll
 0002:00000f50       __imp_??H@YA?BVQString@@ABV0@PBD@Z 10013f50     qt-mt323:qt-mt323.dll
 0002:00000f54       __imp_??H@YA?BVQString@@ABV0@0@Z 10013f54     qt-mt323:qt-mt323.dll
 0002:00000f58       __imp_??8@YA_NABVQString@@PBD@Z 10013f58     qt-mt323:qt-mt323.dll
 0002:00000f5c       __imp_??8@YA_NABVQString@@0@Z 10013f5c     qt-mt323:qt-mt323.dll
 0002:00000f60       __imp_?ascii@QString@@QBEPBDXZ 10013f60     qt-mt323:qt-mt323.dll
 0002:00000f64       __imp_??YQString@@QAEAAV0@PBD@Z 10013f64     qt-mt323:qt-mt323.dll
 0002:00000f68       __imp_??YQString@@QAEAAV0@D@Z 10013f68     qt-mt323:qt-mt323.dll
 0002:00000f6c       __imp_?next@QGList@@IAEPAXXZ 10013f6c     qt-mt323:qt-mt323.dll
 0002:00000f70       __imp_??4QFrame@@QAEAAV0@ABV0@@Z 10013f70     qt-mt323:qt-mt323.dll
 0002:00000f74       __imp_??0QListViewItem@@QAE@PAVQListView@@PAV0@@Z 10013f74     qt-mt323:qt-mt323.dll
 0002:00000f78       __imp_??0QListView@@QAE@ABV0@@Z 10013f78     qt-mt323:qt-mt323.dll
 0002:00000f7c       __imp_?activate_signal_bool@QObject@@IAEXH_N@Z 10013f7c     qt-mt323:qt-mt323.dll
 0002:00000f80       __imp_?staticMetaObject@QListView@@SAPAVQMetaObject@@XZ 10013f80     qt-mt323:qt-mt323.dll
 0002:00000f84       __imp_?static_QUType_bool@@3UQUType_bool@@A 10013f84     qt-mt323:qt-mt323.dll
 0002:00000f88       __imp_??YQString@@QAEAAV0@ABV0@@Z 10013f88     qt-mt323:qt-mt323.dll
 0002:00000f8c       __imp_?upper@QString@@QBE?AV1@XZ 10013f8c     qt-mt323:qt-mt323.dll
 0002:00000f90       __imp_?arg@QString@@QBE?AV1@ABV1@H@Z 10013f90     qt-mt323:qt-mt323.dll
 0002:00000f94       __imp_??4QString@@QAEAAV0@ABV0@@Z 10013f94     qt-mt323:qt-mt323.dll
 0002:00000f98       __imp_??1QString@@QAE@XZ   10013f98     qt-mt323:qt-mt323.dll
 0002:00000f9c       __imp_??0QString@@QAE@PBD@Z 10013f9c     qt-mt323:qt-mt323.dll
 0002:00000fa0       __imp_??0QString@@QAE@ABV0@@Z 10013fa0     qt-mt323:qt-mt323.dll
 0002:00000fa4       __imp_??0QString@@QAE@XZ   10013fa4     qt-mt323:qt-mt323.dll
 0002:00000fa8       __imp_?qDebug@@YAXPBDZZ    10013fa8     qt-mt323:qt-mt323.dll
 0002:00000fac       __imp_??1QGroupBox@@UAE@XZ 10013fac     qt-mt323:qt-mt323.dll
 0002:00000fb0       \177qt-mt323_NULL_THUNK_DATA 10013fb0     qt-mt323:qt-mt323.dll
 0002:00000fb4       ___xc_a                    10013fb4     MSVCRT:cinitexe.obj
 0002:00000fd0       ___xc_z                    10013fd0     MSVCRT:cinitexe.obj
 0002:00000fd4       ___xi_a                    10013fd4     MSVCRT:cinitexe.obj
 0002:00000fe0       ___xi_z                    10013fe0     MSVCRT:cinitexe.obj
 0002:00000ff0       ??_C@_02GIPFHKNO@OK?$AA@   10013ff0     device_type_edit.obj
 0002:00000ffc       ??_SQAction@@6B@           10013ffc     device_type_edit.obj
 0002:0000108c       ??_SQDockWindow@@6BQObject@@@ 1001408c     device_type_edit.obj
 0002:0000129c       ??_SQDockWindow@@6BQPaintDevice@@@ 1001429c     device_type_edit.obj
 0002:000012c4       ??_SQToolBar@@6BQObject@@@ 100142c4     device_type_edit.obj
 0002:000014e0       ??_SQToolBar@@6BQPaintDevice@@@ 100144e0     device_type_edit.obj
 0002:00001504       ??_SQGuardedPtrPrivate@@6B@ 10014504     device_type_edit.obj
 0002:00001558       ??_7QDockWindowList@@6B@   10014558     device_type_edit.obj
 0002:0000157c       ??_SQPopupMenu@@6BQObject@@@ 1001457c     device_type_edit.obj
 0002:0000175c       ??_SQPopupMenu@@6BQPaintDevice@@@ 1001475c     device_type_edit.obj
 0002:00001780       ??_SQPopupMenu@@6B@        10014780     device_type_edit.obj
 0002:000017a4       ??_7?$QPtrList@VQPopupMenu@@@@6B@ 100147a4     device_type_edit.obj
 0002:000017c8       ??_7QPopupMenuList@@6B@    100147c8     device_type_edit.obj
 0002:000017ec       ??_7config_plugin_base@@6BQObject@@@ 100147ec     device_type_edit.obj
 0002:000019c4       ??_7config_plugin_base@@6BQPaintDevice@@@ 100149c4     device_type_edit.obj
 0002:000019e8       ??_C@_0EB@GNDACMDJ@?$CC?5?9?5the?5author?5should?5have?5defin@ 100149e8     device_type_edit.obj
 0002:00001a2c       ??_C@_0CH@BDPDPLDP@This?5is?5the?5default?5?$CCAbout?$CC?5text@ 10014a2c     device_type_edit.obj
 0002:00001a58       ??_7?$QDict@VQAction@@@@6B@ 10014a58     device_type_edit.obj
 0002:00001a78       ??_7device_type_edit@@6BQObject@@@ 10014a78     device_type_edit.obj
 0002:00001c50       ??_7device_type_edit@@6BQPaintDevice@@@ 10014c50     device_type_edit.obj
 0002:00001c70       ??_C@_0BD@LOCLOALI@device_type_edit?3?5?$AA@ 10014c70     device_type_edit.obj
 0002:00001c84       ??_C@_0N@LMCHKLFE@1markDirty?$CI?$CJ?$AA@ 10014c84     device_type_edit.obj
 0002:00001c94       ??_C@_08HNCJCJBC@2dirty?$CI?$CJ?$AA@ 10014c94     device_type_edit.obj
 0002:00001ca0       ??_C@_0BO@DCHMNGHO@?1Template?5Plugin?5Tools?5Window?$AA@ 10014ca0     device_type_edit.obj
 0002:00001cc0       ??_C@_0N@CDOLEPFK@Tools?5Window?$AA@ 10014cc0     device_type_edit.obj
 0002:00001cd0       ??_C@_0BN@LFEKHMAO@1selectType?$CIconst?5QString?5?$CG?$CJ?$AA@ 10014cd0     device_type_edit.obj
 0002:00001cf0       ??_C@_0CB@LDOPJFG@2typeSelected?$CI?5const?5QString?5?$CG?5?$CJ@ 10014cf0     device_type_edit.obj
 0002:00001d14       ??_C@_0BN@HOGOHKFP@1deleteType?$CIconst?5QString?5?$CG?$CJ?$AA@ 10014d14     device_type_edit.obj
 0002:00001d34       ??_C@_0CA@NOLDEGP@2typeDeleted?$CI?5const?5QString?5?$CG?5?$CJ?$AA@ 10014d34     device_type_edit.obj
 0002:00001d54       ??_C@_0BI@DJGPDCG@Template?5Plugin?5Toolbar?$AA@ 10014d54     device_type_edit.obj
 0002:00001d6c       ??_C@_05LHMKEDEH@?$CGEdit?$AA@ 10014d6c     device_type_edit.obj
 0002:00001d74       ??_C@_03CLCAEGCJ@new?$AA@  10014d74     device_type_edit.obj
 0002:00001d78       ??_C@_04CCPFBLLC@?$CGNew?$AA@ 10014d78     device_type_edit.obj
 0002:00001d80       ??_C@_07EJAINBEK@filenew?$AA@ 10014d80     device_type_edit.obj
 0002:00001d88       ??_C@_0BA@NPMEGAC@New?5Application?$AA@ 10014d88     device_type_edit.obj
 0002:00001d98       ??_C@_0L@CINBLJHB@1newFile?$CI?$CJ?$AA@ 10014d98     device_type_edit.obj
 0002:00001da4       ??_C@_0N@KCMOKDBB@2activated?$CI?$CJ?$AA@ 10014da4     device_type_edit.obj
 0002:00001db4       ??_C@_0BH@FJKOLNHB@config?1devicetypes?4xml?$AA@ 10014db4     device_type_edit.obj
 0002:00001dcc       ??_C@_06BNCCALCL@unlock?$AA@ 10014dcc     device_type_edit.obj
 0002:00001dd4       ??_C@_0N@LFOBEKOJ@Unlocking?5?9?5?$AA@ 10014dd4     device_type_edit.obj
 0002:00001de4       ??_C@_08HNIAHLMM@download?$AA@ 10014de4     device_type_edit.obj
 0002:00001df0       ??_C@_01KMDKNFGN@?1?$AA@   10014df0     device_type_edit.obj
 0002:00001df4       ??_C@_04GAOAGNCM@?4xml?$AA@ 10014df4     device_type_edit.obj
 0002:00001dfc       ??_C@_0BE@OJOGEEMJ@config?1devicetypes?1?$AA@ 10014dfc     device_type_edit.obj
 0002:00001e10       ??_C@_0BB@JHLHEMKF@config?1template?1?$AA@ 10014e10     device_type_edit.obj
 0002:00001e21       ??_C@_00CNPNBAHC@?$AA@     10014e21     device_type_edit.obj
 0002:00001e24       ??_C@_05CCAMFJOL@clean?$AA@ 10014e24     device_type_edit.obj
 0002:00001e2c       ??_C@_04MKMCLCOO@lock?$AA@ 10014e2c     device_type_edit.obj
 0002:00001e34       ??_C@_06KAOCKAGB@upload?$AA@ 10014e34     device_type_edit.obj
 0002:00001e3c       ??_C@_0M@EBFEGAAI@Information?$AA@ 10014e3c     device_type_edit.obj
 0002:00001e48       ??_C@_0CO@GKAEALGF@Being?5asked?5to?5navigate?5to?5?$CF1?5wi@ 10014e48     device_type_edit.obj
 0002:00001e78       ??_C@_0N@EHHLDFOB@checkoutFile?$AA@ 10014e78     device_type_edit.obj
 0002:00001e88       ??_C@_0BA@GNHMHBBC@syncDirDownload?$AA@ 10014e88     device_type_edit.obj
 0002:00001e98       ??_C@_0L@CIKGEHEG@uploadFile?$AA@ 10014e98     device_type_edit.obj
 0002:00001ea4       ??_C@_03GJCOJFLC@?4?6?6?$AA@ 10014ea4     device_type_edit.obj
 0002:00001ea8       ??_C@_0BM@CGOIHJMM@Could?5not?5Create?5directory?6?$AA@ 10014ea8     device_type_edit.obj
 0002:00001ec4       ??_C@_0BB@OACMDDDM@Device?5type?5edit?$AA@ 10014ec4     device_type_edit.obj
 0002:00001ed8       ??_C@_0EG@EBHAICDP@?$DMh3?$DODevice?5Type?5editor?5plugin?$DM?1h@ 10014ed8     device_type_edit.obj
 0002:00001f20       ??_C@_08GCOHKBID@13?325?310?$AA@ 10014f20     device_type_edit.obj
 0002:00001f2c       ??_C@_0M@JEDEHNP@Sep?523?52021?$AA@ 10014f2c     device_type_edit.obj
 0002:00001f38       ??_C@_0BD@MKOIHAFG@?5has?5been?5selected?$AA@ 10014f38     device_type_edit.obj
 0002:00001f4c       ??_C@_05CFEJGMAI@dirty?$AA@ 10014f4c     device_type_edit.obj
 0002:00001f5c       ??_SQDomDocument@@6B@      10014f5c     device_type_editdlgimpl.obj
 0002:00002004       ??_SQDomElement@@6B@       10015004     device_type_editdlgimpl.obj
 0002:000020b0       ??_7device_type_editDlg@@6BQObject@@@ 100150b0     device_type_editdlgimpl.obj
 0002:00002268       ??_7device_type_editDlg@@6BQPaintDevice@@@ 10015268     device_type_editdlgimpl.obj
 0002:0000228c       ??_SQListViewItem@@6B@     1001528c     device_type_editdlgimpl.obj
 0002:00002324       ??_C@_0P@GCONKOGG@1selectParam?$CI?$CJ?$AA@ 10015324     device_type_editdlgimpl.obj
 0002:00002334       ??_C@_0BE@BLJBKCLJ@2selectionChanged?$CI?$CJ?$AA@ 10015334     device_type_editdlgimpl.obj
 0002:00002348       ??_C@_0M@DKEJLKC@1paramNew?$CI?$CJ?$AA@ 10015348     device_type_editdlgimpl.obj
 0002:00002354       ??_C@_0L@OELOHDKG@2clicked?$CI?$CJ?$AA@ 10015354     device_type_editdlgimpl.obj
 0002:00002360       ??_C@_0P@NKIEPPPK@1paramRename?$CI?$CJ?$AA@ 10015360     device_type_editdlgimpl.obj
 0002:00002370       ??_C@_0N@HMICGFPC@1paramCopy?$CI?$CJ?$AA@ 10015370     device_type_editdlgimpl.obj
 0002:00002380       ??_C@_0P@GEKAGCMN@1paramDelete?$CI?$CJ?$AA@ 10015380     device_type_editdlgimpl.obj
 0002:00002390       ??_C@_0O@KDDKJPOD@1paramPaste?$CI?$CJ?$AA@ 10015390     device_type_editdlgimpl.obj
 0002:000023a0       ??_C@_0BH@HMNMIPDJ@1checkParamClipboard?$CI?$CJ?$AA@ 100153a0     device_type_editdlgimpl.obj
 0002:000023b8       ??_C@_0P@GLIODLHI@2dataChanged?$CI?$CJ?$AA@ 100153b8     device_type_editdlgimpl.obj
 0002:000023c8       ??_C@_0BE@PIDNAPF@1devTypeChange?$CIint?$CJ?$AA@ 100153c8     device_type_editdlgimpl.obj
 0002:000023dc       ??_C@_0BA@HAKGEOGG@2activated?$CIint?$CJ?$AA@ 100153dc     device_type_editdlgimpl.obj
 0002:000023ec       ??_C@_0BA@BHPINBIH@1markDirty?$CIint?$CJ?$AA@ 100153ec     device_type_editdlgimpl.obj
 0002:000023fc       ??_C@_0BD@OIBDOPAP@2valueChanged?$CIint?$CJ?$AA@ 100153fc     device_type_editdlgimpl.obj
 0002:00002410       ??_C@_0BB@POOMLMGO@2activated?5?$CIint?$CJ?$AA@ 10015410     device_type_editdlgimpl.obj
 0002:00002424       ??_C@_0BL@EHPLENPD@1markDirty?$CIconst?5QString?$CG?$CJ?$AA@ 10015424     device_type_editdlgimpl.obj
 0002:00002440       ??_C@_0BN@HELOKIBG@2textChanged?$CIconst?5QString?$CG?$CJ?$AA@ 10015440     device_type_editdlgimpl.obj
 0002:00002460       ??_C@_05LPIJGKJ@Value?$AA@ 10015460     device_type_editdlgimpl.obj
 0002:00002468       ??_C@_05JNKNAC@State?$AA@  10015468     device_type_editdlgimpl.obj
 0002:00002470       ??_C@_05IHAFCALK@Style?$AA@ 10015470     device_type_editdlgimpl.obj
 0002:00002478       ??_C@_03MLMOILGK@Msg?$AA@  10015478     device_type_editdlgimpl.obj
 0002:0000247c       ??_C@_0DA@GLLECGAF@1enumDblClick?$CIQListViewItem?$CK?0con@ 1001547c     device_type_editdlgimpl.obj
 0002:000024ac       ??_C@_0DB@PONCGDCM@2doubleClicked?$CIQListViewItem?$CK?0co@ 100154ac     device_type_editdlgimpl.obj
 0002:000024e0       ??_C@_0BP@MOMEPNID@1markDirty?$CIQListViewItem?$CK?0int?$CJ?$AA@ 100154e0     device_type_editdlgimpl.obj
 0002:00002500       ??_C@_0CB@FBFODLLH@2itemRenamed?$CIQListViewItem?$CK?0int?$CJ@ 10015500     device_type_editdlgimpl.obj
 0002:00002524       ??_C@_0BA@DOELKFMG@1enumNewState?$CI?$CJ?$AA@ 10015524     device_type_editdlgimpl.obj
 0002:00002534       ??_C@_0BD@DBPMFKCL@1enumDeleteState?$CI?$CJ?$AA@ 10015534     device_type_editdlgimpl.obj
 0002:00002548       ??_C@_0BD@GOCBCOOF@1copyToClipboard?$CI?$CJ?$AA@ 10015548     device_type_editdlgimpl.obj
 0002:0000255c       ??_C@_0N@KCJIABKL@1enumPaste?$CI?$CJ?$AA@ 1001555c     device_type_editdlgimpl.obj
 0002:0000256c       ??_C@_0BC@DLEJKFKG@1setEnabled?$CIbool?$CJ?$AA@ 1001556c     device_type_editdlgimpl.obj
 0002:00002580       ??_C@_0BK@CGPDLMEB@2clipboardDataValid?$CIbool?$CJ?$AA@ 10015580     device_type_editdlgimpl.obj
 0002:0000259c       ??_C@_05OEOKGKGJ@?$DM?1h1?$DO?$AA@ 1001559c     device_type_editdlgimpl.obj
 0002:000025a4       ??_C@_0M@OJJDAEDJ@?$DMh1?$DOType?5?9?5?$AA@ 100155a4     device_type_editdlgimpl.obj
 0002:000025b0       ??_C@_0BI@MBANNBKM@?$CC?$DO?$DM?1device_description?$DO?$AA@ 100155b0     device_type_editdlgimpl.obj
 0002:000025c8       ??_C@_0BL@IINFBLL@?$DMdevice_description?5name?$DN?$CC?$AA@ 100155c8     device_type_editdlgimpl.obj
 0002:000025e4       ??_C@_0DO@ILICBEGG@?$DM?$CBDOCTYPE?5device_description?5SYS@ 100155e4     device_type_editdlgimpl.obj
 0002:00002624       ??_C@_0BI@DOLAIBMO@?$DM?$DPxml?5version?5?$DN?5?81?40?8?$DP?$DO?$AA@ 10015624     device_type_editdlgimpl.obj
 0002:0000263c       ??_C@_0BD@INOIJGBO@device_description?$AA@ 1001563c     device_type_editdlgimpl.obj
 0002:00002650       ??_C@_04MEMAJGDJ@name?$AA@ 10015650     device_type_editdlgimpl.obj
 0002:00002658       ??_C@_0L@NFEMMAMH@drivertype?$AA@ 10015658     device_type_editdlgimpl.obj
 0002:00002664       ??_C@_06KJABCPFL@Router?$AA@ 10015664     device_type_editdlgimpl.obj
 0002:0000266c       ??_C@_03JFHPJKJL@GPI?$AA@  1001566c     device_type_editdlgimpl.obj
 0002:00002670       ??_C@_05LJDNNBIK@param?$AA@ 10015670     device_type_editdlgimpl.obj
 0002:00002678       ??_C@_0CM@IDEEALLJ@?$DMh1?$DOParameter?5?9?5?$CF1?5parameters?5se@ 10015678     device_type_editdlgimpl.obj
 0002:000026a4       ??_C@_0BB@BEKHGIEG@?$DMh1?$DOParameter?5?9?5?$AA@ 100156a4     device_type_editdlgimpl.obj
 0002:000026b8       ??_C@_0BF@MJFJHJNJ@Element?5not?5found?5?9?5?$AA@ 100156b8     device_type_editdlgimpl.obj
 0002:000026d0       ??_C@_0BP@EGHEFDPK@?$DMh1?$DONo?5parameter?5selected?$DM?1h1?$DO?$AA@ 100156d0     device_type_editdlgimpl.obj
 0002:000026f0       ??_C@_04POIHOKKJ@slot?$AA@ 100156f0     device_type_editdlgimpl.obj
 0002:000026f8       ??_C@_05IAKJCFIM@style?$AA@ 100156f8     device_type_editdlgimpl.obj
 0002:00002700       ??_C@_06EBPNOMLE@access?$AA@ 10015700     device_type_editdlgimpl.obj
 0002:00002708       ??_C@_08JOKHDEJH@readonly?$AA@ 10015708     device_type_editdlgimpl.obj
 0002:00002714       ??_C@_09CGKEKDCN@writeonly?$AA@ 10015714     device_type_editdlgimpl.obj
 0002:00002720       ??_C@_08FJNLKCPH@template?$AA@ 10015720     device_type_editdlgimpl.obj
 0002:0000272c       ??_C@_05ENKANFLO@class?$AA@ 1001572c     device_type_editdlgimpl.obj
 0002:00002734       ??_C@_04DBJPMPLO@enum?$AA@ 10015734     device_type_editdlgimpl.obj
 0002:0000273c       ??_C@_04DONFEANM@list?$AA@ 1001573c     device_type_editdlgimpl.obj
 0002:00002744       ??_C@_05CCGOGOBM@range?$AA@ 10015744     device_type_editdlgimpl.obj
 0002:0000274c       ??_C@_06ICGJLFIM@string?$AA@ 1001574c     device_type_editdlgimpl.obj
 0002:00002754       ??_C@_09DOMKHCF@readwrite?$AA@ 10015754     device_type_editdlgimpl.obj
 0002:00002760       ??_C@_05HDBKIDE@state?$AA@ 10015760     device_type_editdlgimpl.obj
 0002:00002768       ??_C@_03GLPMCEFE@msg?$AA@  10015768     device_type_editdlgimpl.obj
 0002:0000276c       ??_C@_07BANDPJOM@caption?$AA@ 1001576c     device_type_editdlgimpl.obj
 0002:00002774       ??_C@_05MFEJDJP@value?$AA@ 10015774     device_type_editdlgimpl.obj
 0002:0000277c       ??_C@_06GEKOPAHD@values?$AA@ 1001577c     device_type_editdlgimpl.obj
 0002:00002784       ??_C@_03KLIPLJLL@min?$AA@  10015784     device_type_editdlgimpl.obj
 0002:00002788       ??_C@_03LJAEFNNE@max?$AA@  10015788     device_type_editdlgimpl.obj
 0002:0000278c       ??_C@_04CNBNFAL@step?$AA@  1001578c     device_type_editdlgimpl.obj
 0002:00002794       ??_C@_07DIMAGMGN@bigstep?$AA@ 10015794     device_type_editdlgimpl.obj
 0002:0000279c       ??_C@_0N@GPEKCLAN@defaultvalue?$AA@ 1001579c     device_type_editdlgimpl.obj
 0002:000027ac       ??_C@_07GCCODDFC@display?$AA@ 100157ac     device_type_editdlgimpl.obj
 0002:000027b4       ??_C@_0L@NBOAACKH@multiplier?$AA@ 100157b4     device_type_editdlgimpl.obj
 0002:000027c0       ??_C@_08OFLDIGMK@inoffset?$AA@ 100157c0     device_type_editdlgimpl.obj
 0002:000027cc       ??_C@_09GHFDDJGJ@outoffset?$AA@ 100157cc     device_type_editdlgimpl.obj
 0002:000027d8       ??_C@_02GAFPDMOH@dp?$AA@   100157d8     device_type_editdlgimpl.obj
 0002:000027dc       ??_C@_05CCBEFJDC@units?$AA@ 100157dc     device_type_editdlgimpl.obj
 0002:000027e4       ??_C@_09GGMBJIEG@maxlength?$AA@ 100157e4     device_type_editdlgimpl.obj
 0002:000027f0       ??_C@_04CKOINMPC@case?$AA@ 100157f0     device_type_editdlgimpl.obj
 0002:000027f8       ??_C@_05IPJEPLHL@lower?$AA@ 100157f8     device_type_editdlgimpl.obj
 0002:00002800       ??_C@_05NECKJAMC@upper?$AA@ 10015800     device_type_editdlgimpl.obj
 0002:00002808       ??_C@_05PHLGJONK@title?$AA@ 10015808     device_type_editdlgimpl.obj
 0002:00002810       ??_C@_01GBGANLPD@0?$AA@    10015810     device_type_editdlgimpl.obj
 0002:00002814       ??_C@_0BN@IOJGLIMN@Entry?5will?5be?5left?5as?5it?5was?$AA@ 10015814     device_type_editdlgimpl.obj
 0002:00002834       ??_C@_0DB@KDPMAMEB@?5exists?5in?5the?5file?0?5but?5does?5no@ 10015834     device_type_editdlgimpl.obj
 0002:00002868       ??_C@_0N@CMAAMPLM@Saving?5Enums?$AA@ 10015868     device_type_editdlgimpl.obj
 0002:00002878       ??_C@_0P@CAFBNFKA@Enter?5a?5value?3?$AA@ 10015878     device_type_editdlgimpl.obj
 0002:00002888       ??_C@_0P@MLPPJMIH@New?5Enum?5Value?$AA@ 10015888     device_type_editdlgimpl.obj
 0002:00002898       ??_C@_0CA@JLCKJLKK@Please?5select?5a?5different?5slot?4?$AA@ 10015898     device_type_editdlgimpl.obj
 0002:000028b8       ??_C@_0BG@FJPMAIKF@?8?5is?5already?5in?5use?4?6?$AA@ 100158b8     device_type_editdlgimpl.obj
 0002:000028d0       ??_C@_07IECBMOKM@Value?5?8?$AA@ 100158d0     device_type_editdlgimpl.obj
 0002:000028d8       ??_C@_01GPOEFGEJ@?7?$AA@   100158d8     device_type_editdlgimpl.obj
 0002:000028dc       ??_C@_0BP@DOPMMOFP@Enter?5a?5unique?5parameter?5name?4?$AA@ 100158dc     device_type_editdlgimpl.obj
 0002:000028fc       ??_C@_0BD@IDPDJCPP@New?5Parameter?5Name?$AA@ 100158fc     device_type_editdlgimpl.obj
 0002:00002910       ??_C@_0BG@BPLNPHHC@You?5must?5enter?5a?5name?$AA@ 10015910     device_type_editdlgimpl.obj
 0002:00002928       ??_C@_0BH@KCKJHNNM@Invalid?5Parameter?5Name?$AA@ 10015928     device_type_editdlgimpl.obj
 0002:00002940       ??_C@_0BC@KMNPDBEN@?5is?5already?5used?$CB?$AA@ 10015940     device_type_editdlgimpl.obj
 0002:00002954       ??_C@_0BF@CGLLMNIC@Name?5for?5pasting?5is?5?$AA@ 10015954     device_type_editdlgimpl.obj
 0002:00002970       ??_7?$QPtrList@VQListViewItem@@@@6B@ 10015970     device_type_editdlgimpl.obj
 0002:00002990       ??_C@_0BK@KECMCOLA@?5in?5file?0?5so?5not?5removed?$CB?$AA@ 10015990     device_type_editdlgimpl.obj
 0002:000029ac       ??_C@_0M@NHLIFGCC@Can?8t?5find?5?$AA@ 100159ac     device_type_editdlgimpl.obj
 0002:000029b8       ??_C@_0BE@KFJDAEOH@Deleting?5Enum?5value?$AA@ 100159b8     device_type_editdlgimpl.obj
 0002:000029cc       ??_C@_05LBDHBNMC@?$CK?4xml?$AA@ 100159cc     device_type_editdlgimpl.obj
 0002:000029d4       __real@00000000            100159d4     device_type_editdlgimpl.obj
 0002:000029d8       __real@3f800000            100159d8     device_type_editdlgimpl.obj
 0002:000029e0       ??_7paramLVI@@6B@          100159e0     paramLVI.obj
 0002:00002a78       ??_C@_09GKIBKPHB@14?514?56?51?$AA@ 10015a78     plugindesc.obj
 0002:00002a84       ??_C@_0M@DKFANHHP@?4?5c?5?$CD000000?$AA@ 10015a84     plugindesc.obj
 0002:00002a90       ??_C@_0M@ECOALFKK@d?5c?5?$CD633000?$AA@ 10015a90     plugindesc.obj
 0002:00002a9c       ??_C@_0M@DNDHEAI@?$CD?5c?5?$CD63ff31?$AA@ 10015a9c     plugindesc.obj
 0002:00002aa8       ??_C@_0M@CINNNEGB@c?5c?5?$CD9c6531?$AA@ 10015aa8     plugindesc.obj
 0002:00002ab4       ??_C@_0M@OCHFMIJJ@a?5c?5?$CDff0000?$AA@ 10015ab4     plugindesc.obj
 0002:00002ac0       ??_C@_0M@EIAONIKM@b?5c?5?$CDffffff?$AA@ 10015ac0     plugindesc.obj
 0002:00002acc       ??_C@_0P@HFKAALMG@?4?4?4?4?4?4?4?4?4?4?4?4?4?4?$AA@ 10015acc     plugindesc.obj
 0002:00002adc       ??_C@_0P@GKFLOHPK@?4?$CD?4?4?$CD?4?4?$CD?4?4?$CD?4?4?4?$AA@ 10015adc     plugindesc.obj
 0002:00002aec       ??_C@_0P@MIHCFHCI@?4?4?4a?4?4a?4?4a?4?4?4?4?$AA@ 10015aec     plugindesc.obj
 0002:00002afc       ??_C@_0P@PEANFGP@bbbbbbbbbbbbbb?$AA@ 10015afc     plugindesc.obj
 0002:00002b0c       ??_C@_0P@EBMAEIBP@bbbbbbbbbcccbb?$AA@ 10015b0c     plugindesc.obj
 0002:00002b1c       ??_C@_0P@LCEHAHDO@bbbbbbbccccddb?$AA@ 10015b1c     plugindesc.obj
 0002:00002b2c       ??_C@_0P@CANIDHJJ@bbbbcccccdddbb?$AA@ 10015b2c     plugindesc.obj
 0002:00002b3c       ??_C@_0P@NFPLNMIF@bbcccccddbbbbb?$AA@ 10015b3c     plugindesc.obj
 0002:00002b4c       ??_C@_0P@GLPGHHPO@bccccddbbbbbbb?$AA@ 10015b4c     plugindesc.obj
 0002:00002b5c       ??_C@_0P@MHFPFAKG@?4ccddbbbbbbbbb?$AA@ 10015b5c     plugindesc.obj
 0002:00002b6c       ??_C@_0P@NIGJJDJN@?4ddbbbbbbbbbbb?$AA@ 10015b6c     plugindesc.obj
 0002:00002b80       ??_7config_plugin_desc_base@@6B@ 10015b80     plugindesc.obj
 0002:00002b94       ??_7plugindesc@@6B@        10015b94     plugindesc.obj
 0002:00002ba4       ??_C@_0CE@BJBDPECI@Home?1System?1Object?1Device?5Type?5E@ 10015ba4     plugindesc.obj
 0002:00002bcc       ??_7toolWindow@@6BQObject@@@ 10015bcc     toolwindowimpl.obj
 0002:00002d84       ??_7toolWindow@@6BQPaintDevice@@@ 10015d84     toolwindowimpl.obj
 0002:00002da4       ??_C@_0BM@GLJFHFDA@1selectType?$CIQListViewItem?$CK?$CJ?$AA@ 10015da4     toolwindowimpl.obj
 0002:00002dc0       ??_C@_0CC@LCOLGNI@2selectionChanged?$CIQListViewItem?$CK@ 10015dc0     toolwindowimpl.obj
 0002:00002de4       ??_C@_0O@BEGAHEPI@1deleteFile?$CI?$CJ?$AA@ 10015de4     toolwindowimpl.obj
 0002:00002df4       ??_C@_0M@EHMABMKM@devicetypes?$AA@ 10015df4     toolwindowimpl.obj
 0002:00002e00       ??_C@_04GPMDFGEJ@type?$AA@ 10015e00     toolwindowimpl.obj
 0002:00002e08       ??_C@_02EGCJHIOB@id?$AA@   10015e08     toolwindowimpl.obj
 0002:00002e0c       ??_C@_06NBOBHOCP@family?$AA@ 10015e0c     toolwindowimpl.obj
 0002:00002e14       ??_C@_0CB@BNNAGILJ@Enter?5a?5unique?5device?5type?5name?4@ 10015e14     toolwindowimpl.obj
 0002:00002e38       ??_C@_0BA@FODFNJLF@New?5Device?5Type?$AA@ 10015e38     toolwindowimpl.obj
 0002:00002e48       ??_C@_0BJ@JALACFMD@Invalid?5device?5type?5name?$AA@ 10015e48     toolwindowimpl.obj
 0002:00002e64       ??_C@_0BH@HDJNCPID@Select?5the?5family?5for?5?$AA@ 10015e64     toolwindowimpl.obj
 0002:00002e7c       ??_C@_0O@HIAPDCAO@Select?5Family?$AA@ 10015e7c     toolwindowimpl.obj
 0002:00002e94       ??_SQWidget@@6BQObject@@@  10015e94     device_type_editdlg.obj
 0002:00003048       ??_SQWidget@@6BQPaintDevice@@@ 10016048     device_type_editdlg.obj
 0002:0000306c       ??_7device_type_editDlgBase@@6BQObject@@@ 1001606c     device_type_editdlg.obj
 0002:00003224       ??_7device_type_editDlgBase@@6BQPaintDevice@@@ 10016224     device_type_editdlg.obj
 0002:0000324c       ??_SQListView@@6BQObject@@@ 1001624c     device_type_editdlg.obj
 0002:00003530       ??_SQListView@@6BQPaintDevice@@@ 10016530     device_type_editdlg.obj
 0002:00003554       ??_SQPushButton@@6BQObject@@@ 10016554     device_type_editdlg.obj
 0002:00003744       ??_SQPushButton@@6BQPaintDevice@@@ 10016744     device_type_editdlg.obj
 0002:0000376c       ??_SQLabel@@6BQObject@@@   1001676c     device_type_editdlg.obj
 0002:00003964       ??_SQLabel@@6BQPaintDevice@@@ 10016964     device_type_editdlg.obj
 0002:0000398c       ??_SQComboBox@@6BQObject@@@ 1001698c     device_type_editdlg.obj
 0002:00003b70       ??_SQComboBox@@6BQPaintDevice@@@ 10016b70     device_type_editdlg.obj
 0002:00003b94       ??_SQGroupBox@@6BQObject@@@ 10016b94     device_type_editdlg.obj
 0002:00003d74       ??_SQGroupBox@@6BQPaintDevice@@@ 10016d74     device_type_editdlg.obj
 0002:00003d9c       ??_SQSpinBox@@6BQObject@@@ 10016d9c     device_type_editdlg.obj
 0002:00003f94       ??_SQSpinBox@@6BQPaintDevice@@@ 10016f94     device_type_editdlg.obj
 0002:00003fb8       ??_SQSpinBox@@6B@          10016fb8     device_type_editdlg.obj
 0002:00003fcc       ??_SQLineEdit@@6BQObject@@@ 10016fcc     device_type_editdlg.obj
 0002:000041f4       ??_SQLineEdit@@6BQPaintDevice@@@ 100171f4     device_type_editdlg.obj
 0002:0000421c       ??_SQWidgetStack@@6BQObject@@@ 1001721c     device_type_editdlg.obj
 0002:000043f4       ??_SQWidgetStack@@6BQPaintDevice@@@ 100173f4     device_type_editdlg.obj
 0002:0000441c       ??_SQCheckBox@@6BQObject@@@ 1001741c     device_type_editdlg.obj
 0002:000045fc       ??_SQCheckBox@@6BQPaintDevice@@@ 100175fc     device_type_editdlg.obj
 0002:00004624       ??_SQSpacerItem@@6B@       10017624     device_type_editdlg.obj
 0002:0000466c       ??_SQGridLayout@@6BQObject@@@ 1001766c     device_type_editdlg.obj
 0002:000046dc       ??_SQGridLayout@@6BQLayoutItem@@@ 100176dc     device_type_editdlg.obj
 0002:00004724       ??_SQHBoxLayout@@6BQObject@@@ 10017724     device_type_editdlg.obj
 0002:0000478c       ??_SQHBoxLayout@@6BQLayoutItem@@@ 1001778c     device_type_editdlg.obj
 0002:000047d4       ??_SQVBoxLayout@@6BQObject@@@ 100177d4     device_type_editdlg.obj
 0002:0000483c       ??_SQVBoxLayout@@6BQLayoutItem@@@ 1001783c     device_type_editdlg.obj
 0002:0000487c       ??_C@_0BI@HIICFJDD@device_type_editDlgBase?$AA@ 1001787c     device_type_editdlg.obj
 0002:00004894       ??_C@_0BO@GELCCPLB@device_type_editDlgBaseLayout?$AA@ 10017894     device_type_editdlg.obj
 0002:000048b4       ??_C@_07OJFJHGCA@lblType?$AA@ 100178b4     device_type_editdlg.obj
 0002:000048bc       ??_C@_08HEFODFJH@layout14?$AA@ 100178bc     device_type_editdlg.obj
 0002:000048c8       ??_C@_0N@GGFNLIAF@textLabel1_3?$AA@ 100178c8     device_type_editdlg.obj
 0002:000048d8       ??_C@_0N@OKABINLF@comboDevType?$AA@ 100178d8     device_type_editdlg.obj
 0002:000048e8       ??_C@_07IBBCGPPB@layout6?$AA@ 100178e8     device_type_editdlg.obj
 0002:000048f0       ??_C@_08GNHGGFDB@lvParams?$AA@ 100178f0     device_type_editdlg.obj
 0002:000048fc       ??_C@_09HPDNJEFH@Parameter?$AA@ 100178fc     device_type_editdlg.obj
 0002:00004908       ??_C@_04DPEGMFKN@Slot?$AA@ 10017908     device_type_editdlg.obj
 0002:00004910       ??_C@_04KOACHJEN@Type?$AA@ 10017910     device_type_editdlg.obj
 0002:00004918       ??_C@_06IOEANFCI@Access?$AA@ 10017918     device_type_editdlg.obj
 0002:00004920       ??_C@_07KKDPDMDC@layout5?$AA@ 10017920     device_type_editdlg.obj
 0002:00004928       ??_C@_0M@JGKOMMLK@btnNewParam?$AA@ 10017928     device_type_editdlg.obj
 0002:00004934       ??_C@_0M@GGFJIOBA@btnDelParam?$AA@ 10017934     device_type_editdlg.obj
 0002:00004940       ??_C@_0N@GIJBKNID@btnCopyParam?$AA@ 10017940     device_type_editdlg.obj
 0002:00004950       ??_C@_0O@HGFEFPAK@btnPasteParam?$AA@ 10017950     device_type_editdlg.obj
 0002:00004960       ??_C@_0P@NCHLOBNP@btnRenameParam?$AA@ 10017960     device_type_editdlg.obj
 0002:00004970       ??_C@_0L@GEIFBDEH@groupParam?$AA@ 10017970     device_type_editdlg.obj
 0002:0000497c       ??_C@_08INNFJCFG@lblParam?$AA@ 1001797c     device_type_editdlg.obj
 0002:00004988       ??_C@_08BADCPAJD@layout10?$AA@ 10017988     device_type_editdlg.obj
 0002:00004994       ??_C@_07GIKHDDO@layout9?$AA@ 10017994     device_type_editdlg.obj
 0002:0000499c       ??_C@_0P@BFGOLANA@textLabel2_2_3?$AA@ 1001799c     device_type_editdlg.obj
 0002:000049ac       ??_C@_0N@GNPDCGKK@textLabel2_2?$AA@ 100179ac     device_type_editdlg.obj
 0002:000049bc       ??_C@_0M@KLFOIEMK@comboAccess?$AA@ 100179bc     device_type_editdlg.obj
 0002:000049c8       ??_C@_09JMMFECAJ@comboType?$AA@ 100179c8     device_type_editdlg.obj
 0002:000049d4       ??_C@_0L@INJINICK@textLabel2?$AA@ 100179d4     device_type_editdlg.obj
 0002:000049e0       ??_C@_0O@KLAOPFEG@comboTemplate?$AA@ 100179e0     device_type_editdlg.obj
 0002:000049f0       ??_C@_08FGMDCPIC@spinSlot?$AA@ 100179f0     device_type_editdlg.obj
 0002:000049fc       ??_C@_08BKBDHJHD@txtStyle?$AA@ 100179fc     device_type_editdlg.obj
 0002:00004a08       ??_C@_0P@MHFIBJB@textLabel2_2_2?$AA@ 10017a08     device_type_editdlg.obj
 0002:00004a18       ??_C@_0BB@MAMJFOAB@textLabel2_2_3_2?$AA@ 10017a18     device_type_editdlg.obj
 0002:00004a2c       ??_C@_09PPLHEDKA@stackType?$AA@ 10017a2c     device_type_editdlg.obj
 0002:00004a38       ??_C@_07CNDDMOPN@Not_Set?$AA@ 10017a38     device_type_editdlg.obj
 0002:00004a40       ??_C@_0N@HPEGIJEE@textLabel1_2?$AA@ 10017a40     device_type_editdlg.obj
 0002:00004a50       ??_C@_04PAFOOALK@Enum?$AA@ 10017a50     device_type_editdlg.obj
 0002:00004a58       ??_C@_0L@MDHOEMNN@EnumLayout?$AA@ 10017a58     device_type_editdlg.obj
 0002:00004a64       ??_C@_08EBBBPHMD@lvStates?$AA@ 10017a64     device_type_editdlg.obj
 0002:00004a70       ??_C@_0L@GNEBAGAL@layout10_2?$AA@ 10017a70     device_type_editdlg.obj
 0002:00004a7c       ??_C@_0L@CCNDADHF@btnEnumNew?$AA@ 10017a7c     device_type_editdlg.obj
 0002:00004a88       ??_C@_0O@JCAHNLLG@btnEnumDelete?$AA@ 10017a88     device_type_editdlg.obj
 0002:00004a98       ??_C@_0M@EMNCKGFP@btnEnumCopy?$AA@ 10017a98     device_type_editdlg.obj
 0002:00004aa4       ??_C@_0N@MDANPDMI@btnEnumPaste?$AA@ 10017aa4     device_type_editdlg.obj
 0002:00004ab4       ??_C@_0P@JDPKMCHO@textLabel1_2_3?$AA@ 10017ab4     device_type_editdlg.obj
 0002:00004ac4       ??_C@_0M@HMMLKJCC@rangeLayout?$AA@ 10017ac4     device_type_editdlg.obj
 0002:00004ad0       ??_C@_07BPJBECHP@layout8?$AA@ 10017ad0     device_type_editdlg.obj
 0002:00004ad8       ??_C@_0BD@PNIEKLPO@textLabel5_2_3_2_2?$AA@ 10017ad8     device_type_editdlg.obj
 0002:00004aec       ??_C@_0P@IGLIAGI@textLabel5_2_3?$AA@ 10017aec     device_type_editdlg.obj
 0002:00004afc       ??_C@_0M@BCGMBKJL@txtRangeMin?$AA@ 10017afc     device_type_editdlg.obj
 0002:00004b08       ??_C@_0O@PIEPDGCB@txtRangeUnits?$AA@ 10017b08     device_type_editdlg.obj
 0002:00004b18       ??_C@_0N@OCFJNFEO@txtRangeJump?$AA@ 10017b18     device_type_editdlg.obj
 0002:00004b28       ??_C@_0N@PACEBOBD@textLabel5_2?$AA@ 10017b28     device_type_editdlg.obj
 0002:00004b38       ??_C@_0L@MCNJEOON@textLabel5?$AA@ 10017b38     device_type_editdlg.obj
 0002:00004b44       ??_C@_0N@DJAGBGGA@txtRangeStep?$AA@ 10017b44     device_type_editdlg.obj
 0002:00004b54       ??_C@_0P@BBHALBCJ@textLabel5_2_2?$AA@ 10017b54     device_type_editdlg.obj
 0002:00004b64       ??_C@_0M@OHPOPE@txtRangeMax?$AA@ 10017b64     device_type_editdlg.obj
 0002:00004b70       ??_C@_0BA@IHJAGGDH@txtRangeDefault?$AA@ 10017b70     device_type_editdlg.obj
 0002:00004b80       ??_C@_0BB@MKAMFHBI@textLabel5_2_3_2?$AA@ 10017b80     device_type_editdlg.obj
 0002:00004b94       ??_C@_0BB@IGDIJAFK@groupCalcDisplay?$AA@ 10017b94     device_type_editdlg.obj
 0002:00004ba8       ??_C@_0P@KJMMNGEM@textLabel5_3_2?$AA@ 10017ba8     device_type_editdlg.obj
 0002:00004bb8       ??_C@_0BA@BBCPMDPP@txtRangeOffsetA?$AA@ 10017bb8     device_type_editdlg.obj
 0002:00004bc8       ??_C@_0N@OJDPCPFC@textLabel5_3?$AA@ 10017bc8     device_type_editdlg.obj
 0002:00004bd8       ??_C@_0L@OJPEBNCO@textLabel6?$AA@ 10017bd8     device_type_editdlg.obj
 0002:00004be4       ??_C@_0BB@LJOMODNI@textLabel5_3_2_2?$AA@ 10017be4     device_type_editdlg.obj
 0002:00004bf8       ??_C@_0L@KGLFILOJ@textLabel1?$AA@ 10017bf8     device_type_editdlg.obj
 0002:00004c04       ??_C@_0O@IHAJBKKN@txtRangeMulti?$AA@ 10017c04     device_type_editdlg.obj
 0002:00004c14       ??_C@_0BA@DKACJADM@txtRangeOffsetB?$AA@ 10017c14     device_type_editdlg.obj
 0002:00004c24       ??_C@_0N@PMLNHDMK@spinRangeDec?$AA@ 10017c24     device_type_editdlg.obj
 0002:00004c34       ??_C@_0P@ENGKKBBC@checkRangeCalc?$AA@ 10017c34     device_type_editdlg.obj
 0002:00004c44       ??_C@_0N@NLCHJEPA@stringLayout?$AA@ 10017c44     device_type_editdlg.obj
 0002:00004c54       ??_C@_0N@HEOIBHOL@textLabel2_3?$AA@ 10017c54     device_type_editdlg.obj
 0002:00004c64       ??_C@_0P@FKCPCGBH@textLabel2_2_4?$AA@ 10017c64     device_type_editdlg.obj
 0002:00004c74       ??_C@_0N@IDGMOKFA@comboStrCase?$AA@ 10017c74     device_type_editdlg.obj
 0002:00004c84       ??_C@_0O@BEDBIKL@spinStrLength?$AA@ 10017c84     device_type_editdlg.obj
 0002:00004c94       ??_C@_0BC@CCKOMJAI@1raiseWidget?$CIint?$CJ?$AA@ 10017c94     device_type_editdlg.obj
 0002:00004ca8       ??_C@_0P@POCECEMJ@2toggled?$CIbool?$CJ?$AA@ 10017ca8     device_type_editdlg.obj
 0002:00004cb8       ??_C@_0BE@BNNIEODF@device_type_editDlg?$AA@ 10017cb8     device_type_editdlg.obj
 0002:00004ccc       ??_C@_0BF@LCDGMGFM@?$DMh1?$DODevice?5Type?$DM?1h1?$DO?$AA@ 10017ccc     device_type_editdlg.obj
 0002:00004ce4       ??_C@_0L@PMICFDLL@DeviceType?$AA@ 10017ce4     device_type_editdlg.obj
 0002:00004cf0       ??_C@_0L@KPCMBCOA@InfoDriver?$AA@ 10017cf0     device_type_editdlg.obj
 0002:00004cfc       ??_C@_03ILBCOJBH@New?$AA@  10017cfc     device_type_editdlg.obj
 0002:00004d00       ??_C@_06JBKGCNBB@Delete?$AA@ 10017d00     device_type_editdlg.obj
 0002:00004d08       ??_C@_04OPMHGHMB@Copy?$AA@ 10017d08     device_type_editdlg.obj
 0002:00004d10       ??_C@_0BG@CODCAOAP@Copy?5to?5the?5clipboard?$AA@ 10017d10     device_type_editdlg.obj
 0002:00004d28       ??_C@_05NEBJFIEK@Paste?$AA@ 10017d28     device_type_editdlg.obj
 0002:00004d30       ??_C@_0DM@CPDIBDFA@Paste?5over?5existing?5parameter?5if@ 10017d30     device_type_editdlg.obj
 0002:00004d6c       ??_C@_0O@MLKCHIAI@Rename?5Param?4?$AA@ 10017d6c     device_type_editdlg.obj
 0002:00004d7c       ??_C@_09JCONGPFK@?$DMh1?$DO?$DM?1h1?$DO?$AA@ 10017d7c     device_type_editdlg.obj
 0002:00004d88       ??_C@_0L@DKONPLBG@Read?1Write?$AA@ 10017d88     device_type_editdlg.obj
 0002:00004d94       ??_C@_09KMNPFIKF@Read?5only?$AA@ 10017d94     device_type_editdlg.obj
 0002:00004da0       ??_C@_0L@EOBCINKH@Write?5only?$AA@ 10017da0     device_type_editdlg.obj
 0002:00004dac       ??_C@_09HCDHCAAF@?$FLNot?5Set?$FN?$AA@ 10017dac     device_type_editdlg.obj
 0002:00004db8       ??_C@_08NLCKCAFE@Template?$AA@ 10017db8     device_type_editdlg.obj
 0002:00004dc4       ??_C@_0BF@CLAADHCK@?$DMh1?$DONo?5type?5set?$DM?1h1?$DO?$AA@ 10017dc4     device_type_editdlg.obj
 0002:00004ddc       ??_C@_0O@OKGOMGEM@?$DMh1?$DOList?$DM?1h1?$DO?$AA@ 10017ddc     device_type_editdlg.obj
 0002:00004dec       ??_C@_05CFLIFMAE@Units?$AA@ 10017dec     device_type_editdlg.obj
 0002:00004df4       ??_C@_08JFEGPOPA@Big?5Step?$AA@ 10017df4     device_type_editdlg.obj
 0002:00004e00       ??_C@_0L@JKHOJFHF@Max?4?5Value?$AA@ 10017e00     device_type_editdlg.obj
 0002:00004e0c       ??_C@_0L@FGHDOOHK@Min?4?5Value?$AA@ 10017e0c     device_type_editdlg.obj
 0002:00004e18       ??_C@_0L@CMBGILKP@Small?5Step?$AA@ 10017e18     device_type_editdlg.obj
 0002:00004e24       ??_C@_07MCAEODGB@Default?$AA@ 10017e24     device_type_editdlg.obj
 0002:00004e2c       ??_C@_0BD@CIGFIKLI@Calculated?5Display?$AA@ 10017e2c     device_type_editdlg.obj
 0002:00004e40       ??_C@_08PCJHPFJ@Offset?5A?$AA@ 10017e40     device_type_editdlg.obj
 0002:00004e4c       ??_C@_0L@FHHMINHA@Multiplier?$AA@ 10017e4c     device_type_editdlg.obj
 0002:00004e58       ??_C@_0CL@LDAMKMFK@Display?5?$DN?5?$CImultiplier?$CIOffsetA?$CLIn@ 10017e58     device_type_editdlg.obj
 0002:00004e84       ??_C@_08CEAECMJK@Offset?5B?$AA@ 10017e84     device_type_editdlg.obj
 0002:00004e90       ??_C@_08DAMBCEIE@Decimals?$AA@ 10017e90     device_type_editdlg.obj
 0002:00004e9c       ??_C@_09NADPJEHH@Calculate?$AA@ 10017e9c     device_type_editdlg.obj
 0002:00004ea8       ??_C@_0L@KADBNAHP@Max?5Length?$AA@ 10017ea8     device_type_editdlg.obj
 0002:00004eb4       ??_C@_04OLCJPDPG@Case?$AA@ 10017eb4     device_type_editdlg.obj
 0002:00004ebc       ??_C@_03OBJFJEBA@any?$AA@  10017ebc     device_type_editdlg.obj
 0002:00004ec0       __xmm@00000030000000f90000001400000014 10017ec0     device_type_editdlg.obj
 0002:00004ed0       ??_C@_0BB@FJCBBIOH@device_type_edit?$AA@ 10017ed0     moc_device_type_edit.obj
 0002:00004ef0       ??_C@_0L@LGCGKDIM@deleteType?$AA@ 10017ef0     moc_device_type_edit.obj
 0002:00004f08       ??_C@_0L@FLBIABLK@selectType?$AA@ 10017f08     moc_device_type_edit.obj
 0002:00004f20       ??_C@_09HIGIDEDO@markDirty?$AA@ 10017f20     moc_device_type_edit.obj
 0002:00004f50       ??_C@_0BL@KIPOLACL@deleteType?$CIconst?5QString?$CG?$CJ?$AA@ 10017f50     moc_device_type_edit.obj
 0002:00004f6c       ??_C@_0BL@ONELGNJL@selectType?$CIconst?5QString?$CG?$CJ?$AA@ 10017f6c     moc_device_type_edit.obj
 0002:00004f88       ??_C@_0M@BCGJBPBD@markDirty?$CI?$CJ?$AA@ 10017f88     moc_device_type_edit.obj
 0002:00004fa0       ??_C@_07KMMNMMFF@command?$AA@ 10017fa0     moc_device_type_edit.obj
 0002:00004fb4       ??_C@_0BJ@FEFNJDLM@command?$CIQString?0QString?$CJ?$AA@ 10017fb4     moc_device_type_edit.obj
 0002:00004fdc       ??_C@_0P@DMEOIADN@languageChange?$AA@ 10017fdc     moc_device_type_editdlg.obj
 0002:00004ff8       ??_C@_0BB@PFEIHPGD@languageChange?$CI?$CJ?$AA@ 10017ff8     moc_device_type_editdlg.obj
 0002:0000500c       ??_C@_03DAPAKLGM@dir?$AA@  1001800c     moc_device_type_editdlgimpl.obj
 0002:0000501c       ??_C@_0O@IGKPFAPL@loadTemplates?$AA@ 1001801c     moc_device_type_editdlgimpl.obj
 0002:00005038       ??_C@_0M@DAEFIJCE@paramDelete?$AA@ 10018038     moc_device_type_editdlgimpl.obj
 0002:00005050       ??_C@_0BE@FIBMIMHP@checkParamClipboard?$AA@ 10018050     moc_device_type_editdlgimpl.obj
 0002:00005070       ??_C@_0L@OGCOBDOL@paramPaste?$AA@ 10018070     moc_device_type_editdlgimpl.obj
 0002:00005088       ??_C@_09OACFON@paramCopy?$AA@ 10018088     moc_device_type_editdlgimpl.obj
 0002:000050a0       ??_C@_0M@NCBOHMBI@paramRename?$AA@ 100180a0     moc_device_type_editdlgimpl.obj
 0002:000050b8       ??_C@_08HJEAOPFE@paramNew?$AA@ 100180b8     moc_device_type_editdlgimpl.obj
 0002:000050d0       ??_C@_09CLOPLGEM@enumPaste?$AA@ 100180d0     moc_device_type_editdlgimpl.obj
 0002:000050e8       ??_C@_0BA@KIPPEHDD@enumDeleteState?$AA@ 100180e8     moc_device_type_editdlgimpl.obj
 0002:00005104       ??_C@_0N@GAGMHFOG@enumNewState?$AA@ 10018104     moc_device_type_editdlgimpl.obj
 0002:00005114       ??_C@_03ELAIKMFE@lvi?$AA@  10018114     moc_device_type_editdlgimpl.obj
 0002:00005118       ??_C@_0O@LAFKAPIP@QListViewItem?$AA@ 10018118     moc_device_type_editdlgimpl.obj
 0002:00005128       ??_C@_01CAKFMAIO@?$AO?$AA@ 10018128     moc_device_type_editdlgimpl.obj
 0002:0000512c       ??_C@_04KOJNECLL@iCol?$AA@ 1001812c     moc_device_type_editdlgimpl.obj
 0002:00005140       ??_C@_0N@ILEGFABJ@enumDblClick?$AA@ 10018140     moc_device_type_editdlgimpl.obj
 0002:0000518c       ??_C@_0M@JNLNKJHL@selectParam?$AA@ 1001818c     moc_device_type_editdlgimpl.obj
 0002:00005198       ??_C@_05FKHKFDID@index?$AA@ 10018198     moc_device_type_editdlgimpl.obj
 0002:000051ac       ??_C@_0O@HCPANIPE@devTypeChange?$AA@ 100181ac     moc_device_type_editdlgimpl.obj
 0002:0000528c       ??_C@_0BH@MCENJHEH@loadTemplates?$CIQString?$CJ?$AA@ 1001828c     moc_device_type_editdlgimpl.obj
 0002:000052a4       ??_C@_0O@BHJEGCNE@paramDelete?$CI?$CJ?$AA@ 100182a4     moc_device_type_editdlgimpl.obj
 0002:000052b4       ??_C@_0BG@DOLBHKJN@checkParamClipboard?$CI?$CJ?$AA@ 100182b4     moc_device_type_editdlgimpl.obj
 0002:000052cc       ??_C@_0N@ELCMAFGE@paramPaste?$CI?$CJ?$AA@ 100182cc     moc_device_type_editdlgimpl.obj
 0002:000052dc       ??_C@_0M@NCMMNBLF@paramCopy?$CI?$CJ?$AA@ 100182dc     moc_device_type_editdlgimpl.obj
 0002:000052e8       ??_C@_0O@KJLAPPOD@paramRename?$CI?$CJ?$AA@ 100182e8     moc_device_type_editdlgimpl.obj
 0002:000052f8       ??_C@_0L@JMHKJGEK@paramNew?$CI?$CJ?$AA@ 100182f8     moc_device_type_editdlgimpl.obj
 0002:00005304       ??_C@_0M@MNGLFOM@enumPaste?$CI?$CJ?$AA@ 10018304     moc_device_type_editdlgimpl.obj
 0002:00005310       ??_C@_0BC@GOMLJBEP@enumDeleteState?$CI?$CJ?$AA@ 10018310     moc_device_type_editdlgimpl.obj
 0002:00005324       ??_C@_0P@FKFDDJAG@enumNewState?$CI?$CJ?$AA@ 10018324     moc_device_type_editdlgimpl.obj
 0002:00005334       ??_C@_0CP@PHFBJBPP@enumDblClick?$CIQListViewItem?$CK?0cons@ 10018334     moc_device_type_editdlgimpl.obj
 0002:00005364       ??_C@_0BK@HOHMEHMM@markDirty?$CIconst?5QString?$CG?$CJ?$AA@ 10018364     moc_device_type_editdlgimpl.obj
 0002:00005380       ??_C@_0P@HDOAENEH@markDirty?$CIint?$CJ?$AA@ 10018380     moc_device_type_editdlgimpl.obj
 0002:00005390       ??_C@_0BO@EANMBGCG@markDirty?$CIQListViewItem?$CK?0int?$CJ?$AA@ 10018390     moc_device_type_editdlgimpl.obj
 0002:000053b0       ??_C@_0O@BBNJKOHP@selectParam?$CI?$CJ?$AA@ 100183b0     moc_device_type_editdlgimpl.obj
 0002:000053c0       ??_C@_0BD@EFADECHP@devTypeChange?$CIint?$CJ?$AA@ 100183c0     moc_device_type_editdlgimpl.obj
 0002:00005404       ??_C@_07POMFAKIB@dirty?$CI?$CJ?$AA@ 10018404     moc_device_type_editdlgimpl.obj
 0002:0000540c       ??_C@_0P@ECKEJGFB@toolWindowBase?$AA@ 1001840c     moc_toolwindow.obj
 0002:00005434       ??_C@_0L@IGMLIIOB@toolWindow?$AA@ 10018434     moc_toolwindowimpl.obj
 0002:0000544c       ??_C@_0L@OJCDGKOF@deleteFile?$AA@ 1001844c     moc_toolwindowimpl.obj
 0002:00005464       ??_C@_07FIMPHEOC@newFile?$AA@ 10018464     moc_toolwindowimpl.obj
 0002:0000549c       ??_C@_0N@PMHGOOHP@deleteFile?$CI?$CJ?$AA@ 1001849c     moc_toolwindowimpl.obj
 0002:000054ac       ??_C@_09EJDIPEDH@newFile?$CI?$CJ?$AA@ 100184ac     moc_toolwindowimpl.obj
 0002:000054b8       ??_C@_0BL@NNMKNPAH@selectType?$CIQListViewItem?$CK?$CJ?$AA@ 100184b8     moc_toolwindowimpl.obj
 0002:000054e0       ??_C@_0N@EIHAHPOH@typeSelected?$AA@ 100184e0     moc_toolwindowimpl.obj
 0002:000054fc       ??_C@_0M@DHNJKGPE@typeDeleted?$AA@ 100184fc     moc_toolwindowimpl.obj
 0002:00005538       ??_C@_0BN@HBDOHOHE@typeSelected?$CIconst?5QString?$CG?$CJ?$AA@ 10018538     moc_toolwindowimpl.obj
 0002:00005558       ??_C@_0BM@HFHIDGDF@typeDeleted?$CIconst?5QString?$CG?$CJ?$AA@ 10018558     moc_toolwindowimpl.obj
 0002:00005578       ??_7toolWindowBase@@6BQObject@@@ 10018578     toolwindow.obj
 0002:00005730       ??_7toolWindowBase@@6BQPaintDevice@@@ 10018730     toolwindow.obj
 0002:00005754       ??_SQTabWidget@@6BQObject@@@ 10018754     toolwindow.obj
 0002:00005928       ??_SQTabWidget@@6BQPaintDevice@@@ 10018928     toolwindow.obj
 0002:00005948       ??_C@_0BF@OGGOGOEO@toolWindowBaseLayout?$AA@ 10018948     toolwindow.obj
 0002:00005960       ??_C@_0L@NNPJCPDK@tabWidget2?$AA@ 10018960     toolwindow.obj
 0002:0000596c       ??_C@_03CEDILPBK@tab?$AA@  1001896c     toolwindow.obj
 0002:00005970       ??_C@_09PEOMDABK@tabLayout?$AA@ 10018970     toolwindow.obj
 0002:0000597c       ??_C@_07MOFDPJDG@layout1?$AA@ 1001897c     toolwindow.obj
 0002:00005984       ??_C@_0L@JDKCOBHF@btnNewType?$AA@ 10018984     toolwindow.obj
 0002:00005990       ??_C@_0O@FMBLAGPA@btnDeleteType?$AA@ 10018990     toolwindow.obj
 0002:000059a0       ??_C@_07NAMNDLEO@lvTypes?$AA@ 100189a0     toolwindow.obj
 0002:000059a8       ??_C@_04FABLJDN@Name?$AA@  100189a8     toolwindow.obj
 0002:000059b0       ??_C@_06BOFMEHLD@Family?$AA@ 100189b0     toolwindow.obj
 0002:000059b8       ??_C@_08COBBAHCH@New?5Type?$AA@ 100189b8     toolwindow.obj
 0002:000059c4       ??_C@_0N@HGJPIPEN@Device?5Types?$AA@ 100189c4     toolwindow.obj
 0002:000059d8       ??_7cfg_ListView@@6BQObject@@@ 100189d8     cfg_widgets001:cfg_ListView.obj
 0002:00005cc4       ??_7cfg_ListView@@6BQPaintDevice@@@ 10018cc4     cfg_widgets001:cfg_ListView.obj
 0002:00005ce4       ??_C@_0BI@DKLEEDHJ@1clipBoardDataChanged?$CI?$CJ?$AA@ 10018ce4     cfg_widgets001:cfg_ListView.obj
 0002:00005cfc       ??_C@_0BA@NOIFKKAG@2dataChanged?5?$CI?$CJ?$AA@ 10018cfc     cfg_widgets001:cfg_ListView.obj
 0002:00005d10       ??_C@_0EB@PMPDJKLD@int?5cfg_ListView?3?3validateRow?$CIiR@ 10018d10     cfg_widgets001:cfg_ListView.obj
 0002:00005d54       ??_C@_0BD@BEIDFIOE@Creating?5new?5entry?$AA@ 10018d54     cfg_widgets001:cfg_ListView.obj
 0002:00005d68       ??_C@_0DO@OOICEDKL@int?5cfg_Table?3?3validateRow?$CIiRow?$CJ@ 10018d68     cfg_widgets001:cfg_ListView.obj
 0002:00005da8       ??_C@_0EN@NNOBKMDG@cfg_ListView?3?3updateEntry?5?9?5newI@ 10018da8     cfg_widgets001:cfg_ListView.obj
 0002:00005df8       ??_C@_0FB@OICAKFGC@int?5cfg_ListView?3?3validateRow?$CIQL@ 10018df8     cfg_widgets001:cfg_ListView.obj
 0002:00005e4c       ??_C@_0N@NAADDCIB@cfg_ListView?$AA@ 10018e4c     cfg_widgets001:moc_cfg_ListView.obj
 0002:00005e68       ??_C@_0L@MLFJPJPC@insertData?$AA@ 10018e68     cfg_widgets001:moc_cfg_ListView.obj
 0002:00005e80       ??_C@_0M@MOKGOAHM@deleteItems?$AA@ 10018e80     cfg_widgets001:moc_cfg_ListView.obj
 0002:00005e98       ??_C@_0BA@FJBCKEJL@copyToClipboard?$AA@ 10018e98     cfg_widgets001:moc_cfg_ListView.obj
 0002:00005eb4       ??_C@_09CLMPBHDI@undoPaste?$AA@ 10018eb4     cfg_widgets001:moc_cfg_ListView.obj
 0002:00005ecc       ??_C@_0M@NOBHHHJI@replaceData?$AA@ 10018ecc     cfg_widgets001:moc_cfg_ListView.obj
 0002:00005ee4       ??_C@_0BF@CDBOAHLL@clipBoardDataChanged?$AA@ 10018ee4     cfg_widgets001:moc_cfg_ListView.obj
 0002:00005f48       ??_C@_0N@JAPDIKGN@insertData?$CI?$CJ?$AA@ 10018f48     cfg_widgets001:moc_cfg_ListView.obj
 0002:00005f58       ??_C@_0O@FBJIJCJH@deleteItems?$CI?$CJ?$AA@ 10018f58     cfg_widgets001:moc_cfg_ListView.obj
 0002:00005f68       ??_C@_0BC@DBBGOFIB@copyToClipboard?$CI?$CJ?$AA@ 10018f68     cfg_widgets001:moc_cfg_ListView.obj
 0002:00005f7c       ??_C@_0M@OGFEJKEA@undoPaste?$CI?$CJ?$AA@ 10018f7c     cfg_widgets001:moc_cfg_ListView.obj
 0002:00005f88       ??_C@_0O@FOBLCCJ@replaceData?$CI?$CJ?$AA@ 10018f88     cfg_widgets001:moc_cfg_ListView.obj
 0002:00005f98       ??_C@_0BH@OLENEJHN@clipBoardDataChanged?$CI?$CJ?$AA@ 10018f98     cfg_widgets001:moc_cfg_ListView.obj
 0002:00005fbc       ??_C@_0L@OIBMJOP@dataPasted?$AA@ 10018fbc     cfg_widgets001:moc_cfg_ListView.obj
 0002:00005fd4       ??_C@_0BD@IALCIEJE@clipboardDataValid?$AA@ 10018fd4     cfg_widgets001:moc_cfg_ListView.obj
 0002:00006000       ??_C@_0N@EJEGBDAF@dataPasted?$CI?$CJ?$AA@ 10019000     cfg_widgets001:moc_cfg_ListView.obj
 0002:00006010       ??_C@_0BJ@FABNKMFK@clipboardDataValid?$CIbool?$CJ?$AA@ 10019010     cfg_widgets001:moc_cfg_ListView.obj
 0002:00006030       ??_7type_info@@6B@         10019030     MSVCRT:ti_inst.obj
 0002:00006034       __pDefaultRawDllMain       10019034     MSVCRT:crtdll.obj
 0002:00006034       __pRawDllMain              10019034     MSVCRT:crtdll.obj
 0002:00006040       __load_config_used         10019040     MSVCRT:loadcfg.obj
 0002:00006088       ??_R3QShared@@8            10019088     device_type_edit.obj
 0002:00006098       ??_R2QShared@@8            10019098     device_type_edit.obj
 0002:000060a0       ??_R1A@?0A@EA@QShared@@8   100190a0     device_type_edit.obj
 0002:000060bc       ??_R1A@?0A@EA@QGList@@8    100190bc     device_type_edit.obj
 0002:000060d8       ??_R3QGList@@8             100190d8     device_type_edit.obj
 0002:000060e8       ??_R2QGList@@8             100190e8     device_type_edit.obj
 0002:000060f4       ??_R1A@?0A@EA@QPtrCollection@@8 100190f4     device_type_edit.obj
 0002:00006110       ??_R3QPtrCollection@@8     10019110     device_type_edit.obj
 0002:00006120       ??_R2QPtrCollection@@8     10019120     device_type_edit.obj
 0002:00006128       ??_R4QToolBar@@6BQObject@@@ 10019128     device_type_edit.obj
 0002:0000613c       ??_R3QToolBar@@8           1001913c     device_type_edit.obj
 0002:0000614c       ??_R2QToolBar@@8           1001914c     device_type_edit.obj
 0002:0000616c       ??_R1A@?0A@EA@QToolBar@@8  1001916c     device_type_edit.obj
 0002:00006188       ??_R1A@?0A@EA@QDockWindow@@8 10019188     device_type_edit.obj
 0002:000061a4       ??_R3QDockWindow@@8        100191a4     device_type_edit.obj
 0002:000061b4       ??_R2QDockWindow@@8        100191b4     device_type_edit.obj
 0002:000061d0       ??_R1A@?0A@EA@QFrame@@8    100191d0     device_type_edit.obj
 0002:000061ec       ??_R3QFrame@@8             100191ec     device_type_edit.obj
 0002:000061fc       ??_R2QFrame@@8             100191fc     device_type_edit.obj
 0002:00006214       ??_R1A@?0A@EA@QWidget@@8   10019214     device_type_edit.obj
 0002:00006230       ??_R3QWidget@@8            10019230     device_type_edit.obj
 0002:00006240       ??_R2QWidget@@8            10019240     device_type_edit.obj
 0002:00006254       ??_R1A@?0A@EA@QObject@@8   10019254     device_type_edit.obj
 0002:00006270       ??_R3QObject@@8            10019270     device_type_edit.obj
 0002:00006280       ??_R2QObject@@8            10019280     device_type_edit.obj
 0002:0000628c       ??_R13?0A@EA@Qt@@8         1001928c     device_type_edit.obj
 0002:000062a8       ??_R3Qt@@8                 100192a8     device_type_edit.obj
 0002:000062b8       ??_R2Qt@@8                 100192b8     device_type_edit.obj
 0002:000062c0       ??_R1A@?0A@EA@Qt@@8        100192c0     device_type_edit.obj
 0002:000062dc       ??_R1CI@?0A@EA@QPaintDevice@@8 100192dc     device_type_edit.obj
 0002:000062f8       ??_R3QPaintDevice@@8       100192f8     device_type_edit.obj
 0002:00006308       ??_R2QPaintDevice@@8       10019308     device_type_edit.obj
 0002:00006310       ??_R1A@?0A@EA@QPaintDevice@@8 10019310     device_type_edit.obj
 0002:0000632c       ??_R4QToolBar@@6BQPaintDevice@@@ 1001932c     device_type_edit.obj
 0002:00006340       ??_R4QPopupMenu@@6BQObject@@@ 10019340     device_type_edit.obj
 0002:00006354       ??_R3QPopupMenu@@8         10019354     device_type_edit.obj
 0002:00006364       ??_R2QPopupMenu@@8         10019364     device_type_edit.obj
 0002:00006384       ??_R1A@?0A@EA@QPopupMenu@@8 10019384     device_type_edit.obj
 0002:000063a0       ??_R1IM@?0A@EA@QMenuData@@8 100193a0     device_type_edit.obj
 0002:000063bc       ??_R3QMenuData@@8          100193bc     device_type_edit.obj
 0002:000063cc       ??_R2QMenuData@@8          100193cc     device_type_edit.obj
 0002:000063d4       ??_R1A@?0A@EA@QMenuData@@8 100193d4     device_type_edit.obj
 0002:000063f0       ??_R4QPopupMenu@@6BQPaintDevice@@@ 100193f0     device_type_edit.obj
 0002:00006404       ??_R4QPopupMenu@@6B@       10019404     device_type_edit.obj
 0002:00006418       ??_R4QDockWindow@@6BQObject@@@ 10019418     device_type_edit.obj
 0002:0000642c       ??_R4QDockWindow@@6BQPaintDevice@@@ 1001942c     device_type_edit.obj
 0002:00006440       ??_R4QAction@@6B@          10019440     device_type_edit.obj
 0002:00006454       ??_R3QAction@@8            10019454     device_type_edit.obj
 0002:00006464       ??_R2QAction@@8            10019464     device_type_edit.obj
 0002:00006474       ??_R1A@?0A@EA@QAction@@8   10019474     device_type_edit.obj
 0002:00006490       ??_R4QGuardedPtrPrivate@@6B@ 10019490     device_type_edit.obj
 0002:000064a4       ??_R3QGuardedPtrPrivate@@8 100194a4     device_type_edit.obj
 0002:000064b4       ??_R2QGuardedPtrPrivate@@8 100194b4     device_type_edit.obj
 0002:000064c8       ??_R1A@?0A@EA@QGuardedPtrPrivate@@8 100194c8     device_type_edit.obj
 0002:000064e4       ??_R1CI@?0A@EA@QShared@@8  100194e4     device_type_edit.obj
 0002:00006500       ??_R4QDockWindowList@@6B@  10019500     device_type_edit.obj
 0002:00006514       ??_R3QDockWindowList@@8    10019514     device_type_edit.obj
 0002:00006524       ??_R2QDockWindowList@@8    10019524     device_type_edit.obj
 0002:00006538       ??_R1A@?0A@EA@QDockWindowList@@8 10019538     device_type_edit.obj
 0002:00006554       ??_R1A@?0A@EA@?$QPtrList@VQDockWindow@@@@8 10019554     device_type_edit.obj
 0002:00006570       ??_R3?$QPtrList@VQDockWindow@@@@8 10019570     device_type_edit.obj
 0002:00006580       ??_R2?$QPtrList@VQDockWindow@@@@8 10019580     device_type_edit.obj
 0002:00006590       ??_R4QPopupMenuList@@6B@   10019590     device_type_edit.obj
 0002:000065a4       ??_R3QPopupMenuList@@8     100195a4     device_type_edit.obj
 0002:000065b4       ??_R2QPopupMenuList@@8     100195b4     device_type_edit.obj
 0002:000065c8       ??_R1A@?0A@EA@QPopupMenuList@@8 100195c8     device_type_edit.obj
 0002:000065e4       ??_R1A@?0A@EA@?$QPtrList@VQPopupMenu@@@@8 100195e4     device_type_edit.obj
 0002:00006600       ??_R3?$QPtrList@VQPopupMenu@@@@8 10019600     device_type_edit.obj
 0002:00006610       ??_R2?$QPtrList@VQPopupMenu@@@@8 10019610     device_type_edit.obj
 0002:00006620       ??_R4?$QPtrList@VQPopupMenu@@@@6B@ 10019620     device_type_edit.obj
 0002:00006634       ??_R4config_plugin_base@@6BQObject@@@ 10019634     device_type_edit.obj
 0002:00006648       ??_R3config_plugin_base@@8 10019648     device_type_edit.obj
 0002:00006658       ??_R2config_plugin_base@@8 10019658     device_type_edit.obj
 0002:00006670       ??_R1A@?0A@EA@config_plugin_base@@8 10019670     device_type_edit.obj
 0002:0000668c       ??_R4config_plugin_base@@6BQPaintDevice@@@ 1001968c     device_type_edit.obj
 0002:000066a0       ??_R1A@?0A@EA@QGDict@@8    100196a0     device_type_edit.obj
 0002:000066bc       ??_R3QGDict@@8             100196bc     device_type_edit.obj
 0002:000066cc       ??_R2QGDict@@8             100196cc     device_type_edit.obj
 0002:000066d8       ??_R4device_type_edit@@6BQObject@@@ 100196d8     device_type_edit.obj
 0002:000066ec       ??_R3device_type_edit@@8   100196ec     device_type_edit.obj
 0002:000066fc       ??_R2device_type_edit@@8   100196fc     device_type_edit.obj
 0002:00006718       ??_R1A@?0A@EA@device_type_edit@@8 10019718     device_type_edit.obj
 0002:00006734       ??_R4device_type_edit@@6BQPaintDevice@@@ 10019734     device_type_edit.obj
 0002:00006748       ??_R4?$QDict@VQAction@@@@6B@ 10019748     device_type_edit.obj
 0002:0000675c       ??_R3?$QDict@VQAction@@@@8 1001975c     device_type_edit.obj
 0002:0000676c       ??_R2?$QDict@VQAction@@@@8 1001976c     device_type_edit.obj
 0002:0000677c       ??_R1A@?0A@EA@?$QDict@VQAction@@@@8 1001977c     device_type_edit.obj
 0002:00006798       ??_R4QListViewItem@@6B@    10019798     device_type_editdlgimpl.obj
 0002:000067ac       ??_R3QListViewItem@@8      100197ac     device_type_editdlgimpl.obj
 0002:000067bc       ??_R2QListViewItem@@8      100197bc     device_type_editdlgimpl.obj
 0002:000067c8       ??_R1A@?0A@EA@QListViewItem@@8 100197c8     device_type_editdlgimpl.obj
 0002:000067e4       ??_R4QDomElement@@6B@      100197e4     device_type_editdlgimpl.obj
 0002:000067f8       ??_R3QDomElement@@8        100197f8     device_type_editdlgimpl.obj
 0002:00006808       ??_R2QDomElement@@8        10019808     device_type_editdlgimpl.obj
 0002:00006814       ??_R1A@?0A@EA@QDomElement@@8 10019814     device_type_editdlgimpl.obj
 0002:00006830       ??_R1A@?0A@EA@QDomNode@@8  10019830     device_type_editdlgimpl.obj
 0002:0000684c       ??_R3QDomNode@@8           1001984c     device_type_editdlgimpl.obj
 0002:0000685c       ??_R2QDomNode@@8           1001985c     device_type_editdlgimpl.obj
 0002:00006864       ??_R4QDomDocument@@6B@     10019864     device_type_editdlgimpl.obj
 0002:00006878       ??_R3QDomDocument@@8       10019878     device_type_editdlgimpl.obj
 0002:00006888       ??_R2QDomDocument@@8       10019888     device_type_editdlgimpl.obj
 0002:00006894       ??_R1A@?0A@EA@QDomDocument@@8 10019894     device_type_editdlgimpl.obj
 0002:000068b0       ??_R4device_type_editDlg@@6BQObject@@@ 100198b0     device_type_editdlgimpl.obj
 0002:000068c4       ??_R3device_type_editDlg@@8 100198c4     device_type_editdlgimpl.obj
 0002:000068d4       ??_R2device_type_editDlg@@8 100198d4     device_type_editdlgimpl.obj
 0002:000068f0       ??_R1A@?0A@EA@device_type_editDlg@@8 100198f0     device_type_editdlgimpl.obj
 0002:0000690c       ??_R1A@?0A@EA@device_type_editDlgBase@@8 1001990c     device_type_editdlgimpl.obj
 0002:00006928       ??_R3device_type_editDlgBase@@8 10019928     device_type_editdlgimpl.obj
 0002:00006938       ??_R2device_type_editDlgBase@@8 10019938     device_type_editdlgimpl.obj
 0002:00006950       ??_R4device_type_editDlg@@6BQPaintDevice@@@ 10019950     device_type_editdlgimpl.obj
 0002:00006964       ??_R4?$QPtrList@VQListViewItem@@@@6B@ 10019964     device_type_editdlgimpl.obj
 0002:00006978       ??_R3?$QPtrList@VQListViewItem@@@@8 10019978     device_type_editdlgimpl.obj
 0002:00006988       ??_R2?$QPtrList@VQListViewItem@@@@8 10019988     device_type_editdlgimpl.obj
 0002:00006998       ??_R1A@?0A@EA@?$QPtrList@VQListViewItem@@@@8 10019998     device_type_editdlgimpl.obj
 0002:000069b4       ??_R4paramLVI@@6B@         100199b4     paramLVI.obj
 0002:000069c8       ??_R3paramLVI@@8           100199c8     paramLVI.obj
 0002:000069d8       ??_R2paramLVI@@8           100199d8     paramLVI.obj
 0002:000069e8       ??_R1A@?0A@EA@paramLVI@@8  100199e8     paramLVI.obj
 0002:00006a04       ??_R4config_plugin_desc_base@@6B@ 10019a04     plugindesc.obj
 0002:00006a18       ??_R3config_plugin_desc_base@@8 10019a18     plugindesc.obj
 0002:00006a28       ??_R2config_plugin_desc_base@@8 10019a28     plugindesc.obj
 0002:00006a30       ??_R1A@?0A@EA@config_plugin_desc_base@@8 10019a30     plugindesc.obj
 0002:00006a4c       ??_R4plugindesc@@6B@       10019a4c     plugindesc.obj
 0002:00006a60       ??_R3plugindesc@@8         10019a60     plugindesc.obj
 0002:00006a70       ??_R2plugindesc@@8         10019a70     plugindesc.obj
 0002:00006a7c       ??_R1A@?0A@EA@plugindesc@@8 10019a7c     plugindesc.obj
 0002:00006a98       ??_R4toolWindow@@6BQObject@@@ 10019a98     toolwindowimpl.obj
 0002:00006aac       ??_R3toolWindow@@8         10019aac     toolwindowimpl.obj
 0002:00006abc       ??_R2toolWindow@@8         10019abc     toolwindowimpl.obj
 0002:00006ad8       ??_R1A@?0A@EA@toolWindow@@8 10019ad8     toolwindowimpl.obj
 0002:00006af4       ??_R1A@?0A@EA@toolWindowBase@@8 10019af4     toolwindowimpl.obj
 0002:00006b10       ??_R3toolWindowBase@@8     10019b10     toolwindowimpl.obj
 0002:00006b20       ??_R2toolWindowBase@@8     10019b20     toolwindowimpl.obj
 0002:00006b38       ??_R4toolWindow@@6BQPaintDevice@@@ 10019b38     toolwindowimpl.obj
 0002:00006b4c       ??_R4QWidget@@6BQObject@@@ 10019b4c     device_type_editdlg.obj
 0002:00006b60       ??_R4QWidget@@6BQPaintDevice@@@ 10019b60     device_type_editdlg.obj
 0002:00006b74       ??_R4QVBoxLayout@@6BQObject@@@ 10019b74     device_type_editdlg.obj
 0002:00006b88       ??_R3QVBoxLayout@@8        10019b88     device_type_editdlg.obj
 0002:00006b98       ??_R2QVBoxLayout@@8        10019b98     device_type_editdlg.obj
 0002:00006bb4       ??_R1A@?0A@EA@QVBoxLayout@@8 10019bb4     device_type_editdlg.obj
 0002:00006bd0       ??_R1A@?0A@EA@QBoxLayout@@8 10019bd0     device_type_editdlg.obj
 0002:00006bec       ??_R3QBoxLayout@@8         10019bec     device_type_editdlg.obj
 0002:00006bfc       ??_R2QBoxLayout@@8         10019bfc     device_type_editdlg.obj
 0002:00006c14       ??_R1A@?0A@EA@QLayout@@8   10019c14     device_type_editdlg.obj
 0002:00006c30       ??_R3QLayout@@8            10019c30     device_type_editdlg.obj
 0002:00006c40       ??_R2QLayout@@8            10019c40     device_type_editdlg.obj
 0002:00006c54       ??_R1CI@?0A@EA@QLayoutItem@@8 10019c54     device_type_editdlg.obj
 0002:00006c70       ??_R3QLayoutItem@@8        10019c70     device_type_editdlg.obj
 0002:00006c80       ??_R2QLayoutItem@@8        10019c80     device_type_editdlg.obj
 0002:00006c88       ??_R1A@?0A@EA@QLayoutItem@@8 10019c88     device_type_editdlg.obj
 0002:00006ca4       ??_R4QVBoxLayout@@6BQLayoutItem@@@ 10019ca4     device_type_editdlg.obj
 0002:00006cb8       ??_R4QHBoxLayout@@6BQObject@@@ 10019cb8     device_type_editdlg.obj
 0002:00006ccc       ??_R3QHBoxLayout@@8        10019ccc     device_type_editdlg.obj
 0002:00006cdc       ??_R2QHBoxLayout@@8        10019cdc     device_type_editdlg.obj
 0002:00006cf8       ??_R1A@?0A@EA@QHBoxLayout@@8 10019cf8     device_type_editdlg.obj
 0002:00006d14       ??_R4QHBoxLayout@@6BQLayoutItem@@@ 10019d14     device_type_editdlg.obj
 0002:00006d28       ??_R4QGridLayout@@6BQObject@@@ 10019d28     device_type_editdlg.obj
 0002:00006d3c       ??_R3QGridLayout@@8        10019d3c     device_type_editdlg.obj
 0002:00006d4c       ??_R2QGridLayout@@8        10019d4c     device_type_editdlg.obj
 0002:00006d64       ??_R1A@?0A@EA@QGridLayout@@8 10019d64     device_type_editdlg.obj
 0002:00006d80       ??_R4QGridLayout@@6BQLayoutItem@@@ 10019d80     device_type_editdlg.obj
 0002:00006d94       ??_R4QLabel@@6BQObject@@@  10019d94     device_type_editdlg.obj
 0002:00006da8       ??_R3QLabel@@8             10019da8     device_type_editdlg.obj
 0002:00006db8       ??_R2QLabel@@8             10019db8     device_type_editdlg.obj
 0002:00006dd4       ??_R1A@?0A@EA@QLabel@@8    10019dd4     device_type_editdlg.obj
 0002:00006df0       ??_R4QLabel@@6BQPaintDevice@@@ 10019df0     device_type_editdlg.obj
 0002:00006e04       ??_R4QComboBox@@6BQObject@@@ 10019e04     device_type_editdlg.obj
 0002:00006e18       ??_R3QComboBox@@8          10019e18     device_type_editdlg.obj
 0002:00006e28       ??_R2QComboBox@@8          10019e28     device_type_editdlg.obj
 0002:00006e40       ??_R1A@?0A@EA@QComboBox@@8 10019e40     device_type_editdlg.obj
 0002:00006e5c       ??_R4QComboBox@@6BQPaintDevice@@@ 10019e5c     device_type_editdlg.obj
 0002:00006e70       ??_R4QListView@@6BQObject@@@ 10019e70     device_type_editdlg.obj
 0002:00006e84       ??_R3QListView@@8          10019e84     device_type_editdlg.obj
 0002:00006e94       ??_R2QListView@@8          10019e94     device_type_editdlg.obj
 0002:00006eb4       ??_R1A@?0A@EA@QListView@@8 10019eb4     device_type_editdlg.obj
 0002:00006ed0       ??_R1A@?0A@EA@QScrollView@@8 10019ed0     device_type_editdlg.obj
 0002:00006eec       ??_R3QScrollView@@8        10019eec     device_type_editdlg.obj
 0002:00006efc       ??_R2QScrollView@@8        10019efc     device_type_editdlg.obj
 0002:00006f18       ??_R4QListView@@6BQPaintDevice@@@ 10019f18     device_type_editdlg.obj
 0002:00006f2c       ??_R4QPushButton@@6BQObject@@@ 10019f2c     device_type_editdlg.obj
 0002:00006f40       ??_R3QPushButton@@8        10019f40     device_type_editdlg.obj
 0002:00006f50       ??_R2QPushButton@@8        10019f50     device_type_editdlg.obj
 0002:00006f6c       ??_R1A@?0A@EA@QPushButton@@8 10019f6c     device_type_editdlg.obj
 0002:00006f88       ??_R1A@?0A@EA@QButton@@8   10019f88     device_type_editdlg.obj
 0002:00006fa4       ??_R3QButton@@8            10019fa4     device_type_editdlg.obj
 0002:00006fb4       ??_R2QButton@@8            10019fb4     device_type_editdlg.obj
 0002:00006fcc       ??_R4QPushButton@@6BQPaintDevice@@@ 10019fcc     device_type_editdlg.obj
 0002:00006fe0       ??_R4QGroupBox@@6BQObject@@@ 10019fe0     device_type_editdlg.obj
 0002:00006ff4       ??_R3QGroupBox@@8          10019ff4     device_type_editdlg.obj
 0002:00007004       ??_R2QGroupBox@@8          1001a004     device_type_editdlg.obj
 0002:00007020       ??_R1A@?0A@EA@QGroupBox@@8 1001a020     device_type_editdlg.obj
 0002:0000703c       ??_R4QGroupBox@@6BQPaintDevice@@@ 1001a03c     device_type_editdlg.obj
 0002:00007050       ??_R4QSpinBox@@6BQObject@@@ 1001a050     device_type_editdlg.obj
 0002:00007064       ??_R3QSpinBox@@8           1001a064     device_type_editdlg.obj
 0002:00007074       ??_R2QSpinBox@@8           1001a074     device_type_editdlg.obj
 0002:00007090       ??_R1A@?0A@EA@QSpinBox@@8  1001a090     device_type_editdlg.obj
 0002:000070ac       ??_R1GM@?0A@EA@QRangeControl@@8 1001a0ac     device_type_editdlg.obj
 0002:000070c8       ??_R3QRangeControl@@8      1001a0c8     device_type_editdlg.obj
 0002:000070d8       ??_R2QRangeControl@@8      1001a0d8     device_type_editdlg.obj
 0002:000070e0       ??_R1A@?0A@EA@QRangeControl@@8 1001a0e0     device_type_editdlg.obj
 0002:000070fc       ??_R4QSpinBox@@6BQPaintDevice@@@ 1001a0fc     device_type_editdlg.obj
 0002:00007110       ??_R4QSpinBox@@6B@         1001a110     device_type_editdlg.obj
 0002:00007124       ??_R4QLineEdit@@6BQObject@@@ 1001a124     device_type_editdlg.obj
 0002:00007138       ??_R3QLineEdit@@8          1001a138     device_type_editdlg.obj
 0002:00007148       ??_R2QLineEdit@@8          1001a148     device_type_editdlg.obj
 0002:00007164       ??_R1A@?0A@EA@QLineEdit@@8 1001a164     device_type_editdlg.obj
 0002:00007180       ??_R4QLineEdit@@6BQPaintDevice@@@ 1001a180     device_type_editdlg.obj
 0002:00007194       ??_R4QWidgetStack@@6BQObject@@@ 1001a194     device_type_editdlg.obj
 0002:000071a8       ??_R3QWidgetStack@@8       1001a1a8     device_type_editdlg.obj
 0002:000071b8       ??_R2QWidgetStack@@8       1001a1b8     device_type_editdlg.obj
 0002:000071d4       ??_R1A@?0A@EA@QWidgetStack@@8 1001a1d4     device_type_editdlg.obj
 0002:000071f0       ??_R4QWidgetStack@@6BQPaintDevice@@@ 1001a1f0     device_type_editdlg.obj
 0002:00007204       ??_R4QCheckBox@@6BQObject@@@ 1001a204     device_type_editdlg.obj
 0002:00007218       ??_R3QCheckBox@@8          1001a218     device_type_editdlg.obj
 0002:00007228       ??_R2QCheckBox@@8          1001a228     device_type_editdlg.obj
 0002:00007244       ??_R1A@?0A@EA@QCheckBox@@8 1001a244     device_type_editdlg.obj
 0002:00007260       ??_R4QCheckBox@@6BQPaintDevice@@@ 1001a260     device_type_editdlg.obj
 0002:00007274       ??_R4device_type_editDlgBase@@6BQObject@@@ 1001a274     device_type_editdlg.obj
 0002:00007288       ??_R4device_type_editDlgBase@@6BQPaintDevice@@@ 1001a288     device_type_editdlg.obj
 0002:0000729c       ??_R4QSpacerItem@@6B@      1001a29c     device_type_editdlg.obj
 0002:000072b0       ??_R3QSpacerItem@@8        1001a2b0     device_type_editdlg.obj
 0002:000072c0       ??_R2QSpacerItem@@8        1001a2c0     device_type_editdlg.obj
 0002:000072cc       ??_R1A@?0A@EA@QSpacerItem@@8 1001a2cc     device_type_editdlg.obj
 0002:000072e8       ??_R4QTabWidget@@6BQObject@@@ 1001a2e8     toolwindow.obj
 0002:000072fc       ??_R3QTabWidget@@8         1001a2fc     toolwindow.obj
 0002:0000730c       ??_R2QTabWidget@@8         1001a30c     toolwindow.obj
 0002:00007324       ??_R1A@?0A@EA@QTabWidget@@8 1001a324     toolwindow.obj
 0002:00007340       ??_R4QTabWidget@@6BQPaintDevice@@@ 1001a340     toolwindow.obj
 0002:00007354       ??_R4toolWindowBase@@6BQObject@@@ 1001a354     toolwindow.obj
 0002:00007368       ??_R4toolWindowBase@@6BQPaintDevice@@@ 1001a368     toolwindow.obj
 0002:0000737c       ??_R4cfg_ListView@@6BQObject@@@ 1001a37c     cfg_widgets001:cfg_ListView.obj
 0002:00007390       ??_R3cfg_ListView@@8       1001a390     cfg_widgets001:cfg_ListView.obj
 0002:000073a0       ??_R2cfg_ListView@@8       1001a3a0     cfg_widgets001:cfg_ListView.obj
 0002:000073c4       ??_R1A@?0A@EA@cfg_ListView@@8 1001a3c4     cfg_widgets001:cfg_ListView.obj
 0002:000073e0       ??_R4cfg_ListView@@6BQPaintDevice@@@ 1001a3e0     cfg_widgets001:cfg_ListView.obj
 0002:000073f4       ??_R4type_info@@6B@        1001a3f4     MSVCRT:ti_inst.obj
 0002:00007408       ??_R3type_info@@8          1001a408     MSVCRT:ti_inst.obj
 0002:00007418       ??_R2type_info@@8          1001a418     MSVCRT:ti_inst.obj
 0002:00007420       ??_R1A@?0A@EA@type_info@@8 1001a420     MSVCRT:ti_inst.obj
 0002:0000743c       ___rtc_iaa                 1001a43c     MSVCRT:initsect.obj
 0002:00007440       ___rtc_izz                 1001a440     MSVCRT:initsect.obj
 0002:00007444       ___rtc_taa                 1001a444     MSVCRT:initsect.obj
 0002:00007448       ___rtc_tzz                 1001a448     MSVCRT:initsect.obj
 0002:0000a1ac       __IMPORT_DESCRIPTOR_config_icons 1001d1ac     config_icons:config_icons.dll
 0002:0000a1c0       __IMPORT_DESCRIPTOR_qt-mt323 1001d1c0     qt-mt323:qt-mt323.dll
 0002:0000a1d4       __IMPORT_DESCRIPTOR_MSVCR120 1001d1d4     MSVCRT:MSVCR120.dll
 0002:0000a1e8       __IMPORT_DESCRIPTOR_KERNEL32 1001d1e8     kernel32:KERNEL32.dll
 0002:0000a1fc       __NULL_IMPORT_DESCRIPTOR   1001d1fc     config_icons:config_icons.dll
 0003:000000b0       ___security_cookie         100290b0     MSVCRT:gs_cookie.obj
 0003:000000b4       ___security_cookie_complement 100290b4     MSVCRT:gs_cookie.obj
 0003:000000c0       ___native_dllmain_reason   100290c0     MSVCRT:natstart.obj
 0003:000000c4       ??_R0?AUQShared@@@8        100290c4     device_type_edit.obj
 0003:000000dc       ??_R0?AVQGList@@@8         100290dc     device_type_edit.obj
 0003:000000f4       ??_R0?AVQPtrCollection@@@8 100290f4     device_type_edit.obj
 0003:00000114       ??_R0?AVQToolBar@@@8       10029114     device_type_edit.obj
 0003:0000012c       ??_R0?AVQDockWindow@@@8    1002912c     device_type_edit.obj
 0003:00000148       ??_R0?AVQFrame@@@8         10029148     device_type_edit.obj
 0003:00000160       ??_R0?AVQWidget@@@8        10029160     device_type_edit.obj
 0003:00000178       ??_R0?AVQObject@@@8        10029178     device_type_edit.obj
 0003:00000190       ??_R0?AVQt@@@8             10029190     device_type_edit.obj
 0003:000001a4       ??_R0?AVQPaintDevice@@@8   100291a4     device_type_edit.obj
 0003:000001c0       ??_R0?AVQPopupMenu@@@8     100291c0     device_type_edit.obj
 0003:000001dc       ??_R0?AVQMenuData@@@8      100291dc     device_type_edit.obj
 0003:000001f4       ??_R0?AVQAction@@@8        100291f4     device_type_edit.obj
 0003:0000020c       ??_R0?AVQGuardedPtrPrivate@@@8 1002920c     device_type_edit.obj
 0003:00000230       ??_R0?AVQDockWindowList@@@8 10029230     device_type_edit.obj
 0003:00000250       ??_R0?AV?$QPtrList@VQDockWindow@@@@@8 10029250     device_type_edit.obj
 0003:00000278       ??_R0?AVQPopupMenuList@@@8 10029278     device_type_edit.obj
 0003:00000298       ??_R0?AV?$QPtrList@VQPopupMenu@@@@@8 10029298     device_type_edit.obj
 0003:000002c0       ??_R0?AVconfig_plugin_base@@@8 100292c0     device_type_edit.obj
 0003:000002e4       ??_R0?AVQGDict@@@8         100292e4     device_type_edit.obj
 0003:000002fc       ??_R0?AVdevice_type_edit@@@8 100292fc     device_type_edit.obj
 0003:0000031c       ??_R0?AV?$QDict@VQAction@@@@@8 1002931c     device_type_edit.obj
 0003:00000340       ??_R0?AVQListViewItem@@@8  10029340     device_type_editdlgimpl.obj
 0003:0000035c       ??_R0?AVQDomElement@@@8    1002935c     device_type_editdlgimpl.obj
 0003:00000378       ??_R0?AVQDomNode@@@8       10029378     device_type_editdlgimpl.obj
 0003:00000390       ??_R0?AVQDomDocument@@@8   10029390     device_type_editdlgimpl.obj
 0003:000003ac       ??_R0?AVdevice_type_editDlg@@@8 100293ac     device_type_editdlgimpl.obj
 0003:000003d0       ??_R0?AVdevice_type_editDlgBase@@@8 100293d0     device_type_editdlgimpl.obj
 0003:000003f8       ??_R0?AV?$QPtrList@VQListViewItem@@@@@8 100293f8     device_type_editdlgimpl.obj
 0003:00000424       ??_R0?AVparamLVI@@@8       10029424     paramLVI.obj
 0003:0000043c       ??_R0?AVconfig_plugin_desc_base@@@8 1002943c     plugindesc.obj
 0003:00000464       ??_R0?AVplugindesc@@@8     10029464     plugindesc.obj
 0003:00000480       ??_R0?AVtoolWindow@@@8     10029480     toolwindowimpl.obj
 0003:0000049c       ??_R0?AVtoolWindowBase@@@8 1002949c     toolwindowimpl.obj
 0003:000004bc       ??_R0?AVQVBoxLayout@@@8    100294bc     device_type_editdlg.obj
 0003:000004d8       ??_R0?AVQBoxLayout@@@8     100294d8     device_type_editdlg.obj
 0003:000004f4       ??_R0?AVQLayout@@@8        100294f4     device_type_editdlg.obj
 0003:0000050c       ??_R0?AVQLayoutItem@@@8    1002950c     device_type_editdlg.obj
 0003:00000528       ??_R0?AVQHBoxLayout@@@8    10029528     device_type_editdlg.obj
 0003:00000544       ??_R0?AVQGridLayout@@@8    10029544     device_type_editdlg.obj
 0003:00000560       ??_R0?AVQLabel@@@8         10029560     device_type_editdlg.obj
 0003:00000578       ??_R0?AVQComboBox@@@8      10029578     device_type_editdlg.obj
 0003:00000590       ??_R0?AVQListView@@@8      10029590     device_type_editdlg.obj
 0003:000005a8       ??_R0?AVQScrollView@@@8    100295a8     device_type_editdlg.obj
 0003:000005c4       ??_R0?AVQPushButton@@@8    100295c4     device_type_editdlg.obj
 0003:000005e0       ??_R0?AVQButton@@@8        100295e0     device_type_editdlg.obj
 0003:000005f8       ??_R0?AVQGroupBox@@@8      100295f8     device_type_editdlg.obj
 0003:00000610       ??_R0?AVQSpinBox@@@8       10029610     device_type_editdlg.obj
 0003:00000628       ??_R0?AVQRangeControl@@@8  10029628     device_type_editdlg.obj
 0003:00000644       ??_R0?AVQLineEdit@@@8      10029644     device_type_editdlg.obj
 0003:0000065c       ??_R0?AVQWidgetStack@@@8   1002965c     device_type_editdlg.obj
 0003:00000678       ??_R0?AVQCheckBox@@@8      10029678     device_type_editdlg.obj
 0003:00000690       ??_R0?AVQSpacerItem@@@8    10029690     device_type_editdlg.obj
 0003:000006ac       ??_R0?AVQTabWidget@@@8     100296ac     toolwindow.obj
 0003:000006c8       ??_R0?AVcfg_ListView@@@8   100296c8     cfg_widgets001:cfg_ListView.obj
 0003:000006e4       ??_R0?AVtype_info@@@8      100296e4     MSVCRT:ti_inst.obj
 0003:00000700       ?metaObj@device_type_edit@@0PAVQMetaObject@@A 10029700     moc_device_type_edit.obj
 0003:0000074c       ?metaObj@device_type_editDlgBase@@0PAVQMetaObject@@A 1002974c     moc_device_type_editdlg.obj
 0003:00000754       ?metaObj@device_type_editDlg@@0PAVQMetaObject@@A 10029754     moc_device_type_editdlgimpl.obj
 0003:000007c0       ?metaObj@toolWindowBase@@0PAVQMetaObject@@A 100297c0     moc_toolwindow.obj
 0003:000007c8       ?metaObj@toolWindow@@0PAVQMetaObject@@A 100297c8     moc_toolwindowimpl.obj
 0003:00000804       ?metaObj@cfg_ListView@@0PAVQMetaObject@@A 10029804     cfg_widgets001:moc_cfg_ListView.obj
 0003:00000b48       ?__type_info_root_node@@3U__type_info_node@@A 10029b48     MSVCRT:tncleanup.obj
 0003:00000b50       ___native_startup_lock     10029b50     <common>
 0003:00000b54       ___native_startup_state    10029b54     <common>
 0003:00000b58       ___dyn_tls_init_callback   10029b58     <common>
 0003:00000b5c       ___onexitend               10029b5c     <common>
 0003:00000b60       ___onexitbegin             10029b60     <common>

 entry point at        0001:0000e8d2

 Static symbols

 0001:00000000       ??__EcleanUp_device_type_edit@@YAXXZ 10001000 f   moc_device_type_edit.obj
 0001:00000021       ??__EcleanUp_device_type_editDlgBase@@YAXXZ 10001021 f   moc_device_type_editdlg.obj
 0001:00000042       ??__EcleanUp_device_type_editDlg@@YAXXZ 10001042 f   moc_device_type_editdlgimpl.obj
 0001:00000063       ??__EcleanUp_toolWindowBase@@YAXXZ 10001063 f   moc_toolwindow.obj
 0001:00000084       ??__EcleanUp_toolWindow@@YAXXZ 10001084 f   moc_toolwindowimpl.obj
 0001:000000a5       ??__EcleanUp_cfg_ListView@@YAXXZ 100010a5 f   cfg_widgets001:moc_cfg_ListView.obj
 0001:0000b985       $LN45                      1000c985     moc_device_type_editdlgimpl.obj
 0001:0000e68f       _pre_c_init                1000f68f f   MSVCRT:crtdll.obj
 0001:0000e8f5       ___DllMainCRTStartup       1000f8f5 f   MSVCRT:crtdll.obj
 0001:0000eb70       $$000000                   1000fb70     MSVCRT:sehprolg4.obj
 0001:0000ee8c       __unwindfunclet$??0config_plugin_base@@QAE@ABVQString@@00@Z$0 1000fe8c f   device_type_edit.obj
 0001:0000ee95       __unwindfunclet$??0config_plugin_base@@QAE@ABVQString@@00@Z$1 1000fe95 f   device_type_edit.obj
 0001:0000eea1       __unwindfunclet$??0config_plugin_base@@QAE@ABVQString@@00@Z$2 1000fea1 f   device_type_edit.obj
 0001:0000eead       __unwindfunclet$??0config_plugin_base@@QAE@ABVQString@@00@Z$3 1000fead f   device_type_edit.obj
 0001:0000eeb9       __ehhandler$??0config_plugin_base@@QAE@ABVQString@@00@Z 1000feb9 f   device_type_edit.obj
 0001:0000eed4       __unwindfunclet$??0device_type_edit@@QAE@ABVQString@@00@Z$0 1000fed4 f   device_type_edit.obj
 0001:0000eedc       __unwindfunclet$??0device_type_edit@@QAE@ABVQString@@00@Z$1 1000fedc f   device_type_edit.obj
 0001:0000eee7       __unwindfunclet$??0device_type_edit@@QAE@ABVQString@@00@Z$2 1000fee7 f   device_type_edit.obj
 0001:0000eef2       __unwindfunclet$??0device_type_edit@@QAE@ABVQString@@00@Z$3 1000fef2 f   device_type_edit.obj
 0001:0000ef00       __unwindfunclet$??0device_type_edit@@QAE@ABVQString@@00@Z$4 1000ff00 f   device_type_edit.obj
 0001:0000ef0e       __unwindfunclet$??0device_type_edit@@QAE@ABVQString@@00@Z$5 1000ff0e f   device_type_edit.obj
 0001:0000ef1c       __unwindfunclet$??0device_type_edit@@QAE@ABVQString@@00@Z$6 1000ff1c f   device_type_edit.obj
 0001:0000ef2b       __unwindfunclet$??0device_type_edit@@QAE@ABVQString@@00@Z$7 1000ff2b f   device_type_edit.obj
 0001:0000ef3a       __unwindfunclet$??0device_type_edit@@QAE@ABVQString@@00@Z$8 1000ff3a f   device_type_edit.obj
 0001:0000ef49       __unwindfunclet$??0device_type_edit@@QAE@ABVQString@@00@Z$9 1000ff49 f   device_type_edit.obj
 0001:0000ef53       __unwindfunclet$??0device_type_edit@@QAE@ABVQString@@00@Z$10 1000ff53 f   device_type_edit.obj
 0001:0000ef5d       __unwindfunclet$??0device_type_edit@@QAE@ABVQString@@00@Z$11 1000ff5d f   device_type_edit.obj
 0001:0000ef77       __unwindfunclet$??0device_type_edit@@QAE@ABVQString@@00@Z$12 1000ff77 f   device_type_edit.obj
 0001:0000ef80       __unwindfunclet$??0device_type_edit@@QAE@ABVQString@@00@Z$13 1000ff80 f   device_type_edit.obj
 0001:0000ef8a       __unwindfunclet$??0device_type_edit@@QAE@ABVQString@@00@Z$14 1000ff8a f   device_type_edit.obj
 0001:0000ef94       __unwindfunclet$??0device_type_edit@@QAE@ABVQString@@00@Z$15 1000ff94 f   device_type_edit.obj
 0001:0000efae       __unwindfunclet$??0device_type_edit@@QAE@ABVQString@@00@Z$16 1000ffae f   device_type_edit.obj
 0001:0000efb8       __unwindfunclet$??0device_type_edit@@QAE@ABVQString@@00@Z$17 1000ffb8 f   device_type_edit.obj
 0001:0000efc2       __unwindfunclet$??0device_type_edit@@QAE@ABVQString@@00@Z$18 1000ffc2 f   device_type_edit.obj
 0001:0000efdc       __unwindfunclet$??0device_type_edit@@QAE@ABVQString@@00@Z$19 1000ffdc f   device_type_edit.obj
 0001:0000eff6       __unwindfunclet$??0device_type_edit@@QAE@ABVQString@@00@Z$20 1000fff6 f   device_type_edit.obj
 0001:0000f010       __unwindfunclet$??0device_type_edit@@QAE@ABVQString@@00@Z$21 10010010 f   device_type_edit.obj
 0001:0000f02a       __unwindfunclet$??0device_type_edit@@QAE@ABVQString@@00@Z$23 1001002a f   device_type_edit.obj
 0001:0000f033       __unwindfunclet$??0device_type_edit@@QAE@ABVQString@@00@Z$24 10010033 f   device_type_edit.obj
 0001:0000f03c       __unwindfunclet$??0device_type_edit@@QAE@ABVQString@@00@Z$25 1001003c f   device_type_edit.obj
 0001:0000f045       __unwindfunclet$??0device_type_edit@@QAE@ABVQString@@00@Z$26 10010045 f   device_type_edit.obj
 0001:0000f04e       __ehhandler$??0device_type_edit@@QAE@ABVQString@@00@Z 1001004e f   device_type_edit.obj
 0001:0000f069       __unwindfunclet$??1?$QDict@VQAction@@@@UAE@XZ$0 10010069 f   device_type_edit.obj
 0001:0000f072       __ehhandler$??1?$QDict@VQAction@@@@UAE@XZ 10010072 f   device_type_edit.obj
 0001:0000f08d       __unwindfunclet$??1QDockWindowList@@UAE@XZ$0 1001008d f   device_type_edit.obj
 0001:0000f096       __unwindfunclet$??1QDockWindowList@@UAE@XZ$1 10010096 f   device_type_edit.obj
 0001:0000f09f       __ehhandler$??1QDockWindowList@@UAE@XZ 1001009f f   device_type_edit.obj
 0001:0000f0ba       __unwindfunclet$??1QPopupMenuList@@UAE@XZ$0 100100ba f   device_type_edit.obj
 0001:0000f0c2       __ehhandler$??1QPopupMenuList@@UAE@XZ 100100c2 f   device_type_edit.obj
 0001:0000f0dd       __unwindfunclet$??1config_plugin_base@@UAE@XZ$0 100100dd f   device_type_edit.obj
 0001:0000f0e6       __unwindfunclet$??1config_plugin_base@@UAE@XZ$1 100100e6 f   device_type_edit.obj
 0001:0000f0f2       __unwindfunclet$??1config_plugin_base@@UAE@XZ$2 100100f2 f   device_type_edit.obj
 0001:0000f0fe       __ehhandler$??1config_plugin_base@@UAE@XZ 100100fe f   device_type_edit.obj
 0001:0000f119       __unwindfunclet$??1device_type_edit@@UAE@XZ$0 10010119 f   device_type_edit.obj
 0001:0000f121       __unwindfunclet$??1device_type_edit@@UAE@XZ$1 10010121 f   device_type_edit.obj
 0001:0000f12c       __unwindfunclet$??1device_type_edit@@UAE@XZ$2 1001012c f   device_type_edit.obj
 0001:0000f137       __unwindfunclet$??1device_type_edit@@UAE@XZ$3 10010137 f   device_type_edit.obj
 0001:0000f145       __unwindfunclet$??1device_type_edit@@UAE@XZ$4 10010145 f   device_type_edit.obj
 0001:0000f153       __unwindfunclet$??1device_type_edit@@UAE@XZ$5 10010153 f   device_type_edit.obj
 0001:0000f161       __unwindfunclet$??1device_type_edit@@UAE@XZ$6 10010161 f   device_type_edit.obj
 0001:0000f170       __unwindfunclet$??1device_type_edit@@UAE@XZ$7 10010170 f   device_type_edit.obj
 0001:0000f17f       __unwindfunclet$??1device_type_edit@@UAE@XZ$8 1001017f f   device_type_edit.obj
 0001:0000f18e       __ehhandler$??1device_type_edit@@UAE@XZ 1001018e f   device_type_edit.obj
 0001:0000f1a9       __unwindfunclet$??0?$QGuardedPtr@VQPopupMenu@@@@QAE@XZ$0 100101a9 f   device_type_edit.obj
 0001:0000f1a9       __unwindfunclet$??4?$QGuardedPtr@VQPopupMenu@@@@QAEAAV0@PAVQPopupMenu@@@Z$0 100101a9 f   device_type_edit.obj
 0001:0000f1a9       __unwindfunclet$?create@plugindesc@@UAEPAVconfig_plugin_base@@ABVQString@@00@Z$0 100101a9 f   device_type_edit.obj
 0001:0000f1a9       __unwindfunclet$??0?$QGuardedPtr@VQDockWindow@@@@QAE@XZ$0 100101a9 f   device_type_edit.obj
 0001:0000f1a9       __unwindfunclet$??4?$QGuardedPtr@VtoolWindow@@@@QAEAAV0@PAVtoolWindow@@@Z$0 100101a9 f   device_type_edit.obj
 0001:0000f1a9       __unwindfunclet$??4?$QGuardedPtr@VQDockWindow@@@@QAEAAV0@PAVQDockWindow@@@Z$0 100101a9 f   device_type_edit.obj
 0001:0000f1a9       __unwindfunclet$?newItem@cfg_ListView@@MAEPAVQListViewItem@@PAVQListView@@PAV2@@Z$0 100101a9 f   device_type_edit.obj
 0001:0000f1a9       __unwindfunclet$??0?$QGuardedPtr@VtoolWindow@@@@QAE@XZ$0 100101a9 f   device_type_edit.obj
 0001:0000f1b3       __ehhandler$?create@plugindesc@@UAEPAVconfig_plugin_base@@ABVQString@@00@Z 100101b3 f   device_type_edit.obj
 0001:0000f1b3       __ehhandler$??0?$QGuardedPtr@VQPopupMenu@@@@QAE@XZ 100101b3 f   device_type_edit.obj
 0001:0000f1b3       __ehhandler$??4?$QGuardedPtr@VQPopupMenu@@@@QAEAAV0@PAVQPopupMenu@@@Z 100101b3 f   device_type_edit.obj
 0001:0000f1b3       __ehhandler$??0?$QGuardedPtr@VQDockWindow@@@@QAE@XZ 100101b3 f   device_type_edit.obj
 0001:0000f1b3       __ehhandler$??4?$QGuardedPtr@VQDockWindow@@@@QAEAAV0@PAVQDockWindow@@@Z 100101b3 f   device_type_edit.obj
 0001:0000f1b3       __ehhandler$??0?$QGuardedPtr@VtoolWindow@@@@QAE@XZ 100101b3 f   device_type_edit.obj
 0001:0000f1b3       __ehhandler$?newItem@cfg_ListView@@MAEPAVQListViewItem@@PAVQListView@@PAV2@@Z 100101b3 f   device_type_edit.obj
 0001:0000f1b3       __ehhandler$??4?$QGuardedPtr@VtoolWindow@@@@QAEAAV0@PAVtoolWindow@@@Z 100101b3 f   device_type_edit.obj
 0001:0000f1ce       __unwindfunclet$?about@config_plugin_base@@UAE?AVQString@@XZ$0 100101ce f   device_type_edit.obj
 0001:0000f1d7       __unwindfunclet$?about@config_plugin_base@@UAE?AVQString@@XZ$1 100101d7 f   device_type_edit.obj
 0001:0000f1f1       __ehhandler$?about@config_plugin_base@@UAE?AVQString@@XZ 100101f1 f   device_type_edit.obj
 0001:0000f20c       __unwindfunclet$?about@device_type_edit@@UAE?AVQString@@XZ$0 1001020c f   device_type_edit.obj
 0001:0000f215       __unwindfunclet$?about@device_type_edit@@UAE?AVQString@@XZ$1 10010215 f   device_type_edit.obj
 0001:0000f21e       __unwindfunclet$?about@device_type_edit@@UAE?AVQString@@XZ$2 1001021e f   device_type_edit.obj
 0001:0000f227       __unwindfunclet$?about@device_type_edit@@UAE?AVQString@@XZ$3 10010227 f   device_type_edit.obj
 0001:0000f230       __unwindfunclet$?about@device_type_edit@@UAE?AVQString@@XZ$4 10010230 f   device_type_edit.obj
 0001:0000f24a       __ehhandler$?about@device_type_edit@@UAE?AVQString@@XZ 1001024a f   device_type_edit.obj
 0001:0000f265       __unwindfunclet$?activate@device_type_edit@@UAEX_N@Z$0 10010265 f   device_type_edit.obj
 0001:0000f26e       __unwindfunclet$?activate@device_type_edit@@UAEX_N@Z$2 1001026e f   device_type_edit.obj
 0001:0000f288       __unwindfunclet$?activate@device_type_edit@@UAEX_N@Z$3 10010288 f   device_type_edit.obj
 0001:0000f2a2       __unwindfunclet$?activate@device_type_edit@@UAEX_N@Z$4 100102a2 f   device_type_edit.obj
 0001:0000f2bc       __unwindfunclet$?activate@device_type_edit@@UAEX_N@Z$5 100102bc f   device_type_edit.obj
 0001:0000f2c5       __unwindfunclet$?activate@device_type_edit@@UAEX_N@Z$7 100102c5 f   device_type_edit.obj
 0001:0000f2ce       __unwindfunclet$?activate@device_type_edit@@UAEX_N@Z$8 100102ce f   device_type_edit.obj
 0001:0000f2d7       __unwindfunclet$?activate@device_type_edit@@UAEX_N@Z$9 100102d7 f   device_type_edit.obj
 0001:0000f2e0       __unwindfunclet$?activate@device_type_edit@@UAEX_N@Z$10 100102e0 f   device_type_edit.obj
 0001:0000f2e9       __ehhandler$?activate@device_type_edit@@UAEX_N@Z 100102e9 f   device_type_edit.obj
 0001:0000f304       __unwindfunclet$?apply@device_type_edit@@UAEXXZ$0 10010304 f   device_type_edit.obj
 0001:0000f30d       __unwindfunclet$?apply@device_type_edit@@UAEXXZ$2 1001030d f   device_type_edit.obj
 0001:0000f316       __unwindfunclet$?apply@device_type_edit@@UAEXXZ$4 10010316 f   device_type_edit.obj
 0001:0000f31f       __unwindfunclet$?apply@device_type_edit@@UAEXXZ$5 1001031f f   device_type_edit.obj
 0001:0000f328       __unwindfunclet$?apply@device_type_edit@@UAEXXZ$6 10010328 f   device_type_edit.obj
 0001:0000f331       __unwindfunclet$?apply@device_type_edit@@UAEXXZ$7 10010331 f   device_type_edit.obj
 0001:0000f33a       __unwindfunclet$?apply@device_type_edit@@UAEXXZ$8 1001033a f   device_type_edit.obj
 0001:0000f343       __unwindfunclet$?apply@device_type_edit@@UAEXXZ$9 10010343 f   device_type_edit.obj
 0001:0000f34c       __unwindfunclet$?apply@device_type_edit@@UAEXXZ$10 1001034c f   device_type_edit.obj
 0001:0000f355       __unwindfunclet$?apply@device_type_edit@@UAEXXZ$11 10010355 f   device_type_edit.obj
 0001:0000f35e       __unwindfunclet$?apply@device_type_edit@@UAEXXZ$12 1001035e f   device_type_edit.obj
 0001:0000f367       __unwindfunclet$?apply@device_type_edit@@UAEXXZ$13 10010367 f   device_type_edit.obj
 0001:0000f370       __unwindfunclet$?apply@device_type_edit@@UAEXXZ$14 10010370 f   device_type_edit.obj
 0001:0000f379       __unwindfunclet$?apply@device_type_edit@@UAEXXZ$15 10010379 f   device_type_edit.obj
 0001:0000f382       __unwindfunclet$?apply@device_type_edit@@UAEXXZ$16 10010382 f   device_type_edit.obj
 0001:0000f38b       __unwindfunclet$?apply@device_type_edit@@UAEXXZ$17 1001038b f   device_type_edit.obj
 0001:0000f394       __unwindfunclet$?apply@device_type_edit@@UAEXXZ$18 10010394 f   device_type_edit.obj
 0001:0000f39d       __unwindfunclet$?apply@device_type_edit@@UAEXXZ$19 1001039d f   device_type_edit.obj
 0001:0000f3a6       __unwindfunclet$?apply@device_type_edit@@UAEXXZ$20 100103a6 f   device_type_edit.obj
 0001:0000f3af       __unwindfunclet$?apply@device_type_edit@@UAEXXZ$21 100103af f   device_type_edit.obj
 0001:0000f3b8       __unwindfunclet$?apply@device_type_edit@@UAEXXZ$22 100103b8 f   device_type_edit.obj
 0001:0000f3c1       __ehhandler$?apply@device_type_edit@@UAEXXZ 100103c1 f   device_type_edit.obj
 0001:0000f3dc       __unwindfunclet$?closeEvent@device_type_edit@@UAEXPAVQCloseEvent@@@Z$0 100103dc f   device_type_edit.obj
 0001:0000f3e5       __unwindfunclet$?closeEvent@device_type_edit@@UAEXPAVQCloseEvent@@@Z$2 100103e5 f   device_type_edit.obj
 0001:0000f3ee       __unwindfunclet$?closeEvent@device_type_edit@@UAEXPAVQCloseEvent@@@Z$4 100103ee f   device_type_edit.obj
 0001:0000f3f7       __unwindfunclet$?closeEvent@device_type_edit@@UAEXPAVQCloseEvent@@@Z$5 100103f7 f   device_type_edit.obj
 0001:0000f400       __ehhandler$?closeEvent@device_type_edit@@UAEXPAVQCloseEvent@@@Z 10010400 f   device_type_edit.obj
 0001:0000f41b       __unwindfunclet$?db@@YAXABVQString@@@Z$0 1001041b f   device_type_edit.obj
 0001:0000f424       __ehhandler$?db@@YAXABVQString@@@Z 10010424 f   device_type_edit.obj
 0001:0000f43f       __unwindfunclet$?deleteType@device_type_edit@@AAEXABVQString@@@Z$0 1001043f f   device_type_edit.obj
 0001:0000f448       __unwindfunclet$?deleteType@device_type_edit@@AAEXABVQString@@@Z$1 10010448 f   device_type_edit.obj
 0001:0000f451       __unwindfunclet$?deleteType@device_type_edit@@AAEXABVQString@@@Z$2 10010451 f   device_type_edit.obj
 0001:0000f45a       __unwindfunclet$?deleteType@device_type_edit@@AAEXABVQString@@@Z$3 1001045a f   device_type_edit.obj
 0001:0000f463       __unwindfunclet$?deleteType@device_type_edit@@AAEXABVQString@@@Z$4 10010463 f   device_type_edit.obj
 0001:0000f46c       __unwindfunclet$?deleteType@device_type_edit@@AAEXABVQString@@@Z$5 1001046c f   device_type_edit.obj
 0001:0000f475       __unwindfunclet$?deleteType@device_type_edit@@AAEXABVQString@@@Z$7 10010475 f   device_type_edit.obj
 0001:0000f47e       __unwindfunclet$?deleteType@device_type_edit@@AAEXABVQString@@@Z$8 1001047e f   device_type_edit.obj
 0001:0000f487       __ehhandler$?deleteType@device_type_edit@@AAEXABVQString@@@Z 10010487 f   device_type_edit.obj
 0001:0000f4a2       __unwindfunclet$?markDirty@device_type_edit@@AAEXXZ$0 100104a2 f   device_type_edit.obj
 0001:0000f4ab       __unwindfunclet$?markDirty@device_type_edit@@AAEXXZ$2 100104ab f   device_type_edit.obj
 0001:0000f4b4       __unwindfunclet$?markDirty@device_type_edit@@AAEXXZ$3 100104b4 f   device_type_edit.obj
 0001:0000f4bd       __unwindfunclet$?markDirty@device_type_edit@@AAEXXZ$4 100104bd f   device_type_edit.obj
 0001:0000f4c6       __unwindfunclet$?markDirty@device_type_edit@@AAEXXZ$5 100104c6 f   device_type_edit.obj
 0001:0000f4cf       __ehhandler$?markDirty@device_type_edit@@AAEXXZ 100104cf f   device_type_edit.obj
 0001:0000f4ea       __unwindfunclet$?menus@device_type_edit@@UAE?AVQPopupMenuList@@XZ$0 100104ea f   device_type_edit.obj
 0001:0000f503       __ehhandler$?menus@device_type_edit@@UAE?AVQPopupMenuList@@XZ 10010503 f   device_type_edit.obj
 0001:0000f51e       __unwindfunclet$?navigate@device_type_edit@@UAEXABVQString@@0@Z$0 1001051e f   device_type_edit.obj
 0001:0000f527       __unwindfunclet$?navigate@device_type_edit@@UAEXABVQString@@0@Z$1 10010527 f   device_type_edit.obj
 0001:0000f530       __unwindfunclet$?navigate@device_type_edit@@UAEXABVQString@@0@Z$2 10010530 f   device_type_edit.obj
 0001:0000f539       __ehhandler$?navigate@device_type_edit@@UAEXABVQString@@0@Z 10010539 f   device_type_edit.obj
 0001:0000f554       __unwindfunclet$?reply@device_type_edit@@UAEXPAVresponse@@@Z$0 10010554 f   device_type_edit.obj
 0001:0000f56e       __unwindfunclet$?reply@device_type_edit@@UAEXPAVresponse@@@Z$1 1001056e f   device_type_edit.obj
 0001:0000f588       __unwindfunclet$?reply@device_type_edit@@UAEXPAVresponse@@@Z$2 10010588 f   device_type_edit.obj
 0001:0000f5a2       __unwindfunclet$?reply@device_type_edit@@UAEXPAVresponse@@@Z$3 100105a2 f   device_type_edit.obj
 0001:0000f5ab       __unwindfunclet$?reply@device_type_edit@@UAEXPAVresponse@@@Z$4 100105ab f   device_type_edit.obj
 0001:0000f5b4       __unwindfunclet$?reply@device_type_edit@@UAEXPAVresponse@@@Z$5 100105b4 f   device_type_edit.obj
 0001:0000f5bd       __unwindfunclet$?reply@device_type_edit@@UAEXPAVresponse@@@Z$6 100105bd f   device_type_edit.obj
 0001:0000f5c6       __unwindfunclet$?reply@device_type_edit@@UAEXPAVresponse@@@Z$8 100105c6 f   device_type_edit.obj
 0001:0000f5e0       __unwindfunclet$?reply@device_type_edit@@UAEXPAVresponse@@@Z$9 100105e0 f   device_type_edit.obj
 0001:0000f5fa       __unwindfunclet$?reply@device_type_edit@@UAEXPAVresponse@@@Z$10 100105fa f   device_type_edit.obj
 0001:0000f614       __unwindfunclet$?reply@device_type_edit@@UAEXPAVresponse@@@Z$11 10010614 f   device_type_edit.obj
 0001:0000f62e       __unwindfunclet$?reply@device_type_edit@@UAEXPAVresponse@@@Z$12 1001062e f   device_type_edit.obj
 0001:0000f64d       __unwindfunclet$?reply@device_type_edit@@UAEXPAVresponse@@@Z$13 1001064d f   device_type_edit.obj
 0001:0000f66c       __unwindfunclet$?reply@device_type_edit@@UAEXPAVresponse@@@Z$14 1001066c f   device_type_edit.obj
 0001:0000f68b       __unwindfunclet$?reply@device_type_edit@@UAEXPAVresponse@@@Z$15 1001068b f   device_type_edit.obj
 0001:0000f6aa       __unwindfunclet$?reply@device_type_edit@@UAEXPAVresponse@@@Z$16 100106aa f   device_type_edit.obj
 0001:0000f6c9       __unwindfunclet$?reply@device_type_edit@@UAEXPAVresponse@@@Z$17 100106c9 f   device_type_edit.obj
 0001:0000f6d2       __unwindfunclet$?reply@device_type_edit@@UAEXPAVresponse@@@Z$19 100106d2 f   device_type_edit.obj
 0001:0000f6db       __unwindfunclet$?reply@device_type_edit@@UAEXPAVresponse@@@Z$21 100106db f   device_type_edit.obj
 0001:0000f6e4       __unwindfunclet$?reply@device_type_edit@@UAEXPAVresponse@@@Z$22 100106e4 f   device_type_edit.obj
 0001:0000f6ed       __unwindfunclet$?reply@device_type_edit@@UAEXPAVresponse@@@Z$23 100106ed f   device_type_edit.obj
 0001:0000f6f6       __unwindfunclet$?reply@device_type_edit@@UAEXPAVresponse@@@Z$24 100106f6 f   device_type_edit.obj
 0001:0000f6ff       __unwindfunclet$?reply@device_type_edit@@UAEXPAVresponse@@@Z$25 100106ff f   device_type_edit.obj
 0001:0000f708       __unwindfunclet$?reply@device_type_edit@@UAEXPAVresponse@@@Z$26 10010708 f   device_type_edit.obj
 0001:0000f711       __unwindfunclet$?reply@device_type_edit@@UAEXPAVresponse@@@Z$27 10010711 f   device_type_edit.obj
 0001:0000f71a       __unwindfunclet$?reply@device_type_edit@@UAEXPAVresponse@@@Z$28 1001071a f   device_type_edit.obj
 0001:0000f723       __unwindfunclet$?reply@device_type_edit@@UAEXPAVresponse@@@Z$29 10010723 f   device_type_edit.obj
 0001:0000f72c       __unwindfunclet$?reply@device_type_edit@@UAEXPAVresponse@@@Z$30 1001072c f   device_type_edit.obj
 0001:0000f735       __unwindfunclet$?reply@device_type_edit@@UAEXPAVresponse@@@Z$32 10010735 f   device_type_edit.obj
 0001:0000f73e       __ehhandler$?reply@device_type_edit@@UAEXPAVresponse@@@Z 1001073e f   device_type_edit.obj
 0001:0000f759       __unwindfunclet$?selectType@device_type_edit@@AAEXABVQString@@@Z$0 10010759 f   device_type_edit.obj
 0001:0000f762       __unwindfunclet$?selectType@device_type_edit@@AAEXABVQString@@@Z$1 10010762 f   device_type_edit.obj
 0001:0000f76b       __unwindfunclet$?selectType@device_type_edit@@AAEXABVQString@@@Z$2 1001076b f   device_type_edit.obj
 0001:0000f774       __unwindfunclet$?selectType@device_type_edit@@AAEXABVQString@@@Z$3 10010774 f   device_type_edit.obj
 0001:0000f77d       __unwindfunclet$?selectType@device_type_edit@@AAEXABVQString@@@Z$4 1001077d f   device_type_edit.obj
 0001:0000f786       __unwindfunclet$?selectType@device_type_edit@@AAEXABVQString@@@Z$5 10010786 f   device_type_edit.obj
 0001:0000f78f       __unwindfunclet$?selectType@device_type_edit@@AAEXABVQString@@@Z$6 1001078f f   device_type_edit.obj
 0001:0000f798       __unwindfunclet$?selectType@device_type_edit@@AAEXABVQString@@@Z$7 10010798 f   device_type_edit.obj
 0001:0000f7a1       __unwindfunclet$?selectType@device_type_edit@@AAEXABVQString@@@Z$8 100107a1 f   device_type_edit.obj
 0001:0000f7aa       __unwindfunclet$?selectType@device_type_edit@@AAEXABVQString@@@Z$9 100107aa f   device_type_edit.obj
 0001:0000f7b3       __unwindfunclet$?selectType@device_type_edit@@AAEXABVQString@@@Z$10 100107b3 f   device_type_edit.obj
 0001:0000f7bc       __unwindfunclet$?selectType@device_type_edit@@AAEXABVQString@@@Z$11 100107bc f   device_type_edit.obj
 0001:0000f7c5       __unwindfunclet$?selectType@device_type_edit@@AAEXABVQString@@@Z$12 100107c5 f   device_type_edit.obj
 0001:0000f7ce       __ehhandler$?selectType@device_type_edit@@AAEXABVQString@@@Z 100107ce f   device_type_edit.obj
 0001:0000f7e9       __unwindfunclet$?toolbars@device_type_edit@@UAE?AVQDockWindowList@@XZ$0 100107e9 f   device_type_edit.obj
 0001:0000f802       __ehhandler$?toolbars@device_type_edit@@UAE?AVQDockWindowList@@XZ 10010802 f   device_type_edit.obj
 0001:0000f81d       __unwindfunclet$??0device_type_editDlg@@QAE@ABVQString@@PAVQWidget@@PBDI@Z$0 1001081d f   device_type_editdlgimpl.obj
 0001:0000f825       __unwindfunclet$??0device_type_editDlg@@QAE@ABVQString@@PAVQWidget@@PBDI@Z$1 10010825 f   device_type_editdlgimpl.obj
 0001:0000f834       __unwindfunclet$??0device_type_editDlg@@QAE@ABVQString@@PAVQWidget@@PBDI@Z$2 10010834 f   device_type_editdlgimpl.obj
 0001:0000f83d       __unwindfunclet$??0device_type_editDlg@@QAE@ABVQString@@PAVQWidget@@PBDI@Z$3 1001083d f   device_type_editdlgimpl.obj
 0001:0000f846       __unwindfunclet$??0device_type_editDlg@@QAE@ABVQString@@PAVQWidget@@PBDI@Z$4 10010846 f   device_type_editdlgimpl.obj
 0001:0000f84f       __unwindfunclet$??0device_type_editDlg@@QAE@ABVQString@@PAVQWidget@@PBDI@Z$5 1001084f f   device_type_editdlgimpl.obj
 0001:0000f858       __unwindfunclet$??0device_type_editDlg@@QAE@ABVQString@@PAVQWidget@@PBDI@Z$6 10010858 f   device_type_editdlgimpl.obj
 0001:0000f861       __ehhandler$??0device_type_editDlg@@QAE@ABVQString@@PAVQWidget@@PBDI@Z 10010861 f   device_type_editdlgimpl.obj
 0001:0000f87c       __unwindfunclet$??1?$QPtrList@VQListViewItem@@@@UAE@XZ$0 1001087c f   device_type_editdlgimpl.obj
 0001:0000f87c       __unwindfunclet$??1?$QPtrList@VQPopupMenu@@@@UAE@XZ$0 1001087c f   device_type_editdlgimpl.obj
 0001:0000f885       __ehhandler$??1?$QPtrList@VQPopupMenu@@@@UAE@XZ 10010885 f   device_type_editdlgimpl.obj
 0001:0000f885       __ehhandler$??1?$QPtrList@VQListViewItem@@@@UAE@XZ 10010885 f   device_type_editdlgimpl.obj
 0001:0000f8a0       __unwindfunclet$??1device_type_editDlg@@UAE@XZ$0 100108a0 f   device_type_editdlgimpl.obj
 0001:0000f8a8       __unwindfunclet$??1device_type_editDlg@@UAE@XZ$1 100108a8 f   device_type_editdlgimpl.obj
 0001:0000f8b7       __ehhandler$??1device_type_editDlg@@UAE@XZ 100108b7 f   device_type_editdlgimpl.obj
 0001:0000f8d2       __unwindfunclet$?checkParamClipboard@device_type_editDlg@@AAEXXZ$0 100108d2 f   device_type_editdlgimpl.obj
 0001:0000f8db       __unwindfunclet$?checkParamClipboard@device_type_editDlg@@AAEXXZ$1 100108db f   device_type_editdlgimpl.obj
 0001:0000f8e4       __unwindfunclet$?checkParamClipboard@device_type_editDlg@@AAEXXZ$2 100108e4 f   device_type_editdlgimpl.obj
 0001:0000f8ed       __unwindfunclet$?checkParamClipboard@device_type_editDlg@@AAEXXZ$3 100108ed f   device_type_editdlgimpl.obj
 0001:0000f8f6       __ehhandler$?checkParamClipboard@device_type_editDlg@@AAEXXZ 100108f6 f   device_type_editdlgimpl.obj
 0001:0000f911       __unwindfunclet$?clearParamView@device_type_editDlg@@AAEXXZ$0 10010911 f   device_type_editdlgimpl.obj
 0001:0000f91a       __unwindfunclet$?clearParamView@device_type_editDlg@@AAEXXZ$1 1001091a f   device_type_editdlgimpl.obj
 0001:0000f923       __ehhandler$?clearParamView@device_type_editDlg@@AAEXXZ 10010923 f   device_type_editdlgimpl.obj
 0001:0000f93e       __unwindfunclet$?devTypeChange@device_type_editDlg@@AAEXH@Z$0 1001093e f   device_type_editdlgimpl.obj
 0001:0000f947       __unwindfunclet$?devTypeChange@device_type_editDlg@@AAEXH@Z$5 10010947 f   device_type_editdlgimpl.obj
 0001:0000f950       __unwindfunclet$?devTypeChange@device_type_editDlg@@AAEXH@Z$3 10010950 f   device_type_editdlgimpl.obj
 0001:0000f959       __unwindfunclet$?devTypeChange@device_type_editDlg@@AAEXH@Z$4 10010959 f   device_type_editdlgimpl.obj
 0001:0000f962       __unwindfunclet$?devTypeChange@device_type_editDlg@@AAEXH@Z$1 10010962 f   device_type_editdlgimpl.obj
 0001:0000f96b       __unwindfunclet$?devTypeChange@device_type_editDlg@@AAEXH@Z$2 1001096b f   device_type_editdlgimpl.obj
 0001:0000f974       __ehhandler$?devTypeChange@device_type_editDlg@@AAEXH@Z 10010974 f   device_type_editdlgimpl.obj
 0001:0000f98f       __unwindfunclet$?displayEnum@device_type_editDlg@@AAEXPAVQDomElement@@@Z$0 1001098f f   device_type_editdlgimpl.obj
 0001:0000f998       __unwindfunclet$?displayEnum@device_type_editDlg@@AAEXPAVQDomElement@@@Z$1 10010998 f   device_type_editdlgimpl.obj
 0001:0000f9a1       __unwindfunclet$?displayEnum@device_type_editDlg@@AAEXPAVQDomElement@@@Z$2 100109a1 f   device_type_editdlgimpl.obj
 0001:0000f9aa       __unwindfunclet$?displayEnum@device_type_editDlg@@AAEXPAVQDomElement@@@Z$3 100109aa f   device_type_editdlgimpl.obj
 0001:0000f9b4       __unwindfunclet$?displayEnum@device_type_editDlg@@AAEXPAVQDomElement@@@Z$4 100109b4 f   device_type_editdlgimpl.obj
 0001:0000f9ce       __unwindfunclet$?displayEnum@device_type_editDlg@@AAEXPAVQDomElement@@@Z$5 100109ce f   device_type_editdlgimpl.obj
 0001:0000f9e8       __unwindfunclet$?displayEnum@device_type_editDlg@@AAEXPAVQDomElement@@@Z$6 100109e8 f   device_type_editdlgimpl.obj
 0001:0000fa02       __unwindfunclet$?displayEnum@device_type_editDlg@@AAEXPAVQDomElement@@@Z$7 10010a02 f   device_type_editdlgimpl.obj
 0001:0000fa1c       __unwindfunclet$?displayEnum@device_type_editDlg@@AAEXPAVQDomElement@@@Z$8 10010a1c f   device_type_editdlgimpl.obj
 0001:0000fa25       __unwindfunclet$?displayEnum@device_type_editDlg@@AAEXPAVQDomElement@@@Z$9 10010a25 f   device_type_editdlgimpl.obj
 0001:0000fa2e       __unwindfunclet$?displayEnum@device_type_editDlg@@AAEXPAVQDomElement@@@Z$10 10010a2e f   device_type_editdlgimpl.obj
 0001:0000fa37       __unwindfunclet$?displayEnum@device_type_editDlg@@AAEXPAVQDomElement@@@Z$11 10010a37 f   device_type_editdlgimpl.obj
 0001:0000fa40       __unwindfunclet$?displayEnum@device_type_editDlg@@AAEXPAVQDomElement@@@Z$12 10010a40 f   device_type_editdlgimpl.obj
 0001:0000fa49       __unwindfunclet$?displayEnum@device_type_editDlg@@AAEXPAVQDomElement@@@Z$13 10010a49 f   device_type_editdlgimpl.obj
 0001:0000fa52       __unwindfunclet$?displayEnum@device_type_editDlg@@AAEXPAVQDomElement@@@Z$14 10010a52 f   device_type_editdlgimpl.obj
 0001:0000fa5b       __unwindfunclet$?displayEnum@device_type_editDlg@@AAEXPAVQDomElement@@@Z$16 10010a5b f   device_type_editdlgimpl.obj
 0001:0000fa64       __ehhandler$?displayEnum@device_type_editDlg@@AAEXPAVQDomElement@@@Z 10010a64 f   device_type_editdlgimpl.obj
 0001:0000fa7f       __unwindfunclet$?displayRange@device_type_editDlg@@AAEXPAVQDomElement@@@Z$0 10010a7f f   device_type_editdlgimpl.obj
 0001:0000fa88       __unwindfunclet$?displayRange@device_type_editDlg@@AAEXPAVQDomElement@@@Z$1 10010a88 f   device_type_editdlgimpl.obj
 0001:0000fa91       __unwindfunclet$?displayRange@device_type_editDlg@@AAEXPAVQDomElement@@@Z$2 10010a91 f   device_type_editdlgimpl.obj
 0001:0000fa9a       __unwindfunclet$?displayRange@device_type_editDlg@@AAEXPAVQDomElement@@@Z$3 10010a9a f   device_type_editdlgimpl.obj
 0001:0000faa3       __unwindfunclet$?displayRange@device_type_editDlg@@AAEXPAVQDomElement@@@Z$4 10010aa3 f   device_type_editdlgimpl.obj
 0001:0000faac       __unwindfunclet$?displayRange@device_type_editDlg@@AAEXPAVQDomElement@@@Z$5 10010aac f   device_type_editdlgimpl.obj
 0001:0000fab5       __unwindfunclet$?displayRange@device_type_editDlg@@AAEXPAVQDomElement@@@Z$6 10010ab5 f   device_type_editdlgimpl.obj
 0001:0000fabe       __unwindfunclet$?displayRange@device_type_editDlg@@AAEXPAVQDomElement@@@Z$7 10010abe f   device_type_editdlgimpl.obj
 0001:0000fac7       __unwindfunclet$?displayRange@device_type_editDlg@@AAEXPAVQDomElement@@@Z$8 10010ac7 f   device_type_editdlgimpl.obj
 0001:0000fad0       __unwindfunclet$?displayRange@device_type_editDlg@@AAEXPAVQDomElement@@@Z$9 10010ad0 f   device_type_editdlgimpl.obj
 0001:0000fad9       __unwindfunclet$?displayRange@device_type_editDlg@@AAEXPAVQDomElement@@@Z$10 10010ad9 f   device_type_editdlgimpl.obj
 0001:0000fae2       __unwindfunclet$?displayRange@device_type_editDlg@@AAEXPAVQDomElement@@@Z$11 10010ae2 f   device_type_editdlgimpl.obj
 0001:0000faeb       __unwindfunclet$?displayRange@device_type_editDlg@@AAEXPAVQDomElement@@@Z$12 10010aeb f   device_type_editdlgimpl.obj
 0001:0000faf4       __unwindfunclet$?displayRange@device_type_editDlg@@AAEXPAVQDomElement@@@Z$13 10010af4 f   device_type_editdlgimpl.obj
 0001:0000fafd       __unwindfunclet$?displayRange@device_type_editDlg@@AAEXPAVQDomElement@@@Z$14 10010afd f   device_type_editdlgimpl.obj
 0001:0000fb06       __unwindfunclet$?displayRange@device_type_editDlg@@AAEXPAVQDomElement@@@Z$15 10010b06 f   device_type_editdlgimpl.obj
 0001:0000fb0f       __unwindfunclet$?displayRange@device_type_editDlg@@AAEXPAVQDomElement@@@Z$16 10010b0f f   device_type_editdlgimpl.obj
 0001:0000fb18       __unwindfunclet$?displayRange@device_type_editDlg@@AAEXPAVQDomElement@@@Z$17 10010b18 f   device_type_editdlgimpl.obj
 0001:0000fb21       __unwindfunclet$?displayRange@device_type_editDlg@@AAEXPAVQDomElement@@@Z$18 10010b21 f   device_type_editdlgimpl.obj
 0001:0000fb2a       __unwindfunclet$?displayRange@device_type_editDlg@@AAEXPAVQDomElement@@@Z$19 10010b2a f   device_type_editdlgimpl.obj
 0001:0000fb33       __unwindfunclet$?displayRange@device_type_editDlg@@AAEXPAVQDomElement@@@Z$20 10010b33 f   device_type_editdlgimpl.obj
 0001:0000fb3c       __unwindfunclet$?displayRange@device_type_editDlg@@AAEXPAVQDomElement@@@Z$21 10010b3c f   device_type_editdlgimpl.obj
 0001:0000fb45       __unwindfunclet$?displayRange@device_type_editDlg@@AAEXPAVQDomElement@@@Z$22 10010b45 f   device_type_editdlgimpl.obj
 0001:0000fb4e       __unwindfunclet$?displayRange@device_type_editDlg@@AAEXPAVQDomElement@@@Z$23 10010b4e f   device_type_editdlgimpl.obj
 0001:0000fb57       __unwindfunclet$?displayRange@device_type_editDlg@@AAEXPAVQDomElement@@@Z$24 10010b57 f   device_type_editdlgimpl.obj
 0001:0000fb60       __unwindfunclet$?displayRange@device_type_editDlg@@AAEXPAVQDomElement@@@Z$25 10010b60 f   device_type_editdlgimpl.obj
 0001:0000fb6c       __ehhandler$?displayRange@device_type_editDlg@@AAEXPAVQDomElement@@@Z 10010b6c f   device_type_editdlgimpl.obj
 0001:0000fb8a       __unwindfunclet$?displayString@device_type_editDlg@@AAEXPAVQDomElement@@@Z$0 10010b8a f   device_type_editdlgimpl.obj
 0001:0000fb93       __unwindfunclet$?displayString@device_type_editDlg@@AAEXPAVQDomElement@@@Z$1 10010b93 f   device_type_editdlgimpl.obj
 0001:0000fb9c       __unwindfunclet$?displayString@device_type_editDlg@@AAEXPAVQDomElement@@@Z$2 10010b9c f   device_type_editdlgimpl.obj
 0001:0000fba5       __unwindfunclet$?displayString@device_type_editDlg@@AAEXPAVQDomElement@@@Z$3 10010ba5 f   device_type_editdlgimpl.obj
 0001:0000fbae       __unwindfunclet$?displayString@device_type_editDlg@@AAEXPAVQDomElement@@@Z$4 10010bae f   device_type_editdlgimpl.obj
 0001:0000fbb7       __unwindfunclet$?displayString@device_type_editDlg@@AAEXPAVQDomElement@@@Z$5 10010bb7 f   device_type_editdlgimpl.obj
 0001:0000fbc0       __unwindfunclet$?displayString@device_type_editDlg@@AAEXPAVQDomElement@@@Z$6 10010bc0 f   device_type_editdlgimpl.obj
 0001:0000fbc9       __unwindfunclet$?displayString@device_type_editDlg@@AAEXPAVQDomElement@@@Z$7 10010bc9 f   device_type_editdlgimpl.obj
 0001:0000fbd2       __ehhandler$?displayString@device_type_editDlg@@AAEXPAVQDomElement@@@Z 10010bd2 f   device_type_editdlgimpl.obj
 0001:0000fbed       __unwindfunclet$?enumDeleteState@device_type_editDlg@@AAE_NVQString@@@Z$0 10010bed f   device_type_editdlgimpl.obj
 0001:0000fbf6       __unwindfunclet$?enumDeleteState@device_type_editDlg@@AAE_NVQString@@@Z$1 10010bf6 f   device_type_editdlgimpl.obj
 0001:0000fbff       __unwindfunclet$?enumDeleteState@device_type_editDlg@@AAE_NVQString@@@Z$2 10010bff f   device_type_editdlgimpl.obj
 0001:0000fc08       __unwindfunclet$?enumDeleteState@device_type_editDlg@@AAE_NVQString@@@Z$3 10010c08 f   device_type_editdlgimpl.obj
 0001:0000fc11       __unwindfunclet$?enumDeleteState@device_type_editDlg@@AAE_NVQString@@@Z$4 10010c11 f   device_type_editdlgimpl.obj
 0001:0000fc1a       __unwindfunclet$?enumDeleteState@device_type_editDlg@@AAE_NVQString@@@Z$5 10010c1a f   device_type_editdlgimpl.obj
 0001:0000fc23       __unwindfunclet$?enumDeleteState@device_type_editDlg@@AAE_NVQString@@@Z$7 10010c23 f   device_type_editdlgimpl.obj
 0001:0000fc2c       __unwindfunclet$?enumDeleteState@device_type_editDlg@@AAE_NVQString@@@Z$8 10010c2c f   device_type_editdlgimpl.obj
 0001:0000fc35       __unwindfunclet$?enumDeleteState@device_type_editDlg@@AAE_NVQString@@@Z$9 10010c35 f   device_type_editdlgimpl.obj
 0001:0000fc3e       __unwindfunclet$?enumDeleteState@device_type_editDlg@@AAE_NVQString@@@Z$10 10010c3e f   device_type_editdlgimpl.obj
 0001:0000fc47       __ehhandler$?enumDeleteState@device_type_editDlg@@AAE_NVQString@@@Z 10010c47 f   device_type_editdlgimpl.obj
 0001:0000fc62       __unwindfunclet$?enumNewState@device_type_editDlg@@AAEXXZ$0 10010c62 f   device_type_editdlgimpl.obj
 0001:0000fc6b       __unwindfunclet$?enumNewState@device_type_editDlg@@AAEXXZ$1 10010c6b f   device_type_editdlgimpl.obj
 0001:0000fc74       __unwindfunclet$?enumNewState@device_type_editDlg@@AAEXXZ$2 10010c74 f   device_type_editdlgimpl.obj
 0001:0000fc7d       __unwindfunclet$?enumNewState@device_type_editDlg@@AAEXXZ$3 10010c7d f   device_type_editdlgimpl.obj
 0001:0000fc86       __unwindfunclet$?enumNewState@device_type_editDlg@@AAEXXZ$4 10010c86 f   device_type_editdlgimpl.obj
 0001:0000fc8f       __unwindfunclet$?enumNewState@device_type_editDlg@@AAEXXZ$5 10010c8f f   device_type_editdlgimpl.obj
 0001:0000fc98       __unwindfunclet$?enumNewState@device_type_editDlg@@AAEXXZ$6 10010c98 f   device_type_editdlgimpl.obj
 0001:0000fca1       __unwindfunclet$?enumNewState@device_type_editDlg@@AAEXXZ$7 10010ca1 f   device_type_editdlgimpl.obj
 0001:0000fcaa       __unwindfunclet$?enumNewState@device_type_editDlg@@AAEXXZ$8 10010caa f   device_type_editdlgimpl.obj
 0001:0000fcb4       __unwindfunclet$?enumNewState@device_type_editDlg@@AAEXXZ$9 10010cb4 f   device_type_editdlgimpl.obj
 0001:0000fcbd       __unwindfunclet$?enumNewState@device_type_editDlg@@AAEXXZ$10 10010cbd f   device_type_editdlgimpl.obj
 0001:0000fcc6       __unwindfunclet$?enumNewState@device_type_editDlg@@AAEXXZ$11 10010cc6 f   device_type_editdlgimpl.obj
 0001:0000fccf       __unwindfunclet$?enumNewState@device_type_editDlg@@AAEXXZ$12 10010ccf f   device_type_editdlgimpl.obj
 0001:0000fcd8       __unwindfunclet$?enumNewState@device_type_editDlg@@AAEXXZ$13 10010cd8 f   device_type_editdlgimpl.obj
 0001:0000fce1       __unwindfunclet$?enumNewState@device_type_editDlg@@AAEXXZ$14 10010ce1 f   device_type_editdlgimpl.obj
 0001:0000fcea       __unwindfunclet$?enumNewState@device_type_editDlg@@AAEXXZ$15 10010cea f   device_type_editdlgimpl.obj
 0001:0000fcf3       __unwindfunclet$?enumNewState@device_type_editDlg@@AAEXXZ$17 10010cf3 f   device_type_editdlgimpl.obj
 0001:0000fcfc       __unwindfunclet$?enumNewState@device_type_editDlg@@AAEXXZ$18 10010cfc f   device_type_editdlgimpl.obj
 0001:0000fd05       __unwindfunclet$?enumNewState@device_type_editDlg@@AAEXXZ$19 10010d05 f   device_type_editdlgimpl.obj
 0001:0000fd0e       __unwindfunclet$?enumNewState@device_type_editDlg@@AAEXXZ$20 10010d0e f   device_type_editdlgimpl.obj
 0001:0000fd17       __unwindfunclet$?enumNewState@device_type_editDlg@@AAEXXZ$21 10010d17 f   device_type_editdlgimpl.obj
 0001:0000fd20       __unwindfunclet$?enumNewState@device_type_editDlg@@AAEXXZ$22 10010d20 f   device_type_editdlgimpl.obj
 0001:0000fd29       __unwindfunclet$?enumNewState@device_type_editDlg@@AAEXXZ$23 10010d29 f   device_type_editdlgimpl.obj
 0001:0000fd32       __unwindfunclet$?enumNewState@device_type_editDlg@@AAEXXZ$24 10010d32 f   device_type_editdlgimpl.obj
 0001:0000fd3b       __unwindfunclet$?enumNewState@device_type_editDlg@@AAEXXZ$25 10010d3b f   device_type_editdlgimpl.obj
 0001:0000fd44       __ehhandler$?enumNewState@device_type_editDlg@@AAEXXZ 10010d44 f   device_type_editdlgimpl.obj
 0001:0000fd62       __unwindfunclet$?enumPaste@device_type_editDlg@@AAEXXZ$0 10010d62 f   device_type_editdlgimpl.obj
 0001:0000fd6b       __unwindfunclet$?enumPaste@device_type_editDlg@@AAEXXZ$1 10010d6b f   device_type_editdlgimpl.obj
 0001:0000fd74       __unwindfunclet$?enumPaste@device_type_editDlg@@AAEXXZ$2 10010d74 f   device_type_editdlgimpl.obj
 0001:0000fd7d       __unwindfunclet$?enumPaste@device_type_editDlg@@AAEXXZ$3 10010d7d f   device_type_editdlgimpl.obj
 0001:0000fd86       __unwindfunclet$?enumPaste@device_type_editDlg@@AAEXXZ$4 10010d86 f   device_type_editdlgimpl.obj
 0001:0000fd8f       __unwindfunclet$?enumPaste@device_type_editDlg@@AAEXXZ$5 10010d8f f   device_type_editdlgimpl.obj
 0001:0000fd98       __unwindfunclet$?enumPaste@device_type_editDlg@@AAEXXZ$6 10010d98 f   device_type_editdlgimpl.obj
 0001:0000fda1       __unwindfunclet$?enumPaste@device_type_editDlg@@AAEXXZ$7 10010da1 f   device_type_editdlgimpl.obj
 0001:0000fdaa       __unwindfunclet$?enumPaste@device_type_editDlg@@AAEXXZ$9 10010daa f   device_type_editdlgimpl.obj
 0001:0000fdb4       __unwindfunclet$?enumPaste@device_type_editDlg@@AAEXXZ$10 10010db4 f   device_type_editdlgimpl.obj
 0001:0000fdbd       __unwindfunclet$?enumPaste@device_type_editDlg@@AAEXXZ$11 10010dbd f   device_type_editdlgimpl.obj
 0001:0000fdc9       __unwindfunclet$?enumPaste@device_type_editDlg@@AAEXXZ$12 10010dc9 f   device_type_editdlgimpl.obj
 0001:0000fdd2       __unwindfunclet$?enumPaste@device_type_editDlg@@AAEXXZ$13 10010dd2 f   device_type_editdlgimpl.obj
 0001:0000fddb       __unwindfunclet$?enumPaste@device_type_editDlg@@AAEXXZ$14 10010ddb f   device_type_editdlgimpl.obj
 0001:0000fde4       __unwindfunclet$?enumPaste@device_type_editDlg@@AAEXXZ$15 10010de4 f   device_type_editdlgimpl.obj
 0001:0000fded       __unwindfunclet$?enumPaste@device_type_editDlg@@AAEXXZ$16 10010ded f   device_type_editdlgimpl.obj
 0001:0000fdf6       __unwindfunclet$?enumPaste@device_type_editDlg@@AAEXXZ$18 10010df6 f   device_type_editdlgimpl.obj
 0001:0000fdff       __unwindfunclet$?enumPaste@device_type_editDlg@@AAEXXZ$19 10010dff f   device_type_editdlgimpl.obj
 0001:0000fe08       __unwindfunclet$?enumPaste@device_type_editDlg@@AAEXXZ$20 10010e08 f   device_type_editdlgimpl.obj
 0001:0000fe11       __unwindfunclet$?enumPaste@device_type_editDlg@@AAEXXZ$21 10010e11 f   device_type_editdlgimpl.obj
 0001:0000fe1a       __unwindfunclet$?enumPaste@device_type_editDlg@@AAEXXZ$22 10010e1a f   device_type_editdlgimpl.obj
 0001:0000fe23       __unwindfunclet$?enumPaste@device_type_editDlg@@AAEXXZ$23 10010e23 f   device_type_editdlgimpl.obj
 0001:0000fe2c       __unwindfunclet$?enumPaste@device_type_editDlg@@AAEXXZ$24 10010e2c f   device_type_editdlgimpl.obj
 0001:0000fe35       __unwindfunclet$?enumPaste@device_type_editDlg@@AAEXXZ$25 10010e35 f   device_type_editdlgimpl.obj
 0001:0000fe3e       __unwindfunclet$?enumPaste@device_type_editDlg@@AAEXXZ$26 10010e3e f   device_type_editdlgimpl.obj
 0001:0000fe47       __unwindfunclet$?enumPaste@device_type_editDlg@@AAEXXZ$27 10010e47 f   device_type_editdlgimpl.obj
 0001:0000fe50       __unwindfunclet$?enumPaste@device_type_editDlg@@AAEXXZ$28 10010e50 f   device_type_editdlgimpl.obj
 0001:0000fe59       __ehhandler$?enumPaste@device_type_editDlg@@AAEXXZ 10010e59 f   device_type_editdlgimpl.obj
 0001:0000fe77       __unwindfunclet$?loadElement@device_type_editDlg@@AAE_NPAVQDomElement@@@Z$0 10010e77 f   device_type_editdlgimpl.obj
 0001:0000fe80       __unwindfunclet$?loadElement@device_type_editDlg@@AAE_NPAVQDomElement@@@Z$1 10010e80 f   device_type_editdlgimpl.obj
 0001:0000fe89       __unwindfunclet$?loadElement@device_type_editDlg@@AAE_NPAVQDomElement@@@Z$2 10010e89 f   device_type_editdlgimpl.obj
 0001:0000fe92       __unwindfunclet$?loadElement@device_type_editDlg@@AAE_NPAVQDomElement@@@Z$3 10010e92 f   device_type_editdlgimpl.obj
 0001:0000fe9b       __unwindfunclet$?loadElement@device_type_editDlg@@AAE_NPAVQDomElement@@@Z$4 10010e9b f   device_type_editdlgimpl.obj
 0001:0000fea4       __unwindfunclet$?loadElement@device_type_editDlg@@AAE_NPAVQDomElement@@@Z$5 10010ea4 f   device_type_editdlgimpl.obj
 0001:0000fead       __unwindfunclet$?loadElement@device_type_editDlg@@AAE_NPAVQDomElement@@@Z$6 10010ead f   device_type_editdlgimpl.obj
 0001:0000feb6       __unwindfunclet$?loadElement@device_type_editDlg@@AAE_NPAVQDomElement@@@Z$7 10010eb6 f   device_type_editdlgimpl.obj
 0001:0000febf       __unwindfunclet$?loadElement@device_type_editDlg@@AAE_NPAVQDomElement@@@Z$8 10010ebf f   device_type_editdlgimpl.obj
 0001:0000fec8       __unwindfunclet$?loadElement@device_type_editDlg@@AAE_NPAVQDomElement@@@Z$9 10010ec8 f   device_type_editdlgimpl.obj
 0001:0000fed1       __unwindfunclet$?loadElement@device_type_editDlg@@AAE_NPAVQDomElement@@@Z$10 10010ed1 f   device_type_editdlgimpl.obj
 0001:0000feda       __ehhandler$?loadElement@device_type_editDlg@@AAE_NPAVQDomElement@@@Z 10010eda f   device_type_editdlgimpl.obj
 0001:0000fef5       __unwindfunclet$?loadFile@device_type_editDlg@@AAE_NABVQString@@0@Z$0 10010ef5 f   device_type_editdlgimpl.obj
 0001:0000fefe       __unwindfunclet$?loadFile@device_type_editDlg@@AAE_NABVQString@@0@Z$1 10010efe f   device_type_editdlgimpl.obj
 0001:0000ff07       __unwindfunclet$?loadFile@device_type_editDlg@@AAE_NABVQString@@0@Z$2 10010f07 f   device_type_editdlgimpl.obj
 0001:0000ff11       __unwindfunclet$?loadFile@device_type_editDlg@@AAE_NABVQString@@0@Z$3 10010f11 f   device_type_editdlgimpl.obj
 0001:0000ff1a       __unwindfunclet$?loadFile@device_type_editDlg@@AAE_NABVQString@@0@Z$4 10010f1a f   device_type_editdlgimpl.obj
 0001:0000ff23       __unwindfunclet$?loadFile@device_type_editDlg@@AAE_NABVQString@@0@Z$5 10010f23 f   device_type_editdlgimpl.obj
 0001:0000ff2c       __unwindfunclet$?loadFile@device_type_editDlg@@AAE_NABVQString@@0@Z$6 10010f2c f   device_type_editdlgimpl.obj
 0001:0000ff35       __unwindfunclet$?loadFile@device_type_editDlg@@AAE_NABVQString@@0@Z$7 10010f35 f   device_type_editdlgimpl.obj
 0001:0000ff3e       __unwindfunclet$?loadFile@device_type_editDlg@@AAE_NABVQString@@0@Z$8 10010f3e f   device_type_editdlgimpl.obj
 0001:0000ff47       __unwindfunclet$?loadFile@device_type_editDlg@@AAE_NABVQString@@0@Z$9 10010f47 f   device_type_editdlgimpl.obj
 0001:0000ff50       __unwindfunclet$?loadFile@device_type_editDlg@@AAE_NABVQString@@0@Z$10 10010f50 f   device_type_editdlgimpl.obj
 0001:0000ff59       __unwindfunclet$?loadFile@device_type_editDlg@@AAE_NABVQString@@0@Z$11 10010f59 f   device_type_editdlgimpl.obj
 0001:0000ff62       __unwindfunclet$?loadFile@device_type_editDlg@@AAE_NABVQString@@0@Z$12 10010f62 f   device_type_editdlgimpl.obj
 0001:0000ff6b       __unwindfunclet$?loadFile@device_type_editDlg@@AAE_NABVQString@@0@Z$13 10010f6b f   device_type_editdlgimpl.obj
 0001:0000ff74       __unwindfunclet$?loadFile@device_type_editDlg@@AAE_NABVQString@@0@Z$14 10010f74 f   device_type_editdlgimpl.obj
 0001:0000ff7d       __unwindfunclet$?loadFile@device_type_editDlg@@AAE_NABVQString@@0@Z$15 10010f7d f   device_type_editdlgimpl.obj
 0001:0000ff86       __unwindfunclet$?loadFile@device_type_editDlg@@AAE_NABVQString@@0@Z$16 10010f86 f   device_type_editdlgimpl.obj
 0001:0000ff8f       __unwindfunclet$?loadFile@device_type_editDlg@@AAE_NABVQString@@0@Z$17 10010f8f f   device_type_editdlgimpl.obj
 0001:0000ff98       __unwindfunclet$?loadFile@device_type_editDlg@@AAE_NABVQString@@0@Z$18 10010f98 f   device_type_editdlgimpl.obj
 0001:0000ffa1       __unwindfunclet$?loadFile@device_type_editDlg@@AAE_NABVQString@@0@Z$19 10010fa1 f   device_type_editdlgimpl.obj
 0001:0000ffaa       __unwindfunclet$?loadFile@device_type_editDlg@@AAE_NABVQString@@0@Z$20 10010faa f   device_type_editdlgimpl.obj
 0001:0000ffb3       __unwindfunclet$?loadFile@device_type_editDlg@@AAE_NABVQString@@0@Z$22 10010fb3 f   device_type_editdlgimpl.obj
 0001:0000ffbc       __ehhandler$?loadFile@device_type_editDlg@@AAE_NABVQString@@0@Z 10010fbc f   device_type_editdlgimpl.obj
 0001:0000ffd7       __unwindfunclet$?loadParamLvi@device_type_editDlg@@AAEXVQString@@PAVQDomElement@@@Z$0 10010fd7 f   device_type_editdlgimpl.obj
 0001:0000ffe0       __unwindfunclet$?loadParamLvi@device_type_editDlg@@AAEXVQString@@PAVQDomElement@@@Z$1 10010fe0 f   device_type_editdlgimpl.obj
 0001:0000ffea       __unwindfunclet$?loadParamLvi@device_type_editDlg@@AAEXVQString@@PAVQDomElement@@@Z$2 10010fea f   device_type_editdlgimpl.obj
 0001:0000fff3       __unwindfunclet$?loadParamLvi@device_type_editDlg@@AAEXVQString@@PAVQDomElement@@@Z$3 10010ff3 f   device_type_editdlgimpl.obj
 0001:0000fffc       __unwindfunclet$?loadParamLvi@device_type_editDlg@@AAEXVQString@@PAVQDomElement@@@Z$4 10010ffc f   device_type_editdlgimpl.obj
 0001:00010005       __unwindfunclet$?loadParamLvi@device_type_editDlg@@AAEXVQString@@PAVQDomElement@@@Z$5 10011005 f   device_type_editdlgimpl.obj
 0001:0001000e       __unwindfunclet$?loadParamLvi@device_type_editDlg@@AAEXVQString@@PAVQDomElement@@@Z$6 1001100e f   device_type_editdlgimpl.obj
 0001:00010017       __unwindfunclet$?loadParamLvi@device_type_editDlg@@AAEXVQString@@PAVQDomElement@@@Z$7 10011017 f   device_type_editdlgimpl.obj
 0001:00010020       __unwindfunclet$?loadParamLvi@device_type_editDlg@@AAEXVQString@@PAVQDomElement@@@Z$8 10011020 f   device_type_editdlgimpl.obj
 0001:00010029       __unwindfunclet$?loadParamLvi@device_type_editDlg@@AAEXVQString@@PAVQDomElement@@@Z$9 10011029 f   device_type_editdlgimpl.obj
 0001:00010032       __unwindfunclet$?loadParamLvi@device_type_editDlg@@AAEXVQString@@PAVQDomElement@@@Z$10 10011032 f   device_type_editdlgimpl.obj
 0001:0001003b       __unwindfunclet$?loadParamLvi@device_type_editDlg@@AAEXVQString@@PAVQDomElement@@@Z$11 1001103b f   device_type_editdlgimpl.obj
 0001:00010044       __ehhandler$?loadParamLvi@device_type_editDlg@@AAEXVQString@@PAVQDomElement@@@Z 10011044 f   device_type_editdlgimpl.obj
 0001:0001005f       __unwindfunclet$?loadTemplates@device_type_editDlg@@AAEXVQString@@@Z$0 1001105f f   device_type_editdlgimpl.obj
 0001:00010068       __unwindfunclet$?loadTemplates@device_type_editDlg@@AAEXVQString@@@Z$1 10011068 f   device_type_editdlgimpl.obj
 0001:00010071       __unwindfunclet$?loadTemplates@device_type_editDlg@@AAEXVQString@@@Z$2 10011071 f   device_type_editdlgimpl.obj
 0001:0001007a       __unwindfunclet$?loadTemplates@device_type_editDlg@@AAEXVQString@@@Z$3 1001107a f   device_type_editdlgimpl.obj
 0001:00010083       __unwindfunclet$?loadTemplates@device_type_editDlg@@AAEXVQString@@@Z$4 10011083 f   device_type_editdlgimpl.obj
 0001:0001008b       __unwindfunclet$?loadTemplates@device_type_editDlg@@AAEXVQString@@@Z$5 1001108b f   device_type_editdlgimpl.obj
 0001:00010094       __ehhandler$?loadTemplates@device_type_editDlg@@AAEXVQString@@@Z 10011094 f   device_type_editdlgimpl.obj
 0001:000100af       __unwindfunclet$?newGetNewParamName@device_type_editDlg@@AAE?AVQString@@V2@@Z$0 100110af f   device_type_editdlgimpl.obj
 0001:000100b8       __unwindfunclet$?newGetNewParamName@device_type_editDlg@@AAE?AVQString@@V2@@Z$1 100110b8 f   device_type_editdlgimpl.obj
 0001:000100c1       __unwindfunclet$?newGetNewParamName@device_type_editDlg@@AAE?AVQString@@V2@@Z$2 100110c1 f   device_type_editdlgimpl.obj
 0001:000100ca       __unwindfunclet$?newGetNewParamName@device_type_editDlg@@AAE?AVQString@@V2@@Z$3 100110ca f   device_type_editdlgimpl.obj
 0001:000100d3       __unwindfunclet$?newGetNewParamName@device_type_editDlg@@AAE?AVQString@@V2@@Z$4 100110d3 f   device_type_editdlgimpl.obj
 0001:000100dc       __unwindfunclet$?newGetNewParamName@device_type_editDlg@@AAE?AVQString@@V2@@Z$6 100110dc f   device_type_editdlgimpl.obj
 0001:000100e5       __unwindfunclet$?newGetNewParamName@device_type_editDlg@@AAE?AVQString@@V2@@Z$7 100110e5 f   device_type_editdlgimpl.obj
 0001:000100ee       __unwindfunclet$?newGetNewParamName@device_type_editDlg@@AAE?AVQString@@V2@@Z$8 100110ee f   device_type_editdlgimpl.obj
 0001:000100f7       __unwindfunclet$?newGetNewParamName@device_type_editDlg@@AAE?AVQString@@V2@@Z$9 100110f7 f   device_type_editdlgimpl.obj
 0001:00010100       __unwindfunclet$?newGetNewParamName@device_type_editDlg@@AAE?AVQString@@V2@@Z$10 10011100 f   device_type_editdlgimpl.obj
 0001:00010109       __unwindfunclet$?newGetNewParamName@device_type_editDlg@@AAE?AVQString@@V2@@Z$11 10011109 f   device_type_editdlgimpl.obj
 0001:00010112       __unwindfunclet$?newGetNewParamName@device_type_editDlg@@AAE?AVQString@@V2@@Z$12 10011112 f   device_type_editdlgimpl.obj
 0001:0001011b       __unwindfunclet$?newGetNewParamName@device_type_editDlg@@AAE?AVQString@@V2@@Z$13 1001111b f   device_type_editdlgimpl.obj
 0001:00010124       __unwindfunclet$?newGetNewParamName@device_type_editDlg@@AAE?AVQString@@V2@@Z$16 10011124 f   device_type_editdlgimpl.obj
 0001:0001012d       __unwindfunclet$?newGetNewParamName@device_type_editDlg@@AAE?AVQString@@V2@@Z$14 1001112d f   device_type_editdlgimpl.obj
 0001:00010136       __unwindfunclet$?newGetNewParamName@device_type_editDlg@@AAE?AVQString@@V2@@Z$15 10011136 f   device_type_editdlgimpl.obj
 0001:0001013f       __unwindfunclet$?newGetNewParamName@device_type_editDlg@@AAE?AVQString@@V2@@Z$5 1001113f f   device_type_editdlgimpl.obj
 0001:00010159       __ehhandler$?newGetNewParamName@device_type_editDlg@@AAE?AVQString@@V2@@Z 10011159 f   device_type_editdlgimpl.obj
 0001:00010174       __unwindfunclet$?paramCopy@device_type_editDlg@@AAEXXZ$0 10011174 f   device_type_editdlgimpl.obj
 0001:0001017d       __unwindfunclet$?paramCopy@device_type_editDlg@@AAEXXZ$1 1001117d f   device_type_editdlgimpl.obj
 0001:00010186       __unwindfunclet$?paramCopy@device_type_editDlg@@AAEXXZ$2 10011186 f   device_type_editdlgimpl.obj
 0001:0001018f       __unwindfunclet$?paramCopy@device_type_editDlg@@AAEXXZ$3 1001118f f   device_type_editdlgimpl.obj
 0001:00010198       __unwindfunclet$?paramCopy@device_type_editDlg@@AAEXXZ$5 10011198 f   device_type_editdlgimpl.obj
 0001:000101a1       __unwindfunclet$?paramCopy@device_type_editDlg@@AAEXXZ$6 100111a1 f   device_type_editdlgimpl.obj
 0001:000101aa       __unwindfunclet$?paramCopy@device_type_editDlg@@AAEXXZ$7 100111aa f   device_type_editdlgimpl.obj
 0001:000101b3       __unwindfunclet$?paramCopy@device_type_editDlg@@AAEXXZ$8 100111b3 f   device_type_editdlgimpl.obj
 0001:000101bc       __unwindfunclet$?paramCopy@device_type_editDlg@@AAEXXZ$9 100111bc f   device_type_editdlgimpl.obj
 0001:000101c5       __unwindfunclet$?paramCopy@device_type_editDlg@@AAEXXZ$10 100111c5 f   device_type_editdlgimpl.obj
 0001:000101ce       __unwindfunclet$?paramCopy@device_type_editDlg@@AAEXXZ$11 100111ce f   device_type_editdlgimpl.obj
 0001:000101d7       __unwindfunclet$?paramCopy@device_type_editDlg@@AAEXXZ$12 100111d7 f   device_type_editdlgimpl.obj
 0001:000101e0       __unwindfunclet$?paramCopy@device_type_editDlg@@AAEXXZ$14 100111e0 f   device_type_editdlgimpl.obj
 0001:000101e9       __unwindfunclet$?paramCopy@device_type_editDlg@@AAEXXZ$15 100111e9 f   device_type_editdlgimpl.obj
 0001:000101f2       __ehhandler$?paramCopy@device_type_editDlg@@AAEXXZ 100111f2 f   device_type_editdlgimpl.obj
 0001:0001020d       __unwindfunclet$?paramDelete@device_type_editDlg@@AAEXXZ$0 1001120d f   device_type_editdlgimpl.obj
 0001:00010215       __unwindfunclet$?paramDelete@device_type_editDlg@@AAEXXZ$1 10011215 f   device_type_editdlgimpl.obj
 0001:0001021e       __unwindfunclet$?paramDelete@device_type_editDlg@@AAEXXZ$2 1001121e f   device_type_editdlgimpl.obj
 0001:00010227       __unwindfunclet$?paramDelete@device_type_editDlg@@AAEXXZ$3 10011227 f   device_type_editdlgimpl.obj
 0001:00010230       __unwindfunclet$?paramDelete@device_type_editDlg@@AAEXXZ$4 10011230 f   device_type_editdlgimpl.obj
 0001:00010239       __unwindfunclet$?paramDelete@device_type_editDlg@@AAEXXZ$5 10011239 f   device_type_editdlgimpl.obj
 0001:00010242       __unwindfunclet$?paramDelete@device_type_editDlg@@AAEXXZ$6 10011242 f   device_type_editdlgimpl.obj
 0001:0001024b       __unwindfunclet$?paramDelete@device_type_editDlg@@AAEXXZ$7 1001124b f   device_type_editdlgimpl.obj
 0001:00010254       __unwindfunclet$?paramDelete@device_type_editDlg@@AAEXXZ$9 10011254 f   device_type_editdlgimpl.obj
 0001:0001025d       __ehhandler$?paramDelete@device_type_editDlg@@AAEXXZ 1001125d f   device_type_editdlgimpl.obj
 0001:00010278       __unwindfunclet$?paramNew@device_type_editDlg@@AAEXXZ$0 10011278 f   device_type_editdlgimpl.obj
 0001:00010281       __unwindfunclet$?paramNew@device_type_editDlg@@AAEXXZ$1 10011281 f   device_type_editdlgimpl.obj
 0001:0001028a       __unwindfunclet$?paramNew@device_type_editDlg@@AAEXXZ$3 1001128a f   device_type_editdlgimpl.obj
 0001:00010293       __unwindfunclet$?paramNew@device_type_editDlg@@AAEXXZ$4 10011293 f   device_type_editdlgimpl.obj
 0001:0001029c       __unwindfunclet$?paramNew@device_type_editDlg@@AAEXXZ$5 1001129c f   device_type_editdlgimpl.obj
 0001:000102a5       __unwindfunclet$?paramNew@device_type_editDlg@@AAEXXZ$6 100112a5 f   device_type_editdlgimpl.obj
 0001:000102ae       __unwindfunclet$?paramNew@device_type_editDlg@@AAEXXZ$7 100112ae f   device_type_editdlgimpl.obj
 0001:000102b7       __unwindfunclet$?paramNew@device_type_editDlg@@AAEXXZ$9 100112b7 f   device_type_editdlgimpl.obj
 0001:000102c0       __ehhandler$?paramNew@device_type_editDlg@@AAEXXZ 100112c0 f   device_type_editdlgimpl.obj
 0001:000102db       __unwindfunclet$?paramPaste@device_type_editDlg@@AAEXXZ$0 100112db f   device_type_editdlgimpl.obj
 0001:000102e4       __unwindfunclet$?paramPaste@device_type_editDlg@@AAEXXZ$1 100112e4 f   device_type_editdlgimpl.obj
 0001:000102ed       __unwindfunclet$?paramPaste@device_type_editDlg@@AAEXXZ$2 100112ed f   device_type_editdlgimpl.obj
 0001:000102f6       __unwindfunclet$?paramPaste@device_type_editDlg@@AAEXXZ$3 100112f6 f   device_type_editdlgimpl.obj
 0001:000102ff       __unwindfunclet$?paramPaste@device_type_editDlg@@AAEXXZ$4 100112ff f   device_type_editdlgimpl.obj
 0001:00010308       __unwindfunclet$?paramPaste@device_type_editDlg@@AAEXXZ$5 10011308 f   device_type_editdlgimpl.obj
 0001:00010311       __unwindfunclet$?paramPaste@device_type_editDlg@@AAEXXZ$6 10011311 f   device_type_editdlgimpl.obj
 0001:0001031a       __unwindfunclet$?paramPaste@device_type_editDlg@@AAEXXZ$7 1001131a f   device_type_editdlgimpl.obj
 0001:00010323       __unwindfunclet$?paramPaste@device_type_editDlg@@AAEXXZ$8 10011323 f   device_type_editdlgimpl.obj
 0001:0001032c       __unwindfunclet$?paramPaste@device_type_editDlg@@AAEXXZ$9 1001132c f   device_type_editdlgimpl.obj
 0001:00010335       __unwindfunclet$?paramPaste@device_type_editDlg@@AAEXXZ$10 10011335 f   device_type_editdlgimpl.obj
 0001:0001033e       __unwindfunclet$?paramPaste@device_type_editDlg@@AAEXXZ$11 1001133e f   device_type_editdlgimpl.obj
 0001:00010347       __unwindfunclet$?paramPaste@device_type_editDlg@@AAEXXZ$12 10011347 f   device_type_editdlgimpl.obj
 0001:00010350       __unwindfunclet$?paramPaste@device_type_editDlg@@AAEXXZ$13 10011350 f   device_type_editdlgimpl.obj
 0001:00010359       __unwindfunclet$?paramPaste@device_type_editDlg@@AAEXXZ$14 10011359 f   device_type_editdlgimpl.obj
 0001:00010362       __unwindfunclet$?paramPaste@device_type_editDlg@@AAEXXZ$15 10011362 f   device_type_editdlgimpl.obj
 0001:0001036b       __unwindfunclet$?paramPaste@device_type_editDlg@@AAEXXZ$18 1001136b f   device_type_editdlgimpl.obj
 0001:00010374       __unwindfunclet$?paramPaste@device_type_editDlg@@AAEXXZ$19 10011374 f   device_type_editdlgimpl.obj
 0001:00010380       __unwindfunclet$?paramPaste@device_type_editDlg@@AAEXXZ$21 10011380 f   device_type_editdlgimpl.obj
 0001:00010389       __unwindfunclet$?paramPaste@device_type_editDlg@@AAEXXZ$23 10011389 f   device_type_editdlgimpl.obj
 0001:00010395       __unwindfunclet$?paramPaste@device_type_editDlg@@AAEXXZ$16 10011395 f   device_type_editdlgimpl.obj
 0001:0001039e       __ehhandler$?paramPaste@device_type_editDlg@@AAEXXZ 1001139e f   device_type_editdlgimpl.obj
 0001:000103bc       __unwindfunclet$?paramRename@device_type_editDlg@@AAEXXZ$1 100113bc f   device_type_editdlgimpl.obj
 0001:000103c5       __unwindfunclet$?paramRename@device_type_editDlg@@AAEXXZ$2 100113c5 f   device_type_editdlgimpl.obj
 0001:000103ce       __unwindfunclet$?paramRename@device_type_editDlg@@AAEXXZ$4 100113ce f   device_type_editdlgimpl.obj
 0001:000103d7       __unwindfunclet$?paramRename@device_type_editDlg@@AAEXXZ$5 100113d7 f   device_type_editdlgimpl.obj
 0001:000103e0       __ehhandler$?paramRename@device_type_editDlg@@AAEXXZ 100113e0 f   device_type_editdlgimpl.obj
 0001:000103fb       __unwindfunclet$?removeSettings@device_type_editDlg@@AAE_NPAVQDomElement@@VQString@@@Z$0 100113fb f   device_type_editdlgimpl.obj
 0001:00010404       __unwindfunclet$?removeSettings@device_type_editDlg@@AAE_NPAVQDomElement@@VQString@@@Z$1 10011404 f   device_type_editdlgimpl.obj
 0001:0001040d       __unwindfunclet$?removeSettings@device_type_editDlg@@AAE_NPAVQDomElement@@VQString@@@Z$2 1001140d f   device_type_editdlgimpl.obj
 0001:00010416       __unwindfunclet$?removeSettings@device_type_editDlg@@AAE_NPAVQDomElement@@VQString@@@Z$3 10011416 f   device_type_editdlgimpl.obj
 0001:0001041f       __unwindfunclet$?removeSettings@device_type_editDlg@@AAE_NPAVQDomElement@@VQString@@@Z$4 1001141f f   device_type_editdlgimpl.obj
 0001:00010428       __unwindfunclet$?removeSettings@device_type_editDlg@@AAE_NPAVQDomElement@@VQString@@@Z$6 10011428 f   device_type_editdlgimpl.obj
 0001:00010431       __unwindfunclet$?removeSettings@device_type_editDlg@@AAE_NPAVQDomElement@@VQString@@@Z$7 10011431 f   device_type_editdlgimpl.obj
 0001:0001043a       __unwindfunclet$?removeSettings@device_type_editDlg@@AAE_NPAVQDomElement@@VQString@@@Z$8 1001143a f   device_type_editdlgimpl.obj
 0001:00010443       __unwindfunclet$?removeSettings@device_type_editDlg@@AAE_NPAVQDomElement@@VQString@@@Z$9 10011443 f   device_type_editdlgimpl.obj
 0001:0001044c       __unwindfunclet$?removeSettings@device_type_editDlg@@AAE_NPAVQDomElement@@VQString@@@Z$11 1001144c f   device_type_editdlgimpl.obj
 0001:00010455       __unwindfunclet$?removeSettings@device_type_editDlg@@AAE_NPAVQDomElement@@VQString@@@Z$12 10011455 f   device_type_editdlgimpl.obj
 0001:0001045e       __unwindfunclet$?removeSettings@device_type_editDlg@@AAE_NPAVQDomElement@@VQString@@@Z$13 1001145e f   device_type_editdlgimpl.obj
 0001:00010467       __unwindfunclet$?removeSettings@device_type_editDlg@@AAE_NPAVQDomElement@@VQString@@@Z$14 10011467 f   device_type_editdlgimpl.obj
 0001:00010470       __unwindfunclet$?removeSettings@device_type_editDlg@@AAE_NPAVQDomElement@@VQString@@@Z$16 10011470 f   device_type_editdlgimpl.obj
 0001:00010479       __unwindfunclet$?removeSettings@device_type_editDlg@@AAE_NPAVQDomElement@@VQString@@@Z$17 10011479 f   device_type_editdlgimpl.obj
 0001:00010482       __unwindfunclet$?removeSettings@device_type_editDlg@@AAE_NPAVQDomElement@@VQString@@@Z$18 10011482 f   device_type_editdlgimpl.obj
 0001:0001048b       __unwindfunclet$?removeSettings@device_type_editDlg@@AAE_NPAVQDomElement@@VQString@@@Z$19 1001148b f   device_type_editdlgimpl.obj
 0001:00010494       __unwindfunclet$?removeSettings@device_type_editDlg@@AAE_NPAVQDomElement@@VQString@@@Z$21 10011494 f   device_type_editdlgimpl.obj
 0001:0001049d       __unwindfunclet$?removeSettings@device_type_editDlg@@AAE_NPAVQDomElement@@VQString@@@Z$22 1001149d f   device_type_editdlgimpl.obj
 0001:000104a6       __unwindfunclet$?removeSettings@device_type_editDlg@@AAE_NPAVQDomElement@@VQString@@@Z$23 100114a6 f   device_type_editdlgimpl.obj
 0001:000104af       __unwindfunclet$?removeSettings@device_type_editDlg@@AAE_NPAVQDomElement@@VQString@@@Z$24 100114af f   device_type_editdlgimpl.obj
 0001:000104b8       __ehhandler$?removeSettings@device_type_editDlg@@AAE_NPAVQDomElement@@VQString@@@Z 100114b8 f   device_type_editdlgimpl.obj
 0001:000104d3       __unwindfunclet$?saveElement@device_type_editDlg@@AAE_NPAVQDomElement@@@Z$0 100114d3 f   device_type_editdlgimpl.obj
 0001:000104dc       __unwindfunclet$?saveElement@device_type_editDlg@@AAE_NPAVQDomElement@@@Z$1 100114dc f   device_type_editdlgimpl.obj
 0001:000104e5       __unwindfunclet$?saveElement@device_type_editDlg@@AAE_NPAVQDomElement@@@Z$2 100114e5 f   device_type_editdlgimpl.obj
 0001:000104ee       __unwindfunclet$?saveElement@device_type_editDlg@@AAE_NPAVQDomElement@@@Z$7 100114ee f   device_type_editdlgimpl.obj
 0001:000104f7       __unwindfunclet$?saveElement@device_type_editDlg@@AAE_NPAVQDomElement@@@Z$8 100114f7 f   device_type_editdlgimpl.obj
 0001:00010500       __unwindfunclet$?saveElement@device_type_editDlg@@AAE_NPAVQDomElement@@@Z$5 10011500 f   device_type_editdlgimpl.obj
 0001:00010509       __unwindfunclet$?saveElement@device_type_editDlg@@AAE_NPAVQDomElement@@@Z$6 10011509 f   device_type_editdlgimpl.obj
 0001:00010512       __unwindfunclet$?saveElement@device_type_editDlg@@AAE_NPAVQDomElement@@@Z$3 10011512 f   device_type_editdlgimpl.obj
 0001:0001051b       __unwindfunclet$?saveElement@device_type_editDlg@@AAE_NPAVQDomElement@@@Z$4 1001151b f   device_type_editdlgimpl.obj
 0001:00010524       __unwindfunclet$?saveElement@device_type_editDlg@@AAE_NPAVQDomElement@@@Z$10 10011524 f   device_type_editdlgimpl.obj
 0001:0001052d       __unwindfunclet$?saveElement@device_type_editDlg@@AAE_NPAVQDomElement@@@Z$11 1001152d f   device_type_editdlgimpl.obj
 0001:00010536       __unwindfunclet$?saveElement@device_type_editDlg@@AAE_NPAVQDomElement@@@Z$12 10011536 f   device_type_editdlgimpl.obj
 0001:0001053f       __unwindfunclet$?saveElement@device_type_editDlg@@AAE_NPAVQDomElement@@@Z$13 1001153f f   device_type_editdlgimpl.obj
 0001:00010548       __unwindfunclet$?saveElement@device_type_editDlg@@AAE_NPAVQDomElement@@@Z$14 10011548 f   device_type_editdlgimpl.obj
 0001:00010551       __ehhandler$?saveElement@device_type_editDlg@@AAE_NPAVQDomElement@@@Z 10011551 f   device_type_editdlgimpl.obj
 0001:0001056c       __unwindfunclet$?saveEnum@device_type_editDlg@@AAE_NPAVQDomElement@@@Z$0 1001156c f   device_type_editdlgimpl.obj
 0001:00010575       __unwindfunclet$?saveEnum@device_type_editDlg@@AAE_NPAVQDomElement@@@Z$1 10011575 f   device_type_editdlgimpl.obj
 0001:0001057e       __unwindfunclet$?saveEnum@device_type_editDlg@@AAE_NPAVQDomElement@@@Z$2 1001157e f   device_type_editdlgimpl.obj
 0001:00010587       __unwindfunclet$?saveEnum@device_type_editDlg@@AAE_NPAVQDomElement@@@Z$3 10011587 f   device_type_editdlgimpl.obj
 0001:00010590       __unwindfunclet$?saveEnum@device_type_editDlg@@AAE_NPAVQDomElement@@@Z$4 10011590 f   device_type_editdlgimpl.obj
 0001:00010599       __unwindfunclet$?saveEnum@device_type_editDlg@@AAE_NPAVQDomElement@@@Z$5 10011599 f   device_type_editdlgimpl.obj
 0001:000105a2       __unwindfunclet$?saveEnum@device_type_editDlg@@AAE_NPAVQDomElement@@@Z$6 100115a2 f   device_type_editdlgimpl.obj
 0001:000105ab       __unwindfunclet$?saveEnum@device_type_editDlg@@AAE_NPAVQDomElement@@@Z$7 100115ab f   device_type_editdlgimpl.obj
 0001:000105b4       __unwindfunclet$?saveEnum@device_type_editDlg@@AAE_NPAVQDomElement@@@Z$8 100115b4 f   device_type_editdlgimpl.obj
 0001:000105bd       __unwindfunclet$?saveEnum@device_type_editDlg@@AAE_NPAVQDomElement@@@Z$9 100115bd f   device_type_editdlgimpl.obj
 0001:000105c6       __unwindfunclet$?saveEnum@device_type_editDlg@@AAE_NPAVQDomElement@@@Z$10 100115c6 f   device_type_editdlgimpl.obj
 0001:000105cf       __unwindfunclet$?saveEnum@device_type_editDlg@@AAE_NPAVQDomElement@@@Z$11 100115cf f   device_type_editdlgimpl.obj
 0001:000105d8       __unwindfunclet$?saveEnum@device_type_editDlg@@AAE_NPAVQDomElement@@@Z$12 100115d8 f   device_type_editdlgimpl.obj
 0001:000105e1       __unwindfunclet$?saveEnum@device_type_editDlg@@AAE_NPAVQDomElement@@@Z$13 100115e1 f   device_type_editdlgimpl.obj
 0001:000105ea       __unwindfunclet$?saveEnum@device_type_editDlg@@AAE_NPAVQDomElement@@@Z$14 100115ea f   device_type_editdlgimpl.obj
 0001:000105f3       __unwindfunclet$?saveEnum@device_type_editDlg@@AAE_NPAVQDomElement@@@Z$15 100115f3 f   device_type_editdlgimpl.obj
 0001:000105fc       __unwindfunclet$?saveEnum@device_type_editDlg@@AAE_NPAVQDomElement@@@Z$16 100115fc f   device_type_editdlgimpl.obj
 0001:00010605       __ehhandler$?saveEnum@device_type_editDlg@@AAE_NPAVQDomElement@@@Z 10011605 f   device_type_editdlgimpl.obj
 0001:00010620       __unwindfunclet$?saveFile@device_type_editDlg@@AAE_NABVQString@@0@Z$0 10011620 f   device_type_editdlgimpl.obj
 0001:00010629       __unwindfunclet$?saveFile@device_type_editDlg@@AAE_NABVQString@@0@Z$1 10011629 f   device_type_editdlgimpl.obj
 0001:00010632       __unwindfunclet$?saveFile@device_type_editDlg@@AAE_NABVQString@@0@Z$2 10011632 f   device_type_editdlgimpl.obj
 0001:0001063b       __unwindfunclet$?saveFile@device_type_editDlg@@AAE_NABVQString@@0@Z$3 1001163b f   device_type_editdlgimpl.obj
 0001:00010644       __unwindfunclet$?saveFile@device_type_editDlg@@AAE_NABVQString@@0@Z$4 10011644 f   device_type_editdlgimpl.obj
 0001:0001064d       __ehhandler$?saveFile@device_type_editDlg@@AAE_NABVQString@@0@Z 1001164d f   device_type_editdlgimpl.obj
 0001:00010668       __unwindfunclet$?saveRange@device_type_editDlg@@AAE_NPAVQDomElement@@@Z$0 10011668 f   device_type_editdlgimpl.obj
 0001:00010671       __unwindfunclet$?saveRange@device_type_editDlg@@AAE_NPAVQDomElement@@@Z$1 10011671 f   device_type_editdlgimpl.obj
 0001:0001067a       __unwindfunclet$?saveRange@device_type_editDlg@@AAE_NPAVQDomElement@@@Z$2 1001167a f   device_type_editdlgimpl.obj
 0001:00010683       __unwindfunclet$?saveRange@device_type_editDlg@@AAE_NPAVQDomElement@@@Z$3 10011683 f   device_type_editdlgimpl.obj
 0001:0001068c       __unwindfunclet$?saveRange@device_type_editDlg@@AAE_NPAVQDomElement@@@Z$4 1001168c f   device_type_editdlgimpl.obj
 0001:00010695       __unwindfunclet$?saveRange@device_type_editDlg@@AAE_NPAVQDomElement@@@Z$5 10011695 f   device_type_editdlgimpl.obj
 0001:0001069e       __unwindfunclet$?saveRange@device_type_editDlg@@AAE_NPAVQDomElement@@@Z$6 1001169e f   device_type_editdlgimpl.obj
 0001:000106a7       __unwindfunclet$?saveRange@device_type_editDlg@@AAE_NPAVQDomElement@@@Z$7 100116a7 f   device_type_editdlgimpl.obj
 0001:000106b0       __unwindfunclet$?saveRange@device_type_editDlg@@AAE_NPAVQDomElement@@@Z$8 100116b0 f   device_type_editdlgimpl.obj
 0001:000106b9       __unwindfunclet$?saveRange@device_type_editDlg@@AAE_NPAVQDomElement@@@Z$10 100116b9 f   device_type_editdlgimpl.obj
 0001:000106c2       __unwindfunclet$?saveRange@device_type_editDlg@@AAE_NPAVQDomElement@@@Z$11 100116c2 f   device_type_editdlgimpl.obj
 0001:000106cb       __unwindfunclet$?saveRange@device_type_editDlg@@AAE_NPAVQDomElement@@@Z$13 100116cb f   device_type_editdlgimpl.obj
 0001:000106d4       __unwindfunclet$?saveRange@device_type_editDlg@@AAE_NPAVQDomElement@@@Z$14 100116d4 f   device_type_editdlgimpl.obj
 0001:000106dd       __unwindfunclet$?saveRange@device_type_editDlg@@AAE_NPAVQDomElement@@@Z$15 100116dd f   device_type_editdlgimpl.obj
 0001:000106e6       __unwindfunclet$?saveRange@device_type_editDlg@@AAE_NPAVQDomElement@@@Z$16 100116e6 f   device_type_editdlgimpl.obj
 0001:000106ef       __unwindfunclet$?saveRange@device_type_editDlg@@AAE_NPAVQDomElement@@@Z$17 100116ef f   device_type_editdlgimpl.obj
 0001:000106f8       __unwindfunclet$?saveRange@device_type_editDlg@@AAE_NPAVQDomElement@@@Z$18 100116f8 f   device_type_editdlgimpl.obj
 0001:00010701       __unwindfunclet$?saveRange@device_type_editDlg@@AAE_NPAVQDomElement@@@Z$19 10011701 f   device_type_editdlgimpl.obj
 0001:0001070a       __unwindfunclet$?saveRange@device_type_editDlg@@AAE_NPAVQDomElement@@@Z$20 1001170a f   device_type_editdlgimpl.obj
 0001:00010713       __unwindfunclet$?saveRange@device_type_editDlg@@AAE_NPAVQDomElement@@@Z$21 10011713 f   device_type_editdlgimpl.obj
 0001:0001071c       __unwindfunclet$?saveRange@device_type_editDlg@@AAE_NPAVQDomElement@@@Z$22 1001171c f   device_type_editdlgimpl.obj
 0001:00010725       __unwindfunclet$?saveRange@device_type_editDlg@@AAE_NPAVQDomElement@@@Z$23 10011725 f   device_type_editdlgimpl.obj
 0001:0001072e       __unwindfunclet$?saveRange@device_type_editDlg@@AAE_NPAVQDomElement@@@Z$24 1001172e f   device_type_editdlgimpl.obj
 0001:00010737       __unwindfunclet$?saveRange@device_type_editDlg@@AAE_NPAVQDomElement@@@Z$25 10011737 f   device_type_editdlgimpl.obj
 0001:00010740       __unwindfunclet$?saveRange@device_type_editDlg@@AAE_NPAVQDomElement@@@Z$26 10011740 f   device_type_editdlgimpl.obj
 0001:00010749       __unwindfunclet$?saveRange@device_type_editDlg@@AAE_NPAVQDomElement@@@Z$27 10011749 f   device_type_editdlgimpl.obj
 0001:00010752       __unwindfunclet$?saveRange@device_type_editDlg@@AAE_NPAVQDomElement@@@Z$28 10011752 f   device_type_editdlgimpl.obj
 0001:0001075b       __unwindfunclet$?saveRange@device_type_editDlg@@AAE_NPAVQDomElement@@@Z$29 1001175b f   device_type_editdlgimpl.obj
 0001:00010764       __unwindfunclet$?saveRange@device_type_editDlg@@AAE_NPAVQDomElement@@@Z$31 10011764 f   device_type_editdlgimpl.obj
 0001:0001076d       __unwindfunclet$?saveRange@device_type_editDlg@@AAE_NPAVQDomElement@@@Z$32 1001176d f   device_type_editdlgimpl.obj
 0001:00010776       __unwindfunclet$?saveRange@device_type_editDlg@@AAE_NPAVQDomElement@@@Z$34 10011776 f   device_type_editdlgimpl.obj
 0001:0001077f       __unwindfunclet$?saveRange@device_type_editDlg@@AAE_NPAVQDomElement@@@Z$35 1001177f f   device_type_editdlgimpl.obj
 0001:00010788       __unwindfunclet$?saveRange@device_type_editDlg@@AAE_NPAVQDomElement@@@Z$36 10011788 f   device_type_editdlgimpl.obj
 0001:00010791       __unwindfunclet$?saveRange@device_type_editDlg@@AAE_NPAVQDomElement@@@Z$37 10011791 f   device_type_editdlgimpl.obj
 0001:0001079a       __unwindfunclet$?saveRange@device_type_editDlg@@AAE_NPAVQDomElement@@@Z$38 1001179a f   device_type_editdlgimpl.obj
 0001:000107a3       __unwindfunclet$?saveRange@device_type_editDlg@@AAE_NPAVQDomElement@@@Z$39 100117a3 f   device_type_editdlgimpl.obj
 0001:000107ac       __unwindfunclet$?saveRange@device_type_editDlg@@AAE_NPAVQDomElement@@@Z$40 100117ac f   device_type_editdlgimpl.obj
 0001:000107b5       __unwindfunclet$?saveRange@device_type_editDlg@@AAE_NPAVQDomElement@@@Z$41 100117b5 f   device_type_editdlgimpl.obj
 0001:000107be       __unwindfunclet$?saveRange@device_type_editDlg@@AAE_NPAVQDomElement@@@Z$42 100117be f   device_type_editdlgimpl.obj
 0001:000107c7       __unwindfunclet$?saveRange@device_type_editDlg@@AAE_NPAVQDomElement@@@Z$43 100117c7 f   device_type_editdlgimpl.obj
 0001:000107d0       __unwindfunclet$?saveRange@device_type_editDlg@@AAE_NPAVQDomElement@@@Z$44 100117d0 f   device_type_editdlgimpl.obj
 0001:000107d9       __unwindfunclet$?saveRange@device_type_editDlg@@AAE_NPAVQDomElement@@@Z$45 100117d9 f   device_type_editdlgimpl.obj
 0001:000107e2       __unwindfunclet$?saveRange@device_type_editDlg@@AAE_NPAVQDomElement@@@Z$46 100117e2 f   device_type_editdlgimpl.obj
 0001:000107eb       __unwindfunclet$?saveRange@device_type_editDlg@@AAE_NPAVQDomElement@@@Z$47 100117eb f   device_type_editdlgimpl.obj
 0001:000107f4       __unwindfunclet$?saveRange@device_type_editDlg@@AAE_NPAVQDomElement@@@Z$48 100117f4 f   device_type_editdlgimpl.obj
 0001:000107fd       __unwindfunclet$?saveRange@device_type_editDlg@@AAE_NPAVQDomElement@@@Z$49 100117fd f   device_type_editdlgimpl.obj
 0001:00010806       __ehhandler$?saveRange@device_type_editDlg@@AAE_NPAVQDomElement@@@Z 10011806 f   device_type_editdlgimpl.obj
 0001:00010821       __unwindfunclet$?saveString@device_type_editDlg@@AAE_NPAVQDomElement@@@Z$0 10011821 f   device_type_editdlgimpl.obj
 0001:0001082a       __unwindfunclet$?saveString@device_type_editDlg@@AAE_NPAVQDomElement@@@Z$1 1001182a f   device_type_editdlgimpl.obj
 0001:00010833       __unwindfunclet$?saveString@device_type_editDlg@@AAE_NPAVQDomElement@@@Z$2 10011833 f   device_type_editdlgimpl.obj
 0001:0001083c       __unwindfunclet$?saveString@device_type_editDlg@@AAE_NPAVQDomElement@@@Z$3 1001183c f   device_type_editdlgimpl.obj
 0001:00010845       __unwindfunclet$?saveString@device_type_editDlg@@AAE_NPAVQDomElement@@@Z$4 10011845 f   device_type_editdlgimpl.obj
 0001:0001084e       __unwindfunclet$?saveString@device_type_editDlg@@AAE_NPAVQDomElement@@@Z$5 1001184e f   device_type_editdlgimpl.obj
 0001:00010857       __unwindfunclet$?saveString@device_type_editDlg@@AAE_NPAVQDomElement@@@Z$6 10011857 f   device_type_editdlgimpl.obj
 0001:00010860       __unwindfunclet$?saveString@device_type_editDlg@@AAE_NPAVQDomElement@@@Z$7 10011860 f   device_type_editdlgimpl.obj
 0001:00010869       __unwindfunclet$?saveString@device_type_editDlg@@AAE_NPAVQDomElement@@@Z$8 10011869 f   device_type_editdlgimpl.obj
 0001:00010872       __unwindfunclet$?saveString@device_type_editDlg@@AAE_NPAVQDomElement@@@Z$10 10011872 f   device_type_editdlgimpl.obj
 0001:0001087b       __unwindfunclet$?saveString@device_type_editDlg@@AAE_NPAVQDomElement@@@Z$11 1001187b f   device_type_editdlgimpl.obj
 0001:00010884       __unwindfunclet$?saveString@device_type_editDlg@@AAE_NPAVQDomElement@@@Z$13 10011884 f   device_type_editdlgimpl.obj
 0001:0001088d       __unwindfunclet$?saveString@device_type_editDlg@@AAE_NPAVQDomElement@@@Z$14 1001188d f   device_type_editdlgimpl.obj
 0001:00010896       __unwindfunclet$?saveString@device_type_editDlg@@AAE_NPAVQDomElement@@@Z$15 10011896 f   device_type_editdlgimpl.obj
 0001:0001089f       __unwindfunclet$?saveString@device_type_editDlg@@AAE_NPAVQDomElement@@@Z$16 1001189f f   device_type_editdlgimpl.obj
 0001:000108a8       __ehhandler$?saveString@device_type_editDlg@@AAE_NPAVQDomElement@@@Z 100118a8 f   device_type_editdlgimpl.obj
 0001:000108c3       __unwindfunclet$?selectParam@device_type_editDlg@@AAEXPAVQListViewItem@@@Z$0 100118c3 f   device_type_editdlgimpl.obj
 0001:000108cc       __unwindfunclet$?selectParam@device_type_editDlg@@AAEXPAVQListViewItem@@@Z$1 100118cc f   device_type_editdlgimpl.obj
 0001:000108d5       __unwindfunclet$?selectParam@device_type_editDlg@@AAEXPAVQListViewItem@@@Z$2 100118d5 f   device_type_editdlgimpl.obj
 0001:000108de       __unwindfunclet$?selectParam@device_type_editDlg@@AAEXPAVQListViewItem@@@Z$3 100118de f   device_type_editdlgimpl.obj
 0001:000108e7       __unwindfunclet$?selectParam@device_type_editDlg@@AAEXPAVQListViewItem@@@Z$4 100118e7 f   device_type_editdlgimpl.obj
 0001:000108f0       __unwindfunclet$?selectParam@device_type_editDlg@@AAEXPAVQListViewItem@@@Z$5 100118f0 f   device_type_editdlgimpl.obj
 0001:000108f9       __unwindfunclet$?selectParam@device_type_editDlg@@AAEXPAVQListViewItem@@@Z$6 100118f9 f   device_type_editdlgimpl.obj
 0001:00010902       __unwindfunclet$?selectParam@device_type_editDlg@@AAEXPAVQListViewItem@@@Z$7 10011902 f   device_type_editdlgimpl.obj
 0001:0001090b       __unwindfunclet$?selectParam@device_type_editDlg@@AAEXPAVQListViewItem@@@Z$8 1001190b f   device_type_editdlgimpl.obj
 0001:00010914       __unwindfunclet$?selectParam@device_type_editDlg@@AAEXPAVQListViewItem@@@Z$10 10011914 f   device_type_editdlgimpl.obj
 0001:0001091d       __unwindfunclet$?selectParam@device_type_editDlg@@AAEXPAVQListViewItem@@@Z$9 1001191d f   device_type_editdlgimpl.obj
 0001:00010927       __unwindfunclet$?selectParam@device_type_editDlg@@AAEXPAVQListViewItem@@@Z$11 10011927 f   device_type_editdlgimpl.obj
 0001:00010930       __ehhandler$?selectParam@device_type_editDlg@@AAEXPAVQListViewItem@@@Z 10011930 f   device_type_editdlgimpl.obj
 0001:0001094b       __unwindfunclet$?selectParam@device_type_editDlg@@AAEXXZ$0 1001194b f   device_type_editdlgimpl.obj
 0001:00010954       __unwindfunclet$?selectParam@device_type_editDlg@@AAEXXZ$1 10011954 f   device_type_editdlgimpl.obj
 0001:0001095d       __unwindfunclet$?selectParam@device_type_editDlg@@AAEXXZ$2 1001195d f   device_type_editdlgimpl.obj
 0001:00010966       __ehhandler$?selectParam@device_type_editDlg@@AAEXXZ 10011966 f   device_type_editdlgimpl.obj
 0001:00010981       __unwindfunclet$?compare@paramLVI@@UBEHPAVQListViewItem@@H_N@Z$0 10011981 f   paramLVI.obj
 0001:0001098a       __unwindfunclet$?compare@paramLVI@@UBEHPAVQListViewItem@@H_N@Z$1 1001198a f   paramLVI.obj
 0001:00010993       __unwindfunclet$?compare@paramLVI@@UBEHPAVQListViewItem@@H_N@Z$2 10011993 f   paramLVI.obj
 0001:0001099c       __unwindfunclet$?compare@paramLVI@@UBEHPAVQListViewItem@@H_N@Z$3 1001199c f   paramLVI.obj
 0001:000109a5       __ehhandler$?compare@paramLVI@@UBEHPAVQListViewItem@@H_N@Z 100119a5 f   paramLVI.obj
 0001:000109c0       __unwindfunclet$?keys@plugindesc@@UAE?AVQStringList@@ABVQString@@0@Z$0 100119c0 f   plugindesc.obj
 0001:000109da       __unwindfunclet$?keys@plugindesc@@UAE?AVQStringList@@ABVQString@@0@Z$1 100119da f   plugindesc.obj
 0001:000109e3       __ehhandler$?keys@plugindesc@@UAE?AVQStringList@@ABVQString@@0@Z 100119e3 f   plugindesc.obj
 0001:000109fe       __unwindfunclet$??0toolWindow@@QAE@PAVQWidget@@PBDI@Z$0 100119fe f   toolwindowimpl.obj
 0001:00010a06       __unwindfunclet$??0toolWindow@@QAE@PAVQWidget@@PBDI@Z$1 10011a06 f   toolwindowimpl.obj
 0001:00010a15       __unwindfunclet$??0toolWindow@@QAE@PAVQWidget@@PBDI@Z$2 10011a15 f   toolwindowimpl.obj
 0001:00010a1e       __ehhandler$??0toolWindow@@QAE@PAVQWidget@@PBDI@Z 10011a1e f   toolwindowimpl.obj
 0001:00010a39       __unwindfunclet$??1toolWindow@@UAE@XZ$0 10011a39 f   toolwindowimpl.obj
 0001:00010a41       __ehhandler$??1toolWindow@@UAE@XZ 10011a41 f   toolwindowimpl.obj
 0001:00010a5c       __unwindfunclet$?deleteFile@toolWindow@@AAEXXZ$0 10011a5c f   toolwindowimpl.obj
 0001:00010a65       __unwindfunclet$?deleteFile@toolWindow@@AAEXXZ$1 10011a65 f   toolwindowimpl.obj
 0001:00010a6e       __unwindfunclet$?deleteFile@toolWindow@@AAEXXZ$2 10011a6e f   toolwindowimpl.obj
 0001:00010a77       __unwindfunclet$?deleteFile@toolWindow@@AAEXXZ$3 10011a77 f   toolwindowimpl.obj
 0001:00010a80       __unwindfunclet$?deleteFile@toolWindow@@AAEXXZ$4 10011a80 f   toolwindowimpl.obj
 0001:00010a89       __unwindfunclet$?deleteFile@toolWindow@@AAEXXZ$5 10011a89 f   toolwindowimpl.obj
 0001:00010a92       __unwindfunclet$?deleteFile@toolWindow@@AAEXXZ$6 10011a92 f   toolwindowimpl.obj
 0001:00010a9b       __unwindfunclet$?deleteFile@toolWindow@@AAEXXZ$8 10011a9b f   toolwindowimpl.obj
 0001:00010aa4       __ehhandler$?deleteFile@toolWindow@@AAEXXZ 10011aa4 f   toolwindowimpl.obj
 0001:00010abf       __unwindfunclet$?loadFile@toolWindow@@QAE_NVQString@@@Z$0 10011abf f   toolwindowimpl.obj
 0001:00010ac8       __unwindfunclet$?loadFile@toolWindow@@QAE_NVQString@@@Z$1 10011ac8 f   toolwindowimpl.obj
 0001:00010ad2       __unwindfunclet$?loadFile@toolWindow@@QAE_NVQString@@@Z$2 10011ad2 f   toolwindowimpl.obj
 0001:00010ade       __unwindfunclet$?loadFile@toolWindow@@QAE_NVQString@@@Z$3 10011ade f   toolwindowimpl.obj
 0001:00010ae7       __unwindfunclet$?loadFile@toolWindow@@QAE_NVQString@@@Z$4 10011ae7 f   toolwindowimpl.obj
 0001:00010af0       __unwindfunclet$?loadFile@toolWindow@@QAE_NVQString@@@Z$5 10011af0 f   toolwindowimpl.obj
 0001:00010af9       __unwindfunclet$?loadFile@toolWindow@@QAE_NVQString@@@Z$6 10011af9 f   toolwindowimpl.obj
 0001:00010b02       __unwindfunclet$?loadFile@toolWindow@@QAE_NVQString@@@Z$7 10011b02 f   toolwindowimpl.obj
 0001:00010b0b       __unwindfunclet$?loadFile@toolWindow@@QAE_NVQString@@@Z$8 10011b0b f   toolwindowimpl.obj
 0001:00010b14       __unwindfunclet$?loadFile@toolWindow@@QAE_NVQString@@@Z$9 10011b14 f   toolwindowimpl.obj
 0001:00010b1d       __unwindfunclet$?loadFile@toolWindow@@QAE_NVQString@@@Z$10 10011b1d f   toolwindowimpl.obj
 0001:00010b26       __unwindfunclet$?loadFile@toolWindow@@QAE_NVQString@@@Z$11 10011b26 f   toolwindowimpl.obj
 0001:00010b2f       __unwindfunclet$?loadFile@toolWindow@@QAE_NVQString@@@Z$12 10011b2f f   toolwindowimpl.obj
 0001:00010b39       __unwindfunclet$?loadFile@toolWindow@@QAE_NVQString@@@Z$13 10011b39 f   toolwindowimpl.obj
 0001:00010b42       __unwindfunclet$?loadFile@toolWindow@@QAE_NVQString@@@Z$14 10011b42 f   toolwindowimpl.obj
 0001:00010b4b       __unwindfunclet$?loadFile@toolWindow@@QAE_NVQString@@@Z$15 10011b4b f   toolwindowimpl.obj
 0001:00010b54       __unwindfunclet$?loadFile@toolWindow@@QAE_NVQString@@@Z$16 10011b54 f   toolwindowimpl.obj
 0001:00010b5d       __unwindfunclet$?loadFile@toolWindow@@QAE_NVQString@@@Z$17 10011b5d f   toolwindowimpl.obj
 0001:00010b66       __unwindfunclet$?loadFile@toolWindow@@QAE_NVQString@@@Z$18 10011b66 f   toolwindowimpl.obj
 0001:00010b6f       __unwindfunclet$?loadFile@toolWindow@@QAE_NVQString@@@Z$19 10011b6f f   toolwindowimpl.obj
 0001:00010b78       __unwindfunclet$?loadFile@toolWindow@@QAE_NVQString@@@Z$21 10011b78 f   toolwindowimpl.obj
 0001:00010b81       __ehhandler$?loadFile@toolWindow@@QAE_NVQString@@@Z 10011b81 f   toolwindowimpl.obj
 0001:00010b9f       __unwindfunclet$?newFile@toolWindow@@AAEXXZ$0 10011b9f f   toolwindowimpl.obj
 0001:00010ba8       __unwindfunclet$?newFile@toolWindow@@AAEXXZ$1 10011ba8 f   toolwindowimpl.obj
 0001:00010bb1       __unwindfunclet$?newFile@toolWindow@@AAEXXZ$2 10011bb1 f   toolwindowimpl.obj
 0001:00010bba       __unwindfunclet$?newFile@toolWindow@@AAEXXZ$3 10011bba f   toolwindowimpl.obj
 0001:00010bc3       __unwindfunclet$?newFile@toolWindow@@AAEXXZ$4 10011bc3 f   toolwindowimpl.obj
 0001:00010bcc       __unwindfunclet$?newFile@toolWindow@@AAEXXZ$5 10011bcc f   toolwindowimpl.obj
 0001:00010bd5       __unwindfunclet$?newFile@toolWindow@@AAEXXZ$6 10011bd5 f   toolwindowimpl.obj
 0001:00010bde       __unwindfunclet$?newFile@toolWindow@@AAEXXZ$7 10011bde f   toolwindowimpl.obj
 0001:00010be7       __unwindfunclet$?newFile@toolWindow@@AAEXXZ$8 10011be7 f   toolwindowimpl.obj
 0001:00010bf0       __unwindfunclet$?newFile@toolWindow@@AAEXXZ$9 10011bf0 f   toolwindowimpl.obj
 0001:00010bf9       __unwindfunclet$?newFile@toolWindow@@AAEXXZ$10 10011bf9 f   toolwindowimpl.obj
 0001:00010c02       __unwindfunclet$?newFile@toolWindow@@AAEXXZ$11 10011c02 f   toolwindowimpl.obj
 0001:00010c0b       __unwindfunclet$?newFile@toolWindow@@AAEXXZ$12 10011c0b f   toolwindowimpl.obj
 0001:00010c14       __unwindfunclet$?newFile@toolWindow@@AAEXXZ$15 10011c14 f   toolwindowimpl.obj
 0001:00010c1d       __unwindfunclet$?newFile@toolWindow@@AAEXXZ$16 10011c1d f   toolwindowimpl.obj
 0001:00010c26       __unwindfunclet$?newFile@toolWindow@@AAEXXZ$18 10011c26 f   toolwindowimpl.obj
 0001:00010c2f       __unwindfunclet$?newFile@toolWindow@@AAEXXZ$19 10011c2f f   toolwindowimpl.obj
 0001:00010c39       __unwindfunclet$?newFile@toolWindow@@AAEXXZ$20 10011c39 f   toolwindowimpl.obj
 0001:00010c42       __unwindfunclet$?newFile@toolWindow@@AAEXXZ$21 10011c42 f   toolwindowimpl.obj
 0001:00010c4b       __unwindfunclet$?newFile@toolWindow@@AAEXXZ$22 10011c4b f   toolwindowimpl.obj
 0001:00010c54       __unwindfunclet$?newFile@toolWindow@@AAEXXZ$23 10011c54 f   toolwindowimpl.obj
 0001:00010c5d       __unwindfunclet$?newFile@toolWindow@@AAEXXZ$24 10011c5d f   toolwindowimpl.obj
 0001:00010c66       __unwindfunclet$?newFile@toolWindow@@AAEXXZ$25 10011c66 f   toolwindowimpl.obj
 0001:00010c6f       __unwindfunclet$?newFile@toolWindow@@AAEXXZ$26 10011c6f f   toolwindowimpl.obj
 0001:00010c78       __unwindfunclet$?newFile@toolWindow@@AAEXXZ$13 10011c78 f   toolwindowimpl.obj
 0001:00010c81       __unwindfunclet$?newFile@toolWindow@@AAEXXZ$14 10011c81 f   toolwindowimpl.obj
 0001:00010c8a       __unwindfunclet$?newFile@toolWindow@@AAEXXZ$28 10011c8a f   toolwindowimpl.obj
 0001:00010c93       __unwindfunclet$?newFile@toolWindow@@AAEXXZ$29 10011c93 f   toolwindowimpl.obj
 0001:00010c9c       __unwindfunclet$?newFile@toolWindow@@AAEXXZ$30 10011c9c f   toolwindowimpl.obj
 0001:00010ca5       __unwindfunclet$?newFile@toolWindow@@AAEXXZ$31 10011ca5 f   toolwindowimpl.obj
 0001:00010cae       __unwindfunclet$?newFile@toolWindow@@AAEXXZ$32 10011cae f   toolwindowimpl.obj
 0001:00010cb7       __unwindfunclet$?newFile@toolWindow@@AAEXXZ$33 10011cb7 f   toolwindowimpl.obj
 0001:00010cc0       __unwindfunclet$?newFile@toolWindow@@AAEXXZ$34 10011cc0 f   toolwindowimpl.obj
 0001:00010cc9       __unwindfunclet$?newFile@toolWindow@@AAEXXZ$35 10011cc9 f   toolwindowimpl.obj
 0001:00010cd2       __ehhandler$?newFile@toolWindow@@AAEXXZ 10011cd2 f   toolwindowimpl.obj
 0001:00010ced       __unwindfunclet$?saveFile@toolWindow@@QAE_NVQString@@@Z$0 10011ced f   toolwindowimpl.obj
 0001:00010cf6       __unwindfunclet$?saveFile@toolWindow@@QAE_NVQString@@@Z$1 10011cf6 f   toolwindowimpl.obj
 0001:00010cff       __unwindfunclet$?saveFile@toolWindow@@QAE_NVQString@@@Z$2 10011cff f   toolwindowimpl.obj
 0001:00010d08       __unwindfunclet$?saveFile@toolWindow@@QAE_NVQString@@@Z$3 10011d08 f   toolwindowimpl.obj
 0001:00010d11       __ehhandler$?saveFile@toolWindow@@QAE_NVQString@@@Z 10011d11 f   toolwindowimpl.obj
 0001:00010d2c       __unwindfunclet$?selectFamily@toolWindow@@AAE?AVQString@@V2@0@Z$0 10011d2c f   toolwindowimpl.obj
 0001:00010d35       __unwindfunclet$?selectFamily@toolWindow@@AAE?AVQString@@V2@0@Z$1 10011d35 f   toolwindowimpl.obj
 0001:00010d3e       __unwindfunclet$?selectFamily@toolWindow@@AAE?AVQString@@V2@0@Z$2 10011d3e f   toolwindowimpl.obj
 0001:00010d47       __unwindfunclet$?selectFamily@toolWindow@@AAE?AVQString@@V2@0@Z$3 10011d47 f   toolwindowimpl.obj
 0001:00010d50       __unwindfunclet$?selectFamily@toolWindow@@AAE?AVQString@@V2@0@Z$4 10011d50 f   toolwindowimpl.obj
 0001:00010d6a       __ehhandler$?selectFamily@toolWindow@@AAE?AVQString@@V2@0@Z 10011d6a f   toolwindowimpl.obj
 0001:00010d85       __unwindfunclet$?selectType@toolWindow@@AAEXPAVQListViewItem@@@Z$0 10011d85 f   toolwindowimpl.obj
 0001:00010d8e       __ehhandler$?selectType@toolWindow@@AAEXPAVQListViewItem@@@Z 10011d8e f   toolwindowimpl.obj
 0001:00010da9       __unwindfunclet$??0device_type_editDlgBase@@QAE@PAVQWidget@@PBDI@Z$0 10011da9 f   device_type_editdlg.obj
 0001:00010db2       __unwindfunclet$??0device_type_editDlgBase@@QAE@PAVQWidget@@PBDI@Z$1 10011db2 f   device_type_editdlg.obj
 0001:00010dc1       __unwindfunclet$??0device_type_editDlgBase@@QAE@PAVQWidget@@PBDI@Z$2 10011dc1 f   device_type_editdlg.obj
 0001:00010dcb       __unwindfunclet$??0device_type_editDlgBase@@QAE@PAVQWidget@@PBDI@Z$3 10011dcb f   device_type_editdlg.obj
 0001:00010dd5       __unwindfunclet$??0device_type_editDlgBase@@QAE@PAVQWidget@@PBDI@Z$4 10011dd5 f   device_type_editdlg.obj
 0001:00010ddf       __unwindfunclet$??0device_type_editDlgBase@@QAE@PAVQWidget@@PBDI@Z$5 10011ddf f   device_type_editdlg.obj
 0001:00010de9       __unwindfunclet$??0device_type_editDlgBase@@QAE@PAVQWidget@@PBDI@Z$6 10011de9 f   device_type_editdlg.obj
 0001:00010df3       __unwindfunclet$??0device_type_editDlgBase@@QAE@PAVQWidget@@PBDI@Z$7 10011df3 f   device_type_editdlg.obj
 0001:00010dfd       __unwindfunclet$??0device_type_editDlgBase@@QAE@PAVQWidget@@PBDI@Z$8 10011dfd f   device_type_editdlg.obj
 0001:00010e07       __unwindfunclet$??0device_type_editDlgBase@@QAE@PAVQWidget@@PBDI@Z$9 10011e07 f   device_type_editdlg.obj
 0001:00010e11       __unwindfunclet$??0device_type_editDlgBase@@QAE@PAVQWidget@@PBDI@Z$10 10011e11 f   device_type_editdlg.obj
 0001:00010e1a       __unwindfunclet$??0device_type_editDlgBase@@QAE@PAVQWidget@@PBDI@Z$11 10011e1a f   device_type_editdlg.obj
 0001:00010e23       __unwindfunclet$??0device_type_editDlgBase@@QAE@PAVQWidget@@PBDI@Z$12 10011e23 f   device_type_editdlg.obj
 0001:00010e2c       __unwindfunclet$??0device_type_editDlgBase@@QAE@PAVQWidget@@PBDI@Z$13 10011e2c f   device_type_editdlg.obj
 0001:00010e35       __unwindfunclet$??0device_type_editDlgBase@@QAE@PAVQWidget@@PBDI@Z$14 10011e35 f   device_type_editdlg.obj
 0001:00010e3e       __unwindfunclet$??0device_type_editDlgBase@@QAE@PAVQWidget@@PBDI@Z$15 10011e3e f   device_type_editdlg.obj
 0001:00010e48       __unwindfunclet$??0device_type_editDlgBase@@QAE@PAVQWidget@@PBDI@Z$16 10011e48 f   device_type_editdlg.obj
 0001:00010e52       __unwindfunclet$??0device_type_editDlgBase@@QAE@PAVQWidget@@PBDI@Z$17 10011e52 f   device_type_editdlg.obj
 0001:00010e5c       __unwindfunclet$??0device_type_editDlgBase@@QAE@PAVQWidget@@PBDI@Z$18 10011e5c f   device_type_editdlg.obj
 0001:00010e66       __unwindfunclet$??0device_type_editDlgBase@@QAE@PAVQWidget@@PBDI@Z$19 10011e66 f   device_type_editdlg.obj
 0001:00010e70       __unwindfunclet$??0device_type_editDlgBase@@QAE@PAVQWidget@@PBDI@Z$20 10011e70 f   device_type_editdlg.obj
 0001:00010e7a       __unwindfunclet$??0device_type_editDlgBase@@QAE@PAVQWidget@@PBDI@Z$21 10011e7a f   device_type_editdlg.obj
 0001:00010e84       __unwindfunclet$??0device_type_editDlgBase@@QAE@PAVQWidget@@PBDI@Z$22 10011e84 f   device_type_editdlg.obj
 0001:00010e8e       __unwindfunclet$??0device_type_editDlgBase@@QAE@PAVQWidget@@PBDI@Z$23 10011e8e f   device_type_editdlg.obj
 0001:00010e98       __unwindfunclet$??0device_type_editDlgBase@@QAE@PAVQWidget@@PBDI@Z$24 10011e98 f   device_type_editdlg.obj
 0001:00010ea2       __unwindfunclet$??0device_type_editDlgBase@@QAE@PAVQWidget@@PBDI@Z$25 10011ea2 f   device_type_editdlg.obj
 0001:00010eac       __unwindfunclet$??0device_type_editDlgBase@@QAE@PAVQWidget@@PBDI@Z$26 10011eac f   device_type_editdlg.obj
 0001:00010eb6       __unwindfunclet$??0device_type_editDlgBase@@QAE@PAVQWidget@@PBDI@Z$27 10011eb6 f   device_type_editdlg.obj
 0001:00010ec0       __unwindfunclet$??0device_type_editDlgBase@@QAE@PAVQWidget@@PBDI@Z$28 10011ec0 f   device_type_editdlg.obj
 0001:00010eca       __unwindfunclet$??0device_type_editDlgBase@@QAE@PAVQWidget@@PBDI@Z$29 10011eca f   device_type_editdlg.obj
 0001:00010ed4       __unwindfunclet$??0device_type_editDlgBase@@QAE@PAVQWidget@@PBDI@Z$30 10011ed4 f   device_type_editdlg.obj
 0001:00010ede       __unwindfunclet$??0device_type_editDlgBase@@QAE@PAVQWidget@@PBDI@Z$31 10011ede f   device_type_editdlg.obj
 0001:00010ee8       __unwindfunclet$??0device_type_editDlgBase@@QAE@PAVQWidget@@PBDI@Z$32 10011ee8 f   device_type_editdlg.obj
 0001:00010ef2       __unwindfunclet$??0device_type_editDlgBase@@QAE@PAVQWidget@@PBDI@Z$33 10011ef2 f   device_type_editdlg.obj
 0001:00010efc       __unwindfunclet$??0device_type_editDlgBase@@QAE@PAVQWidget@@PBDI@Z$34 10011efc f   device_type_editdlg.obj
 0001:00010f06       __unwindfunclet$??0device_type_editDlgBase@@QAE@PAVQWidget@@PBDI@Z$35 10011f06 f   device_type_editdlg.obj
 0001:00010f10       __unwindfunclet$??0device_type_editDlgBase@@QAE@PAVQWidget@@PBDI@Z$36 10011f10 f   device_type_editdlg.obj
 0001:00010f1a       __unwindfunclet$??0device_type_editDlgBase@@QAE@PAVQWidget@@PBDI@Z$37 10011f1a f   device_type_editdlg.obj
 0001:00010f24       __unwindfunclet$??0device_type_editDlgBase@@QAE@PAVQWidget@@PBDI@Z$38 10011f24 f   device_type_editdlg.obj
 0001:00010f2e       __unwindfunclet$??0device_type_editDlgBase@@QAE@PAVQWidget@@PBDI@Z$39 10011f2e f   device_type_editdlg.obj
 0001:00010f38       __unwindfunclet$??0device_type_editDlgBase@@QAE@PAVQWidget@@PBDI@Z$40 10011f38 f   device_type_editdlg.obj
 0001:00010f42       __unwindfunclet$??0device_type_editDlgBase@@QAE@PAVQWidget@@PBDI@Z$41 10011f42 f   device_type_editdlg.obj
 0001:00010f4c       __unwindfunclet$??0device_type_editDlgBase@@QAE@PAVQWidget@@PBDI@Z$42 10011f4c f   device_type_editdlg.obj
 0001:00010f56       __unwindfunclet$??0device_type_editDlgBase@@QAE@PAVQWidget@@PBDI@Z$43 10011f56 f   device_type_editdlg.obj
 0001:00010f60       __unwindfunclet$??0device_type_editDlgBase@@QAE@PAVQWidget@@PBDI@Z$44 10011f60 f   device_type_editdlg.obj
 0001:00010f6a       __unwindfunclet$??0device_type_editDlgBase@@QAE@PAVQWidget@@PBDI@Z$45 10011f6a f   device_type_editdlg.obj
 0001:00010f74       __unwindfunclet$??0device_type_editDlgBase@@QAE@PAVQWidget@@PBDI@Z$46 10011f74 f   device_type_editdlg.obj
 0001:00010f7e       __unwindfunclet$??0device_type_editDlgBase@@QAE@PAVQWidget@@PBDI@Z$47 10011f7e f   device_type_editdlg.obj
 0001:00010f88       __unwindfunclet$??0device_type_editDlgBase@@QAE@PAVQWidget@@PBDI@Z$48 10011f88 f   device_type_editdlg.obj
 0001:00010f92       __unwindfunclet$??0device_type_editDlgBase@@QAE@PAVQWidget@@PBDI@Z$49 10011f92 f   device_type_editdlg.obj
 0001:00010f9c       __unwindfunclet$??0device_type_editDlgBase@@QAE@PAVQWidget@@PBDI@Z$50 10011f9c f   device_type_editdlg.obj
 0001:00010fa6       __unwindfunclet$??0device_type_editDlgBase@@QAE@PAVQWidget@@PBDI@Z$51 10011fa6 f   device_type_editdlg.obj
 0001:00010fb0       __unwindfunclet$??0device_type_editDlgBase@@QAE@PAVQWidget@@PBDI@Z$52 10011fb0 f   device_type_editdlg.obj
 0001:00010fba       __unwindfunclet$??0device_type_editDlgBase@@QAE@PAVQWidget@@PBDI@Z$53 10011fba f   device_type_editdlg.obj
 0001:00010fc4       __unwindfunclet$??0device_type_editDlgBase@@QAE@PAVQWidget@@PBDI@Z$54 10011fc4 f   device_type_editdlg.obj
 0001:00010fce       __unwindfunclet$??0device_type_editDlgBase@@QAE@PAVQWidget@@PBDI@Z$55 10011fce f   device_type_editdlg.obj
 0001:00010fd8       __unwindfunclet$??0device_type_editDlgBase@@QAE@PAVQWidget@@PBDI@Z$56 10011fd8 f   device_type_editdlg.obj
 0001:00010fe2       __unwindfunclet$??0device_type_editDlgBase@@QAE@PAVQWidget@@PBDI@Z$57 10011fe2 f   device_type_editdlg.obj
 0001:00010fec       __unwindfunclet$??0device_type_editDlgBase@@QAE@PAVQWidget@@PBDI@Z$58 10011fec f   device_type_editdlg.obj
 0001:00010ff6       __unwindfunclet$??0device_type_editDlgBase@@QAE@PAVQWidget@@PBDI@Z$59 10011ff6 f   device_type_editdlg.obj
 0001:00011000       __unwindfunclet$??0device_type_editDlgBase@@QAE@PAVQWidget@@PBDI@Z$60 10012000 f   device_type_editdlg.obj
 0001:0001100a       __unwindfunclet$??0device_type_editDlgBase@@QAE@PAVQWidget@@PBDI@Z$61 1001200a f   device_type_editdlg.obj
 0001:00011014       __unwindfunclet$??0device_type_editDlgBase@@QAE@PAVQWidget@@PBDI@Z$62 10012014 f   device_type_editdlg.obj
 0001:0001101e       __unwindfunclet$??0device_type_editDlgBase@@QAE@PAVQWidget@@PBDI@Z$63 1001201e f   device_type_editdlg.obj
 0001:00011028       __unwindfunclet$??0device_type_editDlgBase@@QAE@PAVQWidget@@PBDI@Z$64 10012028 f   device_type_editdlg.obj
 0001:00011032       __unwindfunclet$??0device_type_editDlgBase@@QAE@PAVQWidget@@PBDI@Z$65 10012032 f   device_type_editdlg.obj
 0001:0001103c       __unwindfunclet$??0device_type_editDlgBase@@QAE@PAVQWidget@@PBDI@Z$66 1001203c f   device_type_editdlg.obj
 0001:00011046       __unwindfunclet$??0device_type_editDlgBase@@QAE@PAVQWidget@@PBDI@Z$67 10012046 f   device_type_editdlg.obj
 0001:00011050       __unwindfunclet$??0device_type_editDlgBase@@QAE@PAVQWidget@@PBDI@Z$68 10012050 f   device_type_editdlg.obj
 0001:0001105a       __unwindfunclet$??0device_type_editDlgBase@@QAE@PAVQWidget@@PBDI@Z$69 1001205a f   device_type_editdlg.obj
 0001:00011064       __unwindfunclet$??0device_type_editDlgBase@@QAE@PAVQWidget@@PBDI@Z$70 10012064 f   device_type_editdlg.obj
 0001:0001106e       __unwindfunclet$??0device_type_editDlgBase@@QAE@PAVQWidget@@PBDI@Z$71 1001206e f   device_type_editdlg.obj
 0001:00011078       __unwindfunclet$??0device_type_editDlgBase@@QAE@PAVQWidget@@PBDI@Z$72 10012078 f   device_type_editdlg.obj
 0001:00011082       __unwindfunclet$??0device_type_editDlgBase@@QAE@PAVQWidget@@PBDI@Z$73 10012082 f   device_type_editdlg.obj
 0001:0001108c       __unwindfunclet$??0device_type_editDlgBase@@QAE@PAVQWidget@@PBDI@Z$74 1001208c f   device_type_editdlg.obj
 0001:00011096       __unwindfunclet$??0device_type_editDlgBase@@QAE@PAVQWidget@@PBDI@Z$75 10012096 f   device_type_editdlg.obj
 0001:000110a0       __unwindfunclet$??0device_type_editDlgBase@@QAE@PAVQWidget@@PBDI@Z$76 100120a0 f   device_type_editdlg.obj
 0001:000110aa       __unwindfunclet$??0device_type_editDlgBase@@QAE@PAVQWidget@@PBDI@Z$77 100120aa f   device_type_editdlg.obj
 0001:000110b4       __unwindfunclet$??0device_type_editDlgBase@@QAE@PAVQWidget@@PBDI@Z$78 100120b4 f   device_type_editdlg.obj
 0001:000110be       __unwindfunclet$??0device_type_editDlgBase@@QAE@PAVQWidget@@PBDI@Z$79 100120be f   device_type_editdlg.obj
 0001:000110c8       __unwindfunclet$??0device_type_editDlgBase@@QAE@PAVQWidget@@PBDI@Z$80 100120c8 f   device_type_editdlg.obj
 0001:000110d2       __unwindfunclet$??0device_type_editDlgBase@@QAE@PAVQWidget@@PBDI@Z$81 100120d2 f   device_type_editdlg.obj
 0001:000110dc       __unwindfunclet$??0device_type_editDlgBase@@QAE@PAVQWidget@@PBDI@Z$82 100120dc f   device_type_editdlg.obj
 0001:000110e6       __unwindfunclet$??0device_type_editDlgBase@@QAE@PAVQWidget@@PBDI@Z$83 100120e6 f   device_type_editdlg.obj
 0001:000110f0       __unwindfunclet$??0device_type_editDlgBase@@QAE@PAVQWidget@@PBDI@Z$84 100120f0 f   device_type_editdlg.obj
 0001:000110fa       __unwindfunclet$??0device_type_editDlgBase@@QAE@PAVQWidget@@PBDI@Z$85 100120fa f   device_type_editdlg.obj
 0001:00011104       __unwindfunclet$??0device_type_editDlgBase@@QAE@PAVQWidget@@PBDI@Z$86 10012104 f   device_type_editdlg.obj
 0001:0001110e       __unwindfunclet$??0device_type_editDlgBase@@QAE@PAVQWidget@@PBDI@Z$87 1001210e f   device_type_editdlg.obj
 0001:00011118       __ehhandler$??0device_type_editDlgBase@@QAE@PAVQWidget@@PBDI@Z 10012118 f   device_type_editdlg.obj
 0001:00011133       __unwindfunclet$??1device_type_editDlgBase@@UAE@XZ$0 10012133 f   device_type_editdlg.obj
 0001:0001113c       __ehhandler$??1device_type_editDlgBase@@UAE@XZ 1001213c f   device_type_editdlg.obj
 0001:00011157       __unwindfunclet$?languageChange@device_type_editDlgBase@@MAEXXZ$0 10012157 f   device_type_editdlg.obj
 0001:00011160       __unwindfunclet$?languageChange@device_type_editDlgBase@@MAEXXZ$1 10012160 f   device_type_editdlg.obj
 0001:00011169       __unwindfunclet$?languageChange@device_type_editDlgBase@@MAEXXZ$2 10012169 f   device_type_editdlg.obj
 0001:00011172       __unwindfunclet$?languageChange@device_type_editDlgBase@@MAEXXZ$3 10012172 f   device_type_editdlg.obj
 0001:0001117b       __unwindfunclet$?languageChange@device_type_editDlgBase@@MAEXXZ$4 1001217b f   device_type_editdlg.obj
 0001:00011184       __unwindfunclet$?languageChange@device_type_editDlgBase@@MAEXXZ$5 10012184 f   device_type_editdlg.obj
 0001:0001118d       __unwindfunclet$?languageChange@device_type_editDlgBase@@MAEXXZ$6 1001218d f   device_type_editdlg.obj
 0001:00011196       __unwindfunclet$?languageChange@device_type_editDlgBase@@MAEXXZ$7 10012196 f   device_type_editdlg.obj
 0001:0001119f       __unwindfunclet$?languageChange@device_type_editDlgBase@@MAEXXZ$8 1001219f f   device_type_editdlg.obj
 0001:000111a8       __unwindfunclet$?languageChange@device_type_editDlgBase@@MAEXXZ$9 100121a8 f   device_type_editdlg.obj
 0001:000111b1       __unwindfunclet$?languageChange@device_type_editDlgBase@@MAEXXZ$10 100121b1 f   device_type_editdlg.obj
 0001:000111ba       __unwindfunclet$?languageChange@device_type_editDlgBase@@MAEXXZ$11 100121ba f   device_type_editdlg.obj
 0001:000111c3       __unwindfunclet$?languageChange@device_type_editDlgBase@@MAEXXZ$12 100121c3 f   device_type_editdlg.obj
 0001:000111cc       __unwindfunclet$?languageChange@device_type_editDlgBase@@MAEXXZ$13 100121cc f   device_type_editdlg.obj
 0001:000111d5       __unwindfunclet$?languageChange@device_type_editDlgBase@@MAEXXZ$14 100121d5 f   device_type_editdlg.obj
 0001:000111de       __unwindfunclet$?languageChange@device_type_editDlgBase@@MAEXXZ$15 100121de f   device_type_editdlg.obj
 0001:000111e7       __unwindfunclet$?languageChange@device_type_editDlgBase@@MAEXXZ$16 100121e7 f   device_type_editdlg.obj
 0001:000111f0       __unwindfunclet$?languageChange@device_type_editDlgBase@@MAEXXZ$17 100121f0 f   device_type_editdlg.obj
 0001:000111f9       __unwindfunclet$?languageChange@device_type_editDlgBase@@MAEXXZ$18 100121f9 f   device_type_editdlg.obj
 0001:00011202       __unwindfunclet$?languageChange@device_type_editDlgBase@@MAEXXZ$19 10012202 f   device_type_editdlg.obj
 0001:0001120b       __unwindfunclet$?languageChange@device_type_editDlgBase@@MAEXXZ$20 1001220b f   device_type_editdlg.obj
 0001:00011214       __unwindfunclet$?languageChange@device_type_editDlgBase@@MAEXXZ$21 10012214 f   device_type_editdlg.obj
 0001:0001121d       __unwindfunclet$?languageChange@device_type_editDlgBase@@MAEXXZ$22 1001221d f   device_type_editdlg.obj
 0001:00011226       __unwindfunclet$?languageChange@device_type_editDlgBase@@MAEXXZ$23 10012226 f   device_type_editdlg.obj
 0001:0001122f       __unwindfunclet$?languageChange@device_type_editDlgBase@@MAEXXZ$24 1001222f f   device_type_editdlg.obj
 0001:00011238       __unwindfunclet$?languageChange@device_type_editDlgBase@@MAEXXZ$25 10012238 f   device_type_editdlg.obj
 0001:00011241       __unwindfunclet$?languageChange@device_type_editDlgBase@@MAEXXZ$26 10012241 f   device_type_editdlg.obj
 0001:0001124a       __unwindfunclet$?languageChange@device_type_editDlgBase@@MAEXXZ$27 1001224a f   device_type_editdlg.obj
 0001:00011253       __unwindfunclet$?languageChange@device_type_editDlgBase@@MAEXXZ$28 10012253 f   device_type_editdlg.obj
 0001:0001125c       __unwindfunclet$?languageChange@device_type_editDlgBase@@MAEXXZ$29 1001225c f   device_type_editdlg.obj
 0001:00011265       __unwindfunclet$?languageChange@device_type_editDlgBase@@MAEXXZ$30 10012265 f   device_type_editdlg.obj
 0001:0001126e       __unwindfunclet$?languageChange@device_type_editDlgBase@@MAEXXZ$31 1001226e f   device_type_editdlg.obj
 0001:00011277       __unwindfunclet$?languageChange@device_type_editDlgBase@@MAEXXZ$32 10012277 f   device_type_editdlg.obj
 0001:00011280       __unwindfunclet$?languageChange@device_type_editDlgBase@@MAEXXZ$33 10012280 f   device_type_editdlg.obj
 0001:00011289       __unwindfunclet$?languageChange@device_type_editDlgBase@@MAEXXZ$34 10012289 f   device_type_editdlg.obj
 0001:00011292       __unwindfunclet$?languageChange@device_type_editDlgBase@@MAEXXZ$35 10012292 f   device_type_editdlg.obj
 0001:0001129b       __unwindfunclet$?languageChange@device_type_editDlgBase@@MAEXXZ$36 1001229b f   device_type_editdlg.obj
 0001:000112a4       __unwindfunclet$?languageChange@device_type_editDlgBase@@MAEXXZ$37 100122a4 f   device_type_editdlg.obj
 0001:000112ad       __unwindfunclet$?languageChange@device_type_editDlgBase@@MAEXXZ$38 100122ad f   device_type_editdlg.obj
 0001:000112b6       __unwindfunclet$?languageChange@device_type_editDlgBase@@MAEXXZ$39 100122b6 f   device_type_editdlg.obj
 0001:000112bf       __unwindfunclet$?languageChange@device_type_editDlgBase@@MAEXXZ$40 100122bf f   device_type_editdlg.obj
 0001:000112c8       __unwindfunclet$?languageChange@device_type_editDlgBase@@MAEXXZ$41 100122c8 f   device_type_editdlg.obj
 0001:000112d1       __unwindfunclet$?languageChange@device_type_editDlgBase@@MAEXXZ$42 100122d1 f   device_type_editdlg.obj
 0001:000112da       __unwindfunclet$?languageChange@device_type_editDlgBase@@MAEXXZ$43 100122da f   device_type_editdlg.obj
 0001:000112e3       __unwindfunclet$?languageChange@device_type_editDlgBase@@MAEXXZ$44 100122e3 f   device_type_editdlg.obj
 0001:000112ec       __unwindfunclet$?languageChange@device_type_editDlgBase@@MAEXXZ$45 100122ec f   device_type_editdlg.obj
 0001:000112f5       __unwindfunclet$?languageChange@device_type_editDlgBase@@MAEXXZ$46 100122f5 f   device_type_editdlg.obj
 0001:000112fe       __unwindfunclet$?languageChange@device_type_editDlgBase@@MAEXXZ$47 100122fe f   device_type_editdlg.obj
 0001:00011307       __unwindfunclet$?languageChange@device_type_editDlgBase@@MAEXXZ$48 10012307 f   device_type_editdlg.obj
 0001:00011310       __unwindfunclet$?languageChange@device_type_editDlgBase@@MAEXXZ$49 10012310 f   device_type_editdlg.obj
 0001:00011319       __unwindfunclet$?languageChange@device_type_editDlgBase@@MAEXXZ$50 10012319 f   device_type_editdlg.obj
 0001:00011322       __unwindfunclet$?languageChange@device_type_editDlgBase@@MAEXXZ$51 10012322 f   device_type_editdlg.obj
 0001:0001132b       __unwindfunclet$?languageChange@device_type_editDlgBase@@MAEXXZ$52 1001232b f   device_type_editdlg.obj
 0001:00011334       __unwindfunclet$?languageChange@device_type_editDlgBase@@MAEXXZ$53 10012334 f   device_type_editdlg.obj
 0001:0001133d       __unwindfunclet$?languageChange@device_type_editDlgBase@@MAEXXZ$54 1001233d f   device_type_editdlg.obj
 0001:00011346       __unwindfunclet$?languageChange@device_type_editDlgBase@@MAEXXZ$55 10012346 f   device_type_editdlg.obj
 0001:0001134f       __unwindfunclet$?languageChange@device_type_editDlgBase@@MAEXXZ$56 1001234f f   device_type_editdlg.obj
 0001:00011358       __ehhandler$?languageChange@device_type_editDlgBase@@MAEXXZ 10012358 f   device_type_editdlg.obj
 0001:00011373       __unwindfunclet$?command@device_type_edit@@IAEXVQString@@0@Z$0 10012373 f   moc_device_type_edit.obj
 0001:00011373       __unwindfunclet$?command@device_type_editDlg@@IAEXVQString@@0@Z$0 10012373 f   moc_device_type_edit.obj
 0001:0001137c       __unwindfunclet$?command@device_type_editDlg@@IAEXVQString@@0@Z$1 1001237c f   moc_device_type_edit.obj
 0001:0001137c       __unwindfunclet$?command@device_type_edit@@IAEXVQString@@0@Z$1 1001237c f   moc_device_type_edit.obj
 0001:00011385       __unwindfunclet$?command@device_type_edit@@IAEXVQString@@0@Z$2 10012385 f   moc_device_type_edit.obj
 0001:00011385       __unwindfunclet$?command@device_type_editDlg@@IAEXVQString@@0@Z$2 10012385 f   moc_device_type_edit.obj
 0001:00011399       __ehhandler$?command@device_type_edit@@IAEXVQString@@0@Z 10012399 f   moc_device_type_edit.obj
 0001:00011399       __ehhandler$?command@device_type_editDlg@@IAEXVQString@@0@Z 10012399 f   moc_device_type_edit.obj
 0001:000113be       __unwindfunclet$?qt_emit@device_type_edit@@UAE_NHPAUQUObject@@@Z$0 100123be f   moc_device_type_edit.obj
 0001:000113be       __unwindfunclet$?qt_emit@device_type_editDlg@@UAE_NHPAUQUObject@@@Z$0 100123be f   moc_device_type_edit.obj
 0001:000113c7       __ehhandler$?qt_emit@device_type_edit@@UAE_NHPAUQUObject@@@Z 100123c7 f   moc_device_type_edit.obj
 0001:000113c7       __ehhandler$?qt_emit@device_type_editDlg@@UAE_NHPAUQUObject@@@Z 100123c7 f   moc_device_type_edit.obj
 0001:000113e2       __unwindfunclet$?typeSelected@toolWindow@@IAEXABVQString@@@Z$0 100123e2 f   moc_toolwindowimpl.obj
 0001:000113e2       __unwindfunclet$?typeDeleted@toolWindow@@IAEXABVQString@@@Z$0 100123e2 f   moc_toolwindowimpl.obj
 0001:000113eb       __ehhandler$?typeDeleted@toolWindow@@IAEXABVQString@@@Z 100123eb f   moc_toolwindowimpl.obj
 0001:000113eb       __ehhandler$?typeSelected@toolWindow@@IAEXABVQString@@@Z 100123eb f   moc_toolwindowimpl.obj
 0001:00011406       __unwindfunclet$??0toolWindowBase@@QAE@PAVQWidget@@PBDI@Z$0 10012406 f   toolwindow.obj
 0001:0001140f       __unwindfunclet$??0toolWindowBase@@QAE@PAVQWidget@@PBDI@Z$1 1001240f f   toolwindow.obj
 0001:00011419       __unwindfunclet$??0toolWindowBase@@QAE@PAVQWidget@@PBDI@Z$2 10012419 f   toolwindow.obj
 0001:00011423       __unwindfunclet$??0toolWindowBase@@QAE@PAVQWidget@@PBDI@Z$3 10012423 f   toolwindow.obj
 0001:0001142d       __unwindfunclet$??0toolWindowBase@@QAE@PAVQWidget@@PBDI@Z$4 1001242d f   toolwindow.obj
 0001:00011437       __unwindfunclet$??0toolWindowBase@@QAE@PAVQWidget@@PBDI@Z$5 10012437 f   toolwindow.obj
 0001:00011441       __unwindfunclet$??0toolWindowBase@@QAE@PAVQWidget@@PBDI@Z$6 10012441 f   toolwindow.obj
 0001:0001144b       __unwindfunclet$??0toolWindowBase@@QAE@PAVQWidget@@PBDI@Z$7 1001244b f   toolwindow.obj
 0001:00011455       __unwindfunclet$??0toolWindowBase@@QAE@PAVQWidget@@PBDI@Z$8 10012455 f   toolwindow.obj
 0001:0001145f       __unwindfunclet$??0toolWindowBase@@QAE@PAVQWidget@@PBDI@Z$9 1001245f f   toolwindow.obj
 0001:00011468       __unwindfunclet$??0toolWindowBase@@QAE@PAVQWidget@@PBDI@Z$10 10012468 f   toolwindow.obj
 0001:00011471       __unwindfunclet$??0toolWindowBase@@QAE@PAVQWidget@@PBDI@Z$11 10012471 f   toolwindow.obj
 0001:0001147a       __ehhandler$??0toolWindowBase@@QAE@PAVQWidget@@PBDI@Z 1001247a f   toolwindow.obj
 0001:00011495       __unwindfunclet$?languageChange@toolWindowBase@@MAEXXZ$0 10012495 f   toolwindow.obj
 0001:0001149e       __unwindfunclet$?languageChange@toolWindowBase@@MAEXXZ$1 1001249e f   toolwindow.obj
 0001:000114a7       __unwindfunclet$?languageChange@toolWindowBase@@MAEXXZ$2 100124a7 f   toolwindow.obj
 0001:000114b0       __unwindfunclet$?languageChange@toolWindowBase@@MAEXXZ$3 100124b0 f   toolwindow.obj
 0001:000114b9       __unwindfunclet$?languageChange@toolWindowBase@@MAEXXZ$4 100124b9 f   toolwindow.obj
 0001:000114c2       __unwindfunclet$?languageChange@toolWindowBase@@MAEXXZ$5 100124c2 f   toolwindow.obj
 0001:000114cb       __ehhandler$?languageChange@toolWindowBase@@MAEXXZ 100124cb f   toolwindow.obj
 0001:000114e6       __unwindfunclet$??0cfg_ListView@@QAE@PAVQWidget@@PBD@Z$0 100124e6 f   cfg_widgets001:cfg_ListView.obj
 0001:000114ef       __unwindfunclet$??0cfg_ListView@@QAE@PAVQWidget@@PBD@Z$1 100124ef f   cfg_widgets001:cfg_ListView.obj
 0001:000114f9       __unwindfunclet$??0cfg_ListView@@QAE@PAVQWidget@@PBD@Z$2 100124f9 f   cfg_widgets001:cfg_ListView.obj
 0001:00011503       __ehhandler$??0cfg_ListView@@QAE@PAVQWidget@@PBD@Z 10012503 f   cfg_widgets001:cfg_ListView.obj
 0001:0001151e       __unwindfunclet$??1cfg_ListView@@UAE@XZ$0 1001251e f   cfg_widgets001:cfg_ListView.obj
 0001:00011527       __ehhandler$??1cfg_ListView@@UAE@XZ 10012527 f   cfg_widgets001:cfg_ListView.obj
 0001:00011542       __unwindfunclet$?clipBoardDataChanged@cfg_ListView@@IAEXXZ$0 10012542 f   cfg_widgets001:cfg_ListView.obj
 0001:0001154b       __ehhandler$?clipBoardDataChanged@cfg_ListView@@IAEXXZ 1001254b f   cfg_widgets001:cfg_ListView.obj
 0001:00011566       __unwindfunclet$?copyToClipboard@cfg_ListView@@QAEXXZ$0 10012566 f   cfg_widgets001:cfg_ListView.obj
 0001:0001156f       __unwindfunclet$?copyToClipboard@cfg_ListView@@QAEXXZ$1 1001256f f   cfg_widgets001:cfg_ListView.obj
 0001:00011578       __unwindfunclet$?copyToClipboard@cfg_ListView@@QAEXXZ$2 10012578 f   cfg_widgets001:cfg_ListView.obj
 0001:00011581       __unwindfunclet$?copyToClipboard@cfg_ListView@@QAEXXZ$3 10012581 f   cfg_widgets001:cfg_ListView.obj
 0001:0001158a       __ehhandler$?copyToClipboard@cfg_ListView@@QAEXXZ 1001258a f   cfg_widgets001:cfg_ListView.obj
 0001:000115a5       __unwindfunclet$?deleteItems@cfg_ListView@@QAEXXZ$0 100125a5 f   cfg_widgets001:cfg_ListView.obj
 0001:000115ad       __unwindfunclet$?deleteItems@cfg_ListView@@QAEXXZ$1 100125ad f   cfg_widgets001:cfg_ListView.obj
 0001:000115b6       __ehhandler$?deleteItems@cfg_ListView@@QAEXXZ 100125b6 f   cfg_widgets001:cfg_ListView.obj
 0001:000115d1       __unwindfunclet$?insertData@cfg_ListView@@QAEXXZ$0 100125d1 f   cfg_widgets001:cfg_ListView.obj
 0001:000115da       __unwindfunclet$?insertData@cfg_ListView@@QAEXXZ$1 100125da f   cfg_widgets001:cfg_ListView.obj
 0001:000115e3       __unwindfunclet$?insertData@cfg_ListView@@QAEXXZ$2 100125e3 f   cfg_widgets001:cfg_ListView.obj
 0001:000115ec       __unwindfunclet$?insertData@cfg_ListView@@QAEXXZ$3 100125ec f   cfg_widgets001:cfg_ListView.obj
 0001:000115f5       __ehhandler$?insertData@cfg_ListView@@QAEXXZ 100125f5 f   cfg_widgets001:cfg_ListView.obj
 0001:00011610       __unwindfunclet$?replaceData@cfg_ListView@@QAEXXZ$0 10012610 f   cfg_widgets001:cfg_ListView.obj
 0001:00011618       __unwindfunclet$?replaceData@cfg_ListView@@QAEXXZ$1 10012618 f   cfg_widgets001:cfg_ListView.obj
 0001:00011621       __unwindfunclet$?replaceData@cfg_ListView@@QAEXXZ$2 10012621 f   cfg_widgets001:cfg_ListView.obj
 0001:0001162a       __unwindfunclet$?replaceData@cfg_ListView@@QAEXXZ$3 1001262a f   cfg_widgets001:cfg_ListView.obj
 0001:00011633       __unwindfunclet$?replaceData@cfg_ListView@@QAEXXZ$4 10012633 f   cfg_widgets001:cfg_ListView.obj
 0001:0001163c       __unwindfunclet$?replaceData@cfg_ListView@@QAEXXZ$5 1001263c f   cfg_widgets001:cfg_ListView.obj
 0001:00011645       __ehhandler$?replaceData@cfg_ListView@@QAEXXZ 10012645 f   cfg_widgets001:cfg_ListView.obj
 0001:00011660       __unwindfunclet$?updateEntry@cfg_ListView@@AAEPAVQListViewItem@@QAV2@ABVQString@@_N@Z$0 10012660 f   cfg_widgets001:cfg_ListView.obj
 0001:00011669       __unwindfunclet$?updateEntry@cfg_ListView@@AAEPAVQListViewItem@@QAV2@ABVQString@@_N@Z$1 10012669 f   cfg_widgets001:cfg_ListView.obj
 0001:00011672       __unwindfunclet$?updateEntry@cfg_ListView@@AAEPAVQListViewItem@@QAV2@ABVQString@@_N@Z$2 10012672 f   cfg_widgets001:cfg_ListView.obj
 0001:0001167b       __ehhandler$?updateEntry@cfg_ListView@@AAEPAVQListViewItem@@QAV2@ABVQString@@_N@Z 1001267b f   cfg_widgets001:cfg_ListView.obj
 0001:00011696       ??__FcleanUp_device_type_edit@@YAXXZ 10012696 f   moc_device_type_edit.obj
 0001:000116a1       ??__FcleanUp_device_type_editDlgBase@@YAXXZ 100126a1 f   moc_device_type_editdlg.obj
 0001:000116ac       ??__FcleanUp_device_type_editDlg@@YAXXZ 100126ac f   moc_device_type_editdlgimpl.obj
 0001:000116b7       ??__FcleanUp_toolWindowBase@@YAXXZ 100126b7 f   moc_toolwindow.obj
 0001:000116c2       ??__FcleanUp_toolWindow@@YAXXZ 100126c2 f   moc_toolwindowimpl.obj
 0001:000116cd       ??__FcleanUp_cfg_ListView@@YAXXZ 100126cd f   cfg_widgets001:moc_cfg_ListView.obj
 0002:00000fb8       _cleanUp_device_type_edit$initializer$ 10013fb8     moc_device_type_edit.obj
 0002:00000fbc       _cleanUp_device_type_editDlgBase$initializer$ 10013fbc     moc_device_type_editdlg.obj
 0002:00000fc0       _cleanUp_device_type_editDlg$initializer$ 10013fc0     moc_device_type_editdlgimpl.obj
 0002:00000fc4       _cleanUp_toolWindowBase$initializer$ 10013fc4     moc_toolwindow.obj
 0002:00000fc8       _cleanUp_toolWindow$initializer$ 10013fc8     moc_toolwindowimpl.obj
 0002:00000fcc       _cleanUp_cfg_ListView$initializer$ 10013fcc     cfg_widgets001:moc_cfg_ListView.obj
 0002:00000fd8       _pcinit                    10013fd8     MSVCRT:crtdll.obj
 0002:00000fdc       _pinit                     10013fdc     MSVCRT:atonexit.obj
 0002:00004ee4       ?slot_0@?3??staticMetaObject@device_type_edit@@SAPAVQMetaObject@@XZ@4UQUMethod@@B 10017ee4     moc_device_type_edit.obj
 0002:00004efc       ?slot_1@?3??staticMetaObject@device_type_edit@@SAPAVQMetaObject@@XZ@4UQUMethod@@B 10017efc     moc_device_type_edit.obj
 0002:00004f14       ?slot_2@?3??staticMetaObject@device_type_edit@@SAPAVQMetaObject@@XZ@4UQUMethod@@B 10017f14     moc_device_type_edit.obj
 0002:00004f2c       ?slot_tbl@?3??staticMetaObject@device_type_edit@@SAPAVQMetaObject@@XZ@4QBUQMetaData@@B 10017f2c     moc_device_type_edit.obj
 0002:00004f94       ?signal_0@?3??staticMetaObject@device_type_edit@@SAPAVQMetaObject@@XZ@4UQUMethod@@B 10017f94     moc_device_type_edit.obj
 0002:00004fa8       ?signal_tbl@?3??staticMetaObject@device_type_edit@@SAPAVQMetaObject@@XZ@4QBUQMetaData@@B 10017fa8     moc_device_type_edit.obj
 0002:00004fd0       ?slot_0@?3??staticMetaObject@device_type_editDlgBase@@SAPAVQMetaObject@@XZ@4UQUMethod@@B 10017fd0     moc_device_type_editdlg.obj
 0002:00004fec       ?slot_tbl@?3??staticMetaObject@device_type_editDlgBase@@SAPAVQMetaObject@@XZ@4QBUQMetaData@@B 10017fec     moc_device_type_editdlg.obj
 0002:00005010       ?slot_0@?3??staticMetaObject@device_type_editDlg@@SAPAVQMetaObject@@XZ@4UQUMethod@@B 10018010     moc_device_type_editdlgimpl.obj
 0002:0000502c       ?slot_1@?3??staticMetaObject@device_type_editDlg@@SAPAVQMetaObject@@XZ@4UQUMethod@@B 1001802c     moc_device_type_editdlgimpl.obj
 0002:00005044       ?slot_2@?3??staticMetaObject@device_type_editDlg@@SAPAVQMetaObject@@XZ@4UQUMethod@@B 10018044     moc_device_type_editdlgimpl.obj
 0002:00005064       ?slot_3@?3??staticMetaObject@device_type_editDlg@@SAPAVQMetaObject@@XZ@4UQUMethod@@B 10018064     moc_device_type_editdlgimpl.obj
 0002:0000507c       ?slot_4@?3??staticMetaObject@device_type_editDlg@@SAPAVQMetaObject@@XZ@4UQUMethod@@B 1001807c     moc_device_type_editdlgimpl.obj
 0002:00005094       ?slot_5@?3??staticMetaObject@device_type_editDlg@@SAPAVQMetaObject@@XZ@4UQUMethod@@B 10018094     moc_device_type_editdlgimpl.obj
 0002:000050ac       ?slot_6@?3??staticMetaObject@device_type_editDlg@@SAPAVQMetaObject@@XZ@4UQUMethod@@B 100180ac     moc_device_type_editdlgimpl.obj
 0002:000050c4       ?slot_7@?3??staticMetaObject@device_type_editDlg@@SAPAVQMetaObject@@XZ@4UQUMethod@@B 100180c4     moc_device_type_editdlgimpl.obj
 0002:000050dc       ?slot_8@?3??staticMetaObject@device_type_editDlg@@SAPAVQMetaObject@@XZ@4UQUMethod@@B 100180dc     moc_device_type_editdlgimpl.obj
 0002:000050f8       ?slot_9@?3??staticMetaObject@device_type_editDlg@@SAPAVQMetaObject@@XZ@4UQUMethod@@B 100180f8     moc_device_type_editdlgimpl.obj
 0002:00005134       ?slot_10@?3??staticMetaObject@device_type_editDlg@@SAPAVQMetaObject@@XZ@4UQUMethod@@B 10018134     moc_device_type_editdlgimpl.obj
 0002:00005150       ?slot_11@?3??staticMetaObject@device_type_editDlg@@SAPAVQMetaObject@@XZ@4UQUMethod@@B 10018150     moc_device_type_editdlgimpl.obj
 0002:0000515c       ?slot_12@?3??staticMetaObject@device_type_editDlg@@SAPAVQMetaObject@@XZ@4UQUMethod@@B 1001815c     moc_device_type_editdlgimpl.obj
 0002:00005168       ?slot_13@?3??staticMetaObject@device_type_editDlg@@SAPAVQMetaObject@@XZ@4UQUMethod@@B 10018168     moc_device_type_editdlgimpl.obj
 0002:00005174       ?slot_14@?3??staticMetaObject@device_type_editDlg@@SAPAVQMetaObject@@XZ@4UQUMethod@@B 10018174     moc_device_type_editdlgimpl.obj
 0002:00005180       ?slot_15@?3??staticMetaObject@device_type_editDlg@@SAPAVQMetaObject@@XZ@4UQUMethod@@B 10018180     moc_device_type_editdlgimpl.obj
 0002:000051a0       ?slot_16@?3??staticMetaObject@device_type_editDlg@@SAPAVQMetaObject@@XZ@4UQUMethod@@B 100181a0     moc_device_type_editdlgimpl.obj
 0002:000051c0       ?slot_tbl@?3??staticMetaObject@device_type_editDlg@@SAPAVQMetaObject@@XZ@4QBUQMetaData@@B 100181c0     moc_device_type_editdlgimpl.obj
 0002:000053d4       ?signal_0@?3??staticMetaObject@device_type_editDlg@@SAPAVQMetaObject@@XZ@4UQUMethod@@B 100183d4     moc_device_type_editdlgimpl.obj
 0002:000053e0       ?signal_1@?3??staticMetaObject@device_type_editDlg@@SAPAVQMetaObject@@XZ@4UQUMethod@@B 100183e0     moc_device_type_editdlgimpl.obj
 0002:000053ec       ?signal_tbl@?3??staticMetaObject@device_type_editDlg@@SAPAVQMetaObject@@XZ@4QBUQMetaData@@B 100183ec     moc_device_type_editdlgimpl.obj
 0002:0000541c       ?slot_0@?3??staticMetaObject@toolWindowBase@@SAPAVQMetaObject@@XZ@4UQUMethod@@B 1001841c     moc_toolwindow.obj
 0002:00005428       ?slot_tbl@?3??staticMetaObject@toolWindowBase@@SAPAVQMetaObject@@XZ@4QBUQMetaData@@B 10018428     moc_toolwindow.obj
 0002:00005440       ?slot_0@?3??staticMetaObject@toolWindow@@SAPAVQMetaObject@@XZ@4UQUMethod@@B 10018440     moc_toolwindowimpl.obj
 0002:00005458       ?slot_1@?3??staticMetaObject@toolWindow@@SAPAVQMetaObject@@XZ@4UQUMethod@@B 10018458     moc_toolwindowimpl.obj
 0002:0000546c       ?slot_2@?3??staticMetaObject@toolWindow@@SAPAVQMetaObject@@XZ@4UQUMethod@@B 1001846c     moc_toolwindowimpl.obj
 0002:00005478       ?slot_tbl@?3??staticMetaObject@toolWindow@@SAPAVQMetaObject@@XZ@4QBUQMetaData@@B 10018478     moc_toolwindowimpl.obj
 0002:000054d4       ?signal_0@?3??staticMetaObject@toolWindow@@SAPAVQMetaObject@@XZ@4UQUMethod@@B 100184d4     moc_toolwindowimpl.obj
 0002:000054f0       ?signal_1@?3??staticMetaObject@toolWindow@@SAPAVQMetaObject@@XZ@4UQUMethod@@B 100184f0     moc_toolwindowimpl.obj
 0002:00005508       ?signal_2@?3??staticMetaObject@toolWindow@@SAPAVQMetaObject@@XZ@4UQUMethod@@B 10018508     moc_toolwindowimpl.obj
 0002:00005514       ?signal_tbl@?3??staticMetaObject@toolWindow@@SAPAVQMetaObject@@XZ@4QBUQMetaData@@B 10018514     moc_toolwindowimpl.obj
 0002:00005e5c       ?slot_0@?3??staticMetaObject@cfg_ListView@@SAPAVQMetaObject@@XZ@4UQUMethod@@B 10018e5c     cfg_widgets001:moc_cfg_ListView.obj
 0002:00005e74       ?slot_1@?3??staticMetaObject@cfg_ListView@@SAPAVQMetaObject@@XZ@4UQUMethod@@B 10018e74     cfg_widgets001:moc_cfg_ListView.obj
 0002:00005e8c       ?slot_2@?3??staticMetaObject@cfg_ListView@@SAPAVQMetaObject@@XZ@4UQUMethod@@B 10018e8c     cfg_widgets001:moc_cfg_ListView.obj
 0002:00005ea8       ?slot_3@?3??staticMetaObject@cfg_ListView@@SAPAVQMetaObject@@XZ@4UQUMethod@@B 10018ea8     cfg_widgets001:moc_cfg_ListView.obj
 0002:00005ec0       ?slot_4@?3??staticMetaObject@cfg_ListView@@SAPAVQMetaObject@@XZ@4UQUMethod@@B 10018ec0     cfg_widgets001:moc_cfg_ListView.obj
 0002:00005ed8       ?slot_5@?3??staticMetaObject@cfg_ListView@@SAPAVQMetaObject@@XZ@4UQUMethod@@B 10018ed8     cfg_widgets001:moc_cfg_ListView.obj
 0002:00005f00       ?slot_tbl@?3??staticMetaObject@cfg_ListView@@SAPAVQMetaObject@@XZ@4QBUQMetaData@@B 10018f00     cfg_widgets001:moc_cfg_ListView.obj
 0002:00005fb0       ?signal_0@?3??staticMetaObject@cfg_ListView@@SAPAVQMetaObject@@XZ@4UQUMethod@@B 10018fb0     cfg_widgets001:moc_cfg_ListView.obj
 0002:00005fc8       ?signal_1@?3??staticMetaObject@cfg_ListView@@SAPAVQMetaObject@@XZ@4UQUMethod@@B 10018fc8     cfg_widgets001:moc_cfg_ListView.obj
 0002:00005fe8       ?signal_tbl@?3??staticMetaObject@cfg_ListView@@SAPAVQMetaObject@@XZ@4QBUQMetaData@@B 10018fe8     cfg_widgets001:moc_cfg_ListView.obj
 0002:00006038       _GS_ExceptionPointers      10019038     MSVCRT:gs_report.obj
 0002:00007450       __unwindtable$??1QDockWindowList@@UAE@XZ 1001a450     device_type_edit.obj
 0002:00007460       __ehfuncinfo$??1QDockWindowList@@UAE@XZ 1001a460     device_type_edit.obj
 0002:00007484       __unwindtable$??1QPopupMenuList@@UAE@XZ 1001a484     device_type_edit.obj
 0002:0000748c       __ehfuncinfo$??1QPopupMenuList@@UAE@XZ 1001a48c     device_type_edit.obj
 0002:000074b0       __unwindtable$??0config_plugin_base@@QAE@ABVQString@@00@Z 1001a4b0     device_type_edit.obj
 0002:000074d0       __ehfuncinfo$??0config_plugin_base@@QAE@ABVQString@@00@Z 1001a4d0     device_type_edit.obj
 0002:000074f4       __unwindtable$??1config_plugin_base@@UAE@XZ 1001a4f4     device_type_edit.obj
 0002:0000750c       __ehfuncinfo$??1config_plugin_base@@UAE@XZ 1001a50c     device_type_edit.obj
 0002:00007530       __unwindtable$?about@config_plugin_base@@UAE?AVQString@@XZ 1001a530     device_type_edit.obj
 0002:00007540       __ehfuncinfo$?about@config_plugin_base@@UAE?AVQString@@XZ 1001a540     device_type_edit.obj
 0002:00007564       __ehfuncinfo$??0device_type_edit@@QAE@ABVQString@@00@Z 1001a564     device_type_edit.obj
 0002:00007588       __unwindtable$??0device_type_edit@@QAE@ABVQString@@00@Z 1001a588     device_type_edit.obj
 0002:00007688       __ehfuncinfo$??1device_type_edit@@UAE@XZ 1001a688     device_type_edit.obj
 0002:000076ac       __unwindtable$??1device_type_edit@@UAE@XZ 1001a6ac     device_type_edit.obj
 0002:000076f4       __unwindtable$?toolbars@device_type_edit@@UAE?AVQDockWindowList@@XZ 1001a6f4     device_type_edit.obj
 0002:000076fc       __ehfuncinfo$?toolbars@device_type_edit@@UAE?AVQDockWindowList@@XZ 1001a6fc     device_type_edit.obj
 0002:00007720       __unwindtable$?menus@device_type_edit@@UAE?AVQPopupMenuList@@XZ 1001a720     device_type_edit.obj
 0002:00007728       __ehfuncinfo$?menus@device_type_edit@@UAE?AVQPopupMenuList@@XZ 1001a728     device_type_edit.obj
 0002:0000774c       __ehfuncinfo$?reply@device_type_edit@@UAEXPAVresponse@@@Z 1001a74c     device_type_edit.obj
 0002:00007770       __unwindtable$?reply@device_type_edit@@UAEXPAVresponse@@@Z 1001a770     device_type_edit.obj
 0002:00007858       __unwindtable$?navigate@device_type_edit@@UAEXABVQString@@0@Z 1001a858     device_type_edit.obj
 0002:00007870       __ehfuncinfo$?navigate@device_type_edit@@UAEXABVQString@@0@Z 1001a870     device_type_edit.obj
 0002:00007894       __ehfuncinfo$?activate@device_type_edit@@UAEX_N@Z 1001a894     device_type_edit.obj
 0002:000078b8       __unwindtable$?activate@device_type_edit@@UAEX_N@Z 1001a8b8     device_type_edit.obj
 0002:00007900       __unwindtable$?closeEvent@device_type_edit@@UAEXPAVQCloseEvent@@@Z 1001a900     device_type_edit.obj
 0002:00007920       __ehfuncinfo$?closeEvent@device_type_edit@@UAEXPAVQCloseEvent@@@Z 1001a920     device_type_edit.obj
 0002:00007944       __ehfuncinfo$?apply@device_type_edit@@UAEXXZ 1001a944     device_type_edit.obj
 0002:00007968       __unwindtable$?apply@device_type_edit@@UAEXXZ 1001a968     device_type_edit.obj
 0002:00007a20       __ehfuncinfo$?about@device_type_edit@@UAE?AVQString@@XZ 1001aa20     device_type_edit.obj
 0002:00007a44       __unwindtable$?about@device_type_edit@@UAE?AVQString@@XZ 1001aa44     device_type_edit.obj
 0002:00007a6c       __unwindtable$?newItem@cfg_ListView@@MAEPAVQListViewItem@@PAVQListView@@PAV2@@Z 1001aa6c     device_type_edit.obj
 0002:00007a6c       __unwindtable$??0?$QGuardedPtr@VQDockWindow@@@@QAE@XZ 1001aa6c     device_type_edit.obj
 0002:00007a6c       __unwindtable$??4?$QGuardedPtr@VtoolWindow@@@@QAEAAV0@PAVtoolWindow@@@Z 1001aa6c     device_type_edit.obj
 0002:00007a6c       __unwindtable$??4?$QGuardedPtr@VQDockWindow@@@@QAEAAV0@PAVQDockWindow@@@Z 1001aa6c     device_type_edit.obj
 0002:00007a6c       __unwindtable$??0?$QGuardedPtr@VtoolWindow@@@@QAE@XZ 1001aa6c     device_type_edit.obj
 0002:00007a6c       __unwindtable$??4?$QGuardedPtr@VQPopupMenu@@@@QAEAAV0@PAVQPopupMenu@@@Z 1001aa6c     device_type_edit.obj
 0002:00007a6c       __unwindtable$??0?$QGuardedPtr@VQPopupMenu@@@@QAE@XZ 1001aa6c     device_type_edit.obj
 0002:00007a6c       __unwindtable$?create@plugindesc@@UAEPAVconfig_plugin_base@@ABVQString@@00@Z 1001aa6c     device_type_edit.obj
 0002:00007a74       __ehfuncinfo$?newItem@cfg_ListView@@MAEPAVQListViewItem@@PAVQListView@@PAV2@@Z 1001aa74     device_type_edit.obj
 0002:00007a74       __ehfuncinfo$??0?$QGuardedPtr@VtoolWindow@@@@QAE@XZ 1001aa74     device_type_edit.obj
 0002:00007a74       __ehfuncinfo$?create@plugindesc@@UAEPAVconfig_plugin_base@@ABVQString@@00@Z 1001aa74     device_type_edit.obj
 0002:00007a74       __ehfuncinfo$??0?$QGuardedPtr@VQDockWindow@@@@QAE@XZ 1001aa74     device_type_edit.obj
 0002:00007a74       __ehfuncinfo$??0?$QGuardedPtr@VQPopupMenu@@@@QAE@XZ 1001aa74     device_type_edit.obj
 0002:00007a74       __ehfuncinfo$??4?$QGuardedPtr@VtoolWindow@@@@QAEAAV0@PAVtoolWindow@@@Z 1001aa74     device_type_edit.obj
 0002:00007a74       __ehfuncinfo$??4?$QGuardedPtr@VQPopupMenu@@@@QAEAAV0@PAVQPopupMenu@@@Z 1001aa74     device_type_edit.obj
 0002:00007a74       __ehfuncinfo$??4?$QGuardedPtr@VQDockWindow@@@@QAEAAV0@PAVQDockWindow@@@Z 1001aa74     device_type_edit.obj
 0002:00007a98       __unwindtable$??1?$QDict@VQAction@@@@UAE@XZ 1001aa98     device_type_edit.obj
 0002:00007aa0       __ehfuncinfo$??1?$QDict@VQAction@@@@UAE@XZ 1001aaa0     device_type_edit.obj
 0002:00007ac4       __ehfuncinfo$?deleteType@device_type_edit@@AAEXABVQString@@@Z 1001aac4     device_type_edit.obj
 0002:00007ae8       __unwindtable$?deleteType@device_type_edit@@AAEXABVQString@@@Z 1001aae8     device_type_edit.obj
 0002:00007b40       __ehfuncinfo$?selectType@device_type_edit@@AAEXABVQString@@@Z 1001ab40     device_type_edit.obj
 0002:00007b64       __unwindtable$?selectType@device_type_edit@@AAEXABVQString@@@Z 1001ab64     device_type_edit.obj
 0002:00007bcc       __ehfuncinfo$?markDirty@device_type_edit@@AAEXXZ 1001abcc     device_type_edit.obj
 0002:00007bf0       __unwindtable$?markDirty@device_type_edit@@AAEXXZ 1001abf0     device_type_edit.obj
 0002:00007c20       __unwindtable$?db@@YAXABVQString@@@Z 1001ac20     device_type_edit.obj
 0002:00007c28       __ehfuncinfo$?db@@YAXABVQString@@@Z 1001ac28     device_type_edit.obj
 0002:00007c4c       __ehfuncinfo$??0device_type_editDlg@@QAE@ABVQString@@PAVQWidget@@PBDI@Z 1001ac4c     device_type_editdlgimpl.obj
 0002:00007c70       __unwindtable$??0device_type_editDlg@@QAE@ABVQString@@PAVQWidget@@PBDI@Z 1001ac70     device_type_editdlgimpl.obj
 0002:00007ca8       __unwindtable$??1device_type_editDlg@@UAE@XZ 1001aca8     device_type_editdlgimpl.obj
 0002:00007cb8       __ehfuncinfo$??1device_type_editDlg@@UAE@XZ 1001acb8     device_type_editdlgimpl.obj
 0002:00007cdc       __ehfuncinfo$?enumDeleteState@device_type_editDlg@@AAE_NVQString@@@Z 1001acdc     device_type_editdlgimpl.obj
 0002:00007d00       __unwindtable$?enumDeleteState@device_type_editDlg@@AAE_NVQString@@@Z 1001ad00     device_type_editdlgimpl.obj
 0002:00007d50       __ehfuncinfo$?saveString@device_type_editDlg@@AAE_NPAVQDomElement@@@Z 1001ad50     device_type_editdlgimpl.obj
 0002:00007d74       __unwindtable$?saveString@device_type_editDlg@@AAE_NPAVQDomElement@@@Z 1001ad74     device_type_editdlgimpl.obj
 0002:00007dfc       __ehfuncinfo$?displayString@device_type_editDlg@@AAEXPAVQDomElement@@@Z 1001adfc     device_type_editdlgimpl.obj
 0002:00007e20       __unwindtable$?displayString@device_type_editDlg@@AAEXPAVQDomElement@@@Z 1001ae20     device_type_editdlgimpl.obj
 0002:00007e68       __ehfuncinfo$?newGetNewParamName@device_type_editDlg@@AAE?AVQString@@V2@@Z 1001ae68     device_type_editdlgimpl.obj
 0002:00007e8c       __unwindtable$?newGetNewParamName@device_type_editDlg@@AAE?AVQString@@V2@@Z 1001ae8c     device_type_editdlgimpl.obj
 0002:00007f14       __ehfuncinfo$?loadParamLvi@device_type_editDlg@@AAEXVQString@@PAVQDomElement@@@Z 1001af14     device_type_editdlgimpl.obj
 0002:00007f38       __unwindtable$?loadParamLvi@device_type_editDlg@@AAEXVQString@@PAVQDomElement@@@Z 1001af38     device_type_editdlgimpl.obj
 0002:00007fa0       __ehfuncinfo$?removeSettings@device_type_editDlg@@AAE_NPAVQDomElement@@VQString@@@Z 1001afa0     device_type_editdlgimpl.obj
 0002:00007fc4       __unwindtable$?removeSettings@device_type_editDlg@@AAE_NPAVQDomElement@@VQString@@@Z 1001afc4     device_type_editdlgimpl.obj
 0002:0000806c       __ehfuncinfo$?loadFile@device_type_editDlg@@AAE_NABVQString@@0@Z 1001b06c     device_type_editdlgimpl.obj
 0002:00008090       __unwindtable$?loadFile@device_type_editDlg@@AAE_NABVQString@@0@Z 1001b090     device_type_editdlgimpl.obj
 0002:00008178       __ehfuncinfo$?saveFile@device_type_editDlg@@AAE_NABVQString@@0@Z 1001b178     device_type_editdlgimpl.obj
 0002:0000819c       __unwindtable$?saveFile@device_type_editDlg@@AAE_NABVQString@@0@Z 1001b19c     device_type_editdlgimpl.obj
 0002:000081d4       __ehfuncinfo$?displayRange@device_type_editDlg@@AAEXPAVQDomElement@@@Z 1001b1d4     device_type_editdlgimpl.obj
 0002:000081f8       __unwindtable$?displayRange@device_type_editDlg@@AAEXPAVQDomElement@@@Z 1001b1f8     device_type_editdlgimpl.obj
 0002:000082c8       __ehfuncinfo$?saveRange@device_type_editDlg@@AAE_NPAVQDomElement@@@Z 1001b2c8     device_type_editdlgimpl.obj
 0002:000082ec       __unwindtable$?saveRange@device_type_editDlg@@AAE_NPAVQDomElement@@@Z 1001b2ec     device_type_editdlgimpl.obj
 0002:0000847c       __ehfuncinfo$?displayEnum@device_type_editDlg@@AAEXPAVQDomElement@@@Z 1001b47c     device_type_editdlgimpl.obj
 0002:000084a0       __unwindtable$?displayEnum@device_type_editDlg@@AAEXPAVQDomElement@@@Z 1001b4a0     device_type_editdlgimpl.obj
 0002:00008540       __ehfuncinfo$?saveEnum@device_type_editDlg@@AAE_NPAVQDomElement@@@Z 1001b540     device_type_editdlgimpl.obj
 0002:00008564       __unwindtable$?saveEnum@device_type_editDlg@@AAE_NPAVQDomElement@@@Z 1001b564     device_type_editdlgimpl.obj
 0002:000085f4       __ehfuncinfo$?saveElement@device_type_editDlg@@AAE_NPAVQDomElement@@@Z 1001b5f4     device_type_editdlgimpl.obj
 0002:00008618       __unwindtable$?saveElement@device_type_editDlg@@AAE_NPAVQDomElement@@@Z 1001b618     device_type_editdlgimpl.obj
 0002:00008690       __ehfuncinfo$?loadElement@device_type_editDlg@@AAE_NPAVQDomElement@@@Z 1001b690     device_type_editdlgimpl.obj
 0002:000086b4       __unwindtable$?loadElement@device_type_editDlg@@AAE_NPAVQDomElement@@@Z 1001b6b4     device_type_editdlgimpl.obj
 0002:0000870c       __unwindtable$?clearParamView@device_type_editDlg@@AAEXXZ 1001b70c     device_type_editdlgimpl.obj
 0002:0000871c       __ehfuncinfo$?clearParamView@device_type_editDlg@@AAEXXZ 1001b71c     device_type_editdlgimpl.obj
 0002:00008740       __ehfuncinfo$?selectParam@device_type_editDlg@@AAEXPAVQListViewItem@@@Z 1001b740     device_type_editdlgimpl.obj
 0002:00008764       __unwindtable$?selectParam@device_type_editDlg@@AAEXPAVQListViewItem@@@Z 1001b764     device_type_editdlgimpl.obj
 0002:000087c4       __ehfuncinfo$?loadTemplates@device_type_editDlg@@AAEXVQString@@@Z 1001b7c4     device_type_editdlgimpl.obj
 0002:000087e8       __unwindtable$?loadTemplates@device_type_editDlg@@AAEXVQString@@@Z 1001b7e8     device_type_editdlgimpl.obj
 0002:00008818       __ehfuncinfo$?paramDelete@device_type_editDlg@@AAEXXZ 1001b818     device_type_editdlgimpl.obj
 0002:0000883c       __unwindtable$?paramDelete@device_type_editDlg@@AAEXXZ 1001b83c     device_type_editdlgimpl.obj
 0002:00008884       __unwindtable$?checkParamClipboard@device_type_editDlg@@AAEXXZ 1001b884     device_type_editdlgimpl.obj
 0002:000088a4       __ehfuncinfo$?checkParamClipboard@device_type_editDlg@@AAEXXZ 1001b8a4     device_type_editdlgimpl.obj
 0002:000088c8       __ehfuncinfo$?paramPaste@device_type_editDlg@@AAEXXZ 1001b8c8     device_type_editdlgimpl.obj
 0002:000088ec       __unwindtable$?paramPaste@device_type_editDlg@@AAEXXZ 1001b8ec     device_type_editdlgimpl.obj
 0002:0000899c       __ehfuncinfo$?paramCopy@device_type_editDlg@@AAEXXZ 1001b99c     device_type_editdlgimpl.obj
 0002:000089c0       __unwindtable$?paramCopy@device_type_editDlg@@AAEXXZ 1001b9c0     device_type_editdlgimpl.obj
 0002:00008a40       __unwindtable$?paramRename@device_type_editDlg@@AAEXXZ 1001ba40     device_type_editdlgimpl.obj
 0002:00008a60       __ehfuncinfo$?paramRename@device_type_editDlg@@AAEXXZ 1001ba60     device_type_editdlgimpl.obj
 0002:00008a84       __ehfuncinfo$?paramNew@device_type_editDlg@@AAEXXZ 1001ba84     device_type_editdlgimpl.obj
 0002:00008aa8       __unwindtable$?paramNew@device_type_editDlg@@AAEXXZ 1001baa8     device_type_editdlgimpl.obj
 0002:00008af0       __ehfuncinfo$?enumPaste@device_type_editDlg@@AAEXXZ 1001baf0     device_type_editdlgimpl.obj
 0002:00008b14       __unwindtable$?enumPaste@device_type_editDlg@@AAEXXZ 1001bb14     device_type_editdlgimpl.obj
 0002:00008bfc       __ehfuncinfo$?enumNewState@device_type_editDlg@@AAEXXZ 1001bbfc     device_type_editdlgimpl.obj
 0002:00008c20       __unwindtable$?enumNewState@device_type_editDlg@@AAEXXZ 1001bc20     device_type_editdlgimpl.obj
 0002:00008d00       __unwindtable$?selectParam@device_type_editDlg@@AAEXXZ 1001bd00     device_type_editdlgimpl.obj
 0002:00008d18       __ehfuncinfo$?selectParam@device_type_editDlg@@AAEXXZ 1001bd18     device_type_editdlgimpl.obj
 0002:00008d3c       __ehfuncinfo$?devTypeChange@device_type_editDlg@@AAEXH@Z 1001bd3c     device_type_editdlgimpl.obj
 0002:00008d60       __unwindtable$?devTypeChange@device_type_editDlg@@AAEXH@Z 1001bd60     device_type_editdlgimpl.obj
 0002:00008d90       __unwindtable$??1?$QPtrList@VQListViewItem@@@@UAE@XZ 1001bd90     device_type_editdlgimpl.obj
 0002:00008d90       __unwindtable$??1?$QPtrList@VQPopupMenu@@@@UAE@XZ 1001bd90     device_type_editdlgimpl.obj
 0002:00008d98       __ehfuncinfo$??1?$QPtrList@VQListViewItem@@@@UAE@XZ 1001bd98     device_type_editdlgimpl.obj
 0002:00008d98       __ehfuncinfo$??1?$QPtrList@VQPopupMenu@@@@UAE@XZ 1001bd98     device_type_editdlgimpl.obj
 0002:00008dbc       __unwindtable$?compare@paramLVI@@UBEHPAVQListViewItem@@H_N@Z 1001bdbc     paramLVI.obj
 0002:00008ddc       __ehfuncinfo$?compare@paramLVI@@UBEHPAVQListViewItem@@H_N@Z 1001bddc     paramLVI.obj
 0002:00008e00       __unwindtable$?keys@plugindesc@@UAE?AVQStringList@@ABVQString@@0@Z 1001be00     plugindesc.obj
 0002:00008e10       __ehfuncinfo$?keys@plugindesc@@UAE?AVQStringList@@ABVQString@@0@Z 1001be10     plugindesc.obj
 0002:00008e34       __unwindtable$?saveFile@toolWindow@@QAE_NVQString@@@Z 1001be34     toolwindowimpl.obj
 0002:00008e54       __ehfuncinfo$?saveFile@toolWindow@@QAE_NVQString@@@Z 1001be54     toolwindowimpl.obj
 0002:00008e78       __ehfuncinfo$?loadFile@toolWindow@@QAE_NVQString@@@Z 1001be78     toolwindowimpl.obj
 0002:00008e9c       __unwindtable$?loadFile@toolWindow@@QAE_NVQString@@@Z 1001be9c     toolwindowimpl.obj
 0002:00008f54       __unwindtable$??0toolWindow@@QAE@PAVQWidget@@PBDI@Z 1001bf54     toolwindowimpl.obj
 0002:00008f6c       __ehfuncinfo$??0toolWindow@@QAE@PAVQWidget@@PBDI@Z 1001bf6c     toolwindowimpl.obj
 0002:00008f90       __unwindtable$??1toolWindow@@UAE@XZ 1001bf90     toolwindowimpl.obj
 0002:00008f98       __ehfuncinfo$??1toolWindow@@UAE@XZ 1001bf98     toolwindowimpl.obj
 0002:00008fbc       __ehfuncinfo$?deleteFile@toolWindow@@AAEXXZ 1001bfbc     toolwindowimpl.obj
 0002:00008fe0       __unwindtable$?deleteFile@toolWindow@@AAEXXZ 1001bfe0     toolwindowimpl.obj
 0002:00009020       __ehfuncinfo$?newFile@toolWindow@@AAEXXZ 1001c020     toolwindowimpl.obj
 0002:00009044       __unwindtable$?newFile@toolWindow@@AAEXXZ 1001c044     toolwindowimpl.obj
 0002:00009164       __unwindtable$?selectType@toolWindow@@AAEXPAVQListViewItem@@@Z 1001c164     toolwindowimpl.obj
 0002:0000916c       __ehfuncinfo$?selectType@toolWindow@@AAEXPAVQListViewItem@@@Z 1001c16c     toolwindowimpl.obj
 0002:00009190       __ehfuncinfo$?selectFamily@toolWindow@@AAE?AVQString@@V2@0@Z 1001c190     toolwindowimpl.obj
 0002:000091b4       __unwindtable$?selectFamily@toolWindow@@AAE?AVQString@@V2@0@Z 1001c1b4     toolwindowimpl.obj
 0002:000091dc       __ehfuncinfo$??0device_type_editDlgBase@@QAE@PAVQWidget@@PBDI@Z 1001c1dc     device_type_editdlg.obj
 0002:00009200       __unwindtable$??0device_type_editDlgBase@@QAE@PAVQWidget@@PBDI@Z 1001c200     device_type_editdlg.obj
 0002:000094c0       __unwindtable$??1device_type_editDlgBase@@UAE@XZ 1001c4c0     device_type_editdlg.obj
 0002:000094c8       __ehfuncinfo$??1device_type_editDlgBase@@UAE@XZ 1001c4c8     device_type_editdlg.obj
 0002:000094ec       __ehfuncinfo$?languageChange@device_type_editDlgBase@@MAEXXZ 1001c4ec     device_type_editdlg.obj
 0002:00009510       __unwindtable$?languageChange@device_type_editDlgBase@@MAEXXZ 1001c510     device_type_editdlg.obj
 0002:000096d8       __unwindtable$?qt_emit@device_type_editDlg@@UAE_NHPAUQUObject@@@Z 1001c6d8     moc_device_type_edit.obj
 0002:000096d8       __unwindtable$?qt_emit@device_type_edit@@UAE_NHPAUQUObject@@@Z 1001c6d8     moc_device_type_edit.obj
 0002:000096e0       __ehfuncinfo$?qt_emit@device_type_edit@@UAE_NHPAUQUObject@@@Z 1001c6e0     moc_device_type_edit.obj
 0002:000096e0       __ehfuncinfo$?qt_emit@device_type_editDlg@@UAE_NHPAUQUObject@@@Z 1001c6e0     moc_device_type_edit.obj
 0002:00009704       __unwindtable$?command@device_type_editDlg@@IAEXVQString@@0@Z 1001c704     moc_device_type_edit.obj
 0002:00009704       __unwindtable$?command@device_type_edit@@IAEXVQString@@0@Z 1001c704     moc_device_type_edit.obj
 0002:0000971c       __ehfuncinfo$?command@device_type_edit@@IAEXVQString@@0@Z 1001c71c     moc_device_type_edit.obj
 0002:0000971c       __ehfuncinfo$?command@device_type_editDlg@@IAEXVQString@@0@Z 1001c71c     moc_device_type_edit.obj
 0002:00009740       __unwindtable$?typeDeleted@toolWindow@@IAEXABVQString@@@Z 1001c740     moc_toolwindowimpl.obj
 0002:00009740       __unwindtable$?typeSelected@toolWindow@@IAEXABVQString@@@Z 1001c740     moc_toolwindowimpl.obj
 0002:00009748       __ehfuncinfo$?typeSelected@toolWindow@@IAEXABVQString@@@Z 1001c748     moc_toolwindowimpl.obj
 0002:00009748       __ehfuncinfo$?typeDeleted@toolWindow@@IAEXABVQString@@@Z 1001c748     moc_toolwindowimpl.obj
 0002:0000976c       __ehfuncinfo$??0toolWindowBase@@QAE@PAVQWidget@@PBDI@Z 1001c76c     toolwindow.obj
 0002:00009790       __unwindtable$??0toolWindowBase@@QAE@PAVQWidget@@PBDI@Z 1001c790     toolwindow.obj
 0002:000097f0       __ehfuncinfo$?languageChange@toolWindowBase@@MAEXXZ 1001c7f0     toolwindow.obj
 0002:00009814       __unwindtable$?languageChange@toolWindowBase@@MAEXXZ 1001c814     toolwindow.obj
 0002:00009844       __unwindtable$??0cfg_ListView@@QAE@PAVQWidget@@PBD@Z 1001c844     cfg_widgets001:cfg_ListView.obj
 0002:0000985c       __ehfuncinfo$??0cfg_ListView@@QAE@PAVQWidget@@PBD@Z 1001c85c     cfg_widgets001:cfg_ListView.obj
 0002:00009880       __unwindtable$??1cfg_ListView@@UAE@XZ 1001c880     cfg_widgets001:cfg_ListView.obj
 0002:00009888       __ehfuncinfo$??1cfg_ListView@@UAE@XZ 1001c888     cfg_widgets001:cfg_ListView.obj
 0002:000098ac       __ehfuncinfo$?insertData@cfg_ListView@@QAEXXZ 1001c8ac     cfg_widgets001:cfg_ListView.obj
 0002:000098d0       __unwindtable$?insertData@cfg_ListView@@QAEXXZ 1001c8d0     cfg_widgets001:cfg_ListView.obj
 0002:000098f8       __unwindtable$?deleteItems@cfg_ListView@@QAEXXZ 1001c8f8     cfg_widgets001:cfg_ListView.obj
 0002:00009908       __ehfuncinfo$?deleteItems@cfg_ListView@@QAEXXZ 1001c908     cfg_widgets001:cfg_ListView.obj
 0002:0000992c       __unwindtable$?copyToClipboard@cfg_ListView@@QAEXXZ 1001c92c     cfg_widgets001:cfg_ListView.obj
 0002:0000994c       __ehfuncinfo$?copyToClipboard@cfg_ListView@@QAEXXZ 1001c94c     cfg_widgets001:cfg_ListView.obj
 0002:00009970       __ehfuncinfo$?replaceData@cfg_ListView@@QAEXXZ 1001c970     cfg_widgets001:cfg_ListView.obj
 0002:00009994       __unwindtable$?replaceData@cfg_ListView@@QAEXXZ 1001c994     cfg_widgets001:cfg_ListView.obj
 0002:000099cc       __unwindtable$?clipBoardDataChanged@cfg_ListView@@IAEXXZ 1001c9cc     cfg_widgets001:cfg_ListView.obj
 0002:000099d4       __ehfuncinfo$?clipBoardDataChanged@cfg_ListView@@IAEXXZ 1001c9d4     cfg_widgets001:cfg_ListView.obj
 0002:000099f8       __unwindtable$?updateEntry@cfg_ListView@@AAEPAVQListViewItem@@QAV2@ABVQString@@_N@Z 1001c9f8     cfg_widgets001:cfg_ListView.obj
 0002:00009a18       __ehfuncinfo$?updateEntry@cfg_ListView@@AAEPAVQListViewItem@@QAV2@ABVQString@@_N@Z 1001ca18     cfg_widgets001:cfg_ListView.obj
 0002:00009a40       __sehtable$??_L@YGXPAXIHP6EX0@Z1@Z 1001ca40     MSVCRT:ehvecctr.obj
 0002:00009a60       __sehtable$??_M@YGXPAXIHP6EX0@Z@Z 1001ca60     MSVCRT:ehvecdtr.obj
 0002:00009a80       __sehtable$?__ArrayUnwind@@YGXPAXIHP6EX0@Z@Z 1001ca80     MSVCRT:ehvecdtr.obj
 0002:00009aa0       __sehtable$__onexit        1001caa0     MSVCRT:atonexit.obj
 0002:00009ac0       __sehtable$___DllMainCRTStartup 1001cac0     MSVCRT:crtdll.obj
 0002:00009ae8       __sehtable$__IsNonwritableInCurrentImage 1001cae8     MSVCRT:pesect.obj
 0002:00009b10       .edata                     1001cb10     config_device_type_edit.exp
 0002:00009b38       rgpv                       1001cb38     config_device_type_edit.exp
 0002:00009bb8       rgszName                   1001cbb8     config_device_type_edit.exp
 0002:00009c38       rgwOrd                     1001cc38     config_device_type_edit.exp
 0002:00009c78       szName                     1001cc78     config_device_type_edit.exp
 0002:00009c94       $N00001                    1001cc94     config_device_type_edit.exp
 0002:00009cb1       $N00002                    1001ccb1     config_device_type_edit.exp
 0002:00009cd8       $N00003                    1001ccd8     config_device_type_edit.exp
 0002:00009cf0       $N00004                    1001ccf0     config_device_type_edit.exp
 0002:00009d11       $N00005                    1001cd11     config_device_type_edit.exp
 0002:00009d30       $N00006                    1001cd30     config_device_type_edit.exp
 0002:00009d54       $N00007                    1001cd54     config_device_type_edit.exp
 0002:00009d6d       $N00008                    1001cd6d     config_device_type_edit.exp
 0002:00009d8f       $N00009                    1001cd8f     config_device_type_edit.exp
 0002:00009daf       $N00010                    1001cdaf     config_device_type_edit.exp
 0002:00009dda       $N00011                    1001cdda     config_device_type_edit.exp
 0002:00009e05       $N00012                    1001ce05     config_device_type_edit.exp
 0002:00009e2b       $N00013                    1001ce2b     config_device_type_edit.exp
 0002:00009e4c       $N00014                    1001ce4c     config_device_type_edit.exp
 0002:00009e6e       $N00015                    1001ce6e     config_device_type_edit.exp
 0002:00009e8f       $N00016                    1001ce8f     config_device_type_edit.exp
 0002:00009eb9       $N00017                    1001ceb9     config_device_type_edit.exp
 0002:00009ee9       $N00018                    1001cee9     config_device_type_edit.exp
 0002:00009f2b       $N00019                    1001cf2b     config_device_type_edit.exp
 0002:00009f54       $N00020                    1001cf54     config_device_type_edit.exp
 0002:00009f77       $N00021                    1001cf77     config_device_type_edit.exp
 0002:00009fa4       $N00022                    1001cfa4     config_device_type_edit.exp
 0002:00009fd3       $N00023                    1001cfd3     config_device_type_edit.exp
 0002:0000a005       $N00024                    1001d005     config_device_type_edit.exp
 0002:0000a049       $N00025                    1001d049     config_device_type_edit.exp
 0002:0000a06b       $N00026                    1001d06b     config_device_type_edit.exp
 0002:0000a0a0       $N00027                    1001d0a0     config_device_type_edit.exp
 0002:0000a0c7       $N00028                    1001d0c7     config_device_type_edit.exp
 0002:0000a0f2       $N00029                    1001d0f2     config_device_type_edit.exp
 0002:0000a112       $N00030                    1001d112     config_device_type_edit.exp
 0002:0000a158       $N00031                    1001d158     config_device_type_edit.exp
 0002:0000a18c       $N00032                    1001d18c     config_device_type_edit.exp
 0002:0000b1e4       .idata$6                   1001e1e4     config_icons:config_icons.dll
 0002:00015182       .idata$6                   10028182     qt-mt323:qt-mt323.dll
 0002:000151d2       .idata$6                   100281d2     MSVCRT:MSVCR120.dll
 0002:0001550a       .idata$6                   1002850a     kernel32:KERNEL32.dll
 0003:00000000       _device_type_edit_XPM      10029000     plugindesc.obj
 0003:00000054       ?param_slot_0@?3??staticMetaObject@device_type_editDlg@@SAPAVQMetaObject@@XZ@4QBUQUParameter@@B 10029054     moc_device_type_editdlgimpl.obj
 0003:00000064       ?param_slot_10@?3??staticMetaObject@device_type_editDlg@@SAPAVQMetaObject@@XZ@4QBUQUParameter@@B 10029064     moc_device_type_editdlgimpl.obj
 0003:00000094       ?param_slot_16@?3??staticMetaObject@device_type_editDlg@@SAPAVQMetaObject@@XZ@4QBUQUParameter@@B 10029094     moc_device_type_editdlgimpl.obj
 0003:00000704       _cleanUp_device_type_edit  10029704     moc_device_type_edit.obj
 0003:00000708       ?param_slot_0@?3??staticMetaObject@device_type_edit@@SAPAVQMetaObject@@XZ@4QBUQUParameter@@B 10029708     moc_device_type_edit.obj
 0003:00000718       ?$S1@?3??staticMetaObject@device_type_edit@@SAPAVQMetaObject@@XZ@4IA 10029718     moc_device_type_edit.obj
 0003:0000071c       ?param_slot_1@?3??staticMetaObject@device_type_edit@@SAPAVQMetaObject@@XZ@4QBUQUParameter@@B 1002971c     moc_device_type_edit.obj
 0003:0000072c       ?param_signal_0@?3??staticMetaObject@device_type_edit@@SAPAVQMetaObject@@XZ@4QBUQUParameter@@B 1002972c     moc_device_type_edit.obj
 0003:00000750       _cleanUp_device_type_editDlgBase 10029750     moc_device_type_editdlg.obj
 0003:00000758       _cleanUp_device_type_editDlg 10029758     moc_device_type_editdlgimpl.obj
 0003:0000075c       ?$S1@?3??staticMetaObject@device_type_editDlg@@SAPAVQMetaObject@@XZ@4IA 1002975c     moc_device_type_editdlgimpl.obj
 0003:00000760       ?param_slot_11@?3??staticMetaObject@device_type_editDlg@@SAPAVQMetaObject@@XZ@4QBUQUParameter@@B 10029760     moc_device_type_editdlgimpl.obj
 0003:00000770       ?param_slot_13@?3??staticMetaObject@device_type_editDlg@@SAPAVQMetaObject@@XZ@4QBUQUParameter@@B 10029770     moc_device_type_editdlgimpl.obj
 0003:00000780       ?param_slot_14@?3??staticMetaObject@device_type_editDlg@@SAPAVQMetaObject@@XZ@4QBUQUParameter@@B 10029780     moc_device_type_editdlgimpl.obj
 0003:000007a0       ?param_signal_0@?3??staticMetaObject@device_type_editDlg@@SAPAVQMetaObject@@XZ@4QBUQUParameter@@B 100297a0     moc_device_type_editdlgimpl.obj
 0003:000007c4       _cleanUp_toolWindowBase    100297c4     moc_toolwindow.obj
 0003:000007cc       _cleanUp_toolWindow        100297cc     moc_toolwindowimpl.obj
 0003:000007d0       ?param_slot_2@?3??staticMetaObject@toolWindow@@SAPAVQMetaObject@@XZ@4QBUQUParameter@@B 100297d0     moc_toolwindowimpl.obj
 0003:000007e0       ?$S1@?3??staticMetaObject@toolWindow@@SAPAVQMetaObject@@XZ@4IA 100297e0     moc_toolwindowimpl.obj
 0003:000007e4       ?param_signal_0@?3??staticMetaObject@toolWindow@@SAPAVQMetaObject@@XZ@4QBUQUParameter@@B 100297e4     moc_toolwindowimpl.obj
 0003:000007f4       ?param_signal_1@?3??staticMetaObject@toolWindow@@SAPAVQMetaObject@@XZ@4QBUQUParameter@@B 100297f4     moc_toolwindowimpl.obj
 0003:00000808       _cleanUp_cfg_ListView      10029808     cfg_widgets001:moc_cfg_ListView.obj
 0003:0000080c       ?param_signal_1@?3??staticMetaObject@cfg_ListView@@SAPAVQMetaObject@@XZ@4QBUQUParameter@@B 1002980c     cfg_widgets001:moc_cfg_ListView.obj
 0003:0000081c       ?$S1@?3??staticMetaObject@cfg_ListView@@SAPAVQMetaObject@@XZ@4IA 1002981c     cfg_widgets001:moc_cfg_ListView.obj
 0003:00000820       ___proc_attached           10029820     MSVCRT:crtdll.obj
 0003:00000828       _GS_ExceptionRecord        10029828     MSVCRT:gs_report.obj
 0003:00000878       _GS_ContextRecord          10029878     MSVCRT:gs_report.obj
 0003:00000b44       _DebuggerWasPresent        10029b44     MSVCRT:gs_report.obj
 0004:000000a0       $R000000                   1002a0a0     Script1.res
 0004:00000540       $R0004A0                   1002a540     Script1.res
